 ControlsDLL

 Timestamp is 56cd513e (Wed Feb 24 15:44:14 2016)

 Preferred load address is 10000000

 Start         Length     Name                   Class
 0001:00000000 0005f4b2H .text                   CODE
 0001:0005f4c0 000013bcH .text$x                 CODE
 0001:00060880 0000008cH .text$yc                CODE
 0001:00060910 000000baH .text$yd                CODE
 0002:00000000 00000340H .idata$5                DATA
 0002:00000340 00000004H .CRT$XCA                DATA
 0002:00000344 00000014H .CRT$XCU                DATA
 0002:00000358 00000004H .CRT$XCZ                DATA
 0002:0000035c 00000004H .CRT$XIA                DATA
 0002:00000360 00000014H .CRT$XIC                DATA
 0002:00000374 00000004H .CRT$XIZ                DATA
 0002:00000378 00000004H .CRT$XPA                DATA
 0002:0000037c 00000004H .CRT$XPX                DATA
 0002:00000380 00000004H .CRT$XPXA               DATA
 0002:00000384 00000004H .CRT$XPZ                DATA
 0002:00000388 00000004H .CRT$XTA                DATA
 0002:0000038c 00000004H .CRT$XTZ                DATA
 0002:00000390 00009408H .rdata                  DATA
 0002:00009798 00000071H .rdata$debug            DATA
 0002:0000980c 00000a20H .rdata$r                DATA
 0002:0000a230 000001dcH .rdata$sxdata           DATA
 0002:0000a40c 00000004H .rtc$IAA                DATA
 0002:0000a410 00000004H .rtc$IZZ                DATA
 0002:0000a414 00000004H .rtc$TAA                DATA
 0002:0000a418 00000004H .rtc$TZZ                DATA
 0002:0000a420 00002180H .xdata$x                DATA
 0002:0000c5a0 00000000H ATL$__a                 DATA
 0002:0000c5a0 00000000H ATL$__z                 DATA
 0002:0000c5a0 0000008cH .idata$2                DATA
 0002:0000c62c 00000014H .idata$3                DATA
 0002:0000c640 00000340H .idata$4                DATA
 0002:0000c980 00000f8eH .idata$6                DATA
 0002:0000d910 00000059H .edata                  DATA
 0003:00000000 00001bf0H .data                   DATA
 0003:00001c00 00006920H .bss                    DATA
 0004:00000000 00000058H .rsrc$01                DATA
 0004:00000060 00000300H .rsrc$02                DATA

  Address         Publics by Value              Rva+Base       Lib:Object

 0000:00000000       __except_list              00000000     <absolute>
 0000:00000077       ___safe_se_handler_count   00000077     <absolute>
 0000:00000000       ___ImageBase               10000000     <linker-defined>
 0001:00000000       _GFXDll_DialogManagerWZ    10001000 f   dllaccess.obj
 0001:000000cb       _DllMain@12                100010cb f   DllEntry.obj
 0001:000000e9       ??0CBaseManager@@QAE@XZ    100010e9 f   BaseManager.obj
 0001:00000182       ??1CBaseManager@@UAE@XZ    10001182 f   BaseManager.obj
 0001:00000203       ?OnCreate@CBaseManager@@UAE_NXZ 10001203 f   BaseManager.obj
 0001:0000020e       ?OnDestroy@CBaseManager@@UAEXXZ 1000120e f   BaseManager.obj
 0001:0000021f       ?RemoveCtrlID@CBaseManager@@QAE_NK@Z 1000121f f   BaseManager.obj
 0001:0000029d       ?CreateID@CBaseManager@@QAEKPAX@Z 1000129d f   BaseManager.obj
 0001:000002ee       ?CreateID@CBaseManager@@QAE_NKPAX@Z 100012ee f   BaseManager.obj
 0001:00000345       ?IsCtrlID@CBaseManager@@QAE_NK@Z 10001345 f   BaseManager.obj
 0001:00000397       ?MoveToTail@CBaseManager@@QAE_NK@Z 10001397 f   BaseManager.obj
 0001:000003e9       ?MoveToHead@CBaseManager@@QAE_NK@Z 100013e9 f   BaseManager.obj
 0001:0000043b       ?FindData@CBaseManager@@QAEPAXK@Z 1000143b f   BaseManager.obj
 0001:00000496       ?FindIndexData@CBaseManager@@QAEPAXK@Z 10001496 f   BaseManager.obj
 0001:0000055b       ?FindIndexID@CBaseManager@@QAEKH@Z 1000155b f   BaseManager.obj
 0001:0000060f       ?RemoveAllCtrlID@CBaseManager@@QAE_NXZ 1000160f f   BaseManager.obj
 0001:0000065a       ?FindDrawList@CBaseManager@@QAE?AV?$_Iterator@$00@?$list@KV?$allocator@K@std@@@std@@K@Z 1000165a f   BaseManager.obj
 0001:00000742       ?ChangeCtrlID@CBaseManager@@QAE_NKK@Z 10001742 f   BaseManager.obj
 0001:00000923       ?MoveToListIndex@CBaseManager@@QAE_NHH@Z 10001923 f   BaseManager.obj
 0001:00000a35       ?SetHeadPosition@CBaseManager@@UAEXXZ 10001a35 f   BaseManager.obj
 0001:00000a8f       ?GetNextDrawInfo@CBaseManager@@UAEPAXXZ 10001a8f f   BaseManager.obj
 0001:00000b87       ?SetTailPosition@CBaseManager@@QAEXXZ 10001b87 f   BaseManager.obj
 0001:00000be5       ?GetPrevDrawInfo@CBaseManager@@QAEPAXXZ 10001be5 f   BaseManager.obj
 0001:00000cf9       ?GetCount@CBaseManager@@QAEKXZ 10001cf9 f   BaseManager.obj
 0001:00000d2e       ??_GCBaseManager@@UAEPAXI@Z 10001d2e f i BaseManager.obj
 0001:00000d2e       ??_ECBaseManager@@UAEPAXI@Z 10001d2e f i BaseManager.obj
 0001:00000d55       ??1?$hash_map@KPAXV?$hash_compare@KU?$less@K@std@@@stdext@@V?$allocator@U?$pair@$$CBKPAX@std@@@std@@@stdext@@QAE@XZ 10001d55 f i BaseManager.obj
 0001:00000d68       ?push_front@?$list@PAVCControlWZ@@V?$allocator@PAVCControlWZ@@@std@@@std@@QAEXABQAVCControlWZ@@@Z 10001d68 f i DialogWZ.obj
 0001:00000d68       ?push_front@?$list@PAXV?$allocator@PAX@std@@@std@@QAEXABQAX@Z 10001d68 f i CtrlListWZ.obj
 0001:00000d68       ?push_front@?$list@KV?$allocator@K@std@@@std@@QAEXABK@Z 10001d68 f i BaseManager.obj
 0001:00000dc9       ?push_back@?$list@PAXV?$allocator@PAX@std@@@std@@QAEXABQAX@Z 10001dc9 f i CtrlListWZ.obj
 0001:00000dc9       ?push_back@?$list@KV?$allocator@K@std@@@std@@QAEXABK@Z 10001dc9 f i BaseManager.obj
 0001:00000e22       ?remove@?$list@PAVCControlWZ@@V?$allocator@PAVCControlWZ@@@std@@@std@@QAEXABQAVCControlWZ@@@Z 10001e22 f i CtrlDxEdit.obj
 0001:00000e22       ?remove@?$list@PAXV?$allocator@PAX@std@@@std@@QAEXABQAX@Z 10001e22 f i CtrlListWZ.obj
 0001:00000e22       ?remove@?$list@KV?$allocator@K@std@@@std@@QAEXABK@Z 10001e22 f i BaseManager.obj
 0001:00000eb4       ??8?$_Const_iterator@$00@?$list@KV?$allocator@K@std@@@std@@QBE_NABV012@@Z 10001eb4 f i BaseManager.obj
 0001:00000eb4       ??8?$_Const_iterator@$00@?$list@UtagRECT@@V?$allocator@UtagRECT@@@std@@@std@@QBE_NABV012@@Z 10001eb4 f i DialogWZ.obj
 0001:00000eb4       ??8?$_Const_iterator@$00@?$list@U?$pair@$$CBKPAX@std@@V?$allocator@U?$pair@$$CBKPAX@std@@@2@@std@@QBE_NABV012@@Z 10001eb4 f i BaseManager.obj
 0001:00000eb4       ??8?$_Const_iterator@$00@?$list@PAVCControlWZ@@V?$allocator@PAVCControlWZ@@@std@@@std@@QBE_NABV012@@Z 10001eb4 f i CtrlDxEdit.obj
 0001:00000eb4       ??8?$_Const_iterator@$00@?$list@U?$pair@$$CBKV?$basic_string@DU?$char_traits@D@std@@V?$allocator@D@2@@std@@@std@@V?$allocator@U?$pair@$$CBKV?$basic_string@DU?$char_traits@D@std@@V?$allocator@D@2@@std@@@std@@@2@@std@@QBE_NABV012@@Z 10001eb4 f i StringManager.obj
 0001:00000eb4       ??8?$_Const_iterator@$00@?$list@PAXV?$allocator@PAX@std@@@std@@QBE_NABV012@@Z 10001eb4 f i CtrlListWZ.obj
 0001:00000f06       ??A?$hash_map@KPAXV?$hash_compare@KU?$less@K@std@@@stdext@@V?$allocator@U?$pair@$$CBKPAX@std@@@std@@@stdext@@QAEAAPAXABK@Z 10001f06 f i BaseManager.obj
 0001:00000f88       ??1?$_Hash@V?$_Hmap_traits@KPAXV?$hash_compare@KU?$less@K@std@@@stdext@@V?$allocator@U?$pair@$$CBKPAX@std@@@std@@$0A@@stdext@@@stdext@@QAE@XZ 10001f88 f i BaseManager.obj
 0001:00001020       ?end@?$_Hash@V?$_Hmap_traits@KPAXV?$hash_compare@KU?$less@K@std@@@stdext@@V?$allocator@U?$pair@$$CBKPAX@std@@@std@@$0A@@stdext@@@stdext@@QAE?AV?$_Iterator@$00@?$list@U?$pair@$$CBKPAX@std@@V?$allocator@U?$pair@$$CBKPAX@std@@@2@@std@@XZ 10002020 f i BaseManager.obj
 0001:00001020       ?end@?$_Hash@V?$_Hmap_traits@KV?$basic_string@DU?$char_traits@D@std@@V?$allocator@D@2@@std@@V?$hash_compare@KU?$less@K@std@@@stdext@@V?$allocator@U?$pair@$$CBKV?$basic_string@DU?$char_traits@D@std@@V?$allocator@D@2@@std@@@std@@@2@$0A@@stdext@@@stdext@@QAE?AV?$_Iterator@$00@?$list@U?$pair@$$CBKV?$basic_string@DU?$char_traits@D@std@@V?$allocator@D@2@@std@@@std@@V?$allocator@U?$pair@$$CBKV?$basic_string@DU?$char_traits@D@std@@V?$allocator@D@2@@std@@@std@@@2@@std@@XZ 10002020 f i StringManager.obj
 0001:0000106f       ?erase@?$_Hash@V?$_Hmap_traits@KPAXV?$hash_compare@KU?$less@K@std@@@stdext@@V?$allocator@U?$pair@$$CBKPAX@std@@@std@@$0A@@stdext@@@stdext@@QAE?AV?$_Iterator@$00@?$list@U?$pair@$$CBKPAX@std@@V?$allocator@U?$pair@$$CBKPAX@std@@@2@@std@@V?$_Const_iterator@$00@45@@Z 1000206f f i BaseManager.obj
 0001:000011b6       ?_Insert@?$list@KV?$allocator@K@std@@@std@@QAEXV?$_Const_iterator@$00@12@ABK@Z 100021b6 f i BaseManager.obj
 0001:000011b6       ?_Insert@?$list@PAXV?$allocator@PAX@std@@@std@@QAEXV?$_Const_iterator@$00@12@ABQAX@Z 100021b6 f i CtrlListWZ.obj
 0001:000011b6       ?_Insert@?$list@PAVCControlWZ@@V?$allocator@PAVCControlWZ@@@std@@@std@@QAEXV?$_Const_iterator@$00@12@ABQAVCControlWZ@@@Z 100021b6 f i DialogWZ.obj
 0001:00001204       ??F?$_Const_iterator@$00@?$list@KV?$allocator@K@std@@@std@@QAEAAV012@XZ 10002204 f i BaseManager.obj
 0001:00001204       ??F?$_Const_iterator@$00@?$list@U?$pair@$$CBKPAX@std@@V?$allocator@U?$pair@$$CBKPAX@std@@@2@@std@@QAEAAV012@XZ 10002204 f i BaseManager.obj
 0001:00001204       ??F?$_Const_iterator@$00@?$list@U?$pair@$$CBKV?$basic_string@DU?$char_traits@D@std@@V?$allocator@D@2@@std@@@std@@V?$allocator@U?$pair@$$CBKV?$basic_string@DU?$char_traits@D@std@@V?$allocator@D@2@@std@@@std@@@2@@std@@QAEAAV012@XZ 10002204 f i StringManager.obj
 0001:00001281       ??0?$_Hash@V?$_Hmap_traits@KPAXV?$hash_compare@KU?$less@K@std@@@stdext@@V?$allocator@U?$pair@$$CBKPAX@std@@@std@@$0A@@stdext@@@stdext@@QAE@ABV?$hash_compare@KU?$less@K@std@@@1@ABV?$allocator@U?$pair@$$CBKPAX@std@@@std@@@Z 10002281 f i BaseManager.obj
 0001:00001325       ?_Hashval@?$_Hash@V?$_Hmap_traits@KV?$basic_string@DU?$char_traits@D@std@@V?$allocator@D@2@@std@@V?$hash_compare@KU?$less@K@std@@@stdext@@V?$allocator@U?$pair@$$CBKV?$basic_string@DU?$char_traits@D@std@@V?$allocator@D@2@@std@@@std@@@2@$0A@@stdext@@@stdext@@IBEIABK@Z 10002325 f i StringManager.obj
 0001:00001325       ?_Hashval@?$_Hash@V?$_Hmap_traits@KPAXV?$hash_compare@KU?$less@K@std@@@stdext@@V?$allocator@U?$pair@$$CBKPAX@std@@@std@@$0A@@stdext@@@stdext@@IBEIABK@Z 10002325 f i BaseManager.obj
 0001:00001368       ??1?$list@U?$pair@$$CBKPAX@std@@V?$allocator@U?$pair@$$CBKPAX@std@@@2@@std@@QAE@XZ 10002368 f i BaseManager.obj
 0001:00001368       ??1?$list@KV?$allocator@K@std@@@std@@QAE@XZ 10002368 f i CtrlTabWZ.obj
 0001:00001368       ??1?$list@UtagRECT@@V?$allocator@UtagRECT@@@std@@@std@@QAE@XZ 10002368 f i DialogWZ.obj
 0001:000013be       ?_Buynode@?$list@PAVCControlWZ@@V?$allocator@PAVCControlWZ@@@std@@@std@@IAEPAU_Node@?$_List_nod@PAVCControlWZ@@V?$allocator@PAVCControlWZ@@@std@@@2@PAU342@0ABQAVCControlWZ@@@Z 100023be f i DialogWZ.obj
 0001:000013be       ?_Buynode@?$list@PAXV?$allocator@PAX@std@@@std@@IAEPAU_Node@?$_List_nod@PAXV?$allocator@PAX@std@@@2@PAU342@0ABQAX@Z 100023be f i CtrlListWZ.obj
 0001:000013be       ?_Buynode@?$list@KV?$allocator@K@std@@@std@@IAEPAU_Node@?$_List_nod@KV?$allocator@K@std@@@2@PAU342@0ABK@Z 100023be f i BaseManager.obj
 0001:000014c2       ?_Incsize@?$list@PAXV?$allocator@PAX@std@@@std@@IAEXI@Z 100024c2 f i CtrlListWZ.obj
 0001:000014c2       ?_Incsize@?$list@PAVCControlWZ@@V?$allocator@PAVCControlWZ@@@std@@@std@@IAEXI@Z 100024c2 f i DialogWZ.obj
 0001:000014c2       ?_Incsize@?$list@KV?$allocator@K@std@@@std@@IAEXI@Z 100024c2 f i BaseManager.obj
 0001:0000158c       ??0?$_Const_iterator@$00@?$list@U?$pair@$$CBKPAX@std@@V?$allocator@U?$pair@$$CBKPAX@std@@@2@@std@@QAE@PAU_Node@?$_List_nod@U?$pair@$$CBKPAX@std@@V?$allocator@U?$pair@$$CBKPAX@std@@@2@@2@PBV12@@Z 1000258c f i BaseManager.obj
 0001:0000158c       ??0?$_Const_iterator@$00@?$list@U?$pair@$$CBKV?$basic_string@DU?$char_traits@D@std@@V?$allocator@D@2@@std@@@std@@V?$allocator@U?$pair@$$CBKV?$basic_string@DU?$char_traits@D@std@@V?$allocator@D@2@@std@@@std@@@2@@std@@QAE@PAU_Node@?$_List_nod@U?$pair@$$CBKV?$basic_string@DU?$char_traits@D@std@@V?$allocator@D@2@@std@@@std@@V?$allocator@U?$pair@$$CBKV?$basic_string@DU?$char_traits@D@std@@V?$allocator@D@2@@std@@@std@@@2@@2@PBV12@@Z 1000258c f i StringManager.obj
 0001:0000158c       ??0?$_Const_iterator@$00@?$list@PAXV?$allocator@PAX@std@@@std@@QAE@PAU_Node@?$_List_nod@PAXV?$allocator@PAX@std@@@2@PBV12@@Z 1000258c f i CtrlListWZ.obj
 0001:0000158c       ??0?$_Const_iterator@$00@?$list@PAVCControlWZ@@V?$allocator@PAVCControlWZ@@@std@@@std@@QAE@PAU_Node@?$_List_nod@PAVCControlWZ@@V?$allocator@PAVCControlWZ@@@std@@@2@PBV12@@Z 1000258c f i DialogWZ.obj
 0001:0000158c       ??0?$_Const_iterator@$00@?$list@KV?$allocator@K@std@@@std@@QAE@PAU_Node@?$_List_nod@KV?$allocator@K@std@@@2@PBV12@@Z 1000258c f i BaseManager.obj
 0001:000015c7       ?_Insert@?$_Hash@V?$_Hmap_traits@KPAXV?$hash_compare@KU?$less@K@std@@@stdext@@V?$allocator@U?$pair@$$CBKPAX@std@@@std@@$0A@@stdext@@@stdext@@IAE?AU?$pair@V?$_Iterator@$00@?$list@U?$pair@$$CBKPAX@std@@V?$allocator@U?$pair@$$CBKPAX@std@@@2@@std@@_N@std@@ABU?$pair@$$CBKPAX@4@V?$_Iterator@$00@?$list@U?$pair@$$CBKPAX@std@@V?$allocator@U?$pair@$$CBKPAX@std@@@2@@4@@Z 100025c7 f i BaseManager.obj
 0001:00001af9       ??R?$hash_compare@KU?$less@K@std@@@stdext@@QBEIABK@Z 10002af9 f i BaseManager.obj
 0001:00001b60       ??0?$list@U?$pair@$$CBKPAX@std@@V?$allocator@U?$pair@$$CBKPAX@std@@@2@@std@@QAE@ABV?$allocator@U?$pair@$$CBKPAX@std@@@1@@Z 10002b60 f i BaseManager.obj
 0001:00001bd7       ?_Tidy@?$vector@U_List_position@?$_Hash@V?$_Hmap_traits@KV?$basic_string@DU?$char_traits@D@std@@V?$allocator@D@2@@std@@V?$hash_compare@KU?$less@K@std@@@stdext@@V?$allocator@U?$pair@$$CBKV?$basic_string@DU?$char_traits@D@std@@V?$allocator@D@2@@std@@@std@@@2@$0A@@stdext@@@stdext@@V?$allocator@U_List_position@?$_Hash@V?$_Hmap_traits@KV?$basic_string@DU?$char_traits@D@std@@V?$allocator@D@2@@std@@V?$hash_compare@KU?$less@K@std@@@stdext@@V?$allocator@U?$pair@$$CBKV?$basic_string@DU?$char_traits@D@std@@V?$allocator@D@2@@std@@@std@@@2@$0A@@stdext@@@stdext@@@std@@@std@@IAEXXZ 10002bd7 f i StringManager.obj
 0001:00001bd7       ?_Tidy@?$vector@U_List_position@?$_Hash@V?$_Hmap_traits@KPAXV?$hash_compare@KU?$less@K@std@@@stdext@@V?$allocator@U?$pair@$$CBKPAX@std@@@std@@$0A@@stdext@@@stdext@@V?$allocator@U_List_position@?$_Hash@V?$_Hmap_traits@KPAXV?$hash_compare@KU?$less@K@std@@@stdext@@V?$allocator@U?$pair@$$CBKPAX@std@@@std@@$0A@@stdext@@@stdext@@@std@@@std@@IAEXXZ 10002bd7 f i BaseManager.obj
 0001:00001c63       ??0length_error@std@@QAE@ABV01@@Z 10002c63 f i BaseManager.obj
 0001:00001c87       ?load_factor@?$_Hash@V?$_Hmap_traits@KV?$basic_string@DU?$char_traits@D@std@@V?$allocator@D@2@@std@@V?$hash_compare@KU?$less@K@std@@@stdext@@V?$allocator@U?$pair@$$CBKV?$basic_string@DU?$char_traits@D@std@@V?$allocator@D@2@@std@@@std@@@2@$0A@@stdext@@@stdext@@QBEMXZ 10002c87 f i StringManager.obj
 0001:00001c87       ?load_factor@?$_Hash@V?$_Hmap_traits@KPAXV?$hash_compare@KU?$less@K@std@@@stdext@@V?$allocator@U?$pair@$$CBKPAX@std@@@std@@$0A@@stdext@@@stdext@@QBEMXZ 10002c87 f i BaseManager.obj
 0001:00001cc6       ?_Reinsert@?$_Hash@V?$_Hmap_traits@KPAXV?$hash_compare@KU?$less@K@std@@@stdext@@V?$allocator@U?$pair@$$CBKPAX@std@@@std@@$0A@@stdext@@@stdext@@IAEXXZ 10002cc6 f i BaseManager.obj
 0001:00001dd0       ?splice@?$list@U?$pair@$$CBKPAX@std@@V?$allocator@U?$pair@$$CBKPAX@std@@@2@@std@@QAEXV?$_Const_iterator@$00@12@AAV12@0@Z 10002dd0 f i BaseManager.obj
 0001:00001e9a       ?_Buynode@?$list@U?$pair@$$CBKPAX@std@@V?$allocator@U?$pair@$$CBKPAX@std@@@2@@std@@IAEPAU_Node@?$_List_nod@U?$pair@$$CBKPAX@std@@V?$allocator@U?$pair@$$CBKPAX@std@@@2@@2@XZ 10002e9a f i BaseManager.obj
 0001:00001f7c       ??0?$_Const_iterator@$0A@@?$list@U?$pair@$$CBKPAX@std@@V?$allocator@U?$pair@$$CBKPAX@std@@@2@@std@@QAE@PAU_Node@?$_List_nod@U?$pair@$$CBKPAX@std@@V?$allocator@U?$pair@$$CBKPAX@std@@@2@@2@PBV12@@Z 10002f7c f i BaseManager.obj
 0001:00001f7c       ??0?$_Const_iterator@$0A@@?$list@U?$pair@$$CBKV?$basic_string@DU?$char_traits@D@std@@V?$allocator@D@2@@std@@@std@@V?$allocator@U?$pair@$$CBKV?$basic_string@DU?$char_traits@D@std@@V?$allocator@D@2@@std@@@std@@@2@@std@@QAE@PAU_Node@?$_List_nod@U?$pair@$$CBKV?$basic_string@DU?$char_traits@D@std@@V?$allocator@D@2@@std@@@std@@V?$allocator@U?$pair@$$CBKV?$basic_string@DU?$char_traits@D@std@@V?$allocator@D@2@@std@@@std@@@2@@2@PBV12@@Z 10002f7c f i StringManager.obj
 0001:00001fb6       ?_Insert@?$list@U?$pair@$$CBKPAX@std@@V?$allocator@U?$pair@$$CBKPAX@std@@@2@@std@@QAEXV?$_Const_iterator@$00@12@ABU?$pair@$$CBKPAX@2@@Z 10002fb6 f i BaseManager.obj
 0001:00002004       ?_Splice@?$list@U?$pair@$$CBKPAX@std@@V?$allocator@U?$pair@$$CBKPAX@std@@@2@@std@@QAEXV?$_Const_iterator@$00@12@AAV12@00I_N@Z 10003004 f i BaseManager.obj
 0001:0000218d       ?erase@?$list@U?$pair@$$CBKPAX@std@@V?$allocator@U?$pair@$$CBKPAX@std@@@2@@std@@QAE?AV?$_Iterator@$00@12@V?$_Const_iterator@$00@12@0@Z 1000318d f i BaseManager.obj
 0001:000022e5       ?_Buynode@?$list@U?$pair@$$CBKPAX@std@@V?$allocator@U?$pair@$$CBKPAX@std@@@2@@std@@IAEPAU_Node@?$_List_nod@U?$pair@$$CBKPAX@std@@V?$allocator@U?$pair@$$CBKPAX@std@@@2@@2@PAU342@0ABU?$pair@$$CBKPAX@2@@Z 100032e5 f i BaseManager.obj
 0001:000023ef       ?_Incsize@?$list@U?$pair@$$CBKPAX@std@@V?$allocator@U?$pair@$$CBKPAX@std@@@2@@std@@IAEXI@Z 100033ef f i BaseManager.obj
 0001:000024b9       ??8?$_Vector_const_iterator@U_List_position@?$_Hash@V?$_Hmap_traits@KV?$basic_string@DU?$char_traits@D@std@@V?$allocator@D@2@@std@@V?$hash_compare@KU?$less@K@std@@@stdext@@V?$allocator@U?$pair@$$CBKV?$basic_string@DU?$char_traits@D@std@@V?$allocator@D@2@@std@@@std@@@2@$0A@@stdext@@@stdext@@V?$allocator@U_List_position@?$_Hash@V?$_Hmap_traits@KV?$basic_string@DU?$char_traits@D@std@@V?$allocator@D@2@@std@@V?$hash_compare@KU?$less@K@std@@@stdext@@V?$allocator@U?$pair@$$CBKV?$basic_string@DU?$char_traits@D@std@@V?$allocator@D@2@@std@@@std@@@2@$0A@@stdext@@@stdext@@@std@@@std@@QBE_NABV01@@Z 100034b9 f i StringManager.obj
 0001:000024b9       ??8const_iterator@?$_Tree@V?$_Tmap_traits@V?$basic_string@DU?$char_traits@D@std@@V?$allocator@D@2@@std@@PAXU?$less@V?$basic_string@DU?$char_traits@D@std@@V?$allocator@D@2@@std@@@2@V?$allocator@U?$pair@$$CBV?$basic_string@DU?$char_traits@D@std@@V?$allocator@D@2@@std@@PAX@std@@@2@$00@std@@@std@@QBE_NABV012@@Z 100034b9 f i CtrlListWZ.obj
 0001:000024b9       ??8?$_Vector_const_iterator@KV?$allocator@K@std@@@std@@QBE_NABV01@@Z 100034b9 f i CtrlDxEdit.obj
 0001:000024b9       ??8const_iterator@?$_Tree@V?$_Tmap_traits@KPAXU?$less@K@std@@V?$allocator@U?$pair@$$CBKPAX@std@@@2@$0A@@std@@@std@@QBE_NABV012@@Z 100034b9 f i CtrlListWZ.obj
 0001:000024b9       ??8const_iterator@?$_Tree@V?$_Tmap_traits@KPAUCListSellData@CCtrlListWZ@@U?$less@K@std@@V?$allocator@U?$pair@$$CBKPAUCListSellData@CCtrlListWZ@@@std@@@4@$0A@@std@@@std@@QBE_NABV012@@Z 100034b9 f i CtrlListWZ.obj
 0001:000024b9       ??8const_iterator@?$_Tree@V?$_Tmap_traits@KKU?$less@K@std@@V?$allocator@U?$pair@$$CBKK@std@@@2@$0A@@std@@@std@@QBE_NABV012@@Z 100034b9 f i CtrlTabWZ.obj
 0001:000024b9       ??8?$_Vector_const_iterator@U_List_position@?$_Hash@V?$_Hmap_traits@KPAXV?$hash_compare@KU?$less@K@std@@@stdext@@V?$allocator@U?$pair@$$CBKPAX@std@@@std@@$0A@@stdext@@@stdext@@V?$allocator@U_List_position@?$_Hash@V?$_Hmap_traits@KPAXV?$hash_compare@KU?$less@K@std@@@stdext@@V?$allocator@U?$pair@$$CBKPAX@std@@@std@@$0A@@stdext@@@stdext@@@std@@@std@@QBE_NABV01@@Z 100034b9 f i BaseManager.obj
 0001:00002506       ??$_Allocate@U_Node@?$_List_nod@PAXV?$allocator@PAX@std@@@std@@@std@@YAPAU_Node@?$_List_nod@PAXV?$allocator@PAX@std@@@0@IPAU120@@Z 10003506 f i CtrlListWZ.obj
 0001:00002506       ??$_Allocate@U_Node@?$_List_nod@KV?$allocator@K@std@@@std@@@std@@YAPAU_Node@?$_List_nod@KV?$allocator@K@std@@@0@IPAU120@@Z 10003506 f i BaseManager.obj
 0001:00002506       ??$_Allocate@U_Node@?$_List_nod@PAVCControlWZ@@V?$allocator@PAVCControlWZ@@@std@@@std@@@std@@YAPAU_Node@?$_List_nod@PAVCControlWZ@@V?$allocator@PAVCControlWZ@@@std@@@0@IPAU120@@Z 10003506 f i DialogWZ.obj
 0001:00002559       ??1bad_alloc@std@@UAE@XZ   10003559 f i BaseManager.obj
 0001:00002573       ??_Ebad_alloc@std@@UAEPAXI@Z 10003573 f i BaseManager.obj
 0001:00002573       ??_Gbad_alloc@std@@UAEPAXI@Z 10003573 f i BaseManager.obj
 0001:000025a3       ??$_Allocate@U_Node@?$_List_nod@U?$pair@$$CBKPAX@std@@V?$allocator@U?$pair@$$CBKPAX@std@@@2@@std@@@std@@YAPAU_Node@?$_List_nod@U?$pair@$$CBKPAX@std@@V?$allocator@U?$pair@$$CBKPAX@std@@@2@@0@IPAU120@@Z 100035a3 f i BaseManager.obj
 0001:000025f6       ??$unchecked_copy@PAU_List_position@?$_Hash@V?$_Hmap_traits@KPAXV?$hash_compare@KU?$less@K@std@@@stdext@@V?$allocator@U?$pair@$$CBKPAX@std@@@std@@$0A@@stdext@@@stdext@@PAU123@@stdext@@YAPAU_List_position@?$_Hash@V?$_Hmap_traits@KPAXV?$hash_compare@KU?$less@K@std@@@stdext@@V?$allocator@U?$pair@$$CBKPAX@std@@@std@@$0A@@stdext@@@0@PAU120@00@Z 100035f6 f i BaseManager.obj
 0001:000025f6       ??$unchecked_copy@PAU_List_position@?$_Hash@V?$_Hmap_traits@KV?$basic_string@DU?$char_traits@D@std@@V?$allocator@D@2@@std@@V?$hash_compare@KU?$less@K@std@@@stdext@@V?$allocator@U?$pair@$$CBKV?$basic_string@DU?$char_traits@D@std@@V?$allocator@D@2@@std@@@std@@@2@$0A@@stdext@@@stdext@@PAU123@@stdext@@YAPAU_List_position@?$_Hash@V?$_Hmap_traits@KV?$basic_string@DU?$char_traits@D@std@@V?$allocator@D@2@@std@@V?$hash_compare@KU?$less@K@std@@@stdext@@V?$allocator@U?$pair@$$CBKV?$basic_string@DU?$char_traits@D@std@@V?$allocator@D@2@@std@@@std@@@2@$0A@@stdext@@@0@PAU120@00@Z 100035f6 f i StringManager.obj
 0001:00002691       ??1_Container_base_aux@std@@QAE@XZ 10003691 f i BaseManager.obj
 0001:00002691       ??1?$_Hmap_traits@KV?$basic_string@DU?$char_traits@D@std@@V?$allocator@D@2@@std@@V?$hash_compare@KU?$less@K@std@@@stdext@@V?$allocator@U?$pair@$$CBKV?$basic_string@DU?$char_traits@D@std@@V?$allocator@D@2@@std@@@std@@@2@$0A@@stdext@@QAE@XZ 10003691 f i StringManager.obj
 0001:00002691       ??1?$_Hmap_traits@KPAXV?$hash_compare@KU?$less@K@std@@@stdext@@V?$allocator@U?$pair@$$CBKPAX@std@@@std@@$0A@@stdext@@QAE@XZ 10003691 f i BaseManager.obj
 0001:00002691       ?ClearText@CCtrlBaseEdit@@UAEXXZ 10003691 f i CtrlDxEdit.obj
 0001:00002691       ?SetFocusWZ@CCtrlBaseEdit@@UAEXXZ 10003691 f i CtrlDxEdit.obj
 0001:0000269a       ??$_Umove@PAU_List_position@?$_Hash@V?$_Hmap_traits@KV?$basic_string@DU?$char_traits@D@std@@V?$allocator@D@2@@std@@V?$hash_compare@KU?$less@K@std@@@stdext@@V?$allocator@U?$pair@$$CBKV?$basic_string@DU?$char_traits@D@std@@V?$allocator@D@2@@std@@@std@@@2@$0A@@stdext@@@stdext@@@?$vector@U_List_position@?$_Hash@V?$_Hmap_traits@KV?$basic_string@DU?$char_traits@D@std@@V?$allocator@D@2@@std@@V?$hash_compare@KU?$less@K@std@@@stdext@@V?$allocator@U?$pair@$$CBKV?$basic_string@DU?$char_traits@D@std@@V?$allocator@D@2@@std@@@std@@@2@$0A@@stdext@@@stdext@@V?$allocator@U_List_position@?$_Hash@V?$_Hmap_traits@KV?$basic_string@DU?$char_traits@D@std@@V?$allocator@D@2@@std@@V?$hash_compare@KU?$less@K@std@@@stdext@@V?$allocator@U?$pair@$$CBKV?$basic_string@DU?$char_traits@D@std@@V?$allocator@D@2@@std@@@std@@@2@$0A@@stdext@@@stdext@@@std@@@std@@IAEPAU_List_position@?$_Hash@V?$_Hmap_traits@KV?$basic_string@DU?$char_traits@D@std@@V?$allocator@D@2@@std@@V?$hash_compare@KU?$less@K@std@@@stdext@@V?$allocator@U?$pair@$$CBKV?$basic_string@DU?$char_traits@D@std@@V?$allocator@D@2@@std@@@std@@@2@$0A@@stdext@@@stdext@@PAU234@00@Z 1000369a f i StringManager.obj
 0001:0000269a       ??$_Umove@PAU_List_position@?$_Hash@V?$_Hmap_traits@KPAXV?$hash_compare@KU?$less@K@std@@@stdext@@V?$allocator@U?$pair@$$CBKPAX@std@@@std@@$0A@@stdext@@@stdext@@@?$vector@U_List_position@?$_Hash@V?$_Hmap_traits@KPAXV?$hash_compare@KU?$less@K@std@@@stdext@@V?$allocator@U?$pair@$$CBKPAX@std@@@std@@$0A@@stdext@@@stdext@@V?$allocator@U_List_position@?$_Hash@V?$_Hmap_traits@KPAXV?$hash_compare@KU?$less@K@std@@@stdext@@V?$allocator@U?$pair@$$CBKPAX@std@@@std@@$0A@@stdext@@@stdext@@@std@@@std@@IAEPAU_List_position@?$_Hash@V?$_Hmap_traits@KPAXV?$hash_compare@KU?$less@K@std@@@stdext@@V?$allocator@U?$pair@$$CBKPAX@std@@@std@@$0A@@stdext@@@stdext@@PAU234@00@Z 1000369a f i BaseManager.obj
 0001:000026bf       ??$_Unchecked_move_backward@PAU_List_position@?$_Hash@V?$_Hmap_traits@KV?$basic_string@DU?$char_traits@D@std@@V?$allocator@D@2@@std@@V?$hash_compare@KU?$less@K@std@@@stdext@@V?$allocator@U?$pair@$$CBKV?$basic_string@DU?$char_traits@D@std@@V?$allocator@D@2@@std@@@std@@@2@$0A@@stdext@@@stdext@@PAU123@@stdext@@YAPAU_List_position@?$_Hash@V?$_Hmap_traits@KV?$basic_string@DU?$char_traits@D@std@@V?$allocator@D@2@@std@@V?$hash_compare@KU?$less@K@std@@@stdext@@V?$allocator@U?$pair@$$CBKV?$basic_string@DU?$char_traits@D@std@@V?$allocator@D@2@@std@@@std@@@2@$0A@@stdext@@@0@PAU120@00@Z 100036bf f i StringManager.obj
 0001:000026bf       ??$_Unchecked_move_backward@PAU_List_position@?$_Hash@V?$_Hmap_traits@KPAXV?$hash_compare@KU?$less@K@std@@@stdext@@V?$allocator@U?$pair@$$CBKPAX@std@@@std@@$0A@@stdext@@@stdext@@PAU123@@stdext@@YAPAU_List_position@?$_Hash@V?$_Hmap_traits@KPAXV?$hash_compare@KU?$less@K@std@@@stdext@@V?$allocator@U?$pair@$$CBKPAX@std@@@std@@$0A@@stdext@@@0@PAU120@00@Z 100036bf f i BaseManager.obj
 0001:000026fb       ??$_Insert@V?$_Const_iterator@$00@?$list@U?$pair@$$CBKPAX@std@@V?$allocator@U?$pair@$$CBKPAX@std@@@2@@std@@@?$list@U?$pair@$$CBKPAX@std@@V?$allocator@U?$pair@$$CBKPAX@std@@@2@@std@@QAEXV?$_Const_iterator@$00@01@00Uforward_iterator_tag@1@@Z 100036fb f i BaseManager.obj
 0001:00002810       ??0logic_error@std@@QAE@ABV?$basic_string@DU?$char_traits@D@std@@V?$allocator@D@2@@1@@Z 10003810 f i BaseManager.obj
 0001:0000288b       ??$_Unchecked_uninitialized_move@PAU_List_position@?$_Hash@V?$_Hmap_traits@KPAXV?$hash_compare@KU?$less@K@std@@@stdext@@V?$allocator@U?$pair@$$CBKPAX@std@@@std@@$0A@@stdext@@@stdext@@PAU123@V?$allocator@U_List_position@?$_Hash@V?$_Hmap_traits@KPAXV?$hash_compare@KU?$less@K@std@@@stdext@@V?$allocator@U?$pair@$$CBKPAX@std@@@std@@$0A@@stdext@@@stdext@@@std@@@stdext@@YAPAU_List_position@?$_Hash@V?$_Hmap_traits@KPAXV?$hash_compare@KU?$less@K@std@@@stdext@@V?$allocator@U?$pair@$$CBKPAX@std@@@std@@$0A@@stdext@@@0@PAU120@00AAV?$allocator@U_List_position@?$_Hash@V?$_Hmap_traits@KPAXV?$hash_compare@KU?$less@K@std@@@stdext@@V?$allocator@U?$pair@$$CBKPAX@std@@@std@@$0A@@stdext@@@stdext@@@std@@@Z 1000388b f i BaseManager.obj
 0001:0000288b       ??$_Unchecked_uninitialized_move@PAU_List_position@?$_Hash@V?$_Hmap_traits@KV?$basic_string@DU?$char_traits@D@std@@V?$allocator@D@2@@std@@V?$hash_compare@KU?$less@K@std@@@stdext@@V?$allocator@U?$pair@$$CBKV?$basic_string@DU?$char_traits@D@std@@V?$allocator@D@2@@std@@@std@@@2@$0A@@stdext@@@stdext@@PAU123@V?$allocator@U_List_position@?$_Hash@V?$_Hmap_traits@KV?$basic_string@DU?$char_traits@D@std@@V?$allocator@D@2@@std@@V?$hash_compare@KU?$less@K@std@@@stdext@@V?$allocator@U?$pair@$$CBKV?$basic_string@DU?$char_traits@D@std@@V?$allocator@D@2@@std@@@std@@@2@$0A@@stdext@@@stdext@@@std@@@stdext@@YAPAU_List_position@?$_Hash@V?$_Hmap_traits@KV?$basic_string@DU?$char_traits@D@std@@V?$allocator@D@2@@std@@V?$hash_compare@KU?$less@K@std@@@stdext@@V?$allocator@U?$pair@$$CBKV?$basic_string@DU?$char_traits@D@std@@V?$allocator@D@2@@std@@@std@@@2@$0A@@stdext@@@0@PAU120@00AAV?$allocator@U_List_position@?$_Hash@V?$_Hmap_traits@KV?$basic_string@DU?$char_traits@D@std@@V?$allocator@D@2@@std@@V?$hash_compare@KU?$less@K@std@@@stdext@@V?$allocator@U?$pair@$$CBKV?$basic_string@DU?$char_traits@D@std@@V?$allocator@D@2@@std@@@std@@@2@$0A@@stdext@@@stdext@@@std@@@Z 1000388b f i StringManager.obj
 0001:000028fd       ?what@logic_error@std@@UBEPBDXZ 100038fd f i BaseManager.obj
 0001:00002931       ??_Glogic_error@std@@UAEPAXI@Z 10003931 f i BaseManager.obj
 0001:00002931       ??_Elogic_error@std@@UAEPAXI@Z 10003931 f i BaseManager.obj
 0001:0000295a       ??1logic_error@std@@UAE@XZ 1000395a f i BaseManager.obj
 0001:00002985       ??$_Move_backward_opt@PAU_List_position@?$_Hash@V?$_Hmap_traits@KV?$basic_string@DU?$char_traits@D@std@@V?$allocator@D@2@@std@@V?$hash_compare@KU?$less@K@std@@@stdext@@V?$allocator@U?$pair@$$CBKV?$basic_string@DU?$char_traits@D@std@@V?$allocator@D@2@@std@@@std@@@2@$0A@@stdext@@@stdext@@PAU123@Urandom_access_iterator_tag@std@@U_Undefined_move_tag@5@@std@@YAPAU_List_position@?$_Hash@V?$_Hmap_traits@KV?$basic_string@DU?$char_traits@D@std@@V?$allocator@D@2@@std@@V?$hash_compare@KU?$less@K@std@@@stdext@@V?$allocator@U?$pair@$$CBKV?$basic_string@DU?$char_traits@D@std@@V?$allocator@D@2@@std@@@std@@@2@$0A@@stdext@@@stdext@@PAU123@00Urandom_access_iterator_tag@0@U_Undefined_move_tag@0@U_Range_checked_iterator_tag@0@@Z 10003985 f i StringManager.obj
 0001:00002985       ??$_Move_backward_opt@PAU_List_position@?$_Hash@V?$_Hmap_traits@KPAXV?$hash_compare@KU?$less@K@std@@@stdext@@V?$allocator@U?$pair@$$CBKPAX@std@@@std@@$0A@@stdext@@@stdext@@PAU123@Urandom_access_iterator_tag@std@@U_Undefined_move_tag@5@@std@@YAPAU_List_position@?$_Hash@V?$_Hmap_traits@KPAXV?$hash_compare@KU?$less@K@std@@@stdext@@V?$allocator@U?$pair@$$CBKPAX@std@@@std@@$0A@@stdext@@@stdext@@PAU123@00Urandom_access_iterator_tag@0@U_Undefined_move_tag@0@U_Range_checked_iterator_tag@0@@Z 10003985 f i BaseManager.obj
 0001:00002a14       ??1length_error@std@@UAE@XZ 10003a14 f i BaseManager.obj
 0001:00002a30       ??_Glength_error@std@@UAEPAXI@Z 10003a30 f i BaseManager.obj
 0001:00002a30       ??_Elength_error@std@@UAEPAXI@Z 10003a30 f i BaseManager.obj
 0001:00002a62       ??$_Uninit_copy@PAU_List_position@?$_Hash@V?$_Hmap_traits@KPAXV?$hash_compare@KU?$less@K@std@@@stdext@@V?$allocator@U?$pair@$$CBKPAX@std@@@std@@$0A@@stdext@@@stdext@@PAU123@V?$allocator@U_List_position@?$_Hash@V?$_Hmap_traits@KPAXV?$hash_compare@KU?$less@K@std@@@stdext@@V?$allocator@U?$pair@$$CBKPAX@std@@@std@@$0A@@stdext@@@stdext@@@std@@@std@@YAPAU_List_position@?$_Hash@V?$_Hmap_traits@KPAXV?$hash_compare@KU?$less@K@std@@@stdext@@V?$allocator@U?$pair@$$CBKPAX@std@@@std@@$0A@@stdext@@@stdext@@PAU123@00AAV?$allocator@U_List_position@?$_Hash@V?$_Hmap_traits@KPAXV?$hash_compare@KU?$less@K@std@@@stdext@@V?$allocator@U?$pair@$$CBKPAX@std@@@std@@$0A@@stdext@@@stdext@@@0@U_Nonscalar_ptr_iterator_tag@0@U_Range_checked_iterator_tag@0@@Z 10003a62 f i BaseManager.obj
 0001:00002a62       ??$_Uninit_copy@PAU_List_position@?$_Hash@V?$_Hmap_traits@KV?$basic_string@DU?$char_traits@D@std@@V?$allocator@D@2@@std@@V?$hash_compare@KU?$less@K@std@@@stdext@@V?$allocator@U?$pair@$$CBKV?$basic_string@DU?$char_traits@D@std@@V?$allocator@D@2@@std@@@std@@@2@$0A@@stdext@@@stdext@@PAU123@V?$allocator@U_List_position@?$_Hash@V?$_Hmap_traits@KV?$basic_string@DU?$char_traits@D@std@@V?$allocator@D@2@@std@@V?$hash_compare@KU?$less@K@std@@@stdext@@V?$allocator@U?$pair@$$CBKV?$basic_string@DU?$char_traits@D@std@@V?$allocator@D@2@@std@@@std@@@2@$0A@@stdext@@@stdext@@@std@@@std@@YAPAU_List_position@?$_Hash@V?$_Hmap_traits@KV?$basic_string@DU?$char_traits@D@std@@V?$allocator@D@2@@std@@V?$hash_compare@KU?$less@K@std@@@stdext@@V?$allocator@U?$pair@$$CBKV?$basic_string@DU?$char_traits@D@std@@V?$allocator@D@2@@std@@@std@@@2@$0A@@stdext@@@stdext@@PAU123@00AAV?$allocator@U_List_position@?$_Hash@V?$_Hmap_traits@KV?$basic_string@DU?$char_traits@D@std@@V?$allocator@D@2@@std@@V?$hash_compare@KU?$less@K@std@@@stdext@@V?$allocator@U?$pair@$$CBKV?$basic_string@DU?$char_traits@D@std@@V?$allocator@D@2@@std@@@std@@@2@$0A@@stdext@@@stdext@@@0@U_Nonscalar_ptr_iterator_tag@0@U_Range_checked_iterator_tag@0@@Z 10003a62 f i StringManager.obj
 0001:00002b25       ??0logic_error@std@@QAE@ABV01@@Z 10003b25 f i BaseManager.obj
 0001:00002ba7       ??0?$basic_string@DU?$char_traits@D@std@@V?$allocator@D@2@@std@@QAE@PBD@Z 10003ba7 f i BaseManager.obj
 0001:00002bfe       ?assign@?$basic_string@DU?$char_traits@D@std@@V?$allocator@D@2@@std@@QAEAAV12@ABV12@II@Z 10003bfe f i BaseManager.obj
 0001:00002d21       ?_Tidy@?$basic_string@DU?$char_traits@D@std@@V?$allocator@D@2@@std@@IAEX_NI@Z 10003d21 f i BaseManager.obj
 0001:00002dc4       ?assign@?$basic_string@DU?$char_traits@D@std@@V?$allocator@D@2@@std@@QAEAAV12@PBDI@Z 10003dc4 f i BaseManager.obj
 0001:00002ea6       ?erase@?$basic_string@DU?$char_traits@D@std@@V?$allocator@D@2@@std@@QAEAAV12@II@Z 10003ea6 f i BaseManager.obj
 0001:00002faa       ?_Grow@?$basic_string@DU?$char_traits@D@std@@V?$allocator@D@2@@std@@IAE_NI_N@Z 10003faa f i BaseManager.obj
 0001:0000308b       ?_Copy@?$basic_string@DU?$char_traits@D@std@@V?$allocator@D@2@@std@@IAEXII@Z 1000408b f i BaseManager.obj
 0001:000032b7       ?_Inside@?$basic_string@DU?$char_traits@D@std@@V?$allocator@D@2@@std@@IAE_NPBD@Z 100042b7 f i BaseManager.obj
 0001:00003322       ??$_Allocate@D@std@@YAPADIPAD@Z 10004322 f i BaseManager.obj
 0001:00003371       ??0bad_alloc@std@@QAE@ABV01@@Z 10004371 f i BaseManager.obj
 0001:00003393       ??0CStringManager@@QAE@XZ  10004393 f   StringManager.obj
 0001:00003422       ??1CStringManager@@QAE@XZ  10004422 f   StringManager.obj
 0001:00003435       ?OnCreate@CStringManager@@QAEXXZ 10004435 f   StringManager.obj
 0001:00003461       ?OnDestory@CStringManager@@QAEXXZ 10004461 f   StringManager.obj
 0001:00003472       ?OnRelease@CStringManager@@QAEXXZ 10004472 f   StringManager.obj
 0001:000034a9       ?CloseBuffer@CStringManager@@QAEXXZ 100044a9 f   StringManager.obj
 0001:000034e3       ?_clearToken@CStringManager@@AAEXXZ 100044e3 f   StringManager.obj
 0001:000034f3       ?_getchar@CStringManager@@AAEDPAK@Z 100044f3 f   StringManager.obj
 0001:0000354b       ?_getcurchar@CStringManager@@AAEDPAK@Z 1000454b f   StringManager.obj
 0001:00003591       ?_getcurchar@CStringManager@@AAEDK@Z 10004591 f   StringManager.obj
 0001:000035c4       ?_rewind@CStringManager@@AAEXHPAK@Z 100045c4 f   StringManager.obj
 0001:000035eb       ?_isspace@CStringManager@@AAEHD@Z 100045eb f   StringManager.obj
 0001:00003621       ?_isnewline@CStringManager@@AAEHD@Z 10004621 f   StringManager.obj
 0001:00003645       ?_isnumber@CStringManager@@AAE_ND@Z 10004645 f   StringManager.obj
 0001:0000366b       ?_skipComment@CStringManager@@AAEDPAK@Z 1000466b f   StringManager.obj
 0001:0000376d       ?_getNextNewLine@CStringManager@@AAE?AW4eSTRINGTABLE_TOKEN_TYPE@@XZ 1000476d f   StringManager.obj
 0001:00003811       ?_getNextWhiteSpace@CStringManager@@AAE?AW4eSTRINGTABLE_TOKEN_TYPE@@XZ 10004811 f   StringManager.obj
 0001:000038b5       ?FindStr@@YAHHPAD0@Z       100048b5 f   StringManager.obj
 0001:00003954       ?GetLine@@YAHHPAD0@Z       10004954 f   StringManager.obj
 0001:00003a11       ?OnLoad@CStringManager@@QAE_NPBDW4ENUM_LOAD_UITYPE@@@Z 10004a11 f   StringManager.obj
 0001:00003e39       ?OnSave@CStringManager@@QAE_NPBD@Z 10004e39 f   StringManager.obj
 0001:00003fe3       ?FindString@CStringManager@@QAE_NKPAD@Z 10004fe3 f   StringManager.obj
 0001:00004157       ?FindString@CStringManager@@QAEABV?$basic_string@DU?$char_traits@D@std@@V?$allocator@D@2@@std@@K@Z 10005157 f   StringManager.obj
 0001:00004212       ?AddString@CStringManager@@QAE_NKPAD@Z 10005212 f   StringManager.obj
 0001:0000426f       ?RemoveString@CStringManager@@QAE_NK@Z 1000526f f   StringManager.obj
 0001:000042d9       ?GetIndexValue@CStringManager@@QAE_NHPAKPAD@Z 100052d9 f   StringManager.obj
 0001:00004416       ??1?$hash_map@KV?$basic_string@DU?$char_traits@D@std@@V?$allocator@D@2@@std@@V?$hash_compare@KU?$less@K@std@@@stdext@@V?$allocator@U?$pair@$$CBKV?$basic_string@DU?$char_traits@D@std@@V?$allocator@D@2@@std@@@std@@@2@@stdext@@QAE@XZ 10005416 f i StringManager.obj
 0001:00004429       ??A?$hash_map@KV?$basic_string@DU?$char_traits@D@std@@V?$allocator@D@2@@std@@V?$hash_compare@KU?$less@K@std@@@stdext@@V?$allocator@U?$pair@$$CBKV?$basic_string@DU?$char_traits@D@std@@V?$allocator@D@2@@std@@@std@@@2@@stdext@@QAEAAV?$basic_string@DU?$char_traits@D@std@@V?$allocator@D@2@@std@@ABK@Z 10005429 f i StringManager.obj
 0001:00004563       ??1?$_Hash@V?$_Hmap_traits@KV?$basic_string@DU?$char_traits@D@std@@V?$allocator@D@2@@std@@V?$hash_compare@KU?$less@K@std@@@stdext@@V?$allocator@U?$pair@$$CBKV?$basic_string@DU?$char_traits@D@std@@V?$allocator@D@2@@std@@@std@@@2@$0A@@stdext@@@stdext@@QAE@XZ 10005563 f i StringManager.obj
 0001:000045fb       ?erase@?$_Hash@V?$_Hmap_traits@KV?$basic_string@DU?$char_traits@D@std@@V?$allocator@D@2@@std@@V?$hash_compare@KU?$less@K@std@@@stdext@@V?$allocator@U?$pair@$$CBKV?$basic_string@DU?$char_traits@D@std@@V?$allocator@D@2@@std@@@std@@@2@$0A@@stdext@@@stdext@@QAE?AV?$_Iterator@$00@?$list@U?$pair@$$CBKV?$basic_string@DU?$char_traits@D@std@@V?$allocator@D@2@@std@@@std@@V?$allocator@U?$pair@$$CBKV?$basic_string@DU?$char_traits@D@std@@V?$allocator@D@2@@std@@@std@@@2@@std@@V?$_Const_iterator@$00@45@@Z 100055fb f i StringManager.obj
 0001:00004742       ??0?$_Hash@V?$_Hmap_traits@KV?$basic_string@DU?$char_traits@D@std@@V?$allocator@D@2@@std@@V?$hash_compare@KU?$less@K@std@@@stdext@@V?$allocator@U?$pair@$$CBKV?$basic_string@DU?$char_traits@D@std@@V?$allocator@D@2@@std@@@std@@@2@$0A@@stdext@@@stdext@@QAE@ABV?$hash_compare@KU?$less@K@std@@@1@ABV?$allocator@U?$pair@$$CBKV?$basic_string@DU?$char_traits@D@std@@V?$allocator@D@2@@std@@@std@@@std@@@Z 10005742 f i StringManager.obj
 0001:000047e6       ?lower_bound@?$_Hash@V?$_Hmap_traits@KPAXV?$hash_compare@KU?$less@K@std@@@stdext@@V?$allocator@U?$pair@$$CBKPAX@std@@@std@@$0A@@stdext@@@stdext@@QAE?AV?$_Iterator@$00@?$list@U?$pair@$$CBKPAX@std@@V?$allocator@U?$pair@$$CBKPAX@std@@@2@@std@@ABK@Z 100057e6 f i BaseManager.obj
 0001:000047e6       ?lower_bound@?$_Hash@V?$_Hmap_traits@KV?$basic_string@DU?$char_traits@D@std@@V?$allocator@D@2@@std@@V?$hash_compare@KU?$less@K@std@@@stdext@@V?$allocator@U?$pair@$$CBKV?$basic_string@DU?$char_traits@D@std@@V?$allocator@D@2@@std@@@std@@@2@$0A@@stdext@@@stdext@@QAE?AV?$_Iterator@$00@?$list@U?$pair@$$CBKV?$basic_string@DU?$char_traits@D@std@@V?$allocator@D@2@@std@@@std@@V?$allocator@U?$pair@$$CBKV?$basic_string@DU?$char_traits@D@std@@V?$allocator@D@2@@std@@@std@@@2@@std@@ABK@Z 100057e6 f i StringManager.obj
 0001:00004959       ?_Init@?$_Hash@V?$_Hmap_traits@KPAXV?$hash_compare@KU?$less@K@std@@@stdext@@V?$allocator@U?$pair@$$CBKPAX@std@@@std@@$0A@@stdext@@@stdext@@IAEXI@Z 10005959 f i BaseManager.obj
 0001:00004959       ?_Init@?$_Hash@V?$_Hmap_traits@KV?$basic_string@DU?$char_traits@D@std@@V?$allocator@D@2@@std@@V?$hash_compare@KU?$less@K@std@@@stdext@@V?$allocator@U?$pair@$$CBKV?$basic_string@DU?$char_traits@D@std@@V?$allocator@D@2@@std@@@std@@@2@$0A@@stdext@@@stdext@@IAEXI@Z 10005959 f i StringManager.obj
 0001:000049a6       ??1?$list@U?$pair@$$CBKV?$basic_string@DU?$char_traits@D@std@@V?$allocator@D@2@@std@@@std@@V?$allocator@U?$pair@$$CBKV?$basic_string@DU?$char_traits@D@std@@V?$allocator@D@2@@std@@@std@@@2@@std@@QAE@XZ 100059a6 f i StringManager.obj
 0001:000049fc       ?erase@?$list@U?$pair@$$CBKV?$basic_string@DU?$char_traits@D@std@@V?$allocator@D@2@@std@@@std@@V?$allocator@U?$pair@$$CBKV?$basic_string@DU?$char_traits@D@std@@V?$allocator@D@2@@std@@@std@@@2@@std@@QAE?AV?$_Iterator@$00@12@V?$_Const_iterator@$00@12@@Z 100059fc f i StringManager.obj
 0001:00004ab7       ?clear@?$list@U?$pair@$$CBKV?$basic_string@DU?$char_traits@D@std@@V?$allocator@D@2@@std@@@std@@V?$allocator@U?$pair@$$CBKV?$basic_string@DU?$char_traits@D@std@@V?$allocator@D@2@@std@@@std@@@2@@std@@QAEXXZ 10005ab7 f i StringManager.obj
 0001:00004b2d       ??1?$vector@U_List_position@?$_Hash@V?$_Hmap_traits@KPAXV?$hash_compare@KU?$less@K@std@@@stdext@@V?$allocator@U?$pair@$$CBKPAX@std@@@std@@$0A@@stdext@@@stdext@@V?$allocator@U_List_position@?$_Hash@V?$_Hmap_traits@KPAXV?$hash_compare@KU?$less@K@std@@@stdext@@V?$allocator@U?$pair@$$CBKPAX@std@@@std@@$0A@@stdext@@@stdext@@@std@@@std@@QAE@XZ 10005b2d f i BaseManager.obj
 0001:00004b2d       ??1?$vector@U_List_position@?$_Hash@V?$_Hmap_traits@KV?$basic_string@DU?$char_traits@D@std@@V?$allocator@D@2@@std@@V?$hash_compare@KU?$less@K@std@@@stdext@@V?$allocator@U?$pair@$$CBKV?$basic_string@DU?$char_traits@D@std@@V?$allocator@D@2@@std@@@std@@@2@$0A@@stdext@@@stdext@@V?$allocator@U_List_position@?$_Hash@V?$_Hmap_traits@KV?$basic_string@DU?$char_traits@D@std@@V?$allocator@D@2@@std@@V?$hash_compare@KU?$less@K@std@@@stdext@@V?$allocator@U?$pair@$$CBKV?$basic_string@DU?$char_traits@D@std@@V?$allocator@D@2@@std@@@std@@@2@$0A@@stdext@@@stdext@@@std@@@std@@QAE@XZ 10005b2d f i StringManager.obj
 0001:00004b83       ??0_List_position@?$_Hash@V?$_Hmap_traits@KV?$basic_string@DU?$char_traits@D@std@@V?$allocator@D@2@@std@@V?$hash_compare@KU?$less@K@std@@@stdext@@V?$allocator@U?$pair@$$CBKV?$basic_string@DU?$char_traits@D@std@@V?$allocator@D@2@@std@@@std@@@2@$0A@@stdext@@@stdext@@QAE@V?$_Iterator@$00@?$list@U?$pair@$$CBKV?$basic_string@DU?$char_traits@D@std@@V?$allocator@D@2@@std@@@std@@V?$allocator@U?$pair@$$CBKV?$basic_string@DU?$char_traits@D@std@@V?$allocator@D@2@@std@@@std@@@2@@std@@@Z 10005b83 f i StringManager.obj
 0001:00004b83       ??0_List_position@?$_Hash@V?$_Hmap_traits@KPAXV?$hash_compare@KU?$less@K@std@@@stdext@@V?$allocator@U?$pair@$$CBKPAX@std@@@std@@$0A@@stdext@@@stdext@@QAE@V?$_Iterator@$00@?$list@U?$pair@$$CBKPAX@std@@V?$allocator@U?$pair@$$CBKPAX@std@@@2@@std@@@Z 10005b83 f i BaseManager.obj
 0001:00004bdf       ?_Insert@?$_Hash@V?$_Hmap_traits@KV?$basic_string@DU?$char_traits@D@std@@V?$allocator@D@2@@std@@V?$hash_compare@KU?$less@K@std@@@stdext@@V?$allocator@U?$pair@$$CBKV?$basic_string@DU?$char_traits@D@std@@V?$allocator@D@2@@std@@@std@@@2@$0A@@stdext@@@stdext@@IAE?AU?$pair@V?$_Iterator@$00@?$list@U?$pair@$$CBKV?$basic_string@DU?$char_traits@D@std@@V?$allocator@D@2@@std@@@std@@V?$allocator@U?$pair@$$CBKV?$basic_string@DU?$char_traits@D@std@@V?$allocator@D@2@@std@@@std@@@2@@std@@_N@std@@ABU?$pair@$$CBKV?$basic_string@DU?$char_traits@D@std@@V?$allocator@D@2@@std@@@4@V?$_Iterator@$00@?$list@U?$pair@$$CBKV?$basic_string@DU?$char_traits@D@std@@V?$allocator@D@2@@std@@@std@@V?$allocator@U?$pair@$$CBKV?$basic_string@DU?$char_traits@D@std@@V?$allocator@D@2@@std@@@std@@@2@@4@@Z 10005bdf f i StringManager.obj
 0001:00005111       ??0?$list@U?$pair@$$CBKV?$basic_string@DU?$char_traits@D@std@@V?$allocator@D@2@@std@@@std@@V?$allocator@U?$pair@$$CBKV?$basic_string@DU?$char_traits@D@std@@V?$allocator@D@2@@std@@@std@@@2@@std@@QAE@ABV?$allocator@U?$pair@$$CBKV?$basic_string@DU?$char_traits@D@std@@V?$allocator@D@2@@std@@@std@@@1@@Z 10006111 f i StringManager.obj
 0001:00005188       ?_Tidy@?$list@U?$pair@$$CBKV?$basic_string@DU?$char_traits@D@std@@V?$allocator@D@2@@std@@@std@@V?$allocator@U?$pair@$$CBKV?$basic_string@DU?$char_traits@D@std@@V?$allocator@D@2@@std@@@std@@@2@@std@@IAEXXZ 10006188 f i StringManager.obj
 0001:000051bd       ??0?$vector@U_List_position@?$_Hash@V?$_Hmap_traits@KPAXV?$hash_compare@KU?$less@K@std@@@stdext@@V?$allocator@U?$pair@$$CBKPAX@std@@@std@@$0A@@stdext@@@stdext@@V?$allocator@U_List_position@?$_Hash@V?$_Hmap_traits@KPAXV?$hash_compare@KU?$less@K@std@@@stdext@@V?$allocator@U?$pair@$$CBKPAX@std@@@std@@$0A@@stdext@@@stdext@@@std@@@std@@QAE@ABV?$allocator@U_List_position@?$_Hash@V?$_Hmap_traits@KPAXV?$hash_compare@KU?$less@K@std@@@stdext@@V?$allocator@U?$pair@$$CBKPAX@std@@@std@@$0A@@stdext@@@stdext@@@1@@Z 100061bd f i BaseManager.obj
 0001:000051bd       ??0?$vector@U_List_position@?$_Hash@V?$_Hmap_traits@KV?$basic_string@DU?$char_traits@D@std@@V?$allocator@D@2@@std@@V?$hash_compare@KU?$less@K@std@@@stdext@@V?$allocator@U?$pair@$$CBKV?$basic_string@DU?$char_traits@D@std@@V?$allocator@D@2@@std@@@std@@@2@$0A@@stdext@@@stdext@@V?$allocator@U_List_position@?$_Hash@V?$_Hmap_traits@KV?$basic_string@DU?$char_traits@D@std@@V?$allocator@D@2@@std@@V?$hash_compare@KU?$less@K@std@@@stdext@@V?$allocator@U?$pair@$$CBKV?$basic_string@DU?$char_traits@D@std@@V?$allocator@D@2@@std@@@std@@@2@$0A@@stdext@@@stdext@@@std@@@std@@QAE@ABV?$allocator@U_List_position@?$_Hash@V?$_Hmap_traits@KV?$basic_string@DU?$char_traits@D@std@@V?$allocator@D@2@@std@@V?$hash_compare@KU?$less@K@std@@@stdext@@V?$allocator@U?$pair@$$CBKV?$basic_string@DU?$char_traits@D@std@@V?$allocator@D@2@@std@@@std@@@2@$0A@@stdext@@@stdext@@@1@@Z 100061bd f i StringManager.obj
 0001:00005241       ?_Get_iter@_List_position@?$_Hash@V?$_Hmap_traits@KPAXV?$hash_compare@KU?$less@K@std@@@stdext@@V?$allocator@U?$pair@$$CBKPAX@std@@@std@@$0A@@stdext@@@stdext@@QBE?AV?$_Iterator@$00@?$list@U?$pair@$$CBKPAX@std@@V?$allocator@U?$pair@$$CBKPAX@std@@@2@@std@@ABV56@@Z 10006241 f i BaseManager.obj
 0001:00005241       ?_Get_iter@_List_position@?$_Hash@V?$_Hmap_traits@KV?$basic_string@DU?$char_traits@D@std@@V?$allocator@D@2@@std@@V?$hash_compare@KU?$less@K@std@@@stdext@@V?$allocator@U?$pair@$$CBKV?$basic_string@DU?$char_traits@D@std@@V?$allocator@D@2@@std@@@std@@@2@$0A@@stdext@@@stdext@@QBE?AV?$_Iterator@$00@?$list@U?$pair@$$CBKV?$basic_string@DU?$char_traits@D@std@@V?$allocator@D@2@@std@@@std@@V?$allocator@U?$pair@$$CBKV?$basic_string@DU?$char_traits@D@std@@V?$allocator@D@2@@std@@@std@@@2@@std@@ABV56@@Z 10006241 f i StringManager.obj
 0001:00005286       ?_Reinsert@?$_Hash@V?$_Hmap_traits@KV?$basic_string@DU?$char_traits@D@std@@V?$allocator@D@2@@std@@V?$hash_compare@KU?$less@K@std@@@stdext@@V?$allocator@U?$pair@$$CBKV?$basic_string@DU?$char_traits@D@std@@V?$allocator@D@2@@std@@@std@@@2@$0A@@stdext@@@stdext@@IAEXXZ 10006286 f i StringManager.obj
 0001:00005390       ?splice@?$list@U?$pair@$$CBKV?$basic_string@DU?$char_traits@D@std@@V?$allocator@D@2@@std@@@std@@V?$allocator@U?$pair@$$CBKV?$basic_string@DU?$char_traits@D@std@@V?$allocator@D@2@@std@@@std@@@2@@std@@QAEXV?$_Const_iterator@$00@12@AAV12@0@Z 10006390 f i StringManager.obj
 0001:0000545a       ?_Buynode@?$list@U?$pair@$$CBKV?$basic_string@DU?$char_traits@D@std@@V?$allocator@D@2@@std@@@std@@V?$allocator@U?$pair@$$CBKV?$basic_string@DU?$char_traits@D@std@@V?$allocator@D@2@@std@@@std@@@2@@std@@IAEPAU_Node@?$_List_nod@U?$pair@$$CBKV?$basic_string@DU?$char_traits@D@std@@V?$allocator@D@2@@std@@@std@@V?$allocator@U?$pair@$$CBKV?$basic_string@DU?$char_traits@D@std@@V?$allocator@D@2@@std@@@std@@@2@@2@XZ 1000645a f i StringManager.obj
 0001:0000553c       ?_Assign_n@?$vector@U_List_position@?$_Hash@V?$_Hmap_traits@KPAXV?$hash_compare@KU?$less@K@std@@@stdext@@V?$allocator@U?$pair@$$CBKPAX@std@@@std@@$0A@@stdext@@@stdext@@V?$allocator@U_List_position@?$_Hash@V?$_Hmap_traits@KPAXV?$hash_compare@KU?$less@K@std@@@stdext@@V?$allocator@U?$pair@$$CBKPAX@std@@@std@@$0A@@stdext@@@stdext@@@std@@@std@@IAEXIABU_List_position@?$_Hash@V?$_Hmap_traits@KPAXV?$hash_compare@KU?$less@K@std@@@stdext@@V?$allocator@U?$pair@$$CBKPAX@std@@@std@@$0A@@stdext@@@stdext@@@Z 1000653c f i BaseManager.obj
 0001:0000553c       ?_Assign_n@?$vector@U_List_position@?$_Hash@V?$_Hmap_traits@KV?$basic_string@DU?$char_traits@D@std@@V?$allocator@D@2@@std@@V?$hash_compare@KU?$less@K@std@@@stdext@@V?$allocator@U?$pair@$$CBKV?$basic_string@DU?$char_traits@D@std@@V?$allocator@D@2@@std@@@std@@@2@$0A@@stdext@@@stdext@@V?$allocator@U_List_position@?$_Hash@V?$_Hmap_traits@KV?$basic_string@DU?$char_traits@D@std@@V?$allocator@D@2@@std@@V?$hash_compare@KU?$less@K@std@@@stdext@@V?$allocator@U?$pair@$$CBKV?$basic_string@DU?$char_traits@D@std@@V?$allocator@D@2@@std@@@std@@@2@$0A@@stdext@@@stdext@@@std@@@std@@IAEXIABU_List_position@?$_Hash@V?$_Hmap_traits@KV?$basic_string@DU?$char_traits@D@std@@V?$allocator@D@2@@std@@V?$hash_compare@KU?$less@K@std@@@stdext@@V?$allocator@U?$pair@$$CBKV?$basic_string@DU?$char_traits@D@std@@V?$allocator@D@2@@std@@@std@@@2@$0A@@stdext@@@stdext@@@Z 1000653c f i StringManager.obj
 0001:000055c9       ?_Buy@?$vector@U_List_position@?$_Hash@V?$_Hmap_traits@KPAXV?$hash_compare@KU?$less@K@std@@@stdext@@V?$allocator@U?$pair@$$CBKPAX@std@@@std@@$0A@@stdext@@@stdext@@V?$allocator@U_List_position@?$_Hash@V?$_Hmap_traits@KPAXV?$hash_compare@KU?$less@K@std@@@stdext@@V?$allocator@U?$pair@$$CBKPAX@std@@@std@@$0A@@stdext@@@stdext@@@std@@@std@@IAE_NI@Z 100065c9 f i BaseManager.obj
 0001:000055c9       ?_Buy@?$vector@U_List_position@?$_Hash@V?$_Hmap_traits@KV?$basic_string@DU?$char_traits@D@std@@V?$allocator@D@2@@std@@V?$hash_compare@KU?$less@K@std@@@stdext@@V?$allocator@U?$pair@$$CBKV?$basic_string@DU?$char_traits@D@std@@V?$allocator@D@2@@std@@@std@@@2@$0A@@stdext@@@stdext@@V?$allocator@U_List_position@?$_Hash@V?$_Hmap_traits@KV?$basic_string@DU?$char_traits@D@std@@V?$allocator@D@2@@std@@V?$hash_compare@KU?$less@K@std@@@stdext@@V?$allocator@U?$pair@$$CBKV?$basic_string@DU?$char_traits@D@std@@V?$allocator@D@2@@std@@@std@@@2@$0A@@stdext@@@stdext@@@std@@@std@@IAE_NI@Z 100065c9 f i StringManager.obj
 0001:0000567b       ?_Insert@?$list@U?$pair@$$CBKV?$basic_string@DU?$char_traits@D@std@@V?$allocator@D@2@@std@@@std@@V?$allocator@U?$pair@$$CBKV?$basic_string@DU?$char_traits@D@std@@V?$allocator@D@2@@std@@@std@@@2@@std@@QAEXV?$_Const_iterator@$00@12@ABU?$pair@$$CBKV?$basic_string@DU?$char_traits@D@std@@V?$allocator@D@2@@std@@@2@@Z 1000667b f i StringManager.obj
 0001:000056c9       ?_Splice@?$list@U?$pair@$$CBKV?$basic_string@DU?$char_traits@D@std@@V?$allocator@D@2@@std@@@std@@V?$allocator@U?$pair@$$CBKV?$basic_string@DU?$char_traits@D@std@@V?$allocator@D@2@@std@@@std@@@2@@std@@QAEXV?$_Const_iterator@$00@12@AAV12@00I_N@Z 100066c9 f i StringManager.obj
 0001:00005852       ?begin@?$vector@U_List_position@?$_Hash@V?$_Hmap_traits@KPAXV?$hash_compare@KU?$less@K@std@@@stdext@@V?$allocator@U?$pair@$$CBKPAX@std@@@std@@$0A@@stdext@@@stdext@@V?$allocator@U_List_position@?$_Hash@V?$_Hmap_traits@KPAXV?$hash_compare@KU?$less@K@std@@@stdext@@V?$allocator@U?$pair@$$CBKPAX@std@@@std@@$0A@@stdext@@@stdext@@@std@@@std@@QAE?AV?$_Vector_iterator@U_List_position@?$_Hash@V?$_Hmap_traits@KPAXV?$hash_compare@KU?$less@K@std@@@stdext@@V?$allocator@U?$pair@$$CBKPAX@std@@@std@@$0A@@stdext@@@stdext@@V?$allocator@U_List_position@?$_Hash@V?$_Hmap_traits@KPAXV?$hash_compare@KU?$less@K@std@@@stdext@@V?$allocator@U?$pair@$$CBKPAX@std@@@std@@$0A@@stdext@@@stdext@@@std@@@2@XZ 10006852 f i BaseManager.obj
 0001:00005852       ?begin@?$vector@KV?$allocator@K@std@@@std@@QAE?AV?$_Vector_iterator@KV?$allocator@K@std@@@2@XZ 10006852 f i CtrlDxEdit.obj
 0001:00005852       ?begin@?$vector@U_List_position@?$_Hash@V?$_Hmap_traits@KV?$basic_string@DU?$char_traits@D@std@@V?$allocator@D@2@@std@@V?$hash_compare@KU?$less@K@std@@@stdext@@V?$allocator@U?$pair@$$CBKV?$basic_string@DU?$char_traits@D@std@@V?$allocator@D@2@@std@@@std@@@2@$0A@@stdext@@@stdext@@V?$allocator@U_List_position@?$_Hash@V?$_Hmap_traits@KV?$basic_string@DU?$char_traits@D@std@@V?$allocator@D@2@@std@@V?$hash_compare@KU?$less@K@std@@@stdext@@V?$allocator@U?$pair@$$CBKV?$basic_string@DU?$char_traits@D@std@@V?$allocator@D@2@@std@@@std@@@2@$0A@@stdext@@@stdext@@@std@@@std@@QAE?AV?$_Vector_iterator@U_List_position@?$_Hash@V?$_Hmap_traits@KV?$basic_string@DU?$char_traits@D@std@@V?$allocator@D@2@@std@@V?$hash_compare@KU?$less@K@std@@@stdext@@V?$allocator@U?$pair@$$CBKV?$basic_string@DU?$char_traits@D@std@@V?$allocator@D@2@@std@@@std@@@2@$0A@@stdext@@@stdext@@V?$allocator@U_List_position@?$_Hash@V?$_Hmap_traits@KV?$basic_string@DU?$char_traits@D@std@@V?$allocator@D@2@@std@@V?$hash_compare@KU?$less@K@std@@@stdext@@V?$allocator@U?$pair@$$CBKV?$basic_string@DU?$char_traits@D@std@@V?$allocator@D@2@@std@@@std@@@2@$0A@@stdext@@@stdext@@@std@@@2@XZ 10006852 f i StringManager.obj
 0001:000058a8       ?end@?$vector@U_List_position@?$_Hash@V?$_Hmap_traits@KPAXV?$hash_compare@KU?$less@K@std@@@stdext@@V?$allocator@U?$pair@$$CBKPAX@std@@@std@@$0A@@stdext@@@stdext@@V?$allocator@U_List_position@?$_Hash@V?$_Hmap_traits@KPAXV?$hash_compare@KU?$less@K@std@@@stdext@@V?$allocator@U?$pair@$$CBKPAX@std@@@std@@$0A@@stdext@@@stdext@@@std@@@std@@QAE?AV?$_Vector_iterator@U_List_position@?$_Hash@V?$_Hmap_traits@KPAXV?$hash_compare@KU?$less@K@std@@@stdext@@V?$allocator@U?$pair@$$CBKPAX@std@@@std@@$0A@@stdext@@@stdext@@V?$allocator@U_List_position@?$_Hash@V?$_Hmap_traits@KPAXV?$hash_compare@KU?$less@K@std@@@stdext@@V?$allocator@U?$pair@$$CBKPAX@std@@@std@@$0A@@stdext@@@stdext@@@std@@@2@XZ 100068a8 f i BaseManager.obj
 0001:000058a8       ?end@?$vector@KV?$allocator@K@std@@@std@@QAE?AV?$_Vector_iterator@KV?$allocator@K@std@@@2@XZ 100068a8 f i CtrlDxEdit.obj
 0001:000058a8       ?end@?$vector@U_List_position@?$_Hash@V?$_Hmap_traits@KV?$basic_string@DU?$char_traits@D@std@@V?$allocator@D@2@@std@@V?$hash_compare@KU?$less@K@std@@@stdext@@V?$allocator@U?$pair@$$CBKV?$basic_string@DU?$char_traits@D@std@@V?$allocator@D@2@@std@@@std@@@2@$0A@@stdext@@@stdext@@V?$allocator@U_List_position@?$_Hash@V?$_Hmap_traits@KV?$basic_string@DU?$char_traits@D@std@@V?$allocator@D@2@@std@@V?$hash_compare@KU?$less@K@std@@@stdext@@V?$allocator@U?$pair@$$CBKV?$basic_string@DU?$char_traits@D@std@@V?$allocator@D@2@@std@@@std@@@2@$0A@@stdext@@@stdext@@@std@@@std@@QAE?AV?$_Vector_iterator@U_List_position@?$_Hash@V?$_Hmap_traits@KV?$basic_string@DU?$char_traits@D@std@@V?$allocator@D@2@@std@@V?$hash_compare@KU?$less@K@std@@@stdext@@V?$allocator@U?$pair@$$CBKV?$basic_string@DU?$char_traits@D@std@@V?$allocator@D@2@@std@@@std@@@2@$0A@@stdext@@@stdext@@V?$allocator@U_List_position@?$_Hash@V?$_Hmap_traits@KV?$basic_string@DU?$char_traits@D@std@@V?$allocator@D@2@@std@@V?$hash_compare@KU?$less@K@std@@@stdext@@V?$allocator@U?$pair@$$CBKV?$basic_string@DU?$char_traits@D@std@@V?$allocator@D@2@@std@@@std@@@2@$0A@@stdext@@@stdext@@@std@@@2@XZ 100068a8 f i StringManager.obj
 0001:000058fe       ?erase@?$vector@U_List_position@?$_Hash@V?$_Hmap_traits@KV?$basic_string@DU?$char_traits@D@std@@V?$allocator@D@2@@std@@V?$hash_compare@KU?$less@K@std@@@stdext@@V?$allocator@U?$pair@$$CBKV?$basic_string@DU?$char_traits@D@std@@V?$allocator@D@2@@std@@@std@@@2@$0A@@stdext@@@stdext@@V?$allocator@U_List_position@?$_Hash@V?$_Hmap_traits@KV?$basic_string@DU?$char_traits@D@std@@V?$allocator@D@2@@std@@V?$hash_compare@KU?$less@K@std@@@stdext@@V?$allocator@U?$pair@$$CBKV?$basic_string@DU?$char_traits@D@std@@V?$allocator@D@2@@std@@@std@@@2@$0A@@stdext@@@stdext@@@std@@@std@@QAE?AV?$_Vector_iterator@U_List_position@?$_Hash@V?$_Hmap_traits@KV?$basic_string@DU?$char_traits@D@std@@V?$allocator@D@2@@std@@V?$hash_compare@KU?$less@K@std@@@stdext@@V?$allocator@U?$pair@$$CBKV?$basic_string@DU?$char_traits@D@std@@V?$allocator@D@2@@std@@@std@@@2@$0A@@stdext@@@stdext@@V?$allocator@U_List_position@?$_Hash@V?$_Hmap_traits@KV?$basic_string@DU?$char_traits@D@std@@V?$allocator@D@2@@std@@V?$hash_compare@KU?$less@K@std@@@stdext@@V?$allocator@U?$pair@$$CBKV?$basic_string@DU?$char_traits@D@std@@V?$allocator@D@2@@std@@@std@@@2@$0A@@stdext@@@stdext@@@std@@@2@V?$_Vector_const_iterator@U_List_position@?$_Hash@V?$_Hmap_traits@KV?$basic_string@DU?$char_traits@D@std@@V?$allocator@D@2@@std@@V?$hash_compare@KU?$less@K@std@@@stdext@@V?$allocator@U?$pair@$$CBKV?$basic_string@DU?$char_traits@D@std@@V?$allocator@D@2@@std@@@std@@@2@$0A@@stdext@@@stdext@@V?$allocator@U_List_position@?$_Hash@V?$_Hmap_traits@KV?$basic_string@DU?$char_traits@D@std@@V?$allocator@D@2@@std@@V?$hash_compare@KU?$less@K@std@@@stdext@@V?$allocator@U?$pair@$$CBKV?$basic_string@DU?$char_traits@D@std@@V?$allocator@D@2@@std@@@std@@@2@$0A@@stdext@@@stdext@@@std@@@2@0@Z 100068fe f i StringManager.obj
 0001:000058fe       ?erase@?$vector@U_List_position@?$_Hash@V?$_Hmap_traits@KPAXV?$hash_compare@KU?$less@K@std@@@stdext@@V?$allocator@U?$pair@$$CBKPAX@std@@@std@@$0A@@stdext@@@stdext@@V?$allocator@U_List_position@?$_Hash@V?$_Hmap_traits@KPAXV?$hash_compare@KU?$less@K@std@@@stdext@@V?$allocator@U?$pair@$$CBKPAX@std@@@std@@$0A@@stdext@@@stdext@@@std@@@std@@QAE?AV?$_Vector_iterator@U_List_position@?$_Hash@V?$_Hmap_traits@KPAXV?$hash_compare@KU?$less@K@std@@@stdext@@V?$allocator@U?$pair@$$CBKPAX@std@@@std@@$0A@@stdext@@@stdext@@V?$allocator@U_List_position@?$_Hash@V?$_Hmap_traits@KPAXV?$hash_compare@KU?$less@K@std@@@stdext@@V?$allocator@U?$pair@$$CBKPAX@std@@@std@@$0A@@stdext@@@stdext@@@std@@@2@V?$_Vector_const_iterator@U_List_position@?$_Hash@V?$_Hmap_traits@KPAXV?$hash_compare@KU?$less@K@std@@@stdext@@V?$allocator@U?$pair@$$CBKPAX@std@@@std@@$0A@@stdext@@@stdext@@V?$allocator@U_List_position@?$_Hash@V?$_Hmap_traits@KPAXV?$hash_compare@KU?$less@K@std@@@stdext@@V?$allocator@U?$pair@$$CBKPAX@std@@@std@@$0A@@stdext@@@stdext@@@std@@@2@0@Z 100068fe f i BaseManager.obj
 0001:000059a9       ?erase@?$list@U?$pair@$$CBKV?$basic_string@DU?$char_traits@D@std@@V?$allocator@D@2@@std@@@std@@V?$allocator@U?$pair@$$CBKV?$basic_string@DU?$char_traits@D@std@@V?$allocator@D@2@@std@@@std@@@2@@std@@QAE?AV?$_Iterator@$00@12@V?$_Const_iterator@$00@12@0@Z 100069a9 f i StringManager.obj
 0001:00005b01       ?_Buynode@?$list@U?$pair@$$CBKV?$basic_string@DU?$char_traits@D@std@@V?$allocator@D@2@@std@@@std@@V?$allocator@U?$pair@$$CBKV?$basic_string@DU?$char_traits@D@std@@V?$allocator@D@2@@std@@@std@@@2@@std@@IAEPAU_Node@?$_List_nod@U?$pair@$$CBKV?$basic_string@DU?$char_traits@D@std@@V?$allocator@D@2@@std@@@std@@V?$allocator@U?$pair@$$CBKV?$basic_string@DU?$char_traits@D@std@@V?$allocator@D@2@@std@@@std@@@2@@2@PAU342@0ABU?$pair@$$CBKV?$basic_string@DU?$char_traits@D@std@@V?$allocator@D@2@@std@@@2@@Z 10006b01 f i StringManager.obj
 0001:00005beb       ?_Incsize@?$list@U?$pair@$$CBKV?$basic_string@DU?$char_traits@D@std@@V?$allocator@D@2@@std@@@std@@V?$allocator@U?$pair@$$CBKV?$basic_string@DU?$char_traits@D@std@@V?$allocator@D@2@@std@@@std@@@2@@std@@IAEXI@Z 10006beb f i StringManager.obj
 0001:00005cb5       ?_Insert_n@?$vector@U_List_position@?$_Hash@V?$_Hmap_traits@KPAXV?$hash_compare@KU?$less@K@std@@@stdext@@V?$allocator@U?$pair@$$CBKPAX@std@@@std@@$0A@@stdext@@@stdext@@V?$allocator@U_List_position@?$_Hash@V?$_Hmap_traits@KPAXV?$hash_compare@KU?$less@K@std@@@stdext@@V?$allocator@U?$pair@$$CBKPAX@std@@@std@@$0A@@stdext@@@stdext@@@std@@@std@@IAEXV?$_Vector_const_iterator@U_List_position@?$_Hash@V?$_Hmap_traits@KPAXV?$hash_compare@KU?$less@K@std@@@stdext@@V?$allocator@U?$pair@$$CBKPAX@std@@@std@@$0A@@stdext@@@stdext@@V?$allocator@U_List_position@?$_Hash@V?$_Hmap_traits@KPAXV?$hash_compare@KU?$less@K@std@@@stdext@@V?$allocator@U?$pair@$$CBKPAX@std@@@std@@$0A@@stdext@@@stdext@@@std@@@2@IABU_List_position@?$_Hash@V?$_Hmap_traits@KPAXV?$hash_compare@KU?$less@K@std@@@stdext@@V?$allocator@U?$pair@$$CBKPAX@std@@@std@@$0A@@stdext@@@stdext@@@Z 10006cb5 f i BaseManager.obj
 0001:00005cb5       ?_Insert_n@?$vector@U_List_position@?$_Hash@V?$_Hmap_traits@KV?$basic_string@DU?$char_traits@D@std@@V?$allocator@D@2@@std@@V?$hash_compare@KU?$less@K@std@@@stdext@@V?$allocator@U?$pair@$$CBKV?$basic_string@DU?$char_traits@D@std@@V?$allocator@D@2@@std@@@std@@@2@$0A@@stdext@@@stdext@@V?$allocator@U_List_position@?$_Hash@V?$_Hmap_traits@KV?$basic_string@DU?$char_traits@D@std@@V?$allocator@D@2@@std@@V?$hash_compare@KU?$less@K@std@@@stdext@@V?$allocator@U?$pair@$$CBKV?$basic_string@DU?$char_traits@D@std@@V?$allocator@D@2@@std@@@std@@@2@$0A@@stdext@@@stdext@@@std@@@std@@IAEXV?$_Vector_const_iterator@U_List_position@?$_Hash@V?$_Hmap_traits@KV?$basic_string@DU?$char_traits@D@std@@V?$allocator@D@2@@std@@V?$hash_compare@KU?$less@K@std@@@stdext@@V?$allocator@U?$pair@$$CBKV?$basic_string@DU?$char_traits@D@std@@V?$allocator@D@2@@std@@@std@@@2@$0A@@stdext@@@stdext@@V?$allocator@U_List_position@?$_Hash@V?$_Hmap_traits@KV?$basic_string@DU?$char_traits@D@std@@V?$allocator@D@2@@std@@V?$hash_compare@KU?$less@K@std@@@stdext@@V?$allocator@U?$pair@$$CBKV?$basic_string@DU?$char_traits@D@std@@V?$allocator@D@2@@std@@@std@@@2@$0A@@stdext@@@stdext@@@std@@@2@IABU_List_position@?$_Hash@V?$_Hmap_traits@KV?$basic_string@DU?$char_traits@D@std@@V?$allocator@D@2@@std@@V?$hash_compare@KU?$less@K@std@@@stdext@@V?$allocator@U?$pair@$$CBKV?$basic_string@DU?$char_traits@D@std@@V?$allocator@D@2@@std@@@std@@@2@$0A@@stdext@@@stdext@@@Z 10006cb5 f i StringManager.obj
 0001:000063a5       ??$_Allocate@U_Node@?$_List_nod@U?$pair@$$CBKV?$basic_string@DU?$char_traits@D@std@@V?$allocator@D@2@@std@@@std@@V?$allocator@U?$pair@$$CBKV?$basic_string@DU?$char_traits@D@std@@V?$allocator@D@2@@std@@@std@@@2@@std@@@std@@YAPAU_Node@?$_List_nod@U?$pair@$$CBKV?$basic_string@DU?$char_traits@D@std@@V?$allocator@D@2@@std@@@std@@V?$allocator@U?$pair@$$CBKV?$basic_string@DU?$char_traits@D@std@@V?$allocator@D@2@@std@@@std@@@2@@0@IPAU120@@Z 100073a5 f i StringManager.obj
 0001:000063f8       ??$_Allocate@U_List_position@?$_Hash@V?$_Hmap_traits@KV?$basic_string@DU?$char_traits@D@std@@V?$allocator@D@2@@std@@V?$hash_compare@KU?$less@K@std@@@stdext@@V?$allocator@U?$pair@$$CBKV?$basic_string@DU?$char_traits@D@std@@V?$allocator@D@2@@std@@@std@@@2@$0A@@stdext@@@stdext@@@std@@YAPAU_List_position@?$_Hash@V?$_Hmap_traits@KV?$basic_string@DU?$char_traits@D@std@@V?$allocator@D@2@@std@@V?$hash_compare@KU?$less@K@std@@@stdext@@V?$allocator@U?$pair@$$CBKV?$basic_string@DU?$char_traits@D@std@@V?$allocator@D@2@@std@@@std@@@2@$0A@@stdext@@@stdext@@IPAU123@@Z 100073f8 f i StringManager.obj
 0001:000063f8       ??$_Allocate@U_List_position@?$_Hash@V?$_Hmap_traits@KPAXV?$hash_compare@KU?$less@K@std@@@stdext@@V?$allocator@U?$pair@$$CBKPAX@std@@@std@@$0A@@stdext@@@stdext@@@std@@YAPAU_List_position@?$_Hash@V?$_Hmap_traits@KPAXV?$hash_compare@KU?$less@K@std@@@stdext@@V?$allocator@U?$pair@$$CBKPAX@std@@@std@@$0A@@stdext@@@stdext@@IPAU123@@Z 100073f8 f i BaseManager.obj
 0001:0000644b       ??$_Construct@U?$pair@$$CBKV?$basic_string@DU?$char_traits@D@std@@V?$allocator@D@2@@std@@@std@@U12@@std@@YAXPAU?$pair@$$CBKV?$basic_string@DU?$char_traits@D@std@@V?$allocator@D@2@@std@@@0@ABU10@@Z 1000744b f i StringManager.obj
 0001:000064b1       ??_G_Node@?$_List_nod@U?$pair@$$CBKV?$basic_string@DU?$char_traits@D@std@@V?$allocator@D@2@@std@@@std@@V?$allocator@U?$pair@$$CBKV?$basic_string@DU?$char_traits@D@std@@V?$allocator@D@2@@std@@@std@@@2@@std@@QAEPAXI@Z 100074b1 f i StringManager.obj
 0001:000064ea       ??0?$pair@$$CBKV?$basic_string@DU?$char_traits@D@std@@V?$allocator@D@2@@std@@@std@@QAE@ABU01@@Z 100074ea f i StringManager.obj
 0001:00006530       ??$_Insert@V?$_Const_iterator@$00@?$list@U?$pair@$$CBKV?$basic_string@DU?$char_traits@D@std@@V?$allocator@D@2@@std@@@std@@V?$allocator@U?$pair@$$CBKV?$basic_string@DU?$char_traits@D@std@@V?$allocator@D@2@@std@@@std@@@2@@std@@@?$list@U?$pair@$$CBKV?$basic_string@DU?$char_traits@D@std@@V?$allocator@D@2@@std@@@std@@V?$allocator@U?$pair@$$CBKV?$basic_string@DU?$char_traits@D@std@@V?$allocator@D@2@@std@@@std@@@2@@std@@QAEXV?$_Const_iterator@$00@01@00Uforward_iterator_tag@1@@Z 10007530 f i StringManager.obj
 0001:00006645       ??$_Uninit_fill_n@PAU_List_position@?$_Hash@V?$_Hmap_traits@KV?$basic_string@DU?$char_traits@D@std@@V?$allocator@D@2@@std@@V?$hash_compare@KU?$less@K@std@@@stdext@@V?$allocator@U?$pair@$$CBKV?$basic_string@DU?$char_traits@D@std@@V?$allocator@D@2@@std@@@std@@@2@$0A@@stdext@@@stdext@@IU123@V?$allocator@U_List_position@?$_Hash@V?$_Hmap_traits@KV?$basic_string@DU?$char_traits@D@std@@V?$allocator@D@2@@std@@V?$hash_compare@KU?$less@K@std@@@stdext@@V?$allocator@U?$pair@$$CBKV?$basic_string@DU?$char_traits@D@std@@V?$allocator@D@2@@std@@@std@@@2@$0A@@stdext@@@stdext@@@std@@@std@@YAXPAU_List_position@?$_Hash@V?$_Hmap_traits@KV?$basic_string@DU?$char_traits@D@std@@V?$allocator@D@2@@std@@V?$hash_compare@KU?$less@K@std@@@stdext@@V?$allocator@U?$pair@$$CBKV?$basic_string@DU?$char_traits@D@std@@V?$allocator@D@2@@std@@@std@@@2@$0A@@stdext@@@stdext@@IABU123@AAV?$allocator@U_List_position@?$_Hash@V?$_Hmap_traits@KV?$basic_string@DU?$char_traits@D@std@@V?$allocator@D@2@@std@@V?$hash_compare@KU?$less@K@std@@@stdext@@V?$allocator@U?$pair@$$CBKV?$basic_string@DU?$char_traits@D@std@@V?$allocator@D@2@@std@@@std@@@2@$0A@@stdext@@@stdext@@@0@U_Nonscalar_ptr_iterator_tag@0@U_Range_checked_iterator_tag@0@@Z 10007645 f i StringManager.obj
 0001:00006645       ??$_Uninit_fill_n@PAU_List_position@?$_Hash@V?$_Hmap_traits@KPAXV?$hash_compare@KU?$less@K@std@@@stdext@@V?$allocator@U?$pair@$$CBKPAX@std@@@std@@$0A@@stdext@@@stdext@@IU123@V?$allocator@U_List_position@?$_Hash@V?$_Hmap_traits@KPAXV?$hash_compare@KU?$less@K@std@@@stdext@@V?$allocator@U?$pair@$$CBKPAX@std@@@std@@$0A@@stdext@@@stdext@@@std@@@std@@YAXPAU_List_position@?$_Hash@V?$_Hmap_traits@KPAXV?$hash_compare@KU?$less@K@std@@@stdext@@V?$allocator@U?$pair@$$CBKPAX@std@@@std@@$0A@@stdext@@@stdext@@IABU123@AAV?$allocator@U_List_position@?$_Hash@V?$_Hmap_traits@KPAXV?$hash_compare@KU?$less@K@std@@@stdext@@V?$allocator@U?$pair@$$CBKPAX@std@@@std@@$0A@@stdext@@@stdext@@@0@U_Nonscalar_ptr_iterator_tag@0@U_Range_checked_iterator_tag@0@@Z 10007645 f i BaseManager.obj
 0001:00006701       ??3@YAXPAX0@Z              10007701 f i StringManager.obj
 0001:00006706       ??0?$basic_string@DU?$char_traits@D@std@@V?$allocator@D@2@@std@@QAE@ABV01@@Z 10007706 f i StringManager.obj
 0001:00006735       ?IsDigitA@CControlWZ@@SA_NPBD@Z 10007735 f   ControlWZ.obj
 0001:000067a3       ?IsDigitW@CControlWZ@@SA_NPB_W@Z 100077a3 f   ControlWZ.obj
 0001:0000681b       ?MakeMoneyString@CControlWZ@@SA?AV?$basic_string@DU?$char_traits@D@std@@V?$allocator@D@2@@std@@_K@Z 1000781b f   ControlWZ.obj
 0001:000068a6       ??0CControlWZ@@QAE@XZ      100078a6 f   ControlWZ.obj
 0001:00006af8       ??1CControlWZ@@UAE@XZ      10007af8 f   ControlWZ.obj
 0001:00006b6a       ?Release@CControlWZ@@QAEXXZ 10007b6a f   ControlWZ.obj
 0001:00006bf0       ?OnCreate@CControlWZ@@UAE_NKKPAUHWND__@@PAUHINSTANCE__@@PAUtagRECT@@PAX@Z 10007bf0 f   ControlWZ.obj
 0001:00006c7d       ?OnDestroy@CControlWZ@@UAEXXZ 10007c7d f   ControlWZ.obj
 0001:00006c8e       ?IsShow_ToolTip@CControlWZ@@UAE_NXZ 10007c8e f   ControlWZ.obj
 0001:00006ca8       ?OnDoAction_ToolTip@CControlWZ@@UAEXABUtagPOINT@@@Z 10007ca8 f   ControlWZ.obj
 0001:00006d76       ?OnDoAction@CControlWZ@@UAEXXZ 10007d76 f   ControlWZ.obj
 0001:00006d7f       ?DrawImageData@CControlWZ@@QAE_NABUSI_TSUBINFO@@ABUSt_FRect@@@Z 10007d7f f   ControlWZ.obj
 0001:0000812e       ?DrawControlRectangle@CControlWZ@@QAEXABUSI_TSUBINFO@@ABUSt_FRect@@@Z 1000912e f   ControlWZ.obj
 0001:0000817e       ?DrawControlStyle@CControlWZ@@QAEXABUSI_TSUBINFO@@ABUSt_FRect@@@Z 1000917e f   ControlWZ.obj
 0001:00008260       ?DrawCallbackProc@CControlWZ@@QAEXXZ 10009260 f   ControlWZ.obj
 0001:0000828c       ?OnDraw@CControlWZ@@UAE_N_N@Z 1000928c f   ControlWZ.obj
 0001:00008341       ?OnLoad@CControlWZ@@UAEXPAX@Z 10009341 f   ControlWZ.obj
 0001:0000978a       ?ChangeCaptionString@CControlWZ@@UAEXXZ 1000a78a f   ControlWZ.obj
 0001:000097d0       ?OnSave@CControlWZ@@UAEXPAX@Z 1000a7d0 f   ControlWZ.obj
 0001:00009bfe       ?ResetDrawState@CControlWZ@@UAEXXZ 1000abfe f   ControlWZ.obj
 0001:00009c21       ?OnInitialize@CControlWZ@@UAEXXZ 1000ac21 f   ControlWZ.obj
 0001:00009c5b       ?ShowWindowWZ@CControlWZ@@UAEXW4ENUM_STATEWZ@@@Z 1000ac5b f   ControlWZ.obj
 0001:00009c89       ?EnableWindowWZ@CControlWZ@@UAEX_N@Z 1000ac89 f   ControlWZ.obj
 0001:00009cc7       ?GetSizeRect@CControlWZ@@UAE?AUtagRECT@@XZ 1000acc7 f   ControlWZ.obj
 0001:00009d25       ?GetSize@CControlWZ@@UAE?AUtagRECT@@XZ 1000ad25 f   ControlWZ.obj
 0001:00009d6f       ?MoveWindowWZ@CControlWZ@@UAE_NMMMM@Z 1000ad6f f   ControlWZ.obj
 0001:00009da0       ?ChangeSize@CControlWZ@@QAEXMMMM@Z 1000ada0 f   ControlWZ.obj
 0001:00009ddf       ?SetCtrlImageFormat@CControlWZ@@UAEXPAUSI_TFORMAT@@@Z 1000addf f   ControlWZ.obj
 0001:00009e20       ?SetCtrlDetailImageFormat@CControlWZ@@UAEXW4ENUM_DRAWSTATE@@PAUSI_TSUBINFO@@@Z 1000ae20 f   ControlWZ.obj
 0001:00009f12       ?SetToolTipInfo@CControlWZ@@UAEXPAUSI_ToolTip@@@Z 1000af12 f   ControlWZ.obj
 0001:00009f32       ?GetToolTipInfo@CControlWZ@@UAEXPAUSI_ToolTip@@@Z 1000af32 f   ControlWZ.obj
 0001:00009f52       ?ReleaseImage@CControlWZ@@UAEXXZ 1000af52 f   ControlWZ.obj
 0001:00009fd8       ?UpdateWindowWZ@CControlWZ@@UAEXPAUHWND__@@@Z 1000afd8 f   ControlWZ.obj
 0001:0000a1e2       ?SetCtrlID@CControlWZ@@UAE_NK@Z 1000b1e2 f   ControlWZ.obj
 0001:0000a250       ?SendMessageWZ@CControlWZ@@UAE_NPAUSI_MESSAGE@@@Z 1000b250 f   ControlWZ.obj
 0001:0000a3e9       ?Message_MouseLButtonDown@CControlWZ@@MAE_NPAUSI_MESSAGE@@@Z 1000b3e9 f   ControlWZ.obj
 0001:0000a50a       ?Message_MouseLButtonUp@CControlWZ@@MAE_NPAUSI_MESSAGE@@@Z 1000b50a f   ControlWZ.obj
 0001:0000a619       ?Message_MouseLButtonDoubleClick@CControlWZ@@MAE_NPAUSI_MESSAGE@@@Z 1000b619 f   ControlWZ.obj
 0001:0000a747       ?Message_MouseRButtonDown@CControlWZ@@MAE_NPAUSI_MESSAGE@@@Z 1000b747 f   ControlWZ.obj
 0001:0000a84a       ?Message_MouseRButtonUp@CControlWZ@@MAE_NPAUSI_MESSAGE@@@Z 1000b84a f   ControlWZ.obj
 0001:0000a959       ?Message_MouseRButtonDoubleClick@CControlWZ@@MAE_NPAUSI_MESSAGE@@@Z 1000b959 f   ControlWZ.obj
 0001:0000aa5c       ?Message_MouseMove@CControlWZ@@MAE_NPAUSI_MESSAGE@@@Z 1000ba5c f   ControlWZ.obj
 0001:0000ab81       ?Message_KeyDown@CControlWZ@@MAE_NPAUSI_MESSAGE@@@Z 1000bb81 f   ControlWZ.obj
 0001:0000ab8e       ?Message_KeyUp@CControlWZ@@MAE_NPAUSI_MESSAGE@@@Z 1000bb8e f   ControlWZ.obj
 0001:0000ab9b       ?SetMoney@CControlWZ@@UAEX_K@Z 1000bb9b f   ControlWZ.obj
 0001:0000ac1a       ?SetMoneyWithSymbol@CControlWZ@@UAEX_J@Z 1000bc1a f   ControlWZ.obj
 0001:0000acfa       ?OnDraw_Tile_XY@CControlWZ@@EAEXABUSt_FRect@@0PAX@Z 1000bcfa f   ControlWZ.obj
 0001:0000af6d       ?OnDraw_Tile_X@CControlWZ@@EAEXABUSt_FRect@@0PAX@Z 1000bf6d f   ControlWZ.obj
 0001:0000b0d7       ?OnDraw_Tile_Y@CControlWZ@@EAEXABUSt_FRect@@0PAX@Z 1000c0d7 f   ControlWZ.obj
 0001:0000b242       ?GetSoundIndex@CControlWZ@@UBEHW4ENUM_RESULT_MSG@@@Z 1000c242 f   ControlWZ.obj
 0001:0000b2a3       ?GetSoundIndex@CControlWZ@@UBEHW4ControlSoundEventType@@@Z 1000c2a3 f   ControlWZ.obj
 0001:0000b2c5       ?SetSoundIndex@CControlWZ@@UAEXW4ControlSoundEventType@@H@Z 1000c2c5 f   ControlWZ.obj
 0001:0000b2e6       ?SetStyle@CControlWZ@@UAEXK@Z 1000c2e6 f i ControlWZ.obj
 0001:0000b2fa       ?GetCtrlInfo@CControlWZ@@UAEPAUSCTRL_INFO@@XZ 1000c2fa f i ControlWZ.obj
 0001:0000b309       ?GetCtrlImageFormat@CControlWZ@@UAEPAUSI_TFORMAT@@XZ 1000c309 f i ControlWZ.obj
 0001:0000b318       ?GetCtrlID@CControlWZ@@UAEKXZ 1000c318 f i ControlWZ.obj
 0001:0000b327       ?GetState@CControlWZ@@UAE?AW4ENUM_STATEWZ@@XZ 1000c327 f i ControlWZ.obj
 0001:0000b339       ?GetDrawState@CControlWZ@@UAE?AW4ENUM_DRAWSTATE@@XZ 1000c339 f i ControlWZ.obj
 0001:0000b34b       ?AddStyle@CControlWZ@@UAEXK@Z 1000c34b f i ControlWZ.obj
 0001:0000b365       ?GetCtrlStyle@CControlWZ@@UAEKXZ 1000c365 f i ControlWZ.obj
 0001:0000b374       ?GetKind@CControlWZ@@UAEKXZ 1000c374 f i ControlWZ.obj
 0001:0000b383       ?IsKind@CControlWZ@@UAE_NK@Z 1000c383 f i ControlWZ.obj
 0001:0000b39a       ?SetIsOutline@CControlWZ@@UAEX_N@Z 1000c39a f i ControlWZ.obj
 0001:0000b3b1       ?GetIsOutline@CControlWZ@@UAE_NXZ 1000c3b1 f i ControlWZ.obj
 0001:0000b3c3       ?SetOutlineColor@CControlWZ@@UAEXK@Z 1000c3c3 f i ControlWZ.obj
 0001:0000b3da       ?GetOutlineColor@CControlWZ@@UAEKXZ 1000c3da f i ControlWZ.obj
 0001:0000b3ec       ?Set3DShapeState@CControlWZ@@UAEX_N@Z 1000c3ec f i ControlWZ.obj
 0001:0000b403       ?SetShadowState@CControlWZ@@UAEX_N@Z 1000c403 f i ControlWZ.obj
 0001:0000b41a       ?Get3DShapeState@CControlWZ@@UAE_NXZ 1000c41a f i ControlWZ.obj
 0001:0000b42c       ?GetShadowState@CControlWZ@@UAE_NXZ 1000c42c f i ControlWZ.obj
 0001:0000b43e       ?CanHaveFocus@CControlWZ@@UAE_NXZ 1000c43e f i ControlWZ.obj
 0001:0000b449       ?OnFocusIn@CControlWZ@@UAEXXZ 1000c449 f i ControlWZ.obj
 0001:0000b45c       ?OnFocusOut@CControlWZ@@UAEXXZ 1000c45c f i ControlWZ.obj
 0001:0000b47a       ?IsTextReducing@CControlWZ@@UBE_NXZ 1000c47a f i ControlWZ.obj
 0001:0000b47a       ?GetUseIndicator@CCtrlBaseEdit@@UAE_NXZ 1000c47a f i CtrlDxEdit.obj
 0001:0000b47a       ?IsUseDefault@CControlWZ@@UBE_NXZ 1000c47a f i ControlWZ.obj
 0001:0000b47a       ?IsMoneyType@CControlWZ@@UBE_NXZ 1000c47a f i ControlWZ.obj
 0001:0000b485       ?SetTextWZW@CControlWZ@@UAEXPB_W_N@Z 1000c485 f i ControlWZ.obj
 0001:0000b485       ?SetTextWZA@CControlWZ@@UAEXPBD_N@Z 1000c485 f i ControlWZ.obj
 0001:0000b485       ?GetTextWZA@CControlWZ@@UAEXPADH@Z 1000c485 f i ControlWZ.obj
 0001:0000b485       ?GetTextWZW@CControlWZ@@UAEXPA_WH@Z 1000c485 f i ControlWZ.obj
 0001:0000b490       ?SetTransprency@CControlWZ@@UAEXM@Z 1000c490 f i ControlWZ.obj
 0001:0000b4ab       ?GetPosX@CControlWZ@@UAEMXZ 1000c4ab f i ControlWZ.obj
 0001:0000b4ba       ?GetPosY@CControlWZ@@UAEMXZ 1000c4ba f i ControlWZ.obj
 0001:0000b4c9       ?GetSizeWidth@CControlWZ@@UAEMXZ 1000c4c9 f i ControlWZ.obj
 0001:0000b4d8       ?GetSizeHeight@CControlWZ@@UAEMXZ 1000c4d8 f i ControlWZ.obj
 0001:0000b4e7       ?GetOriginRect@CControlWZ@@UAE?AUtagRECT@@XZ 1000c4e7 f i ControlWZ.obj
 0001:0000b509       ?SetNotScaling@CControlWZ@@UAEX_N@Z 1000c509 f i ControlWZ.obj
 0001:0000b520       ?GetNotScaling@CControlWZ@@UAE_NXZ 1000c520 f i ControlWZ.obj
 0001:0000b532       ?SetSizeWidth@CControlWZ@@UAEXJ@Z 1000c532 f i ControlWZ.obj
 0001:0000b54a       ?SetSizeHeight@CControlWZ@@UAEXJ@Z 1000c54a f i ControlWZ.obj
 0001:0000b562       ?IsDiscardMessage@CControlWZ@@UBE_NXZ 1000c562 f i ControlWZ.obj
 0001:0000b574       ?SetDiscardMessage@CControlWZ@@UAEX_N@Z 1000c574 f i ControlWZ.obj
 0001:0000b58b       ?GetUserData@CControlWZ@@UBEKXZ 1000c58b f i ControlWZ.obj
 0001:0000b59d       ?SetUserData@CControlWZ@@UAEXK@Z 1000c59d f i ControlWZ.obj
 0001:0000b5b4       ?SetCallbackDraw@CControlWZ@@UAEXP6AXPAV1@PAX@Z1@Z 1000c5b4 f i ControlWZ.obj
 0001:0000b5d7       ?Initialize@SCTRL_INFO@@QAEXXZ 1000c5d7 f i ControlWZ.obj
 0001:0000b615       ??0SI_TSUBINFO@@QAE@XZ     1000c615 f i ControlWZ.obj
 0001:0000b6d2       ?Initialize@SI_TSUBINFO@@QAEXXZ 1000c6d2 f i ControlWZ.obj
 0001:0000b75c       ?clear@?$basic_string@DU?$char_traits@D@std@@V?$allocator@D@2@@std@@QAEXXZ 1000c75c f i ControlWZ.obj
 0001:0000b7cd       ?erase@?$basic_string@DU?$char_traits@D@std@@V?$allocator@D@2@@std@@QAE?AV?$_String_iterator@DU?$char_traits@D@std@@V?$allocator@D@2@@2@V?$_String_const_iterator@DU?$char_traits@D@std@@V?$allocator@D@2@@2@0@Z 1000c7cd f i ControlWZ.obj
 0001:0000b8bd       ?end@?$basic_string@DU?$char_traits@D@std@@V?$allocator@D@2@@std@@QAE?AV?$_String_iterator@DU?$char_traits@D@std@@V?$allocator@D@2@@2@XZ 1000c8bd f i ControlWZ.obj
 0001:0000b904       ??0?$_String_const_iterator@DU?$char_traits@D@std@@V?$allocator@D@2@@std@@QAE@PBDPBV_Container_base_secure@1@@Z 1000c904 f i ControlWZ.obj
 0001:0000b990       ??G?$_String_const_iterator@DU?$char_traits@D@std@@V?$allocator@D@2@@std@@QBEHABV01@@Z 1000c990 f i ControlWZ.obj
 0001:0000b9e0       ??_ECControlWZ@@UAEPAXI@Z  1000c9e0 f i ControlWZ.obj
 0001:0000b9e0       ??_GCControlWZ@@UAEPAXI@Z  1000c9e0 f i ControlWZ.obj
 0001:0000ba07       ??0SCTRL_INFO@@QAE@XZ      1000ca07 f i ControlWZ.obj
 0001:0000baa5       ??1SI_TFORMAT@@QAE@XZ      1000caa5 f i ControlWZ.obj
 0001:0000babf       ??1?$pair@$$CBKV?$basic_string@DU?$char_traits@D@std@@V?$allocator@D@2@@std@@@std@@QAE@XZ 1000cabf f i StringManager.obj
 0001:0000babf       ??1SI_TSUBINFO@@QAE@XZ     1000cabf f i ControlWZ.obj
 0001:0000bad9       ??4SI_TSUBINFO@@QAEAAU0@ABU0@@Z 1000cad9 f i ControlWZ.obj
 0001:0000bb6d       ??0CCtrlButtonCheckWZ@@QAE@XZ 1000cb6d f   CtrlButtonCheckWZ.obj
 0001:0000bbab       ??1CCtrlButtonCheckWZ@@UAE@XZ 1000cbab f   CtrlButtonCheckWZ.obj
 0001:0000bbc5       ?OnInitialize@CCtrlButtonCheckWZ@@UAEXXZ 1000cbc5 f   CtrlButtonCheckWZ.obj
 0001:0000bbd6       ?OnDraw@CCtrlButtonCheckWZ@@UAE_N_N@Z 1000cbd6 f   CtrlButtonCheckWZ.obj
 0001:0000bf31       ?SendMessageWZ@CCtrlButtonCheckWZ@@UAE_NPAUSI_MESSAGE@@@Z 1000cf31 f   CtrlButtonCheckWZ.obj
 0001:0000bf69       ?GetDrawState@CCtrlButtonCheckWZ@@UAE?AW4ENUM_DRAWSTATE@@XZ 1000cf69 f   CtrlButtonCheckWZ.obj
 0001:0000bfa9       ?Message_MouseLButtonDown@CCtrlButtonCheckWZ@@MAE_NPAUSI_MESSAGE@@@Z 1000cfa9 f   CtrlButtonCheckWZ.obj
 0001:0000c0ca       ?Message_MouseLButtonUp@CCtrlButtonCheckWZ@@MAE_NPAUSI_MESSAGE@@@Z 1000d0ca f   CtrlButtonCheckWZ.obj
 0001:0000c1f5       ?Message_MouseMove@CCtrlButtonCheckWZ@@MAE_NPAUSI_MESSAGE@@@Z 1000d1f5 f   CtrlButtonCheckWZ.obj
 0001:0000c20b       ?SetCheckState@CCtrlButtonCheckWZ@@UAEX_N@Z 1000d20b f   CtrlButtonCheckWZ.obj
 0001:0000c222       ?GetCheckState@CCtrlButtonCheckWZ@@UAE_NXZ 1000d222 f   CtrlButtonCheckWZ.obj
 0001:0000c234       ?IsTextReducing@CCtrlButtonWZ@@UBE_NXZ 1000d234 f i CtrlButtonCheckWZ.obj
 0001:0000c246       ?SetTextReducing@CCtrlButtonWZ@@UAEX_N@Z 1000d246 f i CtrlButtonCheckWZ.obj
 0001:0000c25d       ?IsMoneyType@CCtrlButtonWZ@@UBE_NXZ 1000d25d f i CtrlButtonCheckWZ.obj
 0001:0000c26f       ?SetMoneyType@CCtrlButtonWZ@@UAEX_N@Z 1000d26f f i CtrlButtonCheckWZ.obj
 0001:0000c286       ?IsUseDefault@CCtrlButtonWZ@@UBE_NXZ 1000d286 f i CtrlButtonCheckWZ.obj
 0001:0000c298       ?SetUseDefault@CCtrlButtonWZ@@UAEX_N@Z 1000d298 f i CtrlButtonCheckWZ.obj
 0001:0000c2af       ??_ECCtrlButtonCheckWZ@@UAEPAXI@Z 1000d2af f i CtrlButtonCheckWZ.obj
 0001:0000c2af       ??_GCCtrlButtonCheckWZ@@UAEPAXI@Z 1000d2af f i CtrlButtonCheckWZ.obj
 0001:0000c2d6       ??0CCtrlButtonWZ@@QAE@XZ   1000d2d6 f   CtrlButtonWZ.obj
 0001:0000c3a4       ??1CCtrlButtonWZ@@UAE@XZ   1000d3a4 f   CtrlButtonWZ.obj
 0001:0000c3be       ?OnLoad@CCtrlButtonWZ@@UAEXPAX@Z 1000d3be f   CtrlButtonWZ.obj
 0001:0000c6de       ?OnSave@CCtrlButtonWZ@@UAEXPAX@Z 1000d6de f   CtrlButtonWZ.obj
 0001:0000c844       ?OnDraw@CCtrlButtonWZ@@UAE_N_N@Z 1000d844 f   CtrlButtonWZ.obj
 0001:0000cb30       ?SendMessageWZ@CCtrlButtonWZ@@UAE_NPAUSI_MESSAGE@@@Z 1000db30 f   CtrlButtonWZ.obj
 0001:0000cb46       ?GetTextWZW@CCtrlButtonWZ@@UAEXPA_WH@Z 1000db46 f   CtrlButtonWZ.obj
 0001:0000cc59       ?GetTextWZA@CCtrlButtonWZ@@UAEXPADH@Z 1000dc59 f   CtrlButtonWZ.obj
 0001:0000cce2       ?SetTextWZW@CCtrlButtonWZ@@UAEXPB_W_N@Z 1000dce2 f   CtrlButtonWZ.obj
 0001:0000cd63       ?SetTextWZA@CCtrlButtonWZ@@UAEXPBD_N@Z 1000dd63 f   CtrlButtonWZ.obj
 0001:0000ce4a       ?SetTextID@CCtrlButtonWZ@@UAEXK@Z 1000de4a f   CtrlButtonWZ.obj
 0001:0000cf12       ?GetTextID@CCtrlButtonWZ@@UAEKXZ 1000df12 f   CtrlButtonWZ.obj
 0001:0000cf21       ?SetFontID@CCtrlButtonWZ@@UAEXK@Z 1000df21 f   CtrlButtonWZ.obj
 0001:0000cf38       ?GetFontID@CCtrlButtonWZ@@UAEKXZ 1000df38 f   CtrlButtonWZ.obj
 0001:0000cf4a       ?SetTextKind@CCtrlButtonWZ@@UAEXW4ENUM_TEXT_KIND@@@Z 1000df4a f   CtrlButtonWZ.obj
 0001:0000cf61       ?GetTextKind@CCtrlButtonWZ@@UAE?AW4ENUM_TEXT_KIND@@XZ 1000df61 f   CtrlButtonWZ.obj
 0001:0000cf73       ??_GCCtrlButtonWZ@@UAEPAXI@Z 1000df73 f i CtrlButtonWZ.obj
 0001:0000cf73       ??_ECCtrlButtonWZ@@UAEPAXI@Z 1000df73 f i CtrlButtonWZ.obj
 0001:0000cf9a       ??0CCtrlClientWZ@@QAE@XZ   1000df9a f   CtrlClientWZ.obj
 0001:0000cfce       ??1CCtrlClientWZ@@UAE@XZ   1000dfce f   CtrlClientWZ.obj
 0001:0000cfe8       ?OnCreate@CCtrlClientWZ@@UAE_NKKPAUHWND__@@PAUHINSTANCE__@@PAUtagRECT@@PAX@Z 1000dfe8 f   CtrlClientWZ.obj
 0001:0000d03c       ?OnLoad@CCtrlClientWZ@@UAEXPAX@Z 1000e03c f   CtrlClientWZ.obj
 0001:0000e450       ?OnSave@CCtrlClientWZ@@UAEXPAX@Z 1000f450 f   CtrlClientWZ.obj
 0001:0000e48c       ?OnDraw@CCtrlClientWZ@@UAE_N_N@Z 1000f48c f   CtrlClientWZ.obj
 0001:0000e4c9       ?MoveWindowWZ@CCtrlClientWZ@@UAE_NMMMM@Z 1000f4c9 f   CtrlClientWZ.obj
 0001:0000e514       ?GetControlCount@CCtrlClientWZ@@QAEKXZ 1000f514 f   CtrlClientWZ.obj
 0001:0000e51f       ??_GCCtrlClientWZ@@UAEPAXI@Z 1000f51f f i CtrlClientWZ.obj
 0001:0000e51f       ??_ECCtrlClientWZ@@UAEPAXI@Z 1000f51f f i CtrlClientWZ.obj
 0001:0000e546       ??0CCtrlComboBoxWZ@@QAE@XZ 1000f546 f   CtrlComboBox.obj
 0001:0000e563       ??1CCtrlComboBoxWZ@@UAE@XZ 1000f563 f   CtrlComboBox.obj
 0001:0000e57d       ?SendMessageWZ@CCtrlComboBoxWZ@@UAE_NPAUSI_MESSAGE@@@Z 1000f57d f   CtrlComboBox.obj
 0001:0000e58a       ?OnDraw@CCtrlComboBoxWZ@@UAE_N_N@Z 1000f58a f   CtrlComboBox.obj
 0001:0000e5a7       ?OnLoad@CCtrlComboBoxWZ@@UAEXPAX@Z 1000f5a7 f   CtrlComboBox.obj
 0001:0000e5bd       ?OnSave@CCtrlComboBoxWZ@@UAEXPAX@Z 1000f5bd f   CtrlComboBox.obj
 0001:0000e5d3       ??_GCCtrlComboBoxWZ@@UAEPAXI@Z 1000f5d3 f i CtrlComboBox.obj
 0001:0000e5d3       ??_ECCtrlComboBoxWZ@@UAEPAXI@Z 1000f5d3 f i CtrlComboBox.obj
 0001:0000e5fa       ?Dummy_ScriptApplyDigitSubstitution@CUniBuffer@CCtrlDxEditBox@@CGJPBUtag_SCRIPT_DIGITSUBSTITUTE@@PAUtag_SCRIPT_CONTROL@@PAUtag_SCRIPT_STATE@@@Z 1000f5fa f i CtrlDxEdit.obj
 0001:0000e606       ?Dummy_ScriptStringAnalyse@CUniBuffer@CCtrlDxEditBox@@CGJPAUHDC__@@PBXHHHKHPAUtag_SCRIPT_CONTROL@@PAUtag_SCRIPT_STATE@@PBHPAUtag_SCRIPT_TABDEF@@PBEPAPAX@Z 1000f606 f i CtrlDxEdit.obj
 0001:0000e612       ?Dummy_ScriptStringXtoCP@CUniBuffer@CCtrlDxEditBox@@CGJPAXHPAH1@Z 1000f612 f i CtrlDxEdit.obj
 0001:0000e612       ?Dummy_ScriptStringCPtoX@CUniBuffer@CCtrlDxEditBox@@CGJPAXHHPAH@Z 1000f612 f i CtrlDxEdit.obj
 0001:0000e61e       ?Dummy_ScriptStringFree@CUniBuffer@CCtrlDxEditBox@@CGJPAPAX@Z 1000f61e f i CtrlDxEdit.obj
 0001:0000e62a       ?Dummy_ImmDisableTextFrameService@CCtrlDxIMEEditBox@@KGHK@Z 1000f62a f i CtrlDxEdit.obj
 0001:0000e634       ?Dummy_ImmGetCompositionStringW@CCtrlDxIMEEditBox@@KGJPAUHIMC__@@KPAXK@Z 1000f634 f i CtrlDxEdit.obj
 0001:0000e63e       ?Dummy_ImmNotifyIME@CCtrlDxIMEEditBox@@KGHPAUHIMC__@@KKK@Z 1000f63e f i CtrlDxEdit.obj
 0001:0000e63e       ?Dummy_ImmGetCandidateListW@CCtrlDxIMEEditBox@@KGKPAUHIMC__@@KPAUtagCANDIDATELIST@@K@Z 1000f63e f i CtrlDxEdit.obj
 0001:0000e63e       ?Dummy_VerQueryValueA@CCtrlDxIMEEditBox@@KGHQAXPADPAPAXPAI@Z 1000f63e f i CtrlDxEdit.obj
 0001:0000e63e       ?Dummy_GetFileVersionInfoA@CCtrlDxIMEEditBox@@KGHPADKKPAX@Z 1000f63e f i CtrlDxEdit.obj
 0001:0000e647       ?Dummy_ImmSetConversionStatus@CCtrlDxIMEEditBox@@KGHPAUHIMC__@@KK@Z 1000f647 f i CtrlDxEdit.obj
 0001:0000e647       ?Dummy_ImmGetIMEFileNameA@CCtrlDxIMEEditBox@@KGIPAUHKL__@@PADI@Z 1000f647 f i CtrlDxEdit.obj
 0001:0000e647       ?Dummy_ImmGetConversionStatus@CCtrlDxIMEEditBox@@KGHPAUHIMC__@@PAK1@Z 1000f647 f i CtrlDxEdit.obj
 0001:0000e650       ?Dummy_ImmGetVirtualKey@CCtrlDxIMEEditBox@@KGIPAUHWND__@@@Z 1000f650 f i CtrlDxEdit.obj
 0001:0000e650       ?Dummy_ImmUnlockIMCC@CCtrlDxIMEEditBox@@KGHPAUHIMCC__@@@Z 1000f650 f i CtrlDxEdit.obj
 0001:0000e650       ?Dummy_ImmIsIME@CCtrlDxIMEEditBox@@KGHPAUHKL__@@@Z 1000f650 f i CtrlDxEdit.obj
 0001:0000e650       ?Dummy_ImmGetContext@CCtrlDxIMEEditBox@@KGPAUHIMC__@@PAUHWND__@@@Z 1000f650 f i CtrlDxEdit.obj
 0001:0000e650       ?Dummy_ImmLockIMC@CCtrlDxIMEEditBox@@KGPAU__MIDL___MIDL_itf_dimm_0000_0000_0012@@PAUHIMC__@@@Z 1000f650 f i CtrlDxEdit.obj
 0001:0000e650       ?Dummy_ImmGetOpenStatus@CCtrlDxIMEEditBox@@KGHPAUHIMC__@@@Z 1000f650 f i CtrlDxEdit.obj
 0001:0000e650       ?Dummy_ImmGetDefaultIMEWnd@CCtrlDxIMEEditBox@@KGPAUHWND__@@PAU2@@Z 1000f650 f i CtrlDxEdit.obj
 0001:0000e650       ?Dummy_ScriptString_pLogAttr@CUniBuffer@CCtrlDxEditBox@@CGPBUtag_SCRIPT_LOGATTR@@PAX@Z 1000f650 f i CtrlDxEdit.obj
 0001:0000e650       ?Dummy_ImmLockIMCC@CCtrlDxIMEEditBox@@KGPAXPAUHIMCC__@@@Z 1000f650 f i CtrlDxEdit.obj
 0001:0000e650       ?Dummy_ScriptString_pcOutChars@CUniBuffer@CCtrlDxEditBox@@CGPBHPAX@Z 1000f650 f i CtrlDxEdit.obj
 0001:0000e650       ?Dummy_ImmUnlockIMC@CCtrlDxIMEEditBox@@KGHPAUHIMC__@@@Z 1000f650 f i CtrlDxEdit.obj
 0001:0000e659       ?Dummy_GetFileVersionInfoSizeA@CCtrlDxIMEEditBox@@KGKPADPAK@Z 1000f659 f i CtrlDxEdit.obj
 0001:0000e659       ?Dummy_ImmSetOpenStatus@CCtrlDxIMEEditBox@@KGHPAUHIMC__@@H@Z 1000f659 f i CtrlDxEdit.obj
 0001:0000e659       ?Dummy_ShowReadingWindow@CCtrlDxIMEEditBox@@KGHPAUHIMC__@@H@Z 1000f659 f i CtrlDxEdit.obj
 0001:0000e659       ?Dummy_ImmSetCompositionWindow@CCtrlDxIMEEditBox@@KGHPAUHIMC__@@PAUtagCOMPOSITIONFORM@@@Z 1000f659 f i CtrlDxEdit.obj
 0001:0000e659       ?Dummy_ImmGetProperty@CCtrlDxIMEEditBox@@KGKPAUHKL__@@K@Z 1000f659 f i CtrlDxEdit.obj
 0001:0000e659       ?Dummy_ImmSimulateHotKey@CCtrlDxIMEEditBox@@KGHPAUHWND__@@K@Z 1000f659 f i CtrlDxEdit.obj
 0001:0000e659       ?Dummy_ImmReleaseContext@CCtrlDxIMEEditBox@@KGHPAUHWND__@@PAUHIMC__@@@Z 1000f659 f i CtrlDxEdit.obj
 0001:0000e659       ?Dummy_ImmAssociateContext@CCtrlDxIMEEditBox@@KGPAUHIMC__@@PAUHWND__@@PAU2@@Z 1000f659 f i CtrlDxEdit.obj
 0001:0000e662       ?Dummy_GetReadingString@CCtrlDxIMEEditBox@@KGIPAUHIMC__@@IPA_WPAH2PAI@Z 1000f662 f i CtrlDxEdit.obj
 0001:0000e66b       ??0CCtrlDxEditBox@@QAE@XZ  1000f66b f   CtrlDxEdit.obj
 0001:0000e80d       ??1CCtrlDxEditBox@@UAE@XZ  1000f80d f   CtrlDxEdit.obj
 0001:0000e88b       ?OnInitialize@CCtrlDxEditBox@@UAEXXZ 1000f88b f   CtrlDxEdit.obj
 0001:0000e8a6       ?OnCreate@CCtrlDxEditBox@@UAE_NKKPAUHWND__@@PAUHINSTANCE__@@PAUtagRECT@@PAX@Z 1000f8a6 f   CtrlDxEdit.obj
 0001:0000e94d       ?OnDestroy@CCtrlDxEditBox@@UAEXXZ 1000f94d f   CtrlDxEdit.obj
 0001:0000e9a5       ?OnDoAction@CCtrlDxEditBox@@UAEXXZ 1000f9a5 f   CtrlDxEdit.obj
 0001:0000e9e9       ?OnDraw@CCtrlDxEditBox@@UAE_N_N@Z 1000f9e9 f   CtrlDxEdit.obj
 0001:0000f118       ?OnLoad@CCtrlDxEditBox@@UAEXPAX@Z 10010118 f   CtrlDxEdit.obj
 0001:0000f460       ?OnSave@CCtrlDxEditBox@@UAEXPAX@Z 10010460 f   CtrlDxEdit.obj
 0001:0000f556       ?SetStyle@CCtrlDxEditBox@@UAEXK@Z 10010556 f   CtrlDxEdit.obj
 0001:0000f5cf       ?UpdateWindowWZ@CCtrlDxEditBox@@UAEXPAUHWND__@@@Z 100105cf f   CtrlDxEdit.obj
 0001:0000f5e5       ?ReleaseImage@CCtrlDxEditBox@@UAEXXZ 100105e5 f   CtrlDxEdit.obj
 0001:0000f5f6       ?MoveWindowWZ@CCtrlDxEditBox@@UAE_NMMMM@Z 100105f6 f   CtrlDxEdit.obj
 0001:0000f6b8       ?SetFontID@CCtrlDxEditBox@@UAEXK@Z 100106b8 f   CtrlDxEdit.obj
 0001:0000f6fd       ?GetFontID@CCtrlDxEditBox@@UAEKXZ 100106fd f   CtrlDxEdit.obj
 0001:0000f70f       ?SetColorCaret@CCtrlDxEditBox@@UAEXK@Z 1001070f f   CtrlDxEdit.obj
 0001:0000f726       ?SetColorText@CCtrlDxEditBox@@UAEXK@Z 10010726 f   CtrlDxEdit.obj
 0001:0000f73d       ?SetColorSelBack@CCtrlDxEditBox@@UAEXK@Z 1001073d f   CtrlDxEdit.obj
 0001:0000f754       ?SetColorSelText@CCtrlDxEditBox@@UAEXK@Z 10010754 f   CtrlDxEdit.obj
 0001:0000f76b       ?SetTextKind@CCtrlDxEditBox@@UAEXW4ENUM_TEXT_KIND@@@Z 1001076b f   CtrlDxEdit.obj
 0001:0000f782       ?GetTextKind@CCtrlDxEditBox@@UAE?AW4ENUM_TEXT_KIND@@XZ 10010782 f   CtrlDxEdit.obj
 0001:0000f794       ?SetFocusWZ@CCtrlDxEditBox@@UAEXXZ 10010794 f   CtrlDxEdit.obj
 0001:0000f7c8       ?SetLimitText@CCtrlDxEditBox@@UAEXK@Z 100107c8 f   CtrlDxEdit.obj
 0001:0000f7df       ?SetLimitText_MultibyteCheck@CCtrlDxEditBox@@UAEX_N@Z 100107df f   CtrlDxEdit.obj
 0001:0000f7f6       ?SetLimitLine@CCtrlDxEditBox@@UAEXH@Z 100107f6 f   CtrlDxEdit.obj
 0001:0000f81a       ?IsLimitLine@CCtrlDxEditBox@@MAEHXZ 1001081a f   CtrlDxEdit.obj
 0001:0000f825       ?SetTextWZW@CCtrlDxEditBox@@UAEXPB_W_N@Z 10010825 f   CtrlDxEdit.obj
 0001:0000fa81       ?SetTextWZA@CCtrlDxEditBox@@UAEXPBD_N@Z 10010a81 f   CtrlDxEdit.obj
 0001:0000fce8       ?GetTextWZW@CCtrlDxEditBox@@UAEXPA_WH@Z 10010ce8 f   CtrlDxEdit.obj
 0001:0000fec3       ?GetTextWZA@CCtrlDxEditBox@@UAEXPADH@Z 10010ec3 f   CtrlDxEdit.obj
 0001:0000ff7b       ?ClearText@CCtrlDxEditBox@@UAEXXZ 10010f7b f   CtrlDxEdit.obj
 0001:0000ffd3       ?CanHaveFocus@CCtrlDxEditBox@@UAE_NXZ 10010fd3 f   CtrlDxEdit.obj
 0001:0000ffde       ?GetFontColor@CCtrlDxEditBox@@UAEKXZ 10010fde f   CtrlDxEdit.obj
 0001:0000fff0       ?CheckLimitLine@CCtrlDxEditBox@@MAEHXZ 10010ff0 f   CtrlDxEdit.obj
 0001:0000fffb       ?PlaceCaret@CCtrlDxEditBox@@IAEXH@Z 10010ffb f   CtrlDxEdit.obj
 0001:00010167       ?DeleteSelectionText@CCtrlDxEditBox@@IAEXXZ 10011167 f   CtrlDxEdit.obj
 0001:0001024c       ?ResetCaretBlink@CCtrlDxEditBox@@IAEXXZ 1001124c f   CtrlDxEdit.obj
 0001:00010255       ?CopyToClipboard@CCtrlDxEditBox@@IAEXXZ 10011255 f   CtrlDxEdit.obj
 0001:000103b9       ?PasteFromClipboard@CCtrlDxEditBox@@MAEXXZ 100113b9 f   CtrlDxEdit.obj
 0001:000105cf       ?SetTextNCRect@CCtrlDxEditBox@@UAEXHHHH@Z 100115cf f   CtrlDxEdit.obj
 0001:0001060a       ?SendMessageWZ@CCtrlDxEditBox@@UAE_NPAUSI_MESSAGE@@@Z 1001160a f   CtrlDxEdit.obj
 0001:00011d64       ?ParseFloatArray@CCtrlDxEditBox@@QAEXPAMH@Z 10012d64 f   CtrlDxEdit.obj
 0001:00011eaf       ?SetTextFloatArray@CCtrlDxEditBox@@QAEXPBMH@Z 10012eaf f   CtrlDxEdit.obj
 0001:00011f9a       ?InitializeUniscribe@CUniBuffer@CCtrlDxEditBox@@CAXXZ 10012f9a f   CtrlDxEdit.obj
 0001:0001216a       ?UninitializeUniscribe@CUniBuffer@CCtrlDxEditBox@@CAXXZ 1001316a f   CtrlDxEdit.obj
 0001:000121d1       ?Grow@CUniBuffer@CCtrlDxEditBox@@AAE_NH@Z 100131d1 f   CtrlDxEdit.obj
 0001:000122b9       ?Analyse@CUniBuffer@CCtrlDxEditBox@@AAEJXZ 100132b9 f   CtrlDxEdit.obj
 0001:0001238d       ??0CUniBuffer@CCtrlDxEditBox@@QAE@H@Z 1001338d f   CtrlDxEdit.obj
 0001:000123f5       ??1CUniBuffer@CCtrlDxEditBox@@QAE@XZ 100133f5 f   CtrlDxEdit.obj
 0001:00012426       ?SetBufferSize@CUniBuffer@CCtrlDxEditBox@@QAE_NH@Z 10013426 f   CtrlDxEdit.obj
 0001:00012455       ??ACUniBuffer@CCtrlDxEditBox@@QAEAA_WH@Z 10013455 f   CtrlDxEdit.obj
 0001:00012472       ?Clear@CUniBuffer@CCtrlDxEditBox@@QAEXXZ 10013472 f   CtrlDxEdit.obj
 0001:00012493       ?InsertChar@CUniBuffer@CCtrlDxEditBox@@QAE_NH_W@Z 10013493 f   CtrlDxEdit.obj
 0001:00012542       ?RemoveChar@CUniBuffer@CCtrlDxEditBox@@QAE_NH@Z 10013542 f   CtrlDxEdit.obj
 0001:000125ae       ?InsertString@CUniBuffer@CCtrlDxEditBox@@QAE_NHPB_WH@Z 100135ae f   CtrlDxEdit.obj
 0001:00012696       ?SetText@CUniBuffer@CCtrlDxEditBox@@QAE_NPB_W@Z 10013696 f   CtrlDxEdit.obj
 0001:00012778       ?CPtoX@CUniBuffer@CCtrlDxEditBox@@QAEJHHPAH@Z 10013778 f   CtrlDxEdit.obj
 0001:000127c5       ?XtoCP@CUniBuffer@CCtrlDxEditBox@@QAEJHPAH0@Z 100137c5 f   CtrlDxEdit.obj
 0001:0001285f       ?GetPriorItemPos@CUniBuffer@CCtrlDxEditBox@@QAEXHPAH@Z 1001385f f   CtrlDxEdit.obj
 0001:00012942       ?GetNextItemPos@CUniBuffer@CCtrlDxEditBox@@QAEXHPAH@Z 10013942 f   CtrlDxEdit.obj
 0001:00012a57       ?InitializeImm@CCtrlDxIMEEditBox@@CAXXZ 10013a57 f   CtrlDxEdit.obj
 0001:00012fad       ?UninitializeImm@CCtrlDxIMEEditBox@@CAXXZ 10013fad f   CtrlDxEdit.obj
 0001:00013118       ??0CCtrlDxIMEEditBox@@QAE@XZ 10014118 f   CtrlDxEdit.obj
 0001:00013270       ??1CCtrlDxIMEEditBox@@UAE@XZ 10014270 f   CtrlDxEdit.obj
 0001:000132ca       ?OnCreate@CCtrlDxIMEEditBox@@UAE_NKKPAUHWND__@@PAUHINSTANCE__@@PAUtagRECT@@PAX@Z 100142ca f   CtrlDxEdit.obj
 0001:0001333f       ?MoveWindowWZ@CCtrlDxIMEEditBox@@UAE_NMMMM@Z 1001433f f   CtrlDxEdit.obj
 0001:000133f1       ?OnLoad@CCtrlDxIMEEditBox@@UAEXPAX@Z 100143f1 f   CtrlDxEdit.obj
 0001:000135a0       ?OnSave@CCtrlDxIMEEditBox@@UAEXPAX@Z 100145a0 f   CtrlDxEdit.obj
 0001:0001367a       ?OnDestroy@CCtrlDxIMEEditBox@@UAEXXZ 1001467a f   CtrlDxEdit.obj
 0001:00013699       ?SetHeight@CCtrlDxIMEEditBox@@UAEXK@Z 10014699 f   CtrlDxEdit.obj
 0001:000136a4       ?OnDoAction@CCtrlDxIMEEditBox@@UAEXXZ 100146a4 f   CtrlDxEdit.obj
 0001:000137c6       ?OnDraw@CCtrlDxIMEEditBox@@UAE_N_N@Z 100147c6 f   CtrlDxEdit.obj
 0001:000138a3       ?SendMessageWZ@CCtrlDxIMEEditBox@@UAE_NPAUSI_MESSAGE@@@Z 100148a3 f   CtrlDxEdit.obj
 0001:00015112       ?SendKey@CCtrlDxIMEEditBox@@KAXE@Z 10016112 f   CtrlDxEdit.obj
 0001:00015135       ?StaticOnCreateDevice@CCtrlDxIMEEditBox@@SAJPAUHWND__@@@Z 10016135 f   CtrlDxEdit.obj
 0001:000151af       ?GetImeId@CCtrlDxIMEEditBox@@KAKI@Z 100161af f   CtrlDxEdit.obj
 0001:00015536       ?RenderCandidateReadingWindow@CCtrlDxIMEEditBox@@MAEX_N@Z 10016536 f   CtrlDxEdit.obj
 0001:00015cc5       ?RenderComposition@CCtrlDxIMEEditBox@@MAEXXZ 10016cc5 f   CtrlDxEdit.obj
 0001:00016256       ?RenderIndicator@CCtrlDxIMEEditBox@@MAEXXZ 10017256 f   CtrlDxEdit.obj
 0001:0001634a       ?CheckInputLocale@CCtrlDxIMEEditBox@@KAXXZ 1001734a f   CtrlDxEdit.obj
 0001:000164a9       ?CheckToggleState@CCtrlDxIMEEditBox@@KAXXZ 100174a9 f   CtrlDxEdit.obj
 0001:00016588       ?EnableImeSystem@CCtrlDxIMEEditBox@@SAX_N@Z 10017588 f   CtrlDxEdit.obj
 0001:00016595       ?SetupImeApi@CCtrlDxIMEEditBox@@KAXXZ 10017595 f   CtrlDxEdit.obj
 0001:0001663e       ?ResetCompositionString@CCtrlDxIMEEditBox@@IAEXXZ 1001763e f   CtrlDxEdit.obj
 0001:00016675       ?TruncateCompString@CCtrlDxIMEEditBox@@IAEX_NH@Z 10017675 f   CtrlDxEdit.obj
 0001:000167de       ?SendCompString@CCtrlDxIMEEditBox@@IAEXXZ 100177de f   CtrlDxEdit.obj
 0001:00016871       ?FinalizeString@CCtrlDxIMEEditBox@@IAEX_N@Z 10017871 f   CtrlDxEdit.obj
 0001:00016965       ?GetReadingWindowOrientation@CCtrlDxIMEEditBox@@KAXK@Z 10017965 f   CtrlDxEdit.obj
 0001:00016aee       ?GetPrivateReadingString@CCtrlDxIMEEditBox@@KAXXZ 10017aee f   CtrlDxEdit.obj
 0001:000171bc       ?PumpMessage@CCtrlDxIMEEditBox@@QAEXXZ 100181bc f   CtrlDxEdit.obj
 0001:00017212       ?OnFocusIn@CCtrlDxIMEEditBox@@UAEXXZ 10018212 f   CtrlDxEdit.obj
 0001:00017293       ?OnFocusOut@CCtrlDxIMEEditBox@@UAEXXZ 10018293 f   CtrlDxEdit.obj
 0001:000172c9       ??0CCtrlMultilineEditWZ@@QAE@XZ 100182c9 f   CtrlDxEdit.obj
 0001:00017380       ??1CCtrlMultilineEditWZ@@UAE@XZ 10018380 f   CtrlDxEdit.obj
 0001:0001740f       ?OnCreate@CCtrlMultilineEditWZ@@UAE_NKKPAUHWND__@@PAUHINSTANCE__@@PAUtagRECT@@PAX@Z 1001840f f   CtrlDxEdit.obj
 0001:000175e2       ?OnDestroy@CCtrlMultilineEditWZ@@UAEXXZ 100185e2 f   CtrlDxEdit.obj
 0001:00017618       ?MoveWindowWZ@CCtrlMultilineEditWZ@@UAE_NMMMM@Z 10018618 f   CtrlDxEdit.obj
 0001:0001773b       ?OnDraw@CCtrlMultilineEditWZ@@UAE_N_N@Z 1001873b f   CtrlDxEdit.obj
 0001:000186af       ?RenderComposition@CCtrlMultilineEditWZ@@MAEXXZ 100196af f   CtrlDxEdit.obj
 0001:00018eaa       ?RenderCandidateReadingWindow@CCtrlMultilineEditWZ@@MAEX_N@Z 10019eaa f   CtrlDxEdit.obj
 0001:00019791       ?ResetLineInfo@CCtrlMultilineEditWZ@@IAEXH@Z 1001a791 f   CtrlDxEdit.obj
 0001:00019c0d       ?SendMessageWZ@CCtrlMultilineEditWZ@@UAE_NPAUSI_MESSAGE@@@Z 1001ac0d f   CtrlDxEdit.obj
 0001:0001df50       ?IsLimitLine@CCtrlMultilineEditWZ@@MAEHXZ 1001ef50 f   CtrlDxEdit.obj
 0001:0001df98       ?CheckLimitLine@CCtrlMultilineEditWZ@@MAEHXZ 1001ef98 f   CtrlDxEdit.obj
 0001:0001e172       ?PasteFromClipboard@CCtrlMultilineEditWZ@@MAEXXZ 1001f172 f   CtrlDxEdit.obj
 0001:0001e387       ?OnLoad@CCtrlMultilineEditWZ@@UAEXPAX@Z 1001f387 f   CtrlDxEdit.obj
 0001:0001e3b5       ?OnSave@CCtrlMultilineEditWZ@@UAEXPAX@Z 1001f3b5 f   CtrlDxEdit.obj
 0001:0001e3e3       ?UpdateWindowWZ@CCtrlMultilineEditWZ@@UAEXPAUHWND__@@@Z 1001f3e3 f   CtrlDxEdit.obj
 0001:0001e411       ?ReleaseImage@CCtrlMultilineEditWZ@@UAEXXZ 1001f411 f   CtrlDxEdit.obj
 0001:0001e437       ?SetFontID@CCtrlMultilineEditWZ@@UAEXK@Z 1001f437 f   CtrlDxEdit.obj
 0001:0001e4a4       ?SetTextWZA@CCtrlMultilineEditWZ@@UAEXPBD_N@Z 1001f4a4 f   CtrlDxEdit.obj
 0001:0001e543       ?SetTextWZW@CCtrlMultilineEditWZ@@UAEXPB_W_N@Z 1001f543 f   CtrlDxEdit.obj
 0001:0001e5e2       ?ClearText@CCtrlMultilineEditWZ@@UAEXXZ 1001f5e2 f   CtrlDxEdit.obj
 0001:0001e642       ?SetFocusWZ@CCtrlMultilineEditWZ@@UAEXXZ 1001f642 f   CtrlDxEdit.obj
 0001:0001e653       ?SetHeight@CCtrlMultilineEditWZ@@UAEXK@Z 1001f653 f   CtrlDxEdit.obj
 0001:0001e68f       ?SetVScrollBaseImageFormat@CCtrlMultilineEditWZ@@UAEXPAUSI_TFORMAT@@@Z 1001f68f f   CtrlDxEdit.obj
 0001:0001e6b2       ?SetVScrollArrowUPBTImageFormat@CCtrlMultilineEditWZ@@UAEXPAUSI_TFORMAT@@@Z 1001f6b2 f   CtrlDxEdit.obj
 0001:0001e6d8       ?SetVScrollArrowDownBTImageFormat@CCtrlMultilineEditWZ@@UAEXPAUSI_TFORMAT@@@Z 1001f6d8 f   CtrlDxEdit.obj
 0001:0001e6fe       ?SetVScrollArrowThumbBTImageFormat@CCtrlMultilineEditWZ@@UAEXPAUSI_TFORMAT@@@Z 1001f6fe f   CtrlDxEdit.obj
 0001:0001e724       ?GetVScrollBaseImageFormat@CCtrlMultilineEditWZ@@UAEPAUSI_TFORMAT@@XZ 1001f724 f   CtrlDxEdit.obj
 0001:0001e742       ?GetVScrollArrowUPBTImageFormat@CCtrlMultilineEditWZ@@UAEPAUSI_TFORMAT@@XZ 1001f742 f   CtrlDxEdit.obj
 0001:0001e763       ?GetVScrollArrowDownBTImageFormat@CCtrlMultilineEditWZ@@UAEPAUSI_TFORMAT@@XZ 1001f763 f   CtrlDxEdit.obj
 0001:0001e784       ?GetVScrollArrowThumbBTImageFormat@CCtrlMultilineEditWZ@@UAEPAUSI_TFORMAT@@XZ 1001f784 f   CtrlDxEdit.obj
 0001:0001e7a5       ?SetVScrollBaseIsOutline@CCtrlMultilineEditWZ@@UAEX_N@Z 1001f7a5 f   CtrlDxEdit.obj
 0001:0001e7cb       ?GetVScrollBaseIsOutline@CCtrlMultilineEditWZ@@UAE_NXZ 1001f7cb f   CtrlDxEdit.obj
 0001:0001e7ec       ?SetVScrollBaseOutlineColor@CCtrlMultilineEditWZ@@UAEXK@Z 1001f7ec f   CtrlDxEdit.obj
 0001:0001e812       ?GetVScrollBaseOutlineColor@CCtrlMultilineEditWZ@@UAEKXZ 1001f812 f   CtrlDxEdit.obj
 0001:0001e833       ?SetVScrollArrowUPBTIsOutline@CCtrlMultilineEditWZ@@UAEX_N@Z 1001f833 f   CtrlDxEdit.obj
 0001:0001e859       ?GetVScrollArrowUPBTIsOutline@CCtrlMultilineEditWZ@@UAE_NXZ 1001f859 f   CtrlDxEdit.obj
 0001:0001e87a       ?SetVScrollArrowUPBTOutlineColor@CCtrlMultilineEditWZ@@UAEXK@Z 1001f87a f   CtrlDxEdit.obj
 0001:0001e8a0       ?GetVScrollArrowUPBTOutlineColor@CCtrlMultilineEditWZ@@UAEKXZ 1001f8a0 f   CtrlDxEdit.obj
 0001:0001e8c1       ?SetVScrollArrowDownBTIsOutline@CCtrlMultilineEditWZ@@UAEX_N@Z 1001f8c1 f   CtrlDxEdit.obj
 0001:0001e8e7       ?GetVScrollArrowDownBTIsOutline@CCtrlMultilineEditWZ@@UAE_NXZ 1001f8e7 f   CtrlDxEdit.obj
 0001:0001e908       ?SetVScrollArrowDownBTOutlineColor@CCtrlMultilineEditWZ@@UAEXK@Z 1001f908 f   CtrlDxEdit.obj
 0001:0001e92e       ?GetVScrollArrowDownBTOutlineColor@CCtrlMultilineEditWZ@@UAEKXZ 1001f92e f   CtrlDxEdit.obj
 0001:0001e94f       ?SetVScrollArrowThumbBTIsOutline@CCtrlMultilineEditWZ@@UAEX_N@Z 1001f94f f   CtrlDxEdit.obj
 0001:0001e975       ?GetVScrollArrowThumbBTIsOutline@CCtrlMultilineEditWZ@@UAE_NXZ 1001f975 f   CtrlDxEdit.obj
 0001:0001e996       ?SetVScrollArrowThumbBTOutlineColor@CCtrlMultilineEditWZ@@UAEXK@Z 1001f996 f   CtrlDxEdit.obj
 0001:0001e9bc       ?GetVScrollArrowThumbBTOutlineColor@CCtrlMultilineEditWZ@@UAEKXZ 1001f9bc f   CtrlDxEdit.obj
 0001:0001e9dd       ??1CCtrlBaseEdit@@UAE@XZ   1001f9dd f i CtrlDxEdit.obj
 0001:0001e9f7       ?SetTextID@CControlWZ@@UAEXK@Z 1001f9f7 f i ControlWZ.obj
 0001:0001e9f7       ?SetColorText@CCtrlBaseEdit@@UAEXK@Z 1001f9f7 f i CtrlDxEdit.obj
 0001:0001e9f7       ?SetColorCompText@CCtrlBaseEdit@@UAEXK@Z 1001f9f7 f i CtrlDxEdit.obj
 0001:0001e9f7       ?SetColorCaret@CCtrlBaseEdit@@UAEXK@Z 1001f9f7 f i CtrlDxEdit.obj
 0001:0001e9f7       ?SetTextReducing@CControlWZ@@UAEX_N@Z 1001f9f7 f i ControlWZ.obj
 0001:0001e9f7       ?SetColorCompCaret@CCtrlBaseEdit@@UAEXK@Z 1001f9f7 f i CtrlDxEdit.obj
 0001:0001e9f7       ?SetUseIndicator@CCtrlBaseEdit@@UAEX_N@Z 1001f9f7 f i CtrlDxEdit.obj
 0001:0001e9f7       ?SetFontID@CControlWZ@@UAEXK@Z 1001f9f7 f i ControlWZ.obj
 0001:0001e9f7       ?SetUseDefault@CControlWZ@@UAEX_N@Z 1001f9f7 f i ControlWZ.obj
 0001:0001e9f7       ?SetLimitText@CCtrlBaseEdit@@UAEXK@Z 1001f9f7 f i CtrlDxEdit.obj
 0001:0001e9f7       ?SetColorCompBack@CCtrlBaseEdit@@UAEXK@Z 1001f9f7 f i CtrlDxEdit.obj
 0001:0001e9f7       ?SetColorIndicatorIme@CCtrlBaseEdit@@UAEXK@Z 1001f9f7 f i CtrlDxEdit.obj
 0001:0001e9f7       ?SetFontInfo@CCtrlBaseEdit@@UAEXPAUtagLOGFONTA@@@Z 1001f9f7 f i CtrlDxEdit.obj
 0001:0001e9f7       ?SetColorIndicatorEng@CCtrlBaseEdit@@UAEXK@Z 1001f9f7 f i CtrlDxEdit.obj
 0001:0001e9f7       ?SetColorSelText@CCtrlBaseEdit@@UAEXK@Z 1001f9f7 f i CtrlDxEdit.obj
 0001:0001e9f7       ?SetMoneyType@CControlWZ@@UAEX_N@Z 1001f9f7 f i ControlWZ.obj
 0001:0001e9f7       ?SetTextOutlineColor@CCtrlBaseEdit@@UAEXK@Z 1001f9f7 f i CtrlDxEdit.obj
 0001:0001e9f7       ?SetFontInfo@CCtrlEditWZ@@UAEXPAUtagLOGFONTA@@@Z 1001f9f7 f i CtrlEditWZ.obj
 0001:0001e9f7       ?SetColorSelBack@CCtrlBaseEdit@@UAEXK@Z 1001f9f7 f i CtrlDxEdit.obj
 0001:0001e9f7       ?SetColorIndicatorBK@CCtrlBaseEdit@@UAEXK@Z 1001f9f7 f i CtrlDxEdit.obj
 0001:0001e9f7       ?SetTextKind@CCtrlBaseEdit@@UAEXW4ENUM_TEXT_KIND@@@Z 1001f9f7 f i CtrlDxEdit.obj
 0001:0001e9f7       ?SetFontID@CCtrlBaseEdit@@UAEXK@Z 1001f9f7 f i CtrlDxEdit.obj
 0001:0001ea02       ?GetIndicatorImeColor@CCtrlBaseEdit@@UAEKXZ 1001fa02 f i CtrlDxEdit.obj
 0001:0001ea02       ?GetFontInfo@CCtrlBaseEdit@@UAEPAUtagLOGFONTA@@XZ 1001fa02 f i CtrlDxEdit.obj
 0001:0001ea02       ?GetFontID@CControlWZ@@UAEKXZ 1001fa02 f i ControlWZ.obj
 0001:0001ea02       ?GetIndicatorEngColor@CCtrlBaseEdit@@UAEKXZ 1001fa02 f i CtrlDxEdit.obj
 0001:0001ea02       ?GetEditHwnd@CCtrlBaseEdit@@UAEPAUHWND__@@XZ 1001fa02 f i CtrlDxEdit.obj
 0001:0001ea02       ?GetIndicatorBKColor@CCtrlBaseEdit@@UAEKXZ 1001fa02 f i CtrlDxEdit.obj
 0001:0001ea02       ?GetFontColor@CCtrlBaseEdit@@UAEKXZ 1001fa02 f i CtrlDxEdit.obj
 0001:0001ea02       ?GetFontID@CCtrlBaseEdit@@UAEKXZ 1001fa02 f i CtrlDxEdit.obj
 0001:0001ea02       ?GetSelTextColor@CCtrlBaseEdit@@UAEKXZ 1001fa02 f i CtrlDxEdit.obj
 0001:0001ea02       ?GetCaretColor@CCtrlBaseEdit@@UAEKXZ 1001fa02 f i CtrlDxEdit.obj
 0001:0001ea02       ?GetSelBackColor@CCtrlBaseEdit@@UAEKXZ 1001fa02 f i CtrlDxEdit.obj
 0001:0001ea02       ?GetCompCaretColor@CCtrlBaseEdit@@UAEKXZ 1001fa02 f i CtrlDxEdit.obj
 0001:0001ea02       ?GetTextID@CControlWZ@@UAEKXZ 1001fa02 f i ControlWZ.obj
 0001:0001ea02       ?GetEditHwnd@CCtrlEditWZ@@UAEPAUHWND__@@XZ 1001fa02 f i CtrlEditWZ.obj
 0001:0001ea02       ?GetTextKind@CCtrlBaseEdit@@UAE?AW4ENUM_TEXT_KIND@@XZ 1001fa02 f i CtrlDxEdit.obj
 0001:0001ea02       ?GetCompTextColor@CCtrlBaseEdit@@UAEKXZ 1001fa02 f i CtrlDxEdit.obj
 0001:0001ea02       ?GetCompBackColor@CCtrlBaseEdit@@UAEKXZ 1001fa02 f i CtrlDxEdit.obj
 0001:0001ea0d       ?SetTextNCRect@CCtrlBaseEdit@@UAEXHHHH@Z 1001fa0d f i CtrlDxEdit.obj
 0001:0001ea18       ?GetTextOutlineColor@CCtrlBaseEdit@@UAEKXZ 1001fa18 f i CtrlDxEdit.obj
 0001:0001ea26       ??_GCCtrlBaseEdit@@UAEPAXI@Z 1001fa26 f i CtrlDxEdit.obj
 0001:0001ea26       ??_ECCtrlBaseEdit@@UAEPAXI@Z 1001fa26 f i CtrlDxEdit.obj
 0001:0001ea56       ?GetCaretColor@CCtrlDxEditBox@@UAEKXZ 1001fa56 f i CtrlDxEdit.obj
 0001:0001ea56       ?GetThickness@CCtrlRectangleWZ@@UAEHXZ 1001fa56 f i CtrlRectangleWZ.obj
 0001:0001ea68       ?GetSelBackColor@CCtrlDxEditBox@@UAEKXZ 1001fa68 f i CtrlDxEdit.obj
 0001:0001ea7a       ?GetSelTextColor@CCtrlDxEditBox@@UAEKXZ 1001fa7a f i CtrlDxEdit.obj
 0001:0001ea8c       ?SetTextOutlineColor@CCtrlDxEditBox@@UAEXK@Z 1001fa8c f i CtrlDxEdit.obj
 0001:0001eaa3       ?GetTextOutlineColor@CCtrlDxEditBox@@UAEKXZ 1001faa3 f i CtrlDxEdit.obj
 0001:0001eab5       ?IsNumberic@CCtrlDxEditBox@@UBE_NXZ 1001fab5 f i CtrlDxEdit.obj
 0001:0001eac7       ?SetNumberic@CCtrlDxEditBox@@UAEX_N@Z 1001fac7 f i CtrlDxEdit.obj
 0001:0001eade       ??_GCCtrlDxEditBox@@UAEPAXI@Z 1001fade f i CtrlDxEdit.obj
 0001:0001eade       ??_ECCtrlDxEditBox@@UAEPAXI@Z 1001fade f i CtrlDxEdit.obj
 0001:0001eb05       ?HaveFocus@CCtrlDxIMEEditBox@@UAE_NXZ 1001fb05 f i CtrlDxEdit.obj
 0001:0001eb05       ?HaveFocus@CCtrlEditWZ@@UAE_NXZ 1001fb05 f i CtrlEditWZ.obj
 0001:0001eb17       ?SetColorCompText@CCtrlDxIMEEditBox@@UAEXK@Z 1001fb17 f i CtrlDxEdit.obj
 0001:0001eb2e       ?SetColorCompBack@CCtrlDxIMEEditBox@@UAEXK@Z 1001fb2e f i CtrlDxEdit.obj
 0001:0001eb45       ?SetColorCompCaret@CCtrlDxIMEEditBox@@UAEXK@Z 1001fb45 f i CtrlDxEdit.obj
 0001:0001eb5c       ?SetColorIndicatorIme@CCtrlDxIMEEditBox@@UAEXK@Z 1001fb5c f i CtrlDxEdit.obj
 0001:0001eb73       ?SetColorIndicatorEng@CCtrlDxIMEEditBox@@UAEXK@Z 1001fb73 f i CtrlDxEdit.obj
 0001:0001eb8a       ?SetColorIndicatorBK@CCtrlDxIMEEditBox@@UAEXK@Z 1001fb8a f i CtrlDxEdit.obj
 0001:0001eba1       ?GetCompTextColor@CCtrlDxIMEEditBox@@UAEKXZ 1001fba1 f i CtrlDxEdit.obj
 0001:0001ebb3       ?GetCompBackColor@CCtrlDxIMEEditBox@@UAEKXZ 1001fbb3 f i CtrlDxEdit.obj
 0001:0001ebc5       ?GetCompCaretColor@CCtrlDxIMEEditBox@@UAEKXZ 1001fbc5 f i CtrlDxEdit.obj
 0001:0001ebd7       ?GetIndicatorImeColor@CCtrlDxIMEEditBox@@UAEKXZ 1001fbd7 f i CtrlDxEdit.obj
 0001:0001ebe9       ?GetIndicatorEngColor@CCtrlDxIMEEditBox@@UAEKXZ 1001fbe9 f i CtrlDxEdit.obj
 0001:0001ebfb       ?GetIndicatorBKColor@CCtrlDxIMEEditBox@@UAEKXZ 1001fbfb f i CtrlDxEdit.obj
 0001:0001ec0d       ?SetUseIndicator@CCtrlDxIMEEditBox@@UAEX_N@Z 1001fc0d f i CtrlDxEdit.obj
 0001:0001ec24       ?GetUseIndicator@CCtrlDxIMEEditBox@@UAE_NXZ 1001fc24 f i CtrlDxEdit.obj
 0001:0001ec36       ??_GCCtrlDxIMEEditBox@@UAEPAXI@Z 1001fc36 f i CtrlDxEdit.obj
 0001:0001ec36       ??_ECCtrlDxIMEEditBox@@UAEPAXI@Z 1001fc36 f i CtrlDxEdit.obj
 0001:0001ec5d       ?GetVScroll@CCtrlMultilineEditWZ@@UAEPAVCCtrlVScrollWZ@@XZ 1001fc5d f i CtrlDxEdit.obj
 0001:0001ec6e       ??_GCCtrlMultilineEditWZ@@UAEPAXI@Z 1001fc6e f i CtrlDxEdit.obj
 0001:0001ec6e       ??_ECCtrlMultilineEditWZ@@UAEPAXI@Z 1001fc6e f i CtrlDxEdit.obj
 0001:0001ec95       ?erase@?$basic_string@DU?$char_traits@D@std@@V?$allocator@D@2@@std@@QAE?AV?$_String_iterator@DU?$char_traits@D@std@@V?$allocator@D@2@@2@V?$_String_const_iterator@DU?$char_traits@D@std@@V?$allocator@D@2@@2@@Z 1001fc95 f i CtrlDxEdit.obj
 0001:0001ed51       ??0?$vector@KV?$allocator@K@std@@@std@@QAE@XZ 1001fd51 f i CtrlDxEdit.obj
 0001:0001edd3       ??1?$vector@KV?$allocator@K@std@@@std@@QAE@XZ 1001fdd3 f i CtrlDxEdit.obj
 0001:0001ee29       ?push_back@?$vector@KV?$allocator@K@std@@@std@@QAEXABK@Z 1001fe29 f i CtrlDxEdit.obj
 0001:0001eef3       ?pop_back@?$vector@KV?$allocator@K@std@@@std@@QAEXXZ 1001fef3 f i CtrlDxEdit.obj
 0001:0001ef4f       ?clear@?$vector@KV?$allocator@K@std@@@std@@QAEXXZ 1001ff4f f i CtrlDxEdit.obj
 0001:0001efa0       ?insert@?$basic_string@DU?$char_traits@D@std@@V?$allocator@D@2@@std@@QAEAAV12@IPBDI@Z 1001ffa0 f i CtrlDxEdit.obj
 0001:0001f150       ?end@?$list@KV?$allocator@K@std@@@std@@QAE?AV?$_Iterator@$00@12@XZ 10020150 f i BaseManager.obj
 0001:0001f150       ?end@?$list@PAVCControlWZ@@V?$allocator@PAVCControlWZ@@@std@@@std@@QAE?AV?$_Iterator@$00@12@XZ 10020150 f i CtrlDxEdit.obj
 0001:0001f150       ?end@?$list@PAXV?$allocator@PAX@std@@@std@@QAE?AV?$_Iterator@$00@12@XZ 10020150 f i CtrlListWZ.obj
 0001:0001f150       ?end@?$list@UtagRECT@@V?$allocator@UtagRECT@@@std@@@std@@QAE?AV?$_Iterator@$00@12@XZ 10020150 f i DialogWZ.obj
 0001:0001f195       ?erase@?$list@KV?$allocator@K@std@@@std@@QAE?AV?$_Iterator@$00@12@V?$_Const_iterator@$00@12@@Z 10020195 f i BaseManager.obj
 0001:0001f195       ?erase@?$list@PAXV?$allocator@PAX@std@@@std@@QAE?AV?$_Iterator@$00@12@V?$_Const_iterator@$00@12@@Z 10020195 f i CtrlListWZ.obj
 0001:0001f195       ?erase@?$list@PAVCControlWZ@@V?$allocator@PAVCControlWZ@@@std@@@std@@QAE?AV?$_Iterator@$00@12@V?$_Const_iterator@$00@12@@Z 10020195 f i CtrlDxEdit.obj
 0001:0001f195       ?erase@?$list@U?$pair@$$CBKPAX@std@@V?$allocator@U?$pair@$$CBKPAX@std@@@2@@std@@QAE?AV?$_Iterator@$00@12@V?$_Const_iterator@$00@12@@Z 10020195 f i BaseManager.obj
 0001:0001f246       ?insert@?$vector@KV?$allocator@K@std@@@std@@QAE?AV?$_Vector_iterator@KV?$allocator@K@std@@@2@V?$_Vector_const_iterator@KV?$allocator@K@std@@@2@ABK@Z 10020246 f i CtrlDxEdit.obj
 0001:0001f2d6       ?erase@?$vector@KV?$allocator@K@std@@@std@@QAE?AV?$_Vector_iterator@KV?$allocator@K@std@@@2@V?$_Vector_const_iterator@KV?$allocator@K@std@@@2@0@Z 100202d6 f i CtrlDxEdit.obj
 0001:0001f366       ?_Buy@?$vector@KV?$allocator@K@std@@@std@@IAE_NI@Z 10020366 f i CtrlDxEdit.obj
 0001:0001f418       ?_Tidy@?$vector@KV?$allocator@K@std@@@std@@IAEXXZ 10020418 f i CtrlDxEdit.obj
 0001:0001f489       ?insert@?$basic_string@DU?$char_traits@D@std@@V?$allocator@D@2@@std@@QAEAAV12@IABV12@II@Z 10020489 f i CtrlDxEdit.obj
 0001:0001f6d3       ?_Insert_n@?$vector@KV?$allocator@K@std@@@std@@IAEXV?$_Vector_const_iterator@KV?$allocator@K@std@@@2@IABK@Z 100206d3 f i CtrlDxEdit.obj
 0001:0001fce1       ?_Xlen@?$vector@U_List_position@?$_Hash@V?$_Hmap_traits@KV?$basic_string@DU?$char_traits@D@std@@V?$allocator@D@2@@std@@V?$hash_compare@KU?$less@K@std@@@stdext@@V?$allocator@U?$pair@$$CBKV?$basic_string@DU?$char_traits@D@std@@V?$allocator@D@2@@std@@@std@@@2@$0A@@stdext@@@stdext@@V?$allocator@U_List_position@?$_Hash@V?$_Hmap_traits@KV?$basic_string@DU?$char_traits@D@std@@V?$allocator@D@2@@std@@V?$hash_compare@KU?$less@K@std@@@stdext@@V?$allocator@U?$pair@$$CBKV?$basic_string@DU?$char_traits@D@std@@V?$allocator@D@2@@std@@@std@@@2@$0A@@stdext@@@stdext@@@std@@@std@@KAXXZ 10020ce1 f i StringManager.obj
 0001:0001fce1       ?_Xlen@?$vector@KV?$allocator@K@std@@@std@@KAXXZ 10020ce1 f i CtrlDxEdit.obj
 0001:0001fce1       ?_Xlen@?$vector@U_List_position@?$_Hash@V?$_Hmap_traits@KPAXV?$hash_compare@KU?$less@K@std@@@stdext@@V?$allocator@U?$pair@$$CBKPAX@std@@@std@@$0A@@stdext@@@stdext@@V?$allocator@U_List_position@?$_Hash@V?$_Hmap_traits@KPAXV?$hash_compare@KU?$less@K@std@@@stdext@@V?$allocator@U?$pair@$$CBKPAX@std@@@std@@$0A@@stdext@@@stdext@@@std@@@std@@KAXXZ 10020ce1 f i BaseManager.obj
 0001:0001fd58       ??Y?$_String_const_iterator@DU?$char_traits@D@std@@V?$allocator@D@2@@std@@QAEAAV01@H@Z 10020d58 f i CtrlDxEdit.obj
 0001:0001fe17       ??D?$_Const_iterator@$00@?$list@U?$pair@$$CBKPAX@std@@V?$allocator@U?$pair@$$CBKPAX@std@@@2@@std@@QBEABU?$pair@$$CBKPAX@2@XZ 10020e17 f i BaseManager.obj
 0001:0001fe17       ??D?$_Const_iterator@$00@?$list@PAVCControlWZ@@V?$allocator@PAVCControlWZ@@@std@@@std@@QBEABQAVCControlWZ@@XZ 10020e17 f i CtrlDxEdit.obj
 0001:0001fe17       ??D?$_Const_iterator@$00@?$list@U?$pair@$$CBKV?$basic_string@DU?$char_traits@D@std@@V?$allocator@D@2@@std@@@std@@V?$allocator@U?$pair@$$CBKV?$basic_string@DU?$char_traits@D@std@@V?$allocator@D@2@@std@@@std@@@2@@std@@QBEABU?$pair@$$CBKV?$basic_string@DU?$char_traits@D@std@@V?$allocator@D@2@@std@@@2@XZ 10020e17 f i StringManager.obj
 0001:0001fe17       ??D?$_Const_iterator@$00@?$list@PAXV?$allocator@PAX@std@@@std@@QBEABQAXXZ 10020e17 f i CtrlListWZ.obj
 0001:0001fe17       ??D?$_Const_iterator@$00@?$list@KV?$allocator@K@std@@@std@@QBEABKXZ 10020e17 f i BaseManager.obj
 0001:0001fe17       ??D?$_Const_iterator@$00@?$list@UtagRECT@@V?$allocator@UtagRECT@@@std@@@std@@QBEABUtagRECT@@XZ 10020e17 f i DialogWZ.obj
 0001:0001fe8b       ??G?$_Vector_const_iterator@KV?$allocator@K@std@@@std@@QBEHABV01@@Z 10020e8b f i CtrlDxEdit.obj
 0001:0001fed6       ??0?$_Vector_const_iterator@U_List_position@?$_Hash@V?$_Hmap_traits@KV?$basic_string@DU?$char_traits@D@std@@V?$allocator@D@2@@std@@V?$hash_compare@KU?$less@K@std@@@stdext@@V?$allocator@U?$pair@$$CBKV?$basic_string@DU?$char_traits@D@std@@V?$allocator@D@2@@std@@@std@@@2@$0A@@stdext@@@stdext@@V?$allocator@U_List_position@?$_Hash@V?$_Hmap_traits@KV?$basic_string@DU?$char_traits@D@std@@V?$allocator@D@2@@std@@V?$hash_compare@KU?$less@K@std@@@stdext@@V?$allocator@U?$pair@$$CBKV?$basic_string@DU?$char_traits@D@std@@V?$allocator@D@2@@std@@@std@@@2@$0A@@stdext@@@stdext@@@std@@@std@@QAE@PAU_List_position@?$_Hash@V?$_Hmap_traits@KV?$basic_string@DU?$char_traits@D@std@@V?$allocator@D@2@@std@@V?$hash_compare@KU?$less@K@std@@@stdext@@V?$allocator@U?$pair@$$CBKV?$basic_string@DU?$char_traits@D@std@@V?$allocator@D@2@@std@@@std@@@2@$0A@@stdext@@@stdext@@PBV_Container_base_aux@1@@Z 10020ed6 f i StringManager.obj
 0001:0001fed6       ??0?$_Vector_const_iterator@KV?$allocator@K@std@@@std@@QAE@PAKPBV_Container_base_aux@1@@Z 10020ed6 f i CtrlDxEdit.obj
 0001:0001fed6       ??0?$_Vector_const_iterator@U_List_position@?$_Hash@V?$_Hmap_traits@KPAXV?$hash_compare@KU?$less@K@std@@@stdext@@V?$allocator@U?$pair@$$CBKPAX@std@@@std@@$0A@@stdext@@@stdext@@V?$allocator@U_List_position@?$_Hash@V?$_Hmap_traits@KPAXV?$hash_compare@KU?$less@K@std@@@stdext@@V?$allocator@U?$pair@$$CBKPAX@std@@@std@@$0A@@stdext@@@stdext@@@std@@@std@@QAE@PAU_List_position@?$_Hash@V?$_Hmap_traits@KPAXV?$hash_compare@KU?$less@K@std@@@stdext@@V?$allocator@U?$pair@$$CBKPAX@std@@@std@@$0A@@stdext@@@stdext@@PBV_Container_base_aux@1@@Z 10020ed6 f i BaseManager.obj
 0001:0001ff22       ??Y?$_Vector_const_iterator@KV?$allocator@K@std@@@std@@QAEAAV01@H@Z 10020f22 f i CtrlDxEdit.obj
 0001:0001ffd8       ?SetSize@?$CGrowableArray@UCInputLocale@CCtrlDxIMEEditBox@@@@QAEJH@Z 10020fd8 f i CtrlDxEdit.obj
 0001:00020052       ?Add@?$CGrowableArray@UCInputLocale@CCtrlDxIMEEditBox@@@@QAEJABUCInputLocale@CCtrlDxIMEEditBox@@@Z 10021052 f i CtrlDxEdit.obj
 0001:000200bf       ??$unchecked_copy@PAKPAK@stdext@@YAPAKPAK00@Z 100210bf f i CtrlDxEdit.obj
 0001:00020130       ??$_Umove@PAK@?$vector@KV?$allocator@K@std@@@std@@IAEPAKPAK00@Z 10021130 f i CtrlDxEdit.obj
 0001:0002018d       ??$_Unchecked_move_backward@PAKPAK@stdext@@YAPAKPAK00@Z 1002118d f i CtrlDxEdit.obj
 0001:00020224       ??$_Allocate@K@std@@YAPAKIPAK@Z 10021224 f i CtrlDxEdit.obj
 0001:00020224       ??$_Allocate@V_Aux_cont@std@@@std@@YAPAV_Aux_cont@0@IPAV10@@Z 10021224 f i BaseManager.obj
 0001:00020277       ?SetSizeInternal@?$CGrowableArray@UCInputLocale@CCtrlDxIMEEditBox@@@@IAEJH@Z 10021277 f i CtrlDxEdit.obj
 0001:0002035f       ??$_Unchecked_uninitialized_move@PAKPAKV?$allocator@K@std@@@stdext@@YAPAKPAK00AAV?$allocator@K@std@@@Z 1002135f f i CtrlDxEdit.obj
 0001:000203a1       ??$unchecked_fill_n@PAKIK@stdext@@YAXPAKIABK@Z 100213a1 f i CtrlDxEdit.obj
 0001:0002040b       ??$unchecked_uninitialized_copy@PAKPAKV?$allocator@K@std@@@stdext@@YAPAKPAK00AAV?$allocator@K@std@@@Z 1002140b f i CtrlDxEdit.obj
 0001:00020476       ?GetOSVersion@@YAHPAD0@Z   10021476 f   CtrlEditWZ.obj
 0001:000208bb       ?CCtrlEditBoxWndProc@@YAJPAUHWND__@@IIJ@Z 100218bb f   CtrlEditWZ.obj
 0001:000208ed       ??0CCtrlEditWZ@@QAE@XZ     100218ed f   CtrlEditWZ.obj
 0001:00020ab9       ??1CCtrlEditWZ@@UAE@XZ     10021ab9 f   CtrlEditWZ.obj
 0001:00020adc       ?ReleaseFont@CCtrlEditWZ@@IAEXXZ 10021adc f   CtrlEditWZ.obj
 0001:00020b57       ?ReleaseHDC@CCtrlEditWZ@@IAEXXZ 10021b57 f   CtrlEditWZ.obj
 0001:00020bef       ?OnInitialize@CCtrlEditWZ@@UAEXXZ 10021bef f   CtrlEditWZ.obj
 0001:00020c0a       ?OnLoad@CCtrlEditWZ@@UAEXPAX@Z 10021c0a f   CtrlEditWZ.obj
 0001:00021096       ?OnSave@CCtrlEditWZ@@UAEXPAX@Z 10022096 f   CtrlEditWZ.obj
 0001:000211fc       ?OnCreate@CCtrlEditWZ@@UAE_NKKPAUHWND__@@PAUHINSTANCE__@@PAUtagRECT@@PAX@Z 100221fc f   CtrlEditWZ.obj
 0001:00021645       ?MoveWindowWZ@CCtrlEditWZ@@UAE_NMMMM@Z 10022645 f   CtrlEditWZ.obj
 0001:000218b4       ?SetTextNCRect@CCtrlEditWZ@@UAEXHHHH@Z 100228b4 f   CtrlEditWZ.obj
 0001:000218ef       ?CreateBackBuffer@CCtrlEditWZ@@IAEXHH@Z 100228ef f   CtrlEditWZ.obj
 0001:00021b6c       ?OnDestroy@CCtrlEditWZ@@UAEXXZ 10022b6c f   CtrlEditWZ.obj
 0001:00021bc0       ?OnDoAction@CCtrlEditWZ@@UAEXXZ 10022bc0 f   CtrlEditWZ.obj
 0001:00021f75       ?OnDraw@CCtrlEditWZ@@UAE_N_N@Z 10022f75 f   CtrlEditWZ.obj
 0001:000220b7       ?SetDCToTexture@CCtrlEditWZ@@IAEXXZ 100230b7 f   CtrlEditWZ.obj
 0001:0002227c       ?SetAlphaBuffer@CCtrlEditWZ@@IAEXPAX@Z 1002327c f   CtrlEditWZ.obj
 0001:000222ec       ?ClearBuffer24Bit@CCtrlEditWZ@@IAEXPAEFFF@Z 100232ec f   CtrlEditWZ.obj
 0001:00022399       ?SetStyle@CCtrlEditWZ@@UAEXK@Z 10023399 f   CtrlEditWZ.obj
 0001:000223ad       ?UpdateWindowWZ@CCtrlEditWZ@@UAEXPAUHWND__@@@Z 100233ad f   CtrlEditWZ.obj
 0001:00022461       ?ReleaseImage@CCtrlEditWZ@@UAEXXZ 10023461 f   CtrlEditWZ.obj
 0001:00022495       ?SetLimitText@CCtrlEditWZ@@UAEXK@Z 10023495 f   CtrlEditWZ.obj
 0001:000224b9       ?GetTextWZW@CCtrlEditWZ@@UAEXPA_WH@Z 100234b9 f   CtrlEditWZ.obj
 0001:00022565       ?GetTextWZA@CCtrlEditWZ@@UAEXPADH@Z 10023565 f   CtrlEditWZ.obj
 0001:00022585       ?SetTextWZW@CCtrlEditWZ@@UAEXPB_W_N@Z 10023585 f   CtrlEditWZ.obj
 0001:000225e9       ?SetTextWZA@CCtrlEditWZ@@UAEXPBD_N@Z 100235e9 f   CtrlEditWZ.obj
 0001:000226bc       ?ClearText@CCtrlEditWZ@@UAEXXZ 100236bc f   CtrlEditWZ.obj
 0001:000226d9       ?OnFocusIn@CCtrlEditWZ@@UAEXXZ 100236d9 f   CtrlEditWZ.obj
 0001:000226fa       ?OnFocusOut@CCtrlEditWZ@@UAEXXZ 100236fa f   CtrlEditWZ.obj
 0001:0002272b       ?IsEditFocus@CCtrlEditWZ@@IAE_NXZ 1002372b f   CtrlEditWZ.obj
 0001:0002274b       ?SetFocusWZ@CCtrlEditWZ@@UAEXXZ 1002374b f   CtrlEditWZ.obj
 0001:000227a4       ?SetFontID@CCtrlEditWZ@@UAEXK@Z 100237a4 f   CtrlEditWZ.obj
 0001:00022865       ?GetFontID@CCtrlEditWZ@@UAEKXZ 10023865 f   CtrlEditWZ.obj
 0001:00022877       ?RegisterLogFont@CCtrlEditWZ@@IAEXPAUtagLOGFONTA@@@Z 10023877 f   CtrlEditWZ.obj
 0001:00022969       ?SetColorText@CCtrlEditWZ@@UAEXK@Z 10023969 f   CtrlEditWZ.obj
 0001:00022980       ?SetColorCaret@CCtrlEditWZ@@UAEXK@Z 10023980 f   CtrlEditWZ.obj
 0001:000229a7       ?GetFontColor@CCtrlEditWZ@@UAEKXZ 100239a7 f   CtrlEditWZ.obj
 0001:000229b9       ?SendMessageWZ@CCtrlEditWZ@@UAE_NPAUSI_MESSAGE@@@Z 100239b9 f   CtrlEditWZ.obj
 0001:000229fc       ?Message_MouseLButtonDown@CCtrlEditWZ@@MAE_NPAUSI_MESSAGE@@@Z 100239fc f   CtrlEditWZ.obj
 0001:00022bcc       ?Message_MouseLButtonUp@CCtrlEditWZ@@MAE_NPAUSI_MESSAGE@@@Z 10023bcc f   CtrlEditWZ.obj
 0001:00022cce       ?Message_MouseMove@CCtrlEditWZ@@MAE_NPAUSI_MESSAGE@@@Z 10023cce f   CtrlEditWZ.obj
 0001:00022de6       ?Message_MouseLButtonDoubleClick@CCtrlEditWZ@@MAE_NPAUSI_MESSAGE@@@Z 10023de6 f   CtrlEditWZ.obj
 0001:00022ec7       ?Message_KeyDown@CCtrlEditWZ@@MAE_NPAUSI_MESSAGE@@@Z 10023ec7 f   CtrlEditWZ.obj
 0001:00022f64       ?EditSubProc@CCtrlEditWZ@@QAEJPAUHWND__@@IIJ@Z 10023f64 f   CtrlEditWZ.obj
 0001:00023195       ?GetFontInfo@CCtrlEditWZ@@UAEPAUtagLOGFONTA@@XZ 10024195 f i CtrlEditWZ.obj
 0001:000231a6       ?SetColorSelBack@CCtrlEditWZ@@UAEXK@Z 100241a6 f i CtrlEditWZ.obj
 0001:000231bd       ?SetColorSelText@CCtrlEditWZ@@UAEXK@Z 100241bd f i CtrlEditWZ.obj
 0001:000231d4       ?SetColorCompText@CCtrlEditWZ@@UAEXK@Z 100241d4 f i CtrlEditWZ.obj
 0001:000231eb       ?SetColorCompBack@CCtrlEditWZ@@UAEXK@Z 100241eb f i CtrlEditWZ.obj
 0001:00023202       ?SetColorCompCaret@CCtrlEditWZ@@UAEXK@Z 10024202 f i CtrlEditWZ.obj
 0001:00023219       ?SetColorIndicatorIme@CCtrlEditWZ@@UAEXK@Z 10024219 f i CtrlEditWZ.obj
 0001:00023230       ?SetColorIndicatorEng@CCtrlEditWZ@@UAEXK@Z 10024230 f i CtrlEditWZ.obj
 0001:00023247       ?SetColorIndicatorBK@CCtrlEditWZ@@UAEXK@Z 10024247 f i CtrlEditWZ.obj
 0001:0002325e       ?GetCaretColor@CCtrlEditWZ@@UAEKXZ 1002425e f i CtrlEditWZ.obj
 0001:00023270       ?GetSelBackColor@CCtrlEditWZ@@UAEKXZ 10024270 f i CtrlEditWZ.obj
 0001:00023282       ?GetSelTextColor@CCtrlEditWZ@@UAEKXZ 10024282 f i CtrlEditWZ.obj
 0001:00023294       ?GetCompTextColor@CCtrlEditWZ@@UAEKXZ 10024294 f i CtrlEditWZ.obj
 0001:000232a6       ?GetCompBackColor@CCtrlEditWZ@@UAEKXZ 100242a6 f i CtrlEditWZ.obj
 0001:000232b8       ?GetCompCaretColor@CCtrlEditWZ@@UAEKXZ 100242b8 f i CtrlEditWZ.obj
 0001:000232ca       ?GetIndicatorImeColor@CCtrlEditWZ@@UAEKXZ 100242ca f i CtrlEditWZ.obj
 0001:000232dc       ?GetIndicatorEngColor@CCtrlEditWZ@@UAEKXZ 100242dc f i CtrlEditWZ.obj
 0001:000232ee       ?GetIndicatorBKColor@CCtrlEditWZ@@UAEKXZ 100242ee f i CtrlEditWZ.obj
 0001:00023300       ??_ECCtrlEditWZ@@UAEPAXI@Z 10024300 f i CtrlEditWZ.obj
 0001:00023300       ??_GCCtrlEditWZ@@UAEPAXI@Z 10024300 f i CtrlEditWZ.obj
 0001:00023327       ??0CCtrlHScrollWZ@@QAE@XZ  10024327 f   CtrlHScrollWZ.obj
 0001:0002340f       ??1CCtrlHScrollWZ@@UAE@XZ  1002440f f   CtrlHScrollWZ.obj
 0001:00023490       ?OnCreate@CCtrlHScrollWZ@@UAE_NKKPAUHWND__@@PAUHINSTANCE__@@PAUtagRECT@@PAX@Z 10024490 f   CtrlHScrollWZ.obj
 0001:00023596       ?MoveWindowWZ@CCtrlHScrollWZ@@UAE_NMMMM@Z 10024596 f   CtrlHScrollWZ.obj
 0001:00023be7       ?OnLoad@CCtrlHScrollWZ@@UAEXPAX@Z 10024be7 f   CtrlHScrollWZ.obj
 0001:00023dcf       ?OnSave@CCtrlHScrollWZ@@UAEXPAX@Z 10024dcf f   CtrlHScrollWZ.obj
 0001:00023e65       ?OnInitialize@CCtrlHScrollWZ@@UAEXXZ 10024e65 f   CtrlHScrollWZ.obj
 0001:00023ebf       ?OnDestroy@CCtrlHScrollWZ@@UAEXXZ 10024ebf f   CtrlHScrollWZ.obj
 0001:00023f0f       ?OnDraw@CCtrlHScrollWZ@@UAE_N_N@Z 10024f0f f   CtrlHScrollWZ.obj
 0001:00024047       ?SetStyle@CCtrlHScrollWZ@@UAEXK@Z 10025047 f   CtrlHScrollWZ.obj
 0001:0002405b       ?EnableWindowWZ@CCtrlHScrollWZ@@UAEX_N@Z 1002505b f   CtrlHScrollWZ.obj
 0001:000240b9       ?UpdateWindowWZ@CCtrlHScrollWZ@@UAEXPAUHWND__@@@Z 100250b9 f   CtrlHScrollWZ.obj
 0001:00024117       ?ReleaseImage@CCtrlHScrollWZ@@UAEXXZ 10025117 f   CtrlHScrollWZ.obj
 0001:00024167       ?SetScrollPosWZ@CCtrlHScrollWZ@@UAEHH@Z 10025167 f   CtrlHScrollWZ.obj
 0001:0002418b       ?SetScrollPosWZ@CCtrlHScrollWZ@@UAEHM@Z 1002518b f   CtrlHScrollWZ.obj
 0001:00024337       ?SetScrollRangeWZ@CCtrlHScrollWZ@@UAEXHH@Z 10025337 f   CtrlHScrollWZ.obj
 0001:00024366       ?SetScrollRangeWZ@CCtrlHScrollWZ@@UAEXMM@Z 10025366 f   CtrlHScrollWZ.obj
 0001:00024412       ?GetScrollRangeWZ@CCtrlHScrollWZ@@UAEXPAH0@Z 10025412 f   CtrlHScrollWZ.obj
 0001:0002443d       ?GetScrollRangeWZ@CCtrlHScrollWZ@@UAEXPAM0@Z 1002543d f   CtrlHScrollWZ.obj
 0001:00024464       ?SetChangeSizeThumb@CCtrlHScrollWZ@@UAEXH@Z 10025464 f   CtrlHScrollWZ.obj
 0001:00024539       ?Message_MouseLButtonDown@CCtrlHScrollWZ@@MAE_NPAUSI_MESSAGE@@@Z 10025539 f   CtrlHScrollWZ.obj
 0001:00024960       ?Message_MouseLButtonUp@CCtrlHScrollWZ@@MAE_NPAUSI_MESSAGE@@@Z 10025960 f   CtrlHScrollWZ.obj
 0001:00024ab1       ?Message_MouseMove@CCtrlHScrollWZ@@MAE_NPAUSI_MESSAGE@@@Z 10025ab1 f   CtrlHScrollWZ.obj
 0001:00024e4e       ?SetArrowLeftBTImageFormat@CCtrlHScrollWZ@@UAEXPAUSI_TFORMAT@@@Z 10025e4e f   CtrlHScrollWZ.obj
 0001:00024e71       ?SetArrowRightBTImageFormat@CCtrlHScrollWZ@@UAEXPAUSI_TFORMAT@@@Z 10025e71 f   CtrlHScrollWZ.obj
 0001:00024e94       ?SetArrowThumbBTImageFormat@CCtrlHScrollWZ@@UAEXPAUSI_TFORMAT@@@Z 10025e94 f   CtrlHScrollWZ.obj
 0001:00024eb7       ?GetArrowLeftBTImageFormat@CCtrlHScrollWZ@@UAEPAUSI_TFORMAT@@XZ 10025eb7 f   CtrlHScrollWZ.obj
 0001:00024ed9       ?GetArrowRightBTImageFormat@CCtrlHScrollWZ@@UAEPAUSI_TFORMAT@@XZ 10025ed9 f   CtrlHScrollWZ.obj
 0001:00024efb       ?GetArrowThumbBTImageFormat@CCtrlHScrollWZ@@UAEPAUSI_TFORMAT@@XZ 10025efb f   CtrlHScrollWZ.obj
 0001:00024f1d       ?SetArrowLeftBTIsOutline@CCtrlHScrollWZ@@UAEX_N@Z 10025f1d f   CtrlHScrollWZ.obj
 0001:00024f43       ?GetArrowLeftBTIsOutline@CCtrlHScrollWZ@@UAE_NXZ 10025f43 f   CtrlHScrollWZ.obj
 0001:00024f64       ?SetArrowLeftBTOutlineColor@CCtrlHScrollWZ@@UAEXK@Z 10025f64 f   CtrlHScrollWZ.obj
 0001:00024f8a       ?GetArrowLeftBTOutlineColor@CCtrlHScrollWZ@@UAEKXZ 10025f8a f   CtrlHScrollWZ.obj
 0001:00024fab       ?SetArrowRightBTIsOutline@CCtrlHScrollWZ@@UAEX_N@Z 10025fab f   CtrlHScrollWZ.obj
 0001:00024fd1       ?GetArrowRightBTIsOutline@CCtrlHScrollWZ@@UAE_NXZ 10025fd1 f   CtrlHScrollWZ.obj
 0001:00024ff2       ?SetArrowRightBTOutlineColor@CCtrlHScrollWZ@@UAEXK@Z 10025ff2 f   CtrlHScrollWZ.obj
 0001:00025018       ?GetArrowRightBTOutlineColor@CCtrlHScrollWZ@@UAEKXZ 10026018 f   CtrlHScrollWZ.obj
 0001:00025039       ?SetArrowThumbBTIsOutline@CCtrlHScrollWZ@@UAEX_N@Z 10026039 f   CtrlHScrollWZ.obj
 0001:0002505f       ?GetArrowThumbBTIsOutline@CCtrlHScrollWZ@@UAE_NXZ 1002605f f   CtrlHScrollWZ.obj
 0001:00025080       ?SetArrowThumbBTOutlineColor@CCtrlHScrollWZ@@UAEXK@Z 10026080 f   CtrlHScrollWZ.obj
 0001:000250a6       ?GetArrowThumbBTOutlineColor@CCtrlHScrollWZ@@UAEKXZ 100260a6 f   CtrlHScrollWZ.obj
 0001:000250c7       ?SetArrowLeftSize@CCtrlHScrollWZ@@UAEXAAUtagRECT@@@Z 100260c7 f   CtrlHScrollWZ.obj
 0001:0002511e       ?SetArrowRightSize@CCtrlHScrollWZ@@UAEXAAUtagRECT@@@Z 1002611e f   CtrlHScrollWZ.obj
 0001:00025175       ?SetArrowThumbSize@CCtrlHScrollWZ@@UAEXAAUtagRECT@@@Z 10026175 f   CtrlHScrollWZ.obj
 0001:000251cc       ?GetArrowLeftSize@CCtrlHScrollWZ@@UAE?AUtagRECT@@XZ 100261cc f   CtrlHScrollWZ.obj
 0001:000251f2       ?GetArrowRightSize@CCtrlHScrollWZ@@UAE?AUtagRECT@@XZ 100261f2 f   CtrlHScrollWZ.obj
 0001:00025218       ?GetArrowThumbSize@CCtrlHScrollWZ@@UAE?AUtagRECT@@XZ 10026218 f   CtrlHScrollWZ.obj
 0001:0002523e       ??_ECCtrlHScrollWZ@@UAEPAXI@Z 1002623e f i CtrlHScrollWZ.obj
 0001:0002523e       ??_GCCtrlHScrollWZ@@UAEPAXI@Z 1002623e f i CtrlHScrollWZ.obj
 0001:00025265       ??0CCtrlListWZ@@QAE@XZ     10026265 f   CtrlListWZ.obj
 0001:0002547d       ??1CCtrlListWZ@@UAE@XZ     1002647d f   CtrlListWZ.obj
 0001:0002555a       ?OnCreate@CCtrlListWZ@@UAE_NKKPAUHWND__@@PAUHINSTANCE__@@PAUtagRECT@@PAX@Z 1002655a f   CtrlListWZ.obj
 0001:000255d4       ?OnLoad@CCtrlListWZ@@UAEXPAX@Z 100265d4 f   CtrlListWZ.obj
 0001:00025d75       ?OnSave@CCtrlListWZ@@UAEXPAX@Z 10026d75 f   CtrlListWZ.obj
 0001:00025f7e       ?GetReportButtonInfoPtr@CCtrlListWZ@@IAEPAXH@Z 10026f7e f   CtrlListWZ.obj
 0001:00026027       ?OnInitialize@CCtrlListWZ@@UAEXXZ 10027027 f   CtrlListWZ.obj
 0001:000260df       ?OnDestroy@CCtrlListWZ@@UAEXXZ 100270df f   CtrlListWZ.obj
 0001:000262d9       ?DeleteItem@CCtrlListWZ@@UAEHH@Z 100272d9 f   CtrlListWZ.obj
 0001:0002655b       ?DeleteItemAll@CCtrlListWZ@@UAEXXZ 1002755b f   CtrlListWZ.obj
 0001:0002665a       ?EnableWindowWZ@CCtrlListWZ@@UAEX_N@Z 1002765a f   CtrlListWZ.obj
 0001:00026706       ?UpdateWindowWZ@CCtrlListWZ@@UAEXPAUHWND__@@@Z 10027706 f   CtrlListWZ.obj
 0001:000267b2       ?ReleaseImage@CCtrlListWZ@@UAEXXZ 100277b2 f   CtrlListWZ.obj
 0001:000267c3       ?OnDraw@CCtrlListWZ@@UAE_N_N@Z 100277c3 f   CtrlListWZ.obj
 0001:00026eec       ?DrawListData@CCtrlListWZ@@IAEXHPAXH@Z 10027eec f   CtrlListWZ.obj
 0001:000273a3       ?DrawListSell@CCtrlListWZ@@IAEXHPAUCListSellData@1@UtagRECT@@@Z 100283a3 f   CtrlListWZ.obj
 0001:0002759d       ?MoveWindowWZ@CCtrlListWZ@@UAE_NMMMM@Z 1002859d f   CtrlListWZ.obj
 0001:0002797f       ?SetFontID@CCtrlListWZ@@UAEXK@Z 1002897f f   CtrlListWZ.obj
 0001:00027996       ?GetFontID@CCtrlListWZ@@UAEKXZ 10028996 f   CtrlListWZ.obj
 0001:000279a8       ?GetReportUseCnt@CCtrlListWZ@@UAEFXZ 100289a8 f   CtrlListWZ.obj
 0001:000279bb       ?SetBeginDrawIndex@CCtrlListWZ@@UAEXH@Z 100289bb f   CtrlListWZ.obj
 0001:000279d2       ?SetCurSel@CCtrlListWZ@@UAEXH@Z 100289d2 f   CtrlListWZ.obj
 0001:000279e9       ?GetCurSel@CCtrlListWZ@@UAEHXZ 100289e9 f   CtrlListWZ.obj
 0001:000279fb       ?GetUseReport@CCtrlListWZ@@UAE_NXZ 100289fb f   CtrlListWZ.obj
 0001:00027a0d       ?SetUseReport@CCtrlListWZ@@UAEX_N@Z 10028a0d f   CtrlListWZ.obj
 0001:00027a24       ?GetListRowCnt@CCtrlListWZ@@UAEHXZ 10028a24 f   CtrlListWZ.obj
 0001:00027a3d       ?GetDrawRowCount@CCtrlListWZ@@UAEHXZ 10028a3d f   CtrlListWZ.obj
 0001:00027a6b       ?SetColorText@CCtrlListWZ@@UAEXK@Z 10028a6b f   CtrlListWZ.obj
 0001:00027a82       ?SetColorSelBar@CCtrlListWZ@@UAEXK@Z 10028a82 f   CtrlListWZ.obj
 0001:00027a99       ?SetColorSelBarOnText@CCtrlListWZ@@UAEXK@Z 10028a99 f   CtrlListWZ.obj
 0001:00027ab0       ?SetUnuseSelBar@CCtrlListWZ@@UAEX_N@Z 10028ab0 f   CtrlListWZ.obj
 0001:00027ac7       ?SetTextKind@CCtrlListWZ@@UAEXW4ENUM_TEXT_KIND@@@Z 10028ac7 f   CtrlListWZ.obj
 0001:00027ade       ?GetTextKind@CCtrlListWZ@@UAE?AW4ENUM_TEXT_KIND@@XZ 10028ade f   CtrlListWZ.obj
 0001:00027af0       ?SetRoportButtonImageFormat@CCtrlListWZ@@UAEXPAUSI_TFORMAT@@@Z 10028af0 f   CtrlListWZ.obj
 0001:00027b91       ?GetRoportButtonImageFormat@CCtrlListWZ@@UAEPAUSI_TFORMAT@@XZ 10028b91 f   CtrlListWZ.obj
 0001:00027c25       ?SetReportUseCnt@CCtrlListWZ@@UAEXF@Z 10028c25 f   CtrlListWZ.obj
 0001:00027f66       ?InsertItemBack@CCtrlListWZ@@UAEHXZ 10028f66 f   CtrlListWZ.obj
 0001:00028067       ?InsertItemFront@CCtrlListWZ@@UAEHXZ 10029067 f   CtrlListWZ.obj
 0001:00028151       ?UpdateListDate@CCtrlListWZ@@IAEHPAX@Z 10029151 f   CtrlListWZ.obj
 0001:00028469       ?SetItemWZW@CCtrlListWZ@@UAE_NHPB_WKKKKK@Z 10029469 f   CtrlListWZ.obj
 0001:000284dc       ?SetItemWZA@CCtrlListWZ@@UAE_NHPBDKKKKK@Z 100294dc f   CtrlListWZ.obj
 0001:000286f8       ?SetItemWZW@CCtrlListWZ@@UAE_NHHPB_WKKKKK@Z 100296f8 f   CtrlListWZ.obj
 0001:0002876e       ?SetItemWZA@CCtrlListWZ@@UAE_NHHPBDKKKKK@Z 1002976e f   CtrlListWZ.obj
 0001:00028992       ?SetItemBKColor@CCtrlListWZ@@UAE_NHHK@Z 10029992 f   CtrlListWZ.obj
 0001:00028a3a       ?SetItemTextColor@CCtrlListWZ@@UAE_NHHK@Z 10029a3a f   CtrlListWZ.obj
 0001:00028ae3       ?SetItemSelTextColor@CCtrlListWZ@@UAE_NHHK@Z 10029ae3 f   CtrlListWZ.obj
 0001:00028b8c       ?SetItemUserData@CCtrlListWZ@@UAE_NHHPAX@Z 10029b8c f   CtrlListWZ.obj
 0001:00028c35       ?GetItemUserData@CCtrlListWZ@@UAEPAXHH@Z 10029c35 f   CtrlListWZ.obj
 0001:00028cd5       ?SetItemCallbackDraw@CCtrlListWZ@@UAE_NHHP6AXPAV1@PAUCListSellData@1@HAAUtagRECT@@@Z@Z 10029cd5 f   CtrlListWZ.obj
 0001:00028d7e       ?SetItemFontID@CCtrlListWZ@@UAE_NHHK@Z 10029d7e f   CtrlListWZ.obj
 0001:00028e27       ?SetItemTextStyle@CCtrlListWZ@@UAE_NHHK@Z 10029e27 f   CtrlListWZ.obj
 0001:00028ed0       ?SetSellHeight@CCtrlListWZ@@UAEXH@Z 10029ed0 f   CtrlListWZ.obj
 0001:00028ee7       ?GetSellheight@CCtrlListWZ@@UAEHXZ 10029ee7 f   CtrlListWZ.obj
 0001:00028ef9       ?SetReportHeight@CCtrlListWZ@@UAEXH@Z 10029ef9 f   CtrlListWZ.obj
 0001:00028fac       ?SetItemTextWZW@CCtrlListWZ@@UAE_NHPB_W@Z 10029fac f   CtrlListWZ.obj
 0001:00029010       ?SetItemTextWZA@CCtrlListWZ@@UAE_NHPBD@Z 1002a010 f   CtrlListWZ.obj
 0001:0002904f       ?SetItemTextWZW@CCtrlListWZ@@UAE_NHHPB_W@Z 1002a04f f   CtrlListWZ.obj
 0001:000290b6       ?SetItemTextWZA@CCtrlListWZ@@UAE_NHHPBD@Z 1002a0b6 f   CtrlListWZ.obj
 0001:000290f7       ?SetItemData@CCtrlListWZ@@UAE_NHPAX@Z 1002a0f7 f   CtrlListWZ.obj
 0001:00029126       ?GetItemData@CCtrlListWZ@@UAEPAXH@Z 1002a126 f   CtrlListWZ.obj
 0001:00029157       ?GetItemText@CCtrlListWZ@@UAEPBDHH@Z 1002a157 f   CtrlListWZ.obj
 0001:0002921a       ?GetListInfoDataToIndex@CCtrlListWZ@@IAEPAXH@Z 1002a21a f   CtrlListWZ.obj
 0001:00029475       ?GetIndexToListDataPtr@CCtrlListWZ@@IAEHPAX@Z 1002a475 f   CtrlListWZ.obj
 0001:000296e6       ?SetReportButtonInfoW@CCtrlListWZ@@UAEXHHPB_WK@Z 1002a6e6 f   CtrlListWZ.obj
 0001:00029750       ?SetReportButtonInfoA@CCtrlListWZ@@UAEXHHPBDK@Z 1002a750 f   CtrlListWZ.obj
 0001:00029898       ?GetReportButtonInfoW@CCtrlListWZ@@UAE_NHPAHPA_WHPAK@Z 1002a898 f   CtrlListWZ.obj
 0001:00029953       ?GetReportButtonInfoA@CCtrlListWZ@@UAE_NHPAHPADHPAK@Z 1002a953 f   CtrlListWZ.obj
 0001:00029a8c       ?SelectReportButton@CCtrlListWZ@@UAEXH@Z 1002aa8c f   CtrlListWZ.obj
 0001:00029edf       ?SetReportIsOutline@CCtrlListWZ@@UAEX_N@Z 1002aedf f   CtrlListWZ.obj
 0001:00029f86       ?GetReportIsOutline@CCtrlListWZ@@UAE_NXZ 1002af86 f   CtrlListWZ.obj
 0001:0002a01d       ?SetReportOutlineColor@CCtrlListWZ@@UAEXK@Z 1002b01d f   CtrlListWZ.obj
 0001:0002a0c4       ?GetReportOutlineColor@CCtrlListWZ@@UAEKXZ 1002b0c4 f   CtrlListWZ.obj
 0001:0002a15b       ?Message_MouseLButtonDown@CCtrlListWZ@@MAE_NPAUSI_MESSAGE@@@Z 1002b15b f   CtrlListWZ.obj
 0001:0002a476       ?Message_MouseLButtonUp@CCtrlListWZ@@MAE_NPAUSI_MESSAGE@@@Z 1002b476 f   CtrlListWZ.obj
 0001:0002a6de       ?Message_MouseMove@CCtrlListWZ@@MAE_NPAUSI_MESSAGE@@@Z 1002b6de f   CtrlListWZ.obj
 0001:0002ab85       ?Message_MouseRButtonDown@CCtrlListWZ@@MAE_NPAUSI_MESSAGE@@@Z 1002bb85 f   CtrlListWZ.obj
 0001:0002acae       ?ComputeSel@CCtrlListWZ@@IAEHUtagPOINT@@@Z 1002bcae f   CtrlListWZ.obj
 0001:0002ad7e       ?SetItemFontID@CCtrlListWZ@@UAE_NHHPBD@Z 1002bd7e f i CtrlListWZ.obj
 0001:0002ad8b       ?GetBeginDrawIndex@CCtrlListWZ@@UAEHXZ 1002bd8b f i CtrlListWZ.obj
 0001:0002ad9d       ?SetOverSel@CCtrlListWZ@@UAEXH@Z 1002bd9d f i CtrlListWZ.obj
 0001:0002adb4       ?GetOverSel@CCtrlListWZ@@UAEHXZ 1002bdb4 f i CtrlListWZ.obj
 0001:0002adc6       ?SetStartLineGapTop@CCtrlListWZ@@UAEXH@Z 1002bdc6 f i CtrlListWZ.obj
 0001:0002addd       ?SetStartLineGapLeft@CCtrlListWZ@@UAEXH@Z 1002bddd f i CtrlListWZ.obj
 0001:0002adf4       ?SetStartLineGapRight@CCtrlListWZ@@UAEXH@Z 1002bdf4 f i CtrlListWZ.obj
 0001:0002ae0b       ?IsTextReducing@CCtrlListWZ@@UBE_NXZ 1002be0b f i CtrlListWZ.obj
 0001:0002ae1d       ?SetTextReducing@CCtrlListWZ@@UAEX_N@Z 1002be1d f i CtrlListWZ.obj
 0001:0002ae34       ??_GCCtrlListWZ@@UAEPAXI@Z 1002be34 f i CtrlListWZ.obj
 0001:0002ae34       ??_ECCtrlListWZ@@UAEPAXI@Z 1002be34 f i CtrlListWZ.obj
 0001:0002ae5b       ??1?$multimap@V?$basic_string@DU?$char_traits@D@std@@V?$allocator@D@2@@std@@PAXU?$less@V?$basic_string@DU?$char_traits@D@std@@V?$allocator@D@2@@std@@@2@V?$allocator@U?$pair@$$CBV?$basic_string@DU?$char_traits@D@std@@V?$allocator@D@2@@std@@PAX@std@@@2@@std@@QAE@XZ 1002be5b f i CtrlListWZ.obj
 0001:0002aeb0       ??1CListData@CCtrlListWZ@@QAE@XZ 1002beb0 f i CtrlListWZ.obj
 0001:0002afc0       ??1?$map@KPAXU?$less@K@std@@V?$allocator@U?$pair@$$CBKPAX@std@@@2@@std@@QAE@XZ 1002bfc0 f i CtrlListWZ.obj
 0001:0002afc0       ??1?$map@KPAUCListSellData@CCtrlListWZ@@U?$less@K@std@@V?$allocator@U?$pair@$$CBKPAUCListSellData@CCtrlListWZ@@@std@@@4@@std@@QAE@XZ 1002bfc0 f i CtrlListWZ.obj
 0001:0002b015       ??1SBTData@@QAE@XZ         1002c015 f i CtrlListWZ.obj
 0001:0002b06c       ??0SBTData@@QAE@XZ         1002c06c f i CtrlListWZ.obj
 0001:0002b0e3       ??0CListData@CCtrlListWZ@@QAE@XZ 1002c0e3 f i CtrlListWZ.obj
 0001:0002b117       ??1?$basic_string@DU?$char_traits@D@std@@V?$allocator@D@2@@std@@QAE@XZ 1002c117 f i BaseManager.obj
 0001:0002b117       ??1?$pair@V?$basic_string@DU?$char_traits@D@std@@V?$allocator@D@2@@std@@PAX@std@@QAE@XZ 1002c117 f i CtrlListWZ.obj
 0001:0002b117       ??1?$pair@$$CBV?$basic_string@DU?$char_traits@D@std@@V?$allocator@D@2@@std@@PAX@std@@QAE@XZ 1002c117 f i CtrlListWZ.obj
 0001:0002b12e       ?Add@CListData@CCtrlListWZ@@QAE_NPBDKKKKK@Z 1002c12e f i CtrlListWZ.obj
 0001:0002b22e       ??0CListSellData@CCtrlListWZ@@QAE@XZ 1002c22e f i CtrlListWZ.obj
 0001:0002b28d       ?Add@CListData@CCtrlListWZ@@QAE_NHPBDKKKKK@Z 1002c28d f i CtrlListWZ.obj
 0001:0002b426       ?end@?$_Tree@V?$_Tmap_traits@KPAUCListSellData@CCtrlListWZ@@U?$less@K@std@@V?$allocator@U?$pair@$$CBKPAUCListSellData@CCtrlListWZ@@@std@@@4@$0A@@std@@@std@@QAE?AViterator@12@XZ 1002c426 f i CtrlListWZ.obj
 0001:0002b466       ?find@?$_Tree@V?$_Tmap_traits@KKU?$less@K@std@@V?$allocator@U?$pair@$$CBKK@std@@@2@$0A@@std@@@std@@QAE?AViterator@12@ABK@Z 1002c466 f i CtrlTabWZ.obj
 0001:0002b466       ?find@?$_Tree@V?$_Tmap_traits@KPAXU?$less@K@std@@V?$allocator@U?$pair@$$CBKPAX@std@@@2@$0A@@std@@@std@@QAE?AViterator@12@ABK@Z 1002c466 f i CtrlListWZ.obj
 0001:0002b466       ?find@?$_Tree@V?$_Tmap_traits@KPAUCListSellData@CCtrlListWZ@@U?$less@K@std@@V?$allocator@U?$pair@$$CBKPAUCListSellData@CCtrlListWZ@@@std@@@4@$0A@@std@@@std@@QAE?AViterator@12@ABK@Z 1002c466 f i CtrlListWZ.obj
 0001:0002b539       ?begin@?$_Tree@V?$_Tmap_traits@KPAUCListSellData@CCtrlListWZ@@U?$less@K@std@@V?$allocator@U?$pair@$$CBKPAUCListSellData@CCtrlListWZ@@@std@@@4@$0A@@std@@@std@@QAE?AViterator@12@XZ 1002c539 f i CtrlListWZ.obj
 0001:0002b539       ?begin@?$_Tree@V?$_Tmap_traits@KKU?$less@K@std@@V?$allocator@U?$pair@$$CBKK@std@@@2@$0A@@std@@@std@@QAE?AViterator@12@XZ 1002c539 f i CtrlTabWZ.obj
 0001:0002b539       ?begin@?$_Tree@V?$_Tmap_traits@KPAXU?$less@K@std@@V?$allocator@U?$pair@$$CBKPAX@std@@@2@$0A@@std@@@std@@QAE?AViterator@12@XZ 1002c539 f i CtrlListWZ.obj
 0001:0002b539       ?begin@?$_Tree@V?$_Tmap_traits@V?$basic_string@DU?$char_traits@D@std@@V?$allocator@D@2@@std@@PAXU?$less@V?$basic_string@DU?$char_traits@D@std@@V?$allocator@D@2@@std@@@2@V?$allocator@U?$pair@$$CBV?$basic_string@DU?$char_traits@D@std@@V?$allocator@D@2@@std@@PAX@std@@@2@$00@std@@@std@@QAE?AViterator@12@XZ 1002c539 f i CtrlListWZ.obj
 0001:0002b582       ?erase@?$_Tree@V?$_Tmap_traits@V?$basic_string@DU?$char_traits@D@std@@V?$allocator@D@2@@std@@PAXU?$less@V?$basic_string@DU?$char_traits@D@std@@V?$allocator@D@2@@std@@@2@V?$allocator@U?$pair@$$CBV?$basic_string@DU?$char_traits@D@std@@V?$allocator@D@2@@std@@PAX@std@@@2@$00@std@@@std@@QAE?AViterator@12@Vconst_iterator@12@@Z 1002c582 f i CtrlListWZ.obj
 0001:0002bb66       ??1out_of_range@std@@UAE@XZ 1002cb66 f i CtrlListWZ.obj
 0001:0002bb82       ??_Gout_of_range@std@@UAEPAXI@Z 1002cb82 f i CtrlListWZ.obj
 0001:0002bb82       ??_Eout_of_range@std@@UAEPAXI@Z 1002cb82 f i CtrlListWZ.obj
 0001:0002bbb4       ?clear@?$_Tree@V?$_Tmap_traits@V?$basic_string@DU?$char_traits@D@std@@V?$allocator@D@2@@std@@PAXU?$less@V?$basic_string@DU?$char_traits@D@std@@V?$allocator@D@2@@std@@@2@V?$allocator@U?$pair@$$CBV?$basic_string@DU?$char_traits@D@std@@V?$allocator@D@2@@std@@PAX@std@@@2@$00@std@@@std@@QAEXXZ 1002cbb4 f i CtrlListWZ.obj
 0001:0002bc09       ??C?$_Revranit@Viterator@?$_Tree@V?$_Tmap_traits@V?$basic_string@DU?$char_traits@D@std@@V?$allocator@D@2@@std@@PAXU?$less@V?$basic_string@DU?$char_traits@D@std@@V?$allocator@D@2@@std@@@2@V?$allocator@U?$pair@$$CBV?$basic_string@DU?$char_traits@D@std@@V?$allocator@D@2@@std@@PAX@std@@@2@$00@std@@@std@@U?$iterator@Ubidirectional_iterator_tag@std@@U?$pair@$$CBV?$basic_string@DU?$char_traits@D@std@@V?$allocator@D@2@@std@@PAX@2@HPAU32@AAU32@@3@@std@@QBEPAU?$pair@$$CBV?$basic_string@DU?$char_traits@D@std@@V?$allocator@D@2@@std@@PAX@1@XZ 1002cc09 f i CtrlListWZ.obj
 0001:0002bc32       ??C?$_Revranit@Viterator@?$_Tree@V?$_Tmap_traits@KPAXU?$less@K@std@@V?$allocator@U?$pair@$$CBKPAX@std@@@2@$0A@@std@@@std@@U?$iterator@Ubidirectional_iterator_tag@std@@U?$pair@$$CBKPAX@2@HPAU32@AAU32@@3@@std@@QBEPAU?$pair@$$CBKPAX@1@XZ 1002cc32 f i CtrlListWZ.obj
 0001:0002bc5b       ??1?$_List_val@UtagRECT@@V?$allocator@UtagRECT@@@std@@@std@@QAE@XZ 1002cc5b f i DialogWZ.obj
 0001:0002bc5b       ??1?$_Tree_val@V?$_Tmap_traits@KPAXU?$less@K@std@@V?$allocator@U?$pair@$$CBKPAX@std@@@2@$0A@@std@@@std@@QAE@XZ 1002cc5b f i CtrlListWZ.obj
 0001:0002bc5b       ??1?$_Tree_val@V?$_Tmap_traits@KPAUCListSellData@CCtrlListWZ@@U?$less@K@std@@V?$allocator@U?$pair@$$CBKPAUCListSellData@CCtrlListWZ@@@std@@@4@$0A@@std@@@std@@QAE@XZ 1002cc5b f i CtrlListWZ.obj
 0001:0002bc5b       ??1?$_Vector_val@KV?$allocator@K@std@@@std@@QAE@XZ 1002cc5b f i CtrlDxEdit.obj
 0001:0002bc5b       ??1?$_List_val@KV?$allocator@K@std@@@std@@QAE@XZ 1002cc5b f i BaseManager.obj
 0001:0002bc5b       ??1?$_Vector_val@U_List_position@?$_Hash@V?$_Hmap_traits@KV?$basic_string@DU?$char_traits@D@std@@V?$allocator@D@2@@std@@V?$hash_compare@KU?$less@K@std@@@stdext@@V?$allocator@U?$pair@$$CBKV?$basic_string@DU?$char_traits@D@std@@V?$allocator@D@2@@std@@@std@@@2@$0A@@stdext@@@stdext@@V?$allocator@U_List_position@?$_Hash@V?$_Hmap_traits@KV?$basic_string@DU?$char_traits@D@std@@V?$allocator@D@2@@std@@V?$hash_compare@KU?$less@K@std@@@stdext@@V?$allocator@U?$pair@$$CBKV?$basic_string@DU?$char_traits@D@std@@V?$allocator@D@2@@std@@@std@@@2@$0A@@stdext@@@stdext@@@std@@@std@@QAE@XZ 1002cc5b f i StringManager.obj
 0001:0002bc5b       ??1?$_List_val@PAXV?$allocator@PAX@std@@@std@@QAE@XZ 1002cc5b f i CtrlListWZ.obj
 0001:0002bc5b       ??1?$_Tree_val@V?$_Tmap_traits@V?$basic_string@DU?$char_traits@D@std@@V?$allocator@D@2@@std@@PAXU?$less@V?$basic_string@DU?$char_traits@D@std@@V?$allocator@D@2@@std@@@2@V?$allocator@U?$pair@$$CBV?$basic_string@DU?$char_traits@D@std@@V?$allocator@D@2@@std@@PAX@std@@@2@$00@std@@@std@@QAE@XZ 1002cc5b f i CtrlListWZ.obj
 0001:0002bc5b       ??1?$_Tree_val@V?$_Tmap_traits@KKU?$less@K@std@@V?$allocator@U?$pair@$$CBKK@std@@@2@$0A@@std@@@std@@QAE@XZ 1002cc5b f i CtrlTabWZ.obj
 0001:0002bc5b       ??1?$_Vector_val@U_List_position@?$_Hash@V?$_Hmap_traits@KPAXV?$hash_compare@KU?$less@K@std@@@stdext@@V?$allocator@U?$pair@$$CBKPAX@std@@@std@@$0A@@stdext@@@stdext@@V?$allocator@U_List_position@?$_Hash@V?$_Hmap_traits@KPAXV?$hash_compare@KU?$less@K@std@@@stdext@@V?$allocator@U?$pair@$$CBKPAX@std@@@std@@$0A@@stdext@@@stdext@@@std@@@std@@QAE@XZ 1002cc5b f i BaseManager.obj
 0001:0002bc5b       ??1?$_List_val@U?$pair@$$CBKV?$basic_string@DU?$char_traits@D@std@@V?$allocator@D@2@@std@@@std@@V?$allocator@U?$pair@$$CBKV?$basic_string@DU?$char_traits@D@std@@V?$allocator@D@2@@std@@@std@@@2@@std@@QAE@XZ 1002cc5b f i StringManager.obj
 0001:0002bc5b       ??1?$_List_val@PAVCControlWZ@@V?$allocator@PAVCControlWZ@@@std@@@std@@QAE@XZ 1002cc5b f i DialogWZ.obj
 0001:0002bc5b       ??1?$_List_val@U?$pair@$$CBKPAX@std@@V?$allocator@U?$pair@$$CBKPAX@std@@@2@@std@@QAE@XZ 1002cc5b f i BaseManager.obj
 0001:0002bc76       ??0out_of_range@std@@QAE@ABV01@@Z 1002cc76 f i CtrlListWZ.obj
 0001:0002bc9a       ?_Tidy@?$_Tree@V?$_Tmap_traits@KPAUCListSellData@CCtrlListWZ@@U?$less@K@std@@V?$allocator@U?$pair@$$CBKPAUCListSellData@CCtrlListWZ@@@std@@@4@$0A@@std@@@std@@IAEXXZ 1002cc9a f i CtrlListWZ.obj
 0001:0002bc9a       ?_Tidy@?$_Tree@V?$_Tmap_traits@KPAXU?$less@K@std@@V?$allocator@U?$pair@$$CBKPAX@std@@@2@$0A@@std@@@std@@IAEXXZ 1002cc9a f i CtrlListWZ.obj
 0001:0002bc9a       ?_Tidy@?$_Tree@V?$_Tmap_traits@KKU?$less@K@std@@V?$allocator@U?$pair@$$CBKK@std@@@2@$0A@@std@@@std@@IAEXXZ 1002cc9a f i CtrlTabWZ.obj
 0001:0002bd5a       ??0?$_Tree@V?$_Tmap_traits@V?$basic_string@DU?$char_traits@D@std@@V?$allocator@D@2@@std@@PAXU?$less@V?$basic_string@DU?$char_traits@D@std@@V?$allocator@D@2@@std@@@2@V?$allocator@U?$pair@$$CBV?$basic_string@DU?$char_traits@D@std@@V?$allocator@D@2@@std@@PAX@std@@@2@$00@std@@@std@@QAE@ABU?$less@V?$basic_string@DU?$char_traits@D@std@@V?$allocator@D@2@@std@@@1@ABV?$allocator@U?$pair@$$CBV?$basic_string@DU?$char_traits@D@std@@V?$allocator@D@2@@std@@PAX@std@@@1@@Z 1002cd5a f i CtrlListWZ.obj
 0001:0002bdbb       ?insert@?$_Tree@V?$_Tmap_traits@V?$basic_string@DU?$char_traits@D@std@@V?$allocator@D@2@@std@@PAXU?$less@V?$basic_string@DU?$char_traits@D@std@@V?$allocator@D@2@@std@@@2@V?$allocator@U?$pair@$$CBV?$basic_string@DU?$char_traits@D@std@@V?$allocator@D@2@@std@@PAX@std@@@2@$00@std@@@std@@QAE?AU?$pair@Viterator@?$_Tree@V?$_Tmap_traits@V?$basic_string@DU?$char_traits@D@std@@V?$allocator@D@2@@std@@PAXU?$less@V?$basic_string@DU?$char_traits@D@std@@V?$allocator@D@2@@std@@@2@V?$allocator@U?$pair@$$CBV?$basic_string@DU?$char_traits@D@std@@V?$allocator@D@2@@std@@PAX@std@@@2@$00@std@@@std@@_N@2@ABU?$pair@$$CBV?$basic_string@DU?$char_traits@D@std@@V?$allocator@D@2@@std@@PAX@2@@Z 1002cdbb f i CtrlListWZ.obj
 0001:0002bf97       ?_Erase@?$_Tree@V?$_Tmap_traits@V?$basic_string@DU?$char_traits@D@std@@V?$allocator@D@2@@std@@PAXU?$less@V?$basic_string@DU?$char_traits@D@std@@V?$allocator@D@2@@std@@@2@V?$allocator@U?$pair@$$CBV?$basic_string@DU?$char_traits@D@std@@V?$allocator@D@2@@std@@PAX@std@@@2@$00@std@@@std@@IAEXPAU_Node@?$_Tree_nod@V?$_Tmap_traits@V?$basic_string@DU?$char_traits@D@std@@V?$allocator@D@2@@std@@PAXU?$less@V?$basic_string@DU?$char_traits@D@std@@V?$allocator@D@2@@std@@@2@V?$allocator@U?$pair@$$CBV?$basic_string@DU?$char_traits@D@std@@V?$allocator@D@2@@std@@PAX@std@@@2@$00@std@@@2@@Z 1002cf97 f i CtrlListWZ.obj
 0001:0002bfe7       ?_Lrotate@?$_Tree@V?$_Tmap_traits@V?$basic_string@DU?$char_traits@D@std@@V?$allocator@D@2@@std@@PAXU?$less@V?$basic_string@DU?$char_traits@D@std@@V?$allocator@D@2@@std@@@2@V?$allocator@U?$pair@$$CBV?$basic_string@DU?$char_traits@D@std@@V?$allocator@D@2@@std@@PAX@std@@@2@$00@std@@@std@@IAEXPAU_Node@?$_Tree_nod@V?$_Tmap_traits@V?$basic_string@DU?$char_traits@D@std@@V?$allocator@D@2@@std@@PAXU?$less@V?$basic_string@DU?$char_traits@D@std@@V?$allocator@D@2@@std@@@2@V?$allocator@U?$pair@$$CBV?$basic_string@DU?$char_traits@D@std@@V?$allocator@D@2@@std@@PAX@std@@@2@$00@std@@@2@@Z 1002cfe7 f i CtrlListWZ.obj
 0001:0002c08b       ?_Rrotate@?$_Tree@V?$_Tmap_traits@V?$basic_string@DU?$char_traits@D@std@@V?$allocator@D@2@@std@@PAXU?$less@V?$basic_string@DU?$char_traits@D@std@@V?$allocator@D@2@@std@@@2@V?$allocator@U?$pair@$$CBV?$basic_string@DU?$char_traits@D@std@@V?$allocator@D@2@@std@@PAX@std@@@2@$00@std@@@std@@IAEXPAU_Node@?$_Tree_nod@V?$_Tmap_traits@V?$basic_string@DU?$char_traits@D@std@@V?$allocator@D@2@@std@@PAXU?$less@V?$basic_string@DU?$char_traits@D@std@@V?$allocator@D@2@@std@@@2@V?$allocator@U?$pair@$$CBV?$basic_string@DU?$char_traits@D@std@@V?$allocator@D@2@@std@@PAX@std@@@2@$00@std@@@2@@Z 1002d08b f i CtrlListWZ.obj
 0001:0002c12c       ?_Tidy@?$_Tree@V?$_Tmap_traits@V?$basic_string@DU?$char_traits@D@std@@V?$allocator@D@2@@std@@PAXU?$less@V?$basic_string@DU?$char_traits@D@std@@V?$allocator@D@2@@std@@@2@V?$allocator@U?$pair@$$CBV?$basic_string@DU?$char_traits@D@std@@V?$allocator@D@2@@std@@PAX@std@@@2@$00@std@@@std@@IAEXXZ 1002d12c f i CtrlListWZ.obj
 0001:0002c1ec       ?_Tidy@?$list@PAXV?$allocator@PAX@std@@@std@@IAEXXZ 1002d1ec f i CtrlListWZ.obj
 0001:0002c1ec       ?_Tidy@?$list@PAVCControlWZ@@V?$allocator@PAVCControlWZ@@@std@@@std@@IAEXXZ 1002d1ec f i DialogWZ.obj
 0001:0002c1ec       ?_Tidy@?$list@KV?$allocator@K@std@@@std@@IAEXXZ 1002d1ec f i BaseManager.obj
 0001:0002c1ec       ?_Tidy@?$list@U?$pair@$$CBKPAX@std@@V?$allocator@U?$pair@$$CBKPAX@std@@@2@@std@@IAEXXZ 1002d1ec f i BaseManager.obj
 0001:0002c1ec       ?_Tidy@?$list@UtagRECT@@V?$allocator@UtagRECT@@@std@@@std@@IAEXXZ 1002d1ec f i DialogWZ.obj
 0001:0002c221       ??E?$_Const_iterator@$00@?$list@U?$pair@$$CBKPAX@std@@V?$allocator@U?$pair@$$CBKPAX@std@@@2@@std@@QAEAAV012@XZ 1002d221 f i BaseManager.obj
 0001:0002c221       ??E?$_Const_iterator@$00@?$list@PAXV?$allocator@PAX@std@@@std@@QAEAAV012@XZ 1002d221 f i CtrlListWZ.obj
 0001:0002c221       ??E?$_Const_iterator@$00@?$list@KV?$allocator@K@std@@@std@@QAEAAV012@XZ 1002d221 f i BaseManager.obj
 0001:0002c221       ??E?$_Const_iterator@$00@?$list@U?$pair@$$CBKV?$basic_string@DU?$char_traits@D@std@@V?$allocator@D@2@@std@@@std@@V?$allocator@U?$pair@$$CBKV?$basic_string@DU?$char_traits@D@std@@V?$allocator@D@2@@std@@@std@@@2@@std@@QAEAAV012@XZ 1002d221 f i StringManager.obj
 0001:0002c221       ??E?$_Const_iterator@$00@?$list@PAVCControlWZ@@V?$allocator@PAVCControlWZ@@@std@@@std@@QAEAAV012@XZ 1002d221 f i CtrlDxEdit.obj
 0001:0002c221       ??E?$_Const_iterator@$00@?$list@UtagRECT@@V?$allocator@UtagRECT@@@std@@@std@@QAEAAV012@XZ 1002d221 f i DialogWZ.obj
 0001:0002c2a3       ?erase@?$_Tree@V?$_Tmap_traits@KPAUCListSellData@CCtrlListWZ@@U?$less@K@std@@V?$allocator@U?$pair@$$CBKPAUCListSellData@CCtrlListWZ@@@std@@@4@$0A@@std@@@std@@QAE?AViterator@12@Vconst_iterator@12@0@Z 1002d2a3 f i CtrlListWZ.obj
 0001:0002c2a3       ?erase@?$_Tree@V?$_Tmap_traits@KPAXU?$less@K@std@@V?$allocator@U?$pair@$$CBKPAX@std@@@2@$0A@@std@@@std@@QAE?AViterator@12@Vconst_iterator@12@0@Z 1002d2a3 f i CtrlListWZ.obj
 0001:0002c2a3       ?erase@?$_Tree@V?$_Tmap_traits@KKU?$less@K@std@@V?$allocator@U?$pair@$$CBKK@std@@@2@$0A@@std@@@std@@QAE?AViterator@12@Vconst_iterator@12@0@Z 1002d2a3 f i CtrlTabWZ.obj
 0001:0002c45d       ??9const_iterator@?$_Tree@V?$_Tmap_traits@KPAXU?$less@K@std@@V?$allocator@U?$pair@$$CBKPAX@std@@@2@$0A@@std@@@std@@QBE_NABV012@@Z 1002d45d f i CtrlListWZ.obj
 0001:0002c45d       ??9const_iterator@?$_Tree@V?$_Tmap_traits@KKU?$less@K@std@@V?$allocator@U?$pair@$$CBKK@std@@@2@$0A@@std@@@std@@QBE_NABV012@@Z 1002d45d f i CtrlTabWZ.obj
 0001:0002c45d       ??9const_iterator@?$_Tree@V?$_Tmap_traits@KPAUCListSellData@CCtrlListWZ@@U?$less@K@std@@V?$allocator@U?$pair@$$CBKPAUCListSellData@CCtrlListWZ@@@std@@@4@$0A@@std@@@std@@QBE_NABV012@@Z 1002d45d f i CtrlListWZ.obj
 0001:0002c45d       ??9const_iterator@?$_Tree@V?$_Tmap_traits@V?$basic_string@DU?$char_traits@D@std@@V?$allocator@D@2@@std@@PAXU?$less@V?$basic_string@DU?$char_traits@D@std@@V?$allocator@D@2@@std@@@2@V?$allocator@U?$pair@$$CBV?$basic_string@DU?$char_traits@D@std@@V?$allocator@D@2@@std@@PAX@std@@@2@$00@std@@@std@@QBE_NABV012@@Z 1002d45d f i CtrlListWZ.obj
 0001:0002c4b2       ?_Lbound@?$_Tree@V?$_Tmap_traits@KPAXU?$less@K@std@@V?$allocator@U?$pair@$$CBKPAX@std@@@2@$0A@@std@@@std@@IBEPAU_Node@?$_Tree_nod@V?$_Tmap_traits@KPAXU?$less@K@std@@V?$allocator@U?$pair@$$CBKPAX@std@@@2@$0A@@std@@@2@ABK@Z 1002d4b2 f i CtrlListWZ.obj
 0001:0002c4b2       ?_Lbound@?$_Tree@V?$_Tmap_traits@KPAUCListSellData@CCtrlListWZ@@U?$less@K@std@@V?$allocator@U?$pair@$$CBKPAUCListSellData@CCtrlListWZ@@@std@@@4@$0A@@std@@@std@@IBEPAU_Node@?$_Tree_nod@V?$_Tmap_traits@KPAUCListSellData@CCtrlListWZ@@U?$less@K@std@@V?$allocator@U?$pair@$$CBKPAUCListSellData@CCtrlListWZ@@@std@@@4@$0A@@std@@@2@ABK@Z 1002d4b2 f i CtrlListWZ.obj
 0001:0002c4b2       ?_Lbound@?$_Tree@V?$_Tmap_traits@KKU?$less@K@std@@V?$allocator@U?$pair@$$CBKK@std@@@2@$0A@@std@@@std@@IBEPAU_Node@?$_Tree_nod@V?$_Tmap_traits@KKU?$less@K@std@@V?$allocator@U?$pair@$$CBKK@std@@@2@$0A@@std@@@2@ABK@Z 1002d4b2 f i CtrlTabWZ.obj
 0001:0002c513       ?erase@?$_Tree@V?$_Tmap_traits@V?$basic_string@DU?$char_traits@D@std@@V?$allocator@D@2@@std@@PAXU?$less@V?$basic_string@DU?$char_traits@D@std@@V?$allocator@D@2@@std@@@2@V?$allocator@U?$pair@$$CBV?$basic_string@DU?$char_traits@D@std@@V?$allocator@D@2@@std@@PAX@std@@@2@$00@std@@@std@@QAE?AViterator@12@Vconst_iterator@12@0@Z 1002d513 f i CtrlListWZ.obj
 0001:0002c6cd       ?_Init@?$_Tree@V?$_Tmap_traits@V?$basic_string@DU?$char_traits@D@std@@V?$allocator@D@2@@std@@PAXU?$less@V?$basic_string@DU?$char_traits@D@std@@V?$allocator@D@2@@std@@@2@V?$allocator@U?$pair@$$CBV?$basic_string@DU?$char_traits@D@std@@V?$allocator@D@2@@std@@PAX@std@@@2@$00@std@@@std@@IAEXXZ 1002d6cd f i CtrlListWZ.obj
 0001:0002c728       ?_Insert@?$_Tree@V?$_Tmap_traits@V?$basic_string@DU?$char_traits@D@std@@V?$allocator@D@2@@std@@PAXU?$less@V?$basic_string@DU?$char_traits@D@std@@V?$allocator@D@2@@std@@@2@V?$allocator@U?$pair@$$CBV?$basic_string@DU?$char_traits@D@std@@V?$allocator@D@2@@std@@PAX@std@@@2@$00@std@@@std@@IAE?AViterator@12@_NPAU_Node@?$_Tree_nod@V?$_Tmap_traits@V?$basic_string@DU?$char_traits@D@std@@V?$allocator@D@2@@std@@PAXU?$less@V?$basic_string@DU?$char_traits@D@std@@V?$allocator@D@2@@std@@@2@V?$allocator@U?$pair@$$CBV?$basic_string@DU?$char_traits@D@std@@V?$allocator@D@2@@std@@PAX@std@@@2@$00@std@@@2@ABU?$pair@$$CBV?$basic_string@DU?$char_traits@D@std@@V?$allocator@D@2@@std@@PAX@2@@Z 1002d728 f i CtrlListWZ.obj
 0001:0002cae3       ??0?$_Tree_val@V?$_Tmap_traits@KPAXU?$less@K@std@@V?$allocator@U?$pair@$$CBKPAX@std@@@2@$0A@@std@@@std@@IAE@ABU?$less@K@1@V?$allocator@U?$pair@$$CBKPAX@std@@@1@@Z 1002dae3 f i CtrlListWZ.obj
 0001:0002cae3       ??0?$_Tree_val@V?$_Tmap_traits@KKU?$less@K@std@@V?$allocator@U?$pair@$$CBKK@std@@@2@$0A@@std@@@std@@IAE@ABU?$less@K@1@V?$allocator@U?$pair@$$CBKK@std@@@1@@Z 1002dae3 f i CtrlTabWZ.obj
 0001:0002cae3       ??0?$_Tree_val@V?$_Tmap_traits@KPAUCListSellData@CCtrlListWZ@@U?$less@K@std@@V?$allocator@U?$pair@$$CBKPAUCListSellData@CCtrlListWZ@@@std@@@4@$0A@@std@@@std@@IAE@ABU?$less@K@1@V?$allocator@U?$pair@$$CBKPAUCListSellData@CCtrlListWZ@@@std@@@1@@Z 1002dae3 f i CtrlListWZ.obj
 0001:0002cae3       ??0?$_Tree_val@V?$_Tmap_traits@V?$basic_string@DU?$char_traits@D@std@@V?$allocator@D@2@@std@@PAXU?$less@V?$basic_string@DU?$char_traits@D@std@@V?$allocator@D@2@@std@@@2@V?$allocator@U?$pair@$$CBV?$basic_string@DU?$char_traits@D@std@@V?$allocator@D@2@@std@@PAX@std@@@2@$00@std@@@std@@IAE@ABU?$less@V?$basic_string@DU?$char_traits@D@std@@V?$allocator@D@2@@std@@@1@V?$allocator@U?$pair@$$CBV?$basic_string@DU?$char_traits@D@std@@V?$allocator@D@2@@std@@PAX@std@@@1@@Z 1002dae3 f i CtrlListWZ.obj
 0001:0002cb0a       ??Dconst_iterator@?$_Tree@V?$_Tmap_traits@V?$basic_string@DU?$char_traits@D@std@@V?$allocator@D@2@@std@@PAXU?$less@V?$basic_string@DU?$char_traits@D@std@@V?$allocator@D@2@@std@@@2@V?$allocator@U?$pair@$$CBV?$basic_string@DU?$char_traits@D@std@@V?$allocator@D@2@@std@@PAX@std@@@2@$00@std@@@std@@QBEABU?$pair@$$CBV?$basic_string@DU?$char_traits@D@std@@V?$allocator@D@2@@std@@PAX@2@XZ 1002db0a f i CtrlListWZ.obj
 0001:0002cb0a       ??Dconst_iterator@?$_Tree@V?$_Tmap_traits@KPAXU?$less@K@std@@V?$allocator@U?$pair@$$CBKPAX@std@@@2@$0A@@std@@@std@@QBEABU?$pair@$$CBKPAX@2@XZ 1002db0a f i CtrlListWZ.obj
 0001:0002cb0a       ??Dconst_iterator@?$_Tree@V?$_Tmap_traits@KKU?$less@K@std@@V?$allocator@U?$pair@$$CBKK@std@@@2@$0A@@std@@@std@@QBEABU?$pair@$$CBKK@2@XZ 1002db0a f i CtrlTabWZ.obj
 0001:0002cb0a       ??Dconst_iterator@?$_Tree@V?$_Tmap_traits@KPAUCListSellData@CCtrlListWZ@@U?$less@K@std@@V?$allocator@U?$pair@$$CBKPAUCListSellData@CCtrlListWZ@@@std@@@4@$0A@@std@@@std@@QBEABU?$pair@$$CBKPAUCListSellData@CCtrlListWZ@@@2@XZ 1002db0a f i CtrlListWZ.obj
 0001:0002cb74       ??0const_iterator@?$_Tree@V?$_Tmap_traits@KKU?$less@K@std@@V?$allocator@U?$pair@$$CBKK@std@@@2@$0A@@std@@@std@@QAE@PAU_Node@?$_Tree_nod@V?$_Tmap_traits@KKU?$less@K@std@@V?$allocator@U?$pair@$$CBKK@std@@@2@$0A@@std@@@2@PBV12@@Z 1002db74 f i CtrlTabWZ.obj
 0001:0002cb74       ??0const_iterator@?$_Tree@V?$_Tmap_traits@KPAUCListSellData@CCtrlListWZ@@U?$less@K@std@@V?$allocator@U?$pair@$$CBKPAUCListSellData@CCtrlListWZ@@@std@@@4@$0A@@std@@@std@@QAE@PAU_Node@?$_Tree_nod@V?$_Tmap_traits@KPAUCListSellData@CCtrlListWZ@@U?$less@K@std@@V?$allocator@U?$pair@$$CBKPAUCListSellData@CCtrlListWZ@@@std@@@4@$0A@@std@@@2@PBV12@@Z 1002db74 f i CtrlListWZ.obj
 0001:0002cb74       ??0const_iterator@?$_Tree@V?$_Tmap_traits@KPAXU?$less@K@std@@V?$allocator@U?$pair@$$CBKPAX@std@@@2@$0A@@std@@@std@@QAE@PAU_Node@?$_Tree_nod@V?$_Tmap_traits@KPAXU?$less@K@std@@V?$allocator@U?$pair@$$CBKPAX@std@@@2@$0A@@std@@@2@PBV12@@Z 1002db74 f i CtrlListWZ.obj
 0001:0002cb74       ??0const_iterator@?$_Tree@V?$_Tmap_traits@V?$basic_string@DU?$char_traits@D@std@@V?$allocator@D@2@@std@@PAXU?$less@V?$basic_string@DU?$char_traits@D@std@@V?$allocator@D@2@@std@@@2@V?$allocator@U?$pair@$$CBV?$basic_string@DU?$char_traits@D@std@@V?$allocator@D@2@@std@@PAX@std@@@2@$00@std@@@std@@QAE@PAU_Node@?$_Tree_nod@V?$_Tmap_traits@V?$basic_string@DU?$char_traits@D@std@@V?$allocator@D@2@@std@@PAXU?$less@V?$basic_string@DU?$char_traits@D@std@@V?$allocator@D@2@@std@@@2@V?$allocator@U?$pair@$$CBV?$basic_string@DU?$char_traits@D@std@@V?$allocator@D@2@@std@@PAX@std@@@2@$00@std@@@2@PBV12@@Z 1002db74 f i CtrlListWZ.obj
 0001:0002cbaa       ?_Inc@const_iterator@?$_Tree@V?$_Tmap_traits@KKU?$less@K@std@@V?$allocator@U?$pair@$$CBKK@std@@@2@$0A@@std@@@std@@QAEXXZ 1002dbaa f i CtrlTabWZ.obj
 0001:0002cbaa       ?_Inc@const_iterator@?$_Tree@V?$_Tmap_traits@KPAUCListSellData@CCtrlListWZ@@U?$less@K@std@@V?$allocator@U?$pair@$$CBKPAUCListSellData@CCtrlListWZ@@@std@@@4@$0A@@std@@@std@@QAEXXZ 1002dbaa f i CtrlListWZ.obj
 0001:0002cbaa       ?_Inc@const_iterator@?$_Tree@V?$_Tmap_traits@KPAXU?$less@K@std@@V?$allocator@U?$pair@$$CBKPAX@std@@@2@$0A@@std@@@std@@QAEXXZ 1002dbaa f i CtrlListWZ.obj
 0001:0002cc70       ?_Inc@const_iterator@?$_Tree@V?$_Tmap_traits@V?$basic_string@DU?$char_traits@D@std@@V?$allocator@D@2@@std@@PAXU?$less@V?$basic_string@DU?$char_traits@D@std@@V?$allocator@D@2@@std@@@2@V?$allocator@U?$pair@$$CBV?$basic_string@DU?$char_traits@D@std@@V?$allocator@D@2@@std@@PAX@std@@@2@$00@std@@@std@@QAEXXZ 1002dc70 f i CtrlListWZ.obj
 0001:0002cd36       ?erase@?$_Tree@V?$_Tmap_traits@KPAUCListSellData@CCtrlListWZ@@U?$less@K@std@@V?$allocator@U?$pair@$$CBKPAUCListSellData@CCtrlListWZ@@@std@@@4@$0A@@std@@@std@@QAE?AViterator@12@Vconst_iterator@12@@Z 1002dd36 f i CtrlListWZ.obj
 0001:0002cd36       ?erase@?$_Tree@V?$_Tmap_traits@KPAXU?$less@K@std@@V?$allocator@U?$pair@$$CBKPAX@std@@@2@$0A@@std@@@std@@QAE?AViterator@12@Vconst_iterator@12@@Z 1002dd36 f i CtrlListWZ.obj
 0001:0002cd36       ?erase@?$_Tree@V?$_Tmap_traits@KKU?$less@K@std@@V?$allocator@U?$pair@$$CBKK@std@@@2@$0A@@std@@@std@@QAE?AViterator@12@Vconst_iterator@12@@Z 1002dd36 f i CtrlTabWZ.obj
 0001:0002d311       ?compare@?$basic_string@DU?$char_traits@D@std@@V?$allocator@D@2@@std@@QBEHABV12@@Z 1002e311 f i CtrlListWZ.obj
 0001:0002d35a       ?_Rrotate@?$_Tree@V?$_Tmap_traits@KPAUCListSellData@CCtrlListWZ@@U?$less@K@std@@V?$allocator@U?$pair@$$CBKPAUCListSellData@CCtrlListWZ@@@std@@@4@$0A@@std@@@std@@IAEXPAU_Node@?$_Tree_nod@V?$_Tmap_traits@KPAUCListSellData@CCtrlListWZ@@U?$less@K@std@@V?$allocator@U?$pair@$$CBKPAUCListSellData@CCtrlListWZ@@@std@@@4@$0A@@std@@@2@@Z 1002e35a f i CtrlListWZ.obj
 0001:0002d35a       ?_Rrotate@?$_Tree@V?$_Tmap_traits@KKU?$less@K@std@@V?$allocator@U?$pair@$$CBKK@std@@@2@$0A@@std@@@std@@IAEXPAU_Node@?$_Tree_nod@V?$_Tmap_traits@KKU?$less@K@std@@V?$allocator@U?$pair@$$CBKK@std@@@2@$0A@@std@@@2@@Z 1002e35a f i CtrlTabWZ.obj
 0001:0002d35a       ?_Rrotate@?$_Tree@V?$_Tmap_traits@KPAXU?$less@K@std@@V?$allocator@U?$pair@$$CBKPAX@std@@@2@$0A@@std@@@std@@IAEXPAU_Node@?$_Tree_nod@V?$_Tmap_traits@KPAXU?$less@K@std@@V?$allocator@U?$pair@$$CBKPAX@std@@@2@$0A@@std@@@2@@Z 1002e35a f i CtrlListWZ.obj
 0001:0002d3fb       ?compare@?$basic_string@DU?$char_traits@D@std@@V?$allocator@D@2@@std@@QBEHIIPBDI@Z 1002e3fb f i CtrlListWZ.obj
 0001:0002d4c5       ?_Buynode@?$_Tree@V?$_Tmap_traits@V?$basic_string@DU?$char_traits@D@std@@V?$allocator@D@2@@std@@PAXU?$less@V?$basic_string@DU?$char_traits@D@std@@V?$allocator@D@2@@std@@@2@V?$allocator@U?$pair@$$CBV?$basic_string@DU?$char_traits@D@std@@V?$allocator@D@2@@std@@PAX@std@@@2@$00@std@@@std@@IAEPAU_Node@?$_Tree_nod@V?$_Tmap_traits@V?$basic_string@DU?$char_traits@D@std@@V?$allocator@D@2@@std@@PAXU?$less@V?$basic_string@DU?$char_traits@D@std@@V?$allocator@D@2@@std@@@2@V?$allocator@U?$pair@$$CBV?$basic_string@DU?$char_traits@D@std@@V?$allocator@D@2@@std@@PAX@std@@@2@$00@std@@@2@XZ 1002e4c5 f i CtrlListWZ.obj
 0001:0002d5df       ?_Buynode@?$_Tree@V?$_Tmap_traits@V?$basic_string@DU?$char_traits@D@std@@V?$allocator@D@2@@std@@PAXU?$less@V?$basic_string@DU?$char_traits@D@std@@V?$allocator@D@2@@std@@@2@V?$allocator@U?$pair@$$CBV?$basic_string@DU?$char_traits@D@std@@V?$allocator@D@2@@std@@PAX@std@@@2@$00@std@@@std@@IAEPAU_Node@?$_Tree_nod@V?$_Tmap_traits@V?$basic_string@DU?$char_traits@D@std@@V?$allocator@D@2@@std@@PAXU?$less@V?$basic_string@DU?$char_traits@D@std@@V?$allocator@D@2@@std@@@2@V?$allocator@U?$pair@$$CBV?$basic_string@DU?$char_traits@D@std@@V?$allocator@D@2@@std@@PAX@std@@@2@$00@std@@@2@PAU342@00ABU?$pair@$$CBV?$basic_string@DU?$char_traits@D@std@@V?$allocator@D@2@@std@@PAX@2@D@Z 1002e5df f i CtrlListWZ.obj
 0001:0002d6b5       ??0?$_Tree_ptr@V?$_Tmap_traits@V?$basic_string@DU?$char_traits@D@std@@V?$allocator@D@2@@std@@PAXU?$less@V?$basic_string@DU?$char_traits@D@std@@V?$allocator@D@2@@std@@@2@V?$allocator@U?$pair@$$CBV?$basic_string@DU?$char_traits@D@std@@V?$allocator@D@2@@std@@PAX@std@@@2@$00@std@@@std@@IAE@ABU?$less@V?$basic_string@DU?$char_traits@D@std@@V?$allocator@D@2@@std@@@1@V?$allocator@U?$pair@$$CBV?$basic_string@DU?$char_traits@D@std@@V?$allocator@D@2@@std@@PAX@std@@@1@@Z 1002e6b5 f i CtrlListWZ.obj
 0001:0002d6b5       ??0?$_Tree_ptr@V?$_Tmap_traits@KPAXU?$less@K@std@@V?$allocator@U?$pair@$$CBKPAX@std@@@2@$0A@@std@@@std@@IAE@ABU?$less@K@1@V?$allocator@U?$pair@$$CBKPAX@std@@@1@@Z 1002e6b5 f i CtrlListWZ.obj
 0001:0002d6b5       ??0?$_Tree_ptr@V?$_Tmap_traits@KPAUCListSellData@CCtrlListWZ@@U?$less@K@std@@V?$allocator@U?$pair@$$CBKPAUCListSellData@CCtrlListWZ@@@std@@@4@$0A@@std@@@std@@IAE@ABU?$less@K@1@V?$allocator@U?$pair@$$CBKPAUCListSellData@CCtrlListWZ@@@std@@@1@@Z 1002e6b5 f i CtrlListWZ.obj
 0001:0002d6b5       ??0?$_Tree_ptr@V?$_Tmap_traits@KKU?$less@K@std@@V?$allocator@U?$pair@$$CBKK@std@@@2@$0A@@std@@@std@@IAE@ABU?$less@K@1@V?$allocator@U?$pair@$$CBKK@std@@@1@@Z 1002e6b5 f i CtrlTabWZ.obj
 0001:0002d6f9       ?_Dec@const_iterator@?$_Tree@V?$_Tmap_traits@KPAUCListSellData@CCtrlListWZ@@U?$less@K@std@@V?$allocator@U?$pair@$$CBKPAUCListSellData@CCtrlListWZ@@@std@@@4@$0A@@std@@@std@@QAEXXZ 1002e6f9 f i CtrlListWZ.obj
 0001:0002d6f9       ?_Dec@const_iterator@?$_Tree@V?$_Tmap_traits@KPAXU?$less@K@std@@V?$allocator@U?$pair@$$CBKPAX@std@@@2@$0A@@std@@@std@@QAEXXZ 1002e6f9 f i CtrlListWZ.obj
 0001:0002d6f9       ?_Dec@const_iterator@?$_Tree@V?$_Tmap_traits@KKU?$less@K@std@@V?$allocator@U?$pair@$$CBKK@std@@@2@$0A@@std@@@std@@QAEXXZ 1002e6f9 f i CtrlTabWZ.obj
 0001:0002d7ec       ?_Dec@const_iterator@?$_Tree@V?$_Tmap_traits@V?$basic_string@DU?$char_traits@D@std@@V?$allocator@D@2@@std@@PAXU?$less@V?$basic_string@DU?$char_traits@D@std@@V?$allocator@D@2@@std@@@2@V?$allocator@U?$pair@$$CBV?$basic_string@DU?$char_traits@D@std@@V?$allocator@D@2@@std@@PAX@std@@@2@$00@std@@@std@@QAEXXZ 1002e7ec f i CtrlListWZ.obj
 0001:0002d8df       ??0?$pair@$$CBV?$basic_string@DU?$char_traits@D@std@@V?$allocator@D@2@@std@@PAX@std@@QAE@ABU01@@Z 1002e8df f i CtrlListWZ.obj
 0001:0002d8df       ??$?0V?$basic_string@DU?$char_traits@D@std@@V?$allocator@D@2@@std@@PAX@?$pair@$$CBV?$basic_string@DU?$char_traits@D@std@@V?$allocator@D@2@@std@@PAX@std@@QAE@ABU?$pair@V?$basic_string@DU?$char_traits@D@std@@V?$allocator@D@2@@std@@PAX@1@@Z 1002e8df f i CtrlListWZ.obj
 0001:0002d91a       ??$_Destroy@U_Node@?$_Tree_nod@V?$_Tmap_traits@V?$basic_string@DU?$char_traits@D@std@@V?$allocator@D@2@@std@@PAXU?$less@V?$basic_string@DU?$char_traits@D@std@@V?$allocator@D@2@@std@@@2@V?$allocator@U?$pair@$$CBV?$basic_string@DU?$char_traits@D@std@@V?$allocator@D@2@@std@@PAX@std@@@2@$00@std@@@std@@@std@@YAXPAU_Node@?$_Tree_nod@V?$_Tmap_traits@V?$basic_string@DU?$char_traits@D@std@@V?$allocator@D@2@@std@@PAXU?$less@V?$basic_string@DU?$char_traits@D@std@@V?$allocator@D@2@@std@@@2@V?$allocator@U?$pair@$$CBV?$basic_string@DU?$char_traits@D@std@@V?$allocator@D@2@@std@@PAX@std@@@2@$00@std@@@0@@Z 1002e91a f i CtrlListWZ.obj
 0001:0002d947       ??$_Allocate@U_Node@?$_Tree_nod@V?$_Tmap_traits@V?$basic_string@DU?$char_traits@D@std@@V?$allocator@D@2@@std@@PAXU?$less@V?$basic_string@DU?$char_traits@D@std@@V?$allocator@D@2@@std@@@2@V?$allocator@U?$pair@$$CBV?$basic_string@DU?$char_traits@D@std@@V?$allocator@D@2@@std@@PAX@std@@@2@$00@std@@@std@@@std@@YAPAU_Node@?$_Tree_nod@V?$_Tmap_traits@V?$basic_string@DU?$char_traits@D@std@@V?$allocator@D@2@@std@@PAXU?$less@V?$basic_string@DU?$char_traits@D@std@@V?$allocator@D@2@@std@@@2@V?$allocator@U?$pair@$$CBV?$basic_string@DU?$char_traits@D@std@@V?$allocator@D@2@@std@@PAX@std@@@2@$00@std@@@0@IPAU120@@Z 1002e947 f i CtrlListWZ.obj
 0001:0002d99a       ??0CCtrlPictureWZ@@QAE@XZ  1002e99a f   CtrlPictureWZ.obj
 0001:0002da12       ??1CCtrlPictureWZ@@UAE@XZ  1002ea12 f   CtrlPictureWZ.obj
 0001:0002da2c       ?OnDraw_InnerClip@CCtrlPictureWZ@@QAE_NXZ 1002ea2c f   CtrlPictureWZ.obj
 0001:0002dbef       ?UpdateBlend@CCtrlPictureWZ@@QAEXXZ 1002ebef f   CtrlPictureWZ.obj
 0001:0002dc78       ?EnableBlend@CCtrlPictureWZ@@UAEX_N@Z 1002ec78 f   CtrlPictureWZ.obj
 0001:0002dc8f       ?OnDraw@CCtrlPictureWZ@@UAE_N_N@Z 1002ec8f f   CtrlPictureWZ.obj
 0001:0002dd0a       ?EnableInnerClipDraw@CCtrlPictureWZ@@UAEX_N@Z 1002ed0a f   CtrlPictureWZ.obj
 0001:0002dd21       ?EnableLButtonEvent@CCtrlPictureWZ@@UAEX_N@Z 1002ed21 f   CtrlPictureWZ.obj
 0001:0002dd38       ?Message_MouseLButtonDown@CCtrlPictureWZ@@MAE_NPAUSI_MESSAGE@@@Z 1002ed38 f   CtrlPictureWZ.obj
 0001:0002de6c       ?Message_MouseLButtonUp@CCtrlPictureWZ@@MAE_NPAUSI_MESSAGE@@@Z 1002ee6c f   CtrlPictureWZ.obj
 0001:0002df8e       ?Message_MouseMove@CCtrlPictureWZ@@MAE_NPAUSI_MESSAGE@@@Z 1002ef8e f   CtrlPictureWZ.obj
 0001:0002e0a4       ?SendMessageWZ@CCtrlPictureWZ@@UAE_NPAUSI_MESSAGE@@@Z 1002f0a4 f   CtrlPictureWZ.obj
 0001:0002e139       ?GetClipRateWidth@CCtrlPictureWZ@@UBEMXZ 1002f139 f i CtrlPictureWZ.obj
 0001:0002e14b       ?SetClipRateWidth@CCtrlPictureWZ@@UAEXM@Z 1002f14b f i CtrlPictureWZ.obj
 0001:0002e166       ?GetClipRateHeight@CCtrlPictureWZ@@UBEMXZ 1002f166 f i CtrlPictureWZ.obj
 0001:0002e178       ?SetClipRateHeight@CCtrlPictureWZ@@UAEXM@Z 1002f178 f i CtrlPictureWZ.obj
 0001:0002e193       ??_ECCtrlPictureWZ@@UAEPAXI@Z 1002f193 f i CtrlPictureWZ.obj
 0001:0002e193       ??_GCCtrlPictureWZ@@UAEPAXI@Z 1002f193 f i CtrlPictureWZ.obj
 0001:0002e1ba       ??0CCtrlRectangleWZ@@QAE@XZ 1002f1ba f   CtrlRectangleWZ.obj
 0001:0002e212       ??1CCtrlRectangleWZ@@UAE@XZ 1002f212 f   CtrlRectangleWZ.obj
 0001:0002e22c       ?OnLoad@CCtrlRectangleWZ@@UAEXPAX@Z 1002f22c f   CtrlRectangleWZ.obj
 0001:0002e3b3       ?OnSave@CCtrlRectangleWZ@@UAEXPAX@Z 1002f3b3 f   CtrlRectangleWZ.obj
 0001:0002e448       ?OnDraw@CCtrlRectangleWZ@@UAE_N_N@Z 1002f448 f   CtrlRectangleWZ.obj
 0001:0002e58a       ?SetFill@CCtrlRectangleWZ@@UAEX_N@Z 1002f58a f i CtrlRectangleWZ.obj
 0001:0002e5a1       ?GetFill@CCtrlRectangleWZ@@UAE_NXZ 1002f5a1 f i CtrlRectangleWZ.obj
 0001:0002e5b3       ?SetThickness@CCtrlRectangleWZ@@UAEXH@Z 1002f5b3 f i CtrlRectangleWZ.obj
 0001:0002e5ca       ?SetLineColor@CCtrlRectangleWZ@@UAEXK@Z 1002f5ca f i CtrlRectangleWZ.obj
 0001:0002e5e1       ?GetLineColor@CCtrlRectangleWZ@@UAEXPAK@Z 1002f5e1 f i CtrlRectangleWZ.obj
 0001:0002e5fa       ?Message_MouseMove@CCtrlStaticWZ@@MAE_NPAUSI_MESSAGE@@@Z 1002f5fa f i CtrlStaticWZ.obj
 0001:0002e5fa       ?SendMessageWZ@CCtrlRectangleWZ@@MAE_NPAUSI_MESSAGE@@@Z 1002f5fa f i CtrlRectangleWZ.obj
 0001:0002e607       ??_ECCtrlRectangleWZ@@UAEPAXI@Z 1002f607 f i CtrlRectangleWZ.obj
 0001:0002e607       ??_GCCtrlRectangleWZ@@UAEPAXI@Z 1002f607 f i CtrlRectangleWZ.obj
 0001:0002e62e       ??0CCtrlStaticWZ@@QAE@XZ   1002f62e f   CtrlStaticWZ.obj
 0001:0002e6f5       ??1CCtrlStaticWZ@@UAE@XZ   1002f6f5 f   CtrlStaticWZ.obj
 0001:0002e755       ?OnCreate@CCtrlStaticWZ@@UAE_NKKPAUHWND__@@PAUHINSTANCE__@@PAUtagRECT@@PAX@Z 1002f755 f   CtrlStaticWZ.obj
 0001:0002e77c       ?MoveWindowWZ@CCtrlStaticWZ@@UAE_NMMMM@Z 1002f77c f   CtrlStaticWZ.obj
 0001:0002e7ad       ?OnLoad@CCtrlStaticWZ@@UAEXPAX@Z 1002f7ad f   CtrlStaticWZ.obj
 0001:0002ec49       ?OnSave@CCtrlStaticWZ@@UAEXPAX@Z 1002fc49 f   CtrlStaticWZ.obj
 0001:0002ed07       ?OnInitialize@CCtrlStaticWZ@@UAEXXZ 1002fd07 f   CtrlStaticWZ.obj
 0001:0002ed18       ?OnDestroy@CCtrlStaticWZ@@UAEXXZ 1002fd18 f   CtrlStaticWZ.obj
 0001:0002ed29       ?CheckNewLine@CCtrlStaticWZ@@AAEXPAD@Z 1002fd29 f   CtrlStaticWZ.obj
 0001:0002eeee       ?OnDraw@CCtrlStaticWZ@@UAE_N_N@Z 1002feee f   CtrlStaticWZ.obj
 0001:0002f109       ?ChangeCaptionString@CCtrlStaticWZ@@UAEXXZ 10030109 f   CtrlStaticWZ.obj
 0001:0002f1c6       ?ReleaseImage@CCtrlStaticWZ@@UAEXXZ 100301c6 f   CtrlStaticWZ.obj
 0001:0002f1cf       ?Message_MouseLButtonDown@CCtrlStaticWZ@@MAE_NPAUSI_MESSAGE@@@Z 100301cf f   CtrlStaticWZ.obj
 0001:0002f1dc       ?Message_MouseLButtonUp@CCtrlStaticWZ@@MAE_NPAUSI_MESSAGE@@@Z 100301dc f   CtrlStaticWZ.obj
 0001:0002f1e9       ?SendMessageWZ@CCtrlStaticWZ@@UAE_NPAUSI_MESSAGE@@@Z 100301e9 f   CtrlStaticWZ.obj
 0001:0002f272       ?GetTextWZW@CCtrlStaticWZ@@UAEXPA_WH@Z 10030272 f   CtrlStaticWZ.obj
 0001:0002f385       ?GetTextWZA@CCtrlStaticWZ@@UAEXPADH@Z 10030385 f   CtrlStaticWZ.obj
 0001:0002f40e       ?SetTextWZW@CCtrlStaticWZ@@UAEXPB_W_N@Z 1003040e f   CtrlStaticWZ.obj
 0001:0002f48f       ?SetTextWZA@CCtrlStaticWZ@@UAEXPBD_N@Z 1003048f f   CtrlStaticWZ.obj
 0001:0002f635       ?SetTextID@CCtrlStaticWZ@@UAEXK@Z 10030635 f   CtrlStaticWZ.obj
 0001:0002f657       ?GetTextID@CCtrlStaticWZ@@UAEKXZ 10030657 f   CtrlStaticWZ.obj
 0001:0002f666       ?SetFontID@CCtrlStaticWZ@@UAEXK@Z 10030666 f   CtrlStaticWZ.obj
 0001:0002f67d       ?GetFontID@CCtrlStaticWZ@@UAEKXZ 1003067d f   CtrlStaticWZ.obj
 0001:0002f68f       ?SetTextKind@CCtrlStaticWZ@@UAEXW4ENUM_TEXT_KIND@@@Z 1003068f f   CtrlStaticWZ.obj
 0001:0002f6a6       ?GetTextKind@CCtrlStaticWZ@@UAE?AW4ENUM_TEXT_KIND@@XZ 100306a6 f   CtrlStaticWZ.obj
 0001:0002f6b8       ??0CCtrlImageStaticWZ@@QAE@XZ 100306b8 f   CtrlStaticWZ.obj
 0001:0002f737       ??1CCtrlImageStaticWZ@@UAE@XZ 10030737 f   CtrlStaticWZ.obj
 0001:0002f751       ?OnLoad@CCtrlImageStaticWZ@@UAEXPAX@Z 10030751 f   CtrlStaticWZ.obj
 0001:0002f95e       ?OnSave@CCtrlImageStaticWZ@@UAEXPAX@Z 1003095e f   CtrlStaticWZ.obj
 0001:0002fa1c       ?OnDraw@CCtrlImageStaticWZ@@UAE_N_N@Z 10030a1c f   CtrlStaticWZ.obj
 0001:0002fc67       ?ReleaseImage@CCtrlImageStaticWZ@@UAEXXZ 10030c67 f   CtrlStaticWZ.obj
 0001:0002fc78       ?Message_MouseLButtonDown@CCtrlImageStaticWZ@@MAE_NPAUSI_MESSAGE@@@Z 10030c78 f   CtrlStaticWZ.obj
 0001:0002fc8e       ?Message_MouseLButtonUp@CCtrlImageStaticWZ@@MAE_NPAUSI_MESSAGE@@@Z 10030c8e f   CtrlStaticWZ.obj
 0001:0002fca4       ?Message_MouseMove@CCtrlImageStaticWZ@@MAE_NPAUSI_MESSAGE@@@Z 10030ca4 f   CtrlStaticWZ.obj
 0001:0002fcba       ?IsTextReducing@CCtrlStaticWZ@@UBE_NXZ 10030cba f i CtrlStaticWZ.obj
 0001:0002fccc       ?SetTextReducing@CCtrlStaticWZ@@UAEX_N@Z 10030ccc f i CtrlStaticWZ.obj
 0001:0002fce3       ?IsMoneyType@CCtrlStaticWZ@@UBE_NXZ 10030ce3 f i CtrlStaticWZ.obj
 0001:0002fcf5       ?SetMoneyType@CCtrlStaticWZ@@UAEX_N@Z 10030cf5 f i CtrlStaticWZ.obj
 0001:0002fd0c       ??_ECCtrlStaticWZ@@UAEPAXI@Z 10030d0c f i CtrlStaticWZ.obj
 0001:0002fd0c       ??_GCCtrlStaticWZ@@UAEPAXI@Z 10030d0c f i CtrlStaticWZ.obj
 0001:0002fd33       ?IsUseDefault@CCtrlImageStaticWZ@@UBE_NXZ 10030d33 f i CtrlStaticWZ.obj
 0001:0002fd45       ?SetUseDefault@CCtrlImageStaticWZ@@UAEX_N@Z 10030d45 f i CtrlStaticWZ.obj
 0001:0002fd5c       ??_ECCtrlImageStaticWZ@@UAEPAXI@Z 10030d5c f i CtrlStaticWZ.obj
 0001:0002fd5c       ??_GCCtrlImageStaticWZ@@UAEPAXI@Z 10030d5c f i CtrlStaticWZ.obj
 0001:0002fd83       ??0CCtrlTabWZ@@QAE@XZ      10030d83 f   CtrlTabWZ.obj
 0001:0002fe6b       ??1CCtrlTabWZ@@UAE@XZ      10030e6b f   CtrlTabWZ.obj
 0001:0002fee5       ?OnCreate@CCtrlTabWZ@@UAE_NKKPAUHWND__@@PAUHINSTANCE__@@PAUtagRECT@@PAX@Z 10030ee5 f   CtrlTabWZ.obj
 0001:0002ff25       ?MoveWindowWZ@CCtrlTabWZ@@UAE_NMMMM@Z 10030f25 f   CtrlTabWZ.obj
 0001:000300d1       ?OnLoad@CCtrlTabWZ@@UAEXPAX@Z 100310d1 f   CtrlTabWZ.obj
 0001:0003036f       ?OnSave@CCtrlTabWZ@@UAEXPAX@Z 1003136f f   CtrlTabWZ.obj
 0001:00030518       ?OnInitialize@CCtrlTabWZ@@UAEXXZ 10031518 f   CtrlTabWZ.obj
 0001:00030529       ?OnDestroy@CCtrlTabWZ@@UAEXXZ 10031529 f   CtrlTabWZ.obj
 0001:0003060a       ?OnDraw@CCtrlTabWZ@@UAE_N_N@Z 1003160a f   CtrlTabWZ.obj
 0001:00030690       ?DrawTabPosLeft@CCtrlTabWZ@@IAEXXZ 10031690 f   CtrlTabWZ.obj
 0001:00030e19       ?DrawTabPosRight@CCtrlTabWZ@@IAEXXZ 10031e19 f   CtrlTabWZ.obj
 0001:000315e5       ?DrawTabPosTop@CCtrlTabWZ@@IAEXXZ 100325e5 f   CtrlTabWZ.obj
 0001:00031d47       ?DrawTabPosBottom@CCtrlTabWZ@@IAEXXZ 10032d47 f   CtrlTabWZ.obj
 0001:00032513       ?SetTabPosition@CCtrlTabWZ@@UAEXW4ENUM_TAB_POS@@@Z 10033513 f   CtrlTabWZ.obj
 0001:0003252a       ?ReleaseImage@CCtrlTabWZ@@UAEXXZ 1003352a f   CtrlTabWZ.obj
 0001:00032533       ?Message_MouseLButtonDown@CCtrlTabWZ@@MAE_NPAUSI_MESSAGE@@@Z 10033533 f   CtrlTabWZ.obj
 0001:0003278b       ?Message_MouseLButtonUp@CCtrlTabWZ@@MAE_NPAUSI_MESSAGE@@@Z 1003378b f   CtrlTabWZ.obj
 0001:0003288e       ?Message_MouseMove@CCtrlTabWZ@@MAE_NPAUSI_MESSAGE@@@Z 1003388e f   CtrlTabWZ.obj
 0001:000329a4       ?SetItemCount@CCtrlTabWZ@@UAE_NH@Z 100339a4 f   CtrlTabWZ.obj
 0001:00032b9d       ?SetItemButtonImageFormat@CCtrlTabWZ@@UAEXPAUSI_TFORMAT@@@Z 10033b9d f   CtrlTabWZ.obj
 0001:00032ba8       ?GetItemButtonImageFormat@CCtrlTabWZ@@UAEPAUSI_TFORMAT@@XZ 10033ba8 f   CtrlTabWZ.obj
 0001:00032bb3       ?SetCurSel@CCtrlTabWZ@@UAEXH@Z 10033bb3 f   CtrlTabWZ.obj
 0001:00032bda       ?SelectItemButton@CCtrlTabWZ@@IAEXH@Z 10033bda f   CtrlTabWZ.obj
 0001:00032e13       ?SetHeightRatio@CCtrlTabWZ@@UAEXF@Z 10033e13 f   CtrlTabWZ.obj
 0001:00032ee3       ?SetItemWidth@CCtrlTabWZ@@UAEXJ@Z 10033ee3 f   CtrlTabWZ.obj
 0001:00032f3d       ?GetItemUseIDCount@CCtrlTabWZ@@UAEHH@Z 10033f3d f   CtrlTabWZ.obj
 0001:00032ff6       ?GetItemUseIDIndex@CCtrlTabWZ@@UAEKHH@Z 10033ff6 f   CtrlTabWZ.obj
 0001:000330ae       ?AddItembelongID@CCtrlTabWZ@@UAEXHK@Z 100340ae f   CtrlTabWZ.obj
 0001:00033192       ?RemoveItembelongID@CCtrlTabWZ@@UAEXHK@Z 10034192 f   CtrlTabWZ.obj
 0001:00033261       ?RemoveItemUseIDAll@CCtrlTabWZ@@UAEXH@Z 10034261 f   CtrlTabWZ.obj
 0001:0003330e       ?SetItemButtonIsOutline@CCtrlTabWZ@@UAEX_N@Z 1003430e f   CtrlTabWZ.obj
 0001:00033325       ?GetItemButtonIsOutline@CCtrlTabWZ@@UAE_NXZ 10034325 f   CtrlTabWZ.obj
 0001:0003333b       ?SetItemButtonOutlineColor@CCtrlTabWZ@@UAEXK@Z 1003433b f   CtrlTabWZ.obj
 0001:00033352       ?GetItemButtonOutlineColor@CCtrlTabWZ@@UAEKXZ 10034352 f   CtrlTabWZ.obj
 0001:00033368       ?GetItemCount@CCtrlTabWZ@@UAEHXZ 10034368 f i CtrlTabWZ.obj
 0001:0003337b       ?GetCurSel@CCtrlTabWZ@@UAEHXZ 1003437b f i CtrlTabWZ.obj
 0001:0003338d       ?GetItemWidth@CCtrlTabWZ@@UAEJXZ 1003438d f i CtrlTabWZ.obj
 0001:0003339f       ?GetHeightRatio@CCtrlTabWZ@@UAEFXZ 1003439f f i CtrlTabWZ.obj
 0001:000333b2       ??_ECCtrlTabWZ@@UAEPAXI@Z  100343b2 f i CtrlTabWZ.obj
 0001:000333b2       ??_GCCtrlTabWZ@@UAEPAXI@Z  100343b2 f i CtrlTabWZ.obj
 0001:000333d9       ?IsData@STAB_INFO@@QAE_NK@Z 100343d9 f i CtrlTabWZ.obj
 0001:00033463       ?GetIndex@STAB_INFO@@QAEKH@Z 10034463 f i CtrlTabWZ.obj
 0001:000334f4       ??1STAB_INFO@@QAE@XZ       100344f4 f i CtrlTabWZ.obj
 0001:00033559       ??_GSTAB_INFO@@QAEPAXI@Z   10034559 f i CtrlTabWZ.obj
 0001:00033582       ??A?$map@KKU?$less@K@std@@V?$allocator@U?$pair@$$CBKK@std@@@2@@std@@QAEAAKABK@Z 10034582 f i CtrlTabWZ.obj
 0001:00033582       ??A?$map@KPAUCListSellData@CCtrlListWZ@@U?$less@K@std@@V?$allocator@U?$pair@$$CBKPAUCListSellData@CCtrlListWZ@@@std@@@4@@std@@QAEAAPAUCListSellData@CCtrlListWZ@@ABK@Z 10034582 f i CtrlListWZ.obj
 0001:00033582       ??A?$map@KPAXU?$less@K@std@@V?$allocator@U?$pair@$$CBKPAX@std@@@2@@std@@QAEAAPAXABK@Z 10034582 f i CtrlListWZ.obj
 0001:0003364e       ?clear@?$_Tree@V?$_Tmap_traits@KKU?$less@K@std@@V?$allocator@U?$pair@$$CBKK@std@@@2@$0A@@std@@@std@@QAEXXZ 1003464e f i CtrlTabWZ.obj
 0001:0003364e       ?clear@?$_Tree@V?$_Tmap_traits@KPAXU?$less@K@std@@V?$allocator@U?$pair@$$CBKPAX@std@@@2@$0A@@std@@@std@@QAEXXZ 1003464e f i CtrlListWZ.obj
 0001:0003364e       ?clear@?$_Tree@V?$_Tmap_traits@KPAUCListSellData@CCtrlListWZ@@U?$less@K@std@@V?$allocator@U?$pair@$$CBKPAUCListSellData@CCtrlListWZ@@@std@@@4@$0A@@std@@@std@@QAEXXZ 1003464e f i CtrlListWZ.obj
 0001:000336a3       ??0?$_Tree@V?$_Tmap_traits@KPAXU?$less@K@std@@V?$allocator@U?$pair@$$CBKPAX@std@@@2@$0A@@std@@@std@@QAE@ABU?$less@K@1@ABV?$allocator@U?$pair@$$CBKPAX@std@@@1@@Z 100346a3 f i CtrlListWZ.obj
 0001:000336a3       ??0?$_Tree@V?$_Tmap_traits@KPAUCListSellData@CCtrlListWZ@@U?$less@K@std@@V?$allocator@U?$pair@$$CBKPAUCListSellData@CCtrlListWZ@@@std@@@4@$0A@@std@@@std@@QAE@ABU?$less@K@1@ABV?$allocator@U?$pair@$$CBKPAUCListSellData@CCtrlListWZ@@@std@@@1@@Z 100346a3 f i CtrlListWZ.obj
 0001:000336a3       ??0?$_Tree@V?$_Tmap_traits@KKU?$less@K@std@@V?$allocator@U?$pair@$$CBKK@std@@@2@$0A@@std@@@std@@QAE@ABU?$less@K@1@ABV?$allocator@U?$pair@$$CBKK@std@@@1@@Z 100346a3 f i CtrlTabWZ.obj
 0001:00033704       ?insert@?$_Tree@V?$_Tmap_traits@KPAUCListSellData@CCtrlListWZ@@U?$less@K@std@@V?$allocator@U?$pair@$$CBKPAUCListSellData@CCtrlListWZ@@@std@@@4@$0A@@std@@@std@@QAE?AViterator@12@Vconst_iterator@12@ABU?$pair@$$CBKPAUCListSellData@CCtrlListWZ@@@2@@Z 10034704 f i CtrlListWZ.obj
 0001:00033704       ?insert@?$_Tree@V?$_Tmap_traits@KPAXU?$less@K@std@@V?$allocator@U?$pair@$$CBKPAX@std@@@2@$0A@@std@@@std@@QAE?AViterator@12@Vconst_iterator@12@ABU?$pair@$$CBKPAX@2@@Z 10034704 f i CtrlListWZ.obj
 0001:00033704       ?insert@?$_Tree@V?$_Tmap_traits@KKU?$less@K@std@@V?$allocator@U?$pair@$$CBKK@std@@@2@$0A@@std@@@std@@QAE?AViterator@12@Vconst_iterator@12@ABU?$pair@$$CBKK@2@@Z 10034704 f i CtrlTabWZ.obj
 0001:00033df7       ?_Erase@?$_Tree@V?$_Tmap_traits@KKU?$less@K@std@@V?$allocator@U?$pair@$$CBKK@std@@@2@$0A@@std@@@std@@IAEXPAU_Node@?$_Tree_nod@V?$_Tmap_traits@KKU?$less@K@std@@V?$allocator@U?$pair@$$CBKK@std@@@2@$0A@@std@@@2@@Z 10034df7 f i CtrlTabWZ.obj
 0001:00033df7       ?_Erase@?$_Tree@V?$_Tmap_traits@KPAUCListSellData@CCtrlListWZ@@U?$less@K@std@@V?$allocator@U?$pair@$$CBKPAUCListSellData@CCtrlListWZ@@@std@@@4@$0A@@std@@@std@@IAEXPAU_Node@?$_Tree_nod@V?$_Tmap_traits@KPAUCListSellData@CCtrlListWZ@@U?$less@K@std@@V?$allocator@U?$pair@$$CBKPAUCListSellData@CCtrlListWZ@@@std@@@4@$0A@@std@@@2@@Z 10034df7 f i CtrlListWZ.obj
 0001:00033df7       ?_Erase@?$_Tree@V?$_Tmap_traits@KPAXU?$less@K@std@@V?$allocator@U?$pair@$$CBKPAX@std@@@2@$0A@@std@@@std@@IAEXPAU_Node@?$_Tree_nod@V?$_Tmap_traits@KPAXU?$less@K@std@@V?$allocator@U?$pair@$$CBKPAX@std@@@2@$0A@@std@@@2@@Z 10034df7 f i CtrlListWZ.obj
 0001:00033e3d       ?insert@?$_Tree@V?$_Tmap_traits@KPAUCListSellData@CCtrlListWZ@@U?$less@K@std@@V?$allocator@U?$pair@$$CBKPAUCListSellData@CCtrlListWZ@@@std@@@4@$0A@@std@@@std@@QAE?AU?$pair@Viterator@?$_Tree@V?$_Tmap_traits@KPAUCListSellData@CCtrlListWZ@@U?$less@K@std@@V?$allocator@U?$pair@$$CBKPAUCListSellData@CCtrlListWZ@@@std@@@4@$0A@@std@@@std@@_N@2@ABU?$pair@$$CBKPAUCListSellData@CCtrlListWZ@@@2@@Z 10034e3d f i CtrlListWZ.obj
 0001:00033e3d       ?insert@?$_Tree@V?$_Tmap_traits@KKU?$less@K@std@@V?$allocator@U?$pair@$$CBKK@std@@@2@$0A@@std@@@std@@QAE?AU?$pair@Viterator@?$_Tree@V?$_Tmap_traits@KKU?$less@K@std@@V?$allocator@U?$pair@$$CBKK@std@@@2@$0A@@std@@@std@@_N@2@ABU?$pair@$$CBKK@2@@Z 10034e3d f i CtrlTabWZ.obj
 0001:00033e3d       ?insert@?$_Tree@V?$_Tmap_traits@KPAXU?$less@K@std@@V?$allocator@U?$pair@$$CBKPAX@std@@@2@$0A@@std@@@std@@QAE?AU?$pair@Viterator@?$_Tree@V?$_Tmap_traits@KPAXU?$less@K@std@@V?$allocator@U?$pair@$$CBKPAX@std@@@2@$0A@@std@@@std@@_N@2@ABU?$pair@$$CBKPAX@2@@Z 10034e3d f i CtrlListWZ.obj
 0001:0003400b       ?_Init@?$_Tree@V?$_Tmap_traits@KKU?$less@K@std@@V?$allocator@U?$pair@$$CBKK@std@@@2@$0A@@std@@@std@@IAEXXZ 1003500b f i CtrlTabWZ.obj
 0001:0003400b       ?_Init@?$_Tree@V?$_Tmap_traits@KPAUCListSellData@CCtrlListWZ@@U?$less@K@std@@V?$allocator@U?$pair@$$CBKPAUCListSellData@CCtrlListWZ@@@std@@@4@$0A@@std@@@std@@IAEXXZ 1003500b f i CtrlListWZ.obj
 0001:0003400b       ?_Init@?$_Tree@V?$_Tmap_traits@KPAXU?$less@K@std@@V?$allocator@U?$pair@$$CBKPAX@std@@@2@$0A@@std@@@std@@IAEXXZ 1003500b f i CtrlListWZ.obj
 0001:00034066       ?_Insert@?$_Tree@V?$_Tmap_traits@KPAXU?$less@K@std@@V?$allocator@U?$pair@$$CBKPAX@std@@@2@$0A@@std@@@std@@IAE?AViterator@12@_NPAU_Node@?$_Tree_nod@V?$_Tmap_traits@KPAXU?$less@K@std@@V?$allocator@U?$pair@$$CBKPAX@std@@@2@$0A@@std@@@2@ABU?$pair@$$CBKPAX@2@@Z 10035066 f i CtrlListWZ.obj
 0001:00034066       ?_Insert@?$_Tree@V?$_Tmap_traits@KPAUCListSellData@CCtrlListWZ@@U?$less@K@std@@V?$allocator@U?$pair@$$CBKPAUCListSellData@CCtrlListWZ@@@std@@@4@$0A@@std@@@std@@IAE?AViterator@12@_NPAU_Node@?$_Tree_nod@V?$_Tmap_traits@KPAUCListSellData@CCtrlListWZ@@U?$less@K@std@@V?$allocator@U?$pair@$$CBKPAUCListSellData@CCtrlListWZ@@@std@@@4@$0A@@std@@@2@ABU?$pair@$$CBKPAUCListSellData@CCtrlListWZ@@@2@@Z 10035066 f i CtrlListWZ.obj
 0001:00034066       ?_Insert@?$_Tree@V?$_Tmap_traits@KKU?$less@K@std@@V?$allocator@U?$pair@$$CBKK@std@@@2@$0A@@std@@@std@@IAE?AViterator@12@_NPAU_Node@?$_Tree_nod@V?$_Tmap_traits@KKU?$less@K@std@@V?$allocator@U?$pair@$$CBKK@std@@@2@$0A@@std@@@2@ABU?$pair@$$CBKK@2@@Z 10035066 f i CtrlTabWZ.obj
 0001:00034421       ?_Lrotate@?$_Tree@V?$_Tmap_traits@KKU?$less@K@std@@V?$allocator@U?$pair@$$CBKK@std@@@2@$0A@@std@@@std@@IAEXPAU_Node@?$_Tree_nod@V?$_Tmap_traits@KKU?$less@K@std@@V?$allocator@U?$pair@$$CBKK@std@@@2@$0A@@std@@@2@@Z 10035421 f i CtrlTabWZ.obj
 0001:00034421       ?_Lrotate@?$_Tree@V?$_Tmap_traits@KPAUCListSellData@CCtrlListWZ@@U?$less@K@std@@V?$allocator@U?$pair@$$CBKPAUCListSellData@CCtrlListWZ@@@std@@@4@$0A@@std@@@std@@IAEXPAU_Node@?$_Tree_nod@V?$_Tmap_traits@KPAUCListSellData@CCtrlListWZ@@U?$less@K@std@@V?$allocator@U?$pair@$$CBKPAUCListSellData@CCtrlListWZ@@@std@@@4@$0A@@std@@@2@@Z 10035421 f i CtrlListWZ.obj
 0001:00034421       ?_Lrotate@?$_Tree@V?$_Tmap_traits@KPAXU?$less@K@std@@V?$allocator@U?$pair@$$CBKPAX@std@@@2@$0A@@std@@@std@@IAEXPAU_Node@?$_Tree_nod@V?$_Tmap_traits@KPAXU?$less@K@std@@V?$allocator@U?$pair@$$CBKPAX@std@@@2@$0A@@std@@@2@@Z 10035421 f i CtrlListWZ.obj
 0001:000344c5       ?_Buynode@?$_Tree@V?$_Tmap_traits@KPAUCListSellData@CCtrlListWZ@@U?$less@K@std@@V?$allocator@U?$pair@$$CBKPAUCListSellData@CCtrlListWZ@@@std@@@4@$0A@@std@@@std@@IAEPAU_Node@?$_Tree_nod@V?$_Tmap_traits@KPAUCListSellData@CCtrlListWZ@@U?$less@K@std@@V?$allocator@U?$pair@$$CBKPAUCListSellData@CCtrlListWZ@@@std@@@4@$0A@@std@@@2@XZ 100354c5 f i CtrlListWZ.obj
 0001:000344c5       ?_Buynode@?$_Tree@V?$_Tmap_traits@KKU?$less@K@std@@V?$allocator@U?$pair@$$CBKK@std@@@2@$0A@@std@@@std@@IAEPAU_Node@?$_Tree_nod@V?$_Tmap_traits@KKU?$less@K@std@@V?$allocator@U?$pair@$$CBKK@std@@@2@$0A@@std@@@2@XZ 100354c5 f i CtrlTabWZ.obj
 0001:000344c5       ?_Buynode@?$_Tree@V?$_Tmap_traits@KPAXU?$less@K@std@@V?$allocator@U?$pair@$$CBKPAX@std@@@2@$0A@@std@@@std@@IAEPAU_Node@?$_Tree_nod@V?$_Tmap_traits@KPAXU?$less@K@std@@V?$allocator@U?$pair@$$CBKPAX@std@@@2@$0A@@std@@@2@XZ 100354c5 f i CtrlListWZ.obj
 0001:000345df       ?_Buynode@?$_Tree@V?$_Tmap_traits@KPAXU?$less@K@std@@V?$allocator@U?$pair@$$CBKPAX@std@@@2@$0A@@std@@@std@@IAEPAU_Node@?$_Tree_nod@V?$_Tmap_traits@KPAXU?$less@K@std@@V?$allocator@U?$pair@$$CBKPAX@std@@@2@$0A@@std@@@2@PAU342@00ABU?$pair@$$CBKPAX@2@D@Z 100355df f i CtrlListWZ.obj
 0001:000345df       ?_Buynode@?$_Tree@V?$_Tmap_traits@KPAUCListSellData@CCtrlListWZ@@U?$less@K@std@@V?$allocator@U?$pair@$$CBKPAUCListSellData@CCtrlListWZ@@@std@@@4@$0A@@std@@@std@@IAEPAU_Node@?$_Tree_nod@V?$_Tmap_traits@KPAUCListSellData@CCtrlListWZ@@U?$less@K@std@@V?$allocator@U?$pair@$$CBKPAUCListSellData@CCtrlListWZ@@@std@@@4@$0A@@std@@@2@PAU342@00ABU?$pair@$$CBKPAUCListSellData@CCtrlListWZ@@@2@D@Z 100355df f i CtrlListWZ.obj
 0001:000345df       ?_Buynode@?$_Tree@V?$_Tmap_traits@KKU?$less@K@std@@V?$allocator@U?$pair@$$CBKK@std@@@2@$0A@@std@@@std@@IAEPAU_Node@?$_Tree_nod@V?$_Tmap_traits@KKU?$less@K@std@@V?$allocator@U?$pair@$$CBKK@std@@@2@$0A@@std@@@2@PAU342@00ABU?$pair@$$CBKK@2@D@Z 100355df f i CtrlTabWZ.obj
 0001:000346b0       ??0CCtrlVScrollWZ@@QAE@XZ  100356b0 f   CtrlVScrollWZ.obj
 0001:00034798       ??1CCtrlVScrollWZ@@UAE@XZ  10035798 f   CtrlVScrollWZ.obj
 0001:00034819       ?OnCreate@CCtrlVScrollWZ@@UAE_NKKPAUHWND__@@PAUHINSTANCE__@@PAUtagRECT@@PAX@Z 10035819 f   CtrlVScrollWZ.obj
 0001:0003491f       ?MoveWindowWZ@CCtrlVScrollWZ@@UAE_NMMMM@Z 1003591f f   CtrlVScrollWZ.obj
 0001:00034f70       ?OnLoad@CCtrlVScrollWZ@@UAEXPAX@Z 10035f70 f   CtrlVScrollWZ.obj
 0001:00035158       ?OnSave@CCtrlVScrollWZ@@UAEXPAX@Z 10036158 f   CtrlVScrollWZ.obj
 0001:000351ee       ?OnInitialize@CCtrlVScrollWZ@@UAEXXZ 100361ee f   CtrlVScrollWZ.obj
 0001:00035248       ?OnDestroy@CCtrlVScrollWZ@@UAEXXZ 10036248 f   CtrlVScrollWZ.obj
 0001:00035298       ?OnDraw@CCtrlVScrollWZ@@UAE_N_N@Z 10036298 f   CtrlVScrollWZ.obj
 0001:000353d0       ?EnableWindowWZ@CCtrlVScrollWZ@@UAEX_N@Z 100363d0 f   CtrlVScrollWZ.obj
 0001:0003542e       ?UpdateWindowWZ@CCtrlVScrollWZ@@UAEXPAUHWND__@@@Z 1003642e f   CtrlVScrollWZ.obj
 0001:0003548c       ?ReleaseImage@CCtrlVScrollWZ@@UAEXXZ 1003648c f   CtrlVScrollWZ.obj
 0001:000354dc       ?SetChangeSizeThumb@CCtrlVScrollWZ@@UAEXH@Z 100364dc f   CtrlVScrollWZ.obj
 0001:000355b2       ?SetScrollPosWZ@CCtrlVScrollWZ@@UAEHH@Z 100365b2 f   CtrlVScrollWZ.obj
 0001:000355d6       ?SetScrollPosWZ@CCtrlVScrollWZ@@UAEHM@Z 100365d6 f   CtrlVScrollWZ.obj
 0001:00035763       ?SetScrollRangeWZ@CCtrlVScrollWZ@@UAEXHH@Z 10036763 f   CtrlVScrollWZ.obj
 0001:00035792       ?SetScrollRangeWZ@CCtrlVScrollWZ@@UAEXMM@Z 10036792 f   CtrlVScrollWZ.obj
 0001:0003583e       ?GetScrollRangeWZ@CCtrlVScrollWZ@@UAEXPAH0@Z 1003683e f   CtrlVScrollWZ.obj
 0001:00035869       ?GetScrollRangeWZ@CCtrlVScrollWZ@@UAEXPAM0@Z 10036869 f   CtrlVScrollWZ.obj
 0001:00035890       ?Message_MouseLButtonDown@CCtrlVScrollWZ@@MAE_NPAUSI_MESSAGE@@@Z 10036890 f   CtrlVScrollWZ.obj
 0001:00035cb7       ?Message_MouseLButtonUp@CCtrlVScrollWZ@@MAE_NPAUSI_MESSAGE@@@Z 10036cb7 f   CtrlVScrollWZ.obj
 0001:00035e08       ?Message_MouseMove@CCtrlVScrollWZ@@MAE_NPAUSI_MESSAGE@@@Z 10036e08 f   CtrlVScrollWZ.obj
 0001:000361b3       ?SetArrowUPBTImageFormat@CCtrlVScrollWZ@@UAEXPAUSI_TFORMAT@@@Z 100371b3 f   CtrlVScrollWZ.obj
 0001:000361d6       ?SetArrowDownBTImageFormat@CCtrlVScrollWZ@@UAEXPAUSI_TFORMAT@@@Z 100371d6 f   CtrlVScrollWZ.obj
 0001:000361f9       ?SetArrowThumbBTImageFormat@CCtrlVScrollWZ@@UAEXPAUSI_TFORMAT@@@Z 100371f9 f   CtrlVScrollWZ.obj
 0001:0003621c       ?GetArrowUPBTImageFormat@CCtrlVScrollWZ@@UAEPAUSI_TFORMAT@@XZ 1003721c f   CtrlVScrollWZ.obj
 0001:0003623e       ?GetArrowDownBTImageFormat@CCtrlVScrollWZ@@UAEPAUSI_TFORMAT@@XZ 1003723e f   CtrlVScrollWZ.obj
 0001:00036260       ?GetArrowThumbBTImageFormat@CCtrlVScrollWZ@@UAEPAUSI_TFORMAT@@XZ 10037260 f   CtrlVScrollWZ.obj
 0001:00036282       ?SetArrowUPBTIsOutline@CCtrlVScrollWZ@@UAEX_N@Z 10037282 f   CtrlVScrollWZ.obj
 0001:000362a8       ?GetArrowUPBTIsOutline@CCtrlVScrollWZ@@UAE_NXZ 100372a8 f   CtrlVScrollWZ.obj
 0001:000362c9       ?SetArrowUPBTOutlineColor@CCtrlVScrollWZ@@UAEXK@Z 100372c9 f   CtrlVScrollWZ.obj
 0001:000362ef       ?GetArrowUPBTOutlineColor@CCtrlVScrollWZ@@UAEKXZ 100372ef f   CtrlVScrollWZ.obj
 0001:00036310       ?SetArrowDownBTIsOutline@CCtrlVScrollWZ@@UAEX_N@Z 10037310 f   CtrlVScrollWZ.obj
 0001:00036336       ?GetArrowDownBTIsOutline@CCtrlVScrollWZ@@UAE_NXZ 10037336 f   CtrlVScrollWZ.obj
 0001:00036357       ?SetArrowDownBTOutlineColor@CCtrlVScrollWZ@@UAEXK@Z 10037357 f   CtrlVScrollWZ.obj
 0001:0003637d       ?GetArrowDownBTOutlineColor@CCtrlVScrollWZ@@UAEKXZ 1003737d f   CtrlVScrollWZ.obj
 0001:0003639e       ?SetArrowThumbBTIsOutline@CCtrlVScrollWZ@@UAEX_N@Z 1003739e f   CtrlVScrollWZ.obj
 0001:000363c4       ?GetArrowThumbBTIsOutline@CCtrlVScrollWZ@@UAE_NXZ 100373c4 f   CtrlVScrollWZ.obj
 0001:000363e5       ?SetArrowThumbBTOutlineColor@CCtrlVScrollWZ@@UAEXK@Z 100373e5 f   CtrlVScrollWZ.obj
 0001:0003640b       ?GetArrowThumbBTOutlineColor@CCtrlVScrollWZ@@UAEKXZ 1003740b f   CtrlVScrollWZ.obj
 0001:0003642c       ?SetArrowUPSize@CCtrlVScrollWZ@@UAEXAAUtagRECT@@@Z 1003742c f   CtrlVScrollWZ.obj
 0001:00036483       ?SetArrowDownSize@CCtrlVScrollWZ@@UAEXAAUtagRECT@@@Z 10037483 f   CtrlVScrollWZ.obj
 0001:000364da       ?SetArrowThumbSize@CCtrlVScrollWZ@@UAEXAAUtagRECT@@@Z 100374da f   CtrlVScrollWZ.obj
 0001:00036531       ?GetArrowUPSize@CCtrlVScrollWZ@@UAE?AUtagRECT@@XZ 10037531 f   CtrlVScrollWZ.obj
 0001:00036557       ?GetArrowDownSize@CCtrlVScrollWZ@@UAE?AUtagRECT@@XZ 10037557 f   CtrlVScrollWZ.obj
 0001:0003657d       ?GetArrowThumbSize@CCtrlVScrollWZ@@UAE?AUtagRECT@@XZ 1003757d f   CtrlVScrollWZ.obj
 0001:000365a3       ?GetScrollPosWZ@CCtrlVScrollWZ@@UAEHXZ 100375a3 f i CtrlVScrollWZ.obj
 0001:000365a3       ?GetScrollPosWZ@CCtrlHScrollWZ@@UAEHXZ 100375a3 f i CtrlHScrollWZ.obj
 0001:000365b7       ??_ECCtrlVScrollWZ@@UAEPAXI@Z 100375b7 f i CtrlVScrollWZ.obj
 0001:000365b7       ??_GCCtrlVScrollWZ@@UAEPAXI@Z 100375b7 f i CtrlVScrollWZ.obj
 0001:000365de       ??0CCtrlWebBrowserWZ@@QAE@XZ 100375de f   CtrlWebBrowserWZ.obj
 0001:00036664       ??1CCtrlWebBrowserWZ@@UAE@XZ 10037664 f   CtrlWebBrowserWZ.obj
 0001:0003667e       ?StaticShowState@CCtrlWebBrowserWZ@@SAXW4ENUM_STATEWZ@@@Z 1003767e f   CtrlWebBrowserWZ.obj
 0001:000366b6       ?StaticCreateWebCtrl@CCtrlWebBrowserWZ@@SAXXZ 100376b6 f   CtrlWebBrowserWZ.obj
 0001:000366ed       ?StaticDestroyWebCtrl@CCtrlWebBrowserWZ@@SAXXZ 100376ed f   CtrlWebBrowserWZ.obj
 0001:00036725       ?StaticMoveWebCtrl@CCtrlWebBrowserWZ@@SAXJJ@Z 10037725 f   CtrlWebBrowserWZ.obj
 0001:000367c4       ?OnCreate@CCtrlWebBrowserWZ@@UAE_NKKPAUHWND__@@PAUHINSTANCE__@@PAUtagRECT@@PAX@Z 100377c4 f   CtrlWebBrowserWZ.obj
 0001:000368eb       ?OnDestroy@CCtrlWebBrowserWZ@@UAEXXZ 100378eb f   CtrlWebBrowserWZ.obj
 0001:00036910       ?OnLoad@CCtrlWebBrowserWZ@@UAEXPAX@Z 10037910 f   CtrlWebBrowserWZ.obj
 0001:00036999       ?MoveWindowWZ@CCtrlWebBrowserWZ@@UAE_NMMMM@Z 10037999 f   CtrlWebBrowserWZ.obj
 0001:00036b4b       ?ShowWindowWZ@CCtrlWebBrowserWZ@@UAEXW4ENUM_STATEWZ@@@Z 10037b4b f   CtrlWebBrowserWZ.obj
 0001:00036b89       ?OnDoAction@CCtrlWebBrowserWZ@@UAEXXZ 10037b89 f   CtrlWebBrowserWZ.obj
 0001:00036d98       ?OnDraw@CCtrlWebBrowserWZ@@UAE_N_N@Z 10037d98 f   CtrlWebBrowserWZ.obj
 0001:00036da5       ?GoHome@CCtrlWebBrowserWZ@@UAEXXZ 10037da5 f   CtrlWebBrowserWZ.obj
 0001:00036dc3       ?Navigate@CCtrlWebBrowserWZ@@UAEXPB_W@Z 10037dc3 f   CtrlWebBrowserWZ.obj
 0001:00036ed6       ?Refresh@CCtrlWebBrowserWZ@@UAEXXZ 10037ed6 f   CtrlWebBrowserWZ.obj
 0001:00036ef4       ?Stop@CCtrlWebBrowserWZ@@UAEXXZ 10037ef4 f   CtrlWebBrowserWZ.obj
 0001:00036f12       ?GoBack@CCtrlWebBrowserWZ@@UAEXXZ 10037f12 f   CtrlWebBrowserWZ.obj
 0001:00036f30       ?GoForward@CCtrlWebBrowserWZ@@UAEXXZ 10037f30 f   CtrlWebBrowserWZ.obj
 0001:00036f4e       ??_GCCtrlWebBrowserWZ@@UAEPAXI@Z 10037f4e f i CtrlWebBrowserWZ.obj
 0001:00036f4e       ??_ECCtrlWebBrowserWZ@@UAEPAXI@Z 10037f4e f i CtrlWebBrowserWZ.obj
 0001:00036f75       ?GoHome@IWithWebDialog@@QAEJXZ 10037f75 f i CtrlWebBrowserWZ.obj
 0001:00036fa6       ??0_bstr_t@@QAE@PB_W@Z     10037fa6 f i CtrlWebBrowserWZ.obj
 0001:0003702d       ??1_bstr_t@@QAE@XZ         1003802d f i CtrlWebBrowserWZ.obj
 0001:00037050       ??0Data_t@_bstr_t@@QAE@PB_W@Z 10038050 f i CtrlWebBrowserWZ.obj
 0001:00037095       ?Release@Data_t@_bstr_t@@QAEKXZ 10038095 f i CtrlWebBrowserWZ.obj
 0001:000370f0       ?_Free@Data_t@_bstr_t@@AAEXXZ 100380f0 f i CtrlWebBrowserWZ.obj
 0001:00037128       ??0CComBSTR@ATL@@QAE@PB_W@Z 10038128 f i CtrlWebBrowserWZ.obj
 0001:0003716e       ?AtlThrowImpl@ATL@@YGXJ@Z  1003816e f i CtrlWebBrowserWZ.obj
 0001:00037191       ??1CComBSTR@ATL@@QAE@XZ    10038191 f i CtrlWebBrowserWZ.obj
 0001:000371a5       ??1CComVariant@ATL@@QAE@XZ 100381a5 f i CtrlWebBrowserWZ.obj
 0001:000371b7       ?Refresh@IWithWebDialog@@QAEJXZ 100381b7 f i CtrlWebBrowserWZ.obj
 0001:000371e8       ?Stop@IWithWebDialog@@QAEJXZ 100381e8 f i CtrlWebBrowserWZ.obj
 0001:00037219       ?GoBack@IWithWebDialog@@QAEJXZ 10038219 f i CtrlWebBrowserWZ.obj
 0001:0003724a       ?GoForward@IWithWebDialog@@QAEJXZ 1003824a f i CtrlWebBrowserWZ.obj
 0001:0003727b       ??0CDialogWZ@@QAE@XZ       1003827b f   DialogWZ.obj
 0001:00037437       ??1CDialogWZ@@UAE@XZ       10038437 f   DialogWZ.obj
 0001:00037509       ?OnCreate@CDialogWZ@@UAE_NKKPAUHWND__@@PAUHINSTANCE__@@PAXPAVCDialogManager@@@Z 10038509 f   DialogWZ.obj
 0001:000375f4       ?CreateControllWZ@CDialogWZ@@QAEPAVCControlWZ@@KKKPAUHWND__@@PAUHINSTANCE__@@PAUtagRECT@@PAX@Z 100385f4 f   DialogWZ.obj
 0001:00037ddb       ?OnDestroy@CDialogWZ@@QAEXXZ 10038ddb f   DialogWZ.obj
 0001:00037ef1       ?OnRelease@CDialogWZ@@QAEXXZ 10038ef1 f   DialogWZ.obj
 0001:00037f13       ?ShowWindowWZ@CDialogWZ@@UAEXW4ENUM_STATEWZ@@@Z 10038f13 f   DialogWZ.obj
 0001:000382eb       ?OnInitialize@CDialogWZ@@UAEXXZ 100392eb f   DialogWZ.obj
 0001:00038347       ?OnLoad@CDialogWZ@@UAEXPAX@Z 10039347 f   DialogWZ.obj
 0001:000385ef       ?OnSave@CDialogWZ@@UAEXPAX@Z 100395ef f   DialogWZ.obj
 0001:000387f1       ?RequestFocus@CDialogWZ@@UAEXPAVCControlWZ@@@Z 100397f1 f   DialogWZ.obj
 0001:00038916       ?SetStyle@CDialogWZ@@UAEXK@Z 10039916 f   DialogWZ.obj
 0001:0003893c       ?ReleaseImage@CDialogWZ@@UAEXXZ 1003993c f   DialogWZ.obj
 0001:000389a1       ?UpdateWindowWZ@CDialogWZ@@UAEXPAUHWND__@@@Z 100399a1 f   DialogWZ.obj
 0001:00038a17       ?SetDlgID@CDialogWZ@@UAE_NK@Z 10039a17 f   DialogWZ.obj
 0001:00038a7f       ?GetControlCount@CDialogWZ@@UAEKXZ 10039a7f f   DialogWZ.obj
 0001:00038a93       ?GetControlWZ@CDialogWZ@@UAEPAVCControlWZ@@K@Z 10039a93 f   DialogWZ.obj
 0001:00038abd       ?OnDoAction@CDialogWZ@@UAEXXZ 10039abd f   DialogWZ.obj
 0001:00038be0       ?SetDepth@CDialogWZ@@UAEXM@Z 10039be0 f   DialogWZ.obj
 0001:00038c4d       ?OnDraw@CDialogWZ@@UAEX_N@Z 10039c4d f   DialogWZ.obj
 0001:00039045       ?OnDrawControlWZ@CDialogWZ@@UAE_NK@Z 1003a045 f   DialogWZ.obj
 0001:000390ea       ?RemoveControlWZ@CDialogWZ@@QAE_NK@Z 1003a0ea f   DialogWZ.obj
 0001:0003918c       ?MoveToListIndex@CDialogWZ@@UAEXHH@Z 1003a18c f   DialogWZ.obj
 0001:000391a8       ?SetDialogImageFormat@CDialogWZ@@UAEXPAUSI_TFORMAT@@@Z 1003a1a8 f   DialogWZ.obj
 0001:000391cd       ?SetDialogPartFormat@CDialogWZ@@UAEXPAUSI_TFORMAT@@K@Z 1003a1cd f   DialogWZ.obj
 0001:000391f0       ?GetDialogImageFormat@CDialogWZ@@UAEPAUSI_TFORMAT@@K@Z 1003a1f0 f   DialogWZ.obj
 0001:00039214       ?SetTransparency@CDialogWZ@@UAEXM@Z 1003a214 f   DialogWZ.obj
 0001:0003922f       ?SetControlImageFormat@CDialogWZ@@UAEXKPAUSI_TFORMAT@@@Z 1003a22f f   DialogWZ.obj
 0001:00039260       ?MoveWindowWZ@CDialogWZ@@UAE_NMM@Z 1003a260 f   DialogWZ.obj
 0001:000392d2       ?MoveWindowWZ@CDialogWZ@@UAE_NKMMMM@Z 1003a2d2 f   DialogWZ.obj
 0001:00039322       ?MoveWindowWZ@CDialogWZ@@UAE_NMMMM@Z 1003a322 f   DialogWZ.obj
 0001:0003944d       ?GetDlgPartSizeRect@CDialogWZ@@UAEXPAUtagRECT@@K@Z 1003a44d f   DialogWZ.obj
 0001:00039481       ?SetDlgPartSizeRect@CDialogWZ@@UAEXUtagRECT@@K@Z 1003a481 f   DialogWZ.obj
 0001:000394d3       ?InterSectRect@CDialogWZ@@UAE_NUtagPOINT@@@Z 1003a4d3 f   DialogWZ.obj
 0001:0003964b       ?GetDlgSize@CDialogWZ@@UAEXPAUtagRECT@@@Z 1003a64b f   DialogWZ.obj
 0001:000396ab       ?GetClientRect@CDialogWZ@@UAEXPAUtagRECT@@@Z 1003a6ab f   DialogWZ.obj
 0001:000396d8       ?GetCtrlSize@CDialogWZ@@UAEXKPAUtagRECT@@@Z 1003a6d8 f   DialogWZ.obj
 0001:00039718       ?OnFocusIn@CDialogWZ@@UAEXXZ 1003a718 f   DialogWZ.obj
 0001:0003972b       ?OnFocusOut@CDialogWZ@@UAEXXZ 1003a72b f   DialogWZ.obj
 0001:00039791       ?FindControlWZ@CDialogWZ@@UAEPAVCControlWZ@@H@Z 1003a791 f   DialogWZ.obj
 0001:000397aa       ?SendMessageWZ@CDialogWZ@@QAE_NPAUSI_MESSAGE@@@Z 1003a7aa f   DialogWZ.obj
 0001:0003a146       ?SetTextReducing@CDialogWZ@@UAEX_N@Z 1003b146 f   DialogWZ.obj
 0001:0003a1af       ?SetTextReducing@CDialogWZ@@UAEXK_N@Z 1003b1af f   DialogWZ.obj
 0001:0003a1ee       ?OnKeyDown@CDialogWZ@@QAE_NPAUSI_MESSAGE@@@Z 1003b1ee f   DialogWZ.obj
 0001:0003a378       ?SetScale@CDialogWZ@@UAEXMM@Z 1003b378 f   DialogWZ.obj
 0001:0003a594       ?HaveFocus@CDialogWZ@@UAE_NXZ 1003b594 f i DialogWZ.obj
 0001:0003a5a6       ?GetDlgID@CDialogWZ@@UAEKXZ 1003b5a6 f i DialogWZ.obj
 0001:0003a5b5       ?GetClientWZ@CDialogWZ@@UAEPAVCControlWZ@@XZ 1003b5b5 f i DialogWZ.obj
 0001:0003a5c4       ?SetMoveRECT@CDialogWZ@@UAEXUtagRECT@@@Z 1003b5c4 f i DialogWZ.obj
 0001:0003a5ff       ?GetMoveRECT@CDialogWZ@@UAE?AUtagRECT@@XZ 1003b5ff f i DialogWZ.obj
 0001:0003a621       ?SetIsOutline@CDialogWZ@@UAEX_N@Z 1003b621 f i DialogWZ.obj
 0001:0003a641       ?GetIsOutline@CDialogWZ@@UAE_NXZ 1003b641 f i DialogWZ.obj
 0001:0003a65c       ?SetOutlineColor@CDialogWZ@@UAEXK@Z 1003b65c f i DialogWZ.obj
 0001:0003a67c       ?GetOutlineColor@CDialogWZ@@UAEKXZ 1003b67c f i DialogWZ.obj
 0001:0003a697       ??_GCDialogWZ@@UAEPAXI@Z   1003b697 f i DialogWZ.obj
 0001:0003a697       ??_ECDialogWZ@@UAEPAXI@Z   1003b697 f i DialogWZ.obj
 0001:0003a6be       ??0?$list@UtagRECT@@V?$allocator@UtagRECT@@@std@@@std@@QAE@XZ 1003b6be f i DialogWZ.obj
 0001:0003a733       ?begin@?$list@KV?$allocator@K@std@@@std@@QAE?AV?$_Iterator@$00@12@XZ 1003b733 f i BaseManager.obj
 0001:0003a733       ?begin@?$list@UtagRECT@@V?$allocator@UtagRECT@@@std@@@std@@QAE?AV?$_Iterator@$00@12@XZ 1003b733 f i DialogWZ.obj
 0001:0003a733       ?begin@?$list@U?$pair@$$CBKV?$basic_string@DU?$char_traits@D@std@@V?$allocator@D@2@@std@@@std@@V?$allocator@U?$pair@$$CBKV?$basic_string@DU?$char_traits@D@std@@V?$allocator@D@2@@std@@@std@@@2@@std@@QAE?AV?$_Iterator@$00@12@XZ 1003b733 f i StringManager.obj
 0001:0003a733       ?begin@?$list@PAXV?$allocator@PAX@std@@@std@@QAE?AV?$_Iterator@$00@12@XZ 1003b733 f i CtrlListWZ.obj
 0001:0003a733       ?begin@?$list@PAVCControlWZ@@V?$allocator@PAVCControlWZ@@@std@@@std@@QAE?AV?$_Iterator@$00@12@XZ 1003b733 f i CtrlDxEdit.obj
 0001:0003a781       ?push_back@?$list@UtagRECT@@V?$allocator@UtagRECT@@@std@@@std@@QAEXABUtagRECT@@@Z 1003b781 f i DialogWZ.obj
 0001:0003a7da       ?front@?$list@PAVCControlWZ@@V?$allocator@PAVCControlWZ@@@std@@@std@@QAEAAPAVCControlWZ@@XZ 1003b7da f i DialogWZ.obj
 0001:0003a824       ?_Insert@?$list@UtagRECT@@V?$allocator@UtagRECT@@@std@@@std@@QAEXV?$_Const_iterator@$00@12@ABUtagRECT@@@Z 1003b824 f i DialogWZ.obj
 0001:0003a872       ?_Buynode@?$list@UtagRECT@@V?$allocator@UtagRECT@@@std@@@std@@IAEPAU_Node@?$_List_nod@UtagRECT@@V?$allocator@UtagRECT@@@std@@@2@XZ 1003b872 f i DialogWZ.obj
 0001:0003a954       ?_Buynode@?$list@UtagRECT@@V?$allocator@UtagRECT@@@std@@@std@@IAEPAU_Node@?$_List_nod@UtagRECT@@V?$allocator@UtagRECT@@@std@@@2@PAU342@0ABUtagRECT@@@Z 1003b954 f i DialogWZ.obj
 0001:0003aa58       ?_Incsize@?$list@UtagRECT@@V?$allocator@UtagRECT@@@std@@@std@@IAEXI@Z 1003ba58 f i DialogWZ.obj
 0001:0003ab22       ??$_Allocate@U_Node@?$_Tree_nod@V?$_Tmap_traits@KPAUCListSellData@CCtrlListWZ@@U?$less@K@std@@V?$allocator@U?$pair@$$CBKPAUCListSellData@CCtrlListWZ@@@std@@@4@$0A@@std@@@std@@@std@@YAPAU_Node@?$_Tree_nod@V?$_Tmap_traits@KPAUCListSellData@CCtrlListWZ@@U?$less@K@std@@V?$allocator@U?$pair@$$CBKPAUCListSellData@CCtrlListWZ@@@std@@@4@$0A@@std@@@0@IPAU120@@Z 1003bb22 f i CtrlListWZ.obj
 0001:0003ab22       ??$_Allocate@U_Node@?$_List_nod@UtagRECT@@V?$allocator@UtagRECT@@@std@@@std@@@std@@YAPAU_Node@?$_List_nod@UtagRECT@@V?$allocator@UtagRECT@@@std@@@0@IPAU120@@Z 1003bb22 f i DialogWZ.obj
 0001:0003ab22       ??$_Allocate@U_Node@?$_Tree_nod@V?$_Tmap_traits@KKU?$less@K@std@@V?$allocator@U?$pair@$$CBKK@std@@@2@$0A@@std@@@std@@@std@@YAPAU_Node@?$_Tree_nod@V?$_Tmap_traits@KKU?$less@K@std@@V?$allocator@U?$pair@$$CBKK@std@@@2@$0A@@std@@@0@IPAU120@@Z 1003bb22 f i CtrlTabWZ.obj
 0001:0003ab22       ??$_Allocate@U_Node@?$_Tree_nod@V?$_Tmap_traits@KPAXU?$less@K@std@@V?$allocator@U?$pair@$$CBKPAX@std@@@2@$0A@@std@@@std@@@std@@YAPAU_Node@?$_Tree_nod@V?$_Tmap_traits@KPAXU?$less@K@std@@V?$allocator@U?$pair@$$CBKPAX@std@@@2@$0A@@std@@@0@IPAU120@@Z 1003bb22 f i CtrlListWZ.obj
 0001:0003ab75       ??0?$list@PAXV?$allocator@PAX@std@@@std@@QAE@XZ 1003bb75 f i CtrlListWZ.obj
 0001:0003ab75       ??0?$list@KV?$allocator@K@std@@@std@@QAE@XZ 1003bb75 f i BaseManager.obj
 0001:0003ab75       ??0?$list@PAVCControlWZ@@V?$allocator@PAVCControlWZ@@@std@@@std@@QAE@XZ 1003bb75 f i DialogWZ.obj
 0001:0003abea       ?_Buynode@?$list@PAXV?$allocator@PAX@std@@@std@@IAEPAU_Node@?$_List_nod@PAXV?$allocator@PAX@std@@@2@XZ 1003bbea f i CtrlListWZ.obj
 0001:0003abea       ?_Buynode@?$list@KV?$allocator@K@std@@@std@@IAEPAU_Node@?$_List_nod@KV?$allocator@K@std@@@2@XZ 1003bbea f i BaseManager.obj
 0001:0003abea       ?_Buynode@?$list@PAVCControlWZ@@V?$allocator@PAVCControlWZ@@@std@@@std@@IAEPAU_Node@?$_List_nod@PAVCControlWZ@@V?$allocator@PAVCControlWZ@@@std@@@2@XZ 1003bbea f i DialogWZ.obj
 0001:0003accc       ??0?$_List_ptr@KV?$allocator@K@std@@@std@@IAE@V?$allocator@K@1@@Z 1003bccc f i BaseManager.obj
 0001:0003accc       ??0?$_List_ptr@PAXV?$allocator@PAX@std@@@std@@IAE@V?$allocator@PAX@1@@Z 1003bccc f i CtrlListWZ.obj
 0001:0003accc       ??0?$_List_ptr@PAVCControlWZ@@V?$allocator@PAVCControlWZ@@@std@@@std@@IAE@V?$allocator@PAVCControlWZ@@@1@@Z 1003bccc f i DialogWZ.obj
 0001:0003accc       ??0?$_List_ptr@U?$pair@$$CBKPAX@std@@V?$allocator@U?$pair@$$CBKPAX@std@@@2@@std@@IAE@V?$allocator@U?$pair@$$CBKPAX@std@@@1@@Z 1003bccc f i BaseManager.obj
 0001:0003accc       ??0?$_List_ptr@UtagRECT@@V?$allocator@UtagRECT@@@std@@@std@@IAE@V?$allocator@UtagRECT@@@1@@Z 1003bccc f i DialogWZ.obj
 0001:0003accc       ??0?$_List_ptr@U?$pair@$$CBKV?$basic_string@DU?$char_traits@D@std@@V?$allocator@D@2@@std@@@std@@V?$allocator@U?$pair@$$CBKV?$basic_string@DU?$char_traits@D@std@@V?$allocator@D@2@@std@@@std@@@2@@std@@IAE@V?$allocator@U?$pair@$$CBKV?$basic_string@DU?$char_traits@D@std@@V?$allocator@D@2@@std@@@std@@@1@@Z 1003bccc f i StringManager.obj
 0001:0003acfc       ??0?$_Container_base_aux_alloc_real@V?$allocator@U?$pair@$$CBV?$basic_string@DU?$char_traits@D@std@@V?$allocator@D@2@@std@@PAX@std@@@std@@@std@@IAE@V?$allocator@U?$pair@$$CBV?$basic_string@DU?$char_traits@D@std@@V?$allocator@D@2@@std@@PAX@std@@@1@@Z 1003bcfc f i CtrlListWZ.obj
 0001:0003acfc       ??0?$_Container_base_aux_alloc_real@V?$allocator@U?$pair@$$CBKK@std@@@std@@@std@@IAE@V?$allocator@U?$pair@$$CBKK@std@@@1@@Z 1003bcfc f i CtrlTabWZ.obj
 0001:0003acfc       ??0?$_Container_base_aux_alloc_real@V?$allocator@U?$pair@$$CBKPAUCListSellData@CCtrlListWZ@@@std@@@std@@@std@@IAE@V?$allocator@U?$pair@$$CBKPAUCListSellData@CCtrlListWZ@@@std@@@1@@Z 1003bcfc f i CtrlListWZ.obj
 0001:0003acfc       ??0?$_Container_base_aux_alloc_real@V?$allocator@PAX@std@@@std@@IAE@V?$allocator@PAX@1@@Z 1003bcfc f i CtrlListWZ.obj
 0001:0003acfc       ??0?$_Container_base_aux_alloc_real@V?$allocator@K@std@@@std@@IAE@V?$allocator@K@1@@Z 1003bcfc f i BaseManager.obj
 0001:0003acfc       ??0?$_Container_base_aux_alloc_real@V?$allocator@UtagRECT@@@std@@@std@@IAE@V?$allocator@UtagRECT@@@1@@Z 1003bcfc f i DialogWZ.obj
 0001:0003acfc       ??0?$_Container_base_aux_alloc_real@V?$allocator@PAVCControlWZ@@@std@@@std@@IAE@V?$allocator@PAVCControlWZ@@@1@@Z 1003bcfc f i DialogWZ.obj
 0001:0003acfc       ??0?$_Container_base_aux_alloc_real@V?$allocator@U_List_position@?$_Hash@V?$_Hmap_traits@KV?$basic_string@DU?$char_traits@D@std@@V?$allocator@D@2@@std@@V?$hash_compare@KU?$less@K@std@@@stdext@@V?$allocator@U?$pair@$$CBKV?$basic_string@DU?$char_traits@D@std@@V?$allocator@D@2@@std@@@std@@@2@$0A@@stdext@@@stdext@@@std@@@std@@IAE@V?$allocator@U_List_position@?$_Hash@V?$_Hmap_traits@KV?$basic_string@DU?$char_traits@D@std@@V?$allocator@D@2@@std@@V?$hash_compare@KU?$less@K@std@@@stdext@@V?$allocator@U?$pair@$$CBKV?$basic_string@DU?$char_traits@D@std@@V?$allocator@D@2@@std@@@std@@@2@$0A@@stdext@@@stdext@@@1@@Z 1003bcfc f i StringManager.obj
 0001:0003acfc       ??0?$_Container_base_aux_alloc_real@V?$allocator@U?$pair@$$CBKPAX@std@@@std@@@std@@IAE@V?$allocator@U?$pair@$$CBKPAX@std@@@1@@Z 1003bcfc f i BaseManager.obj
 0001:0003acfc       ??0?$_Container_base_aux_alloc_real@V?$allocator@U_List_position@?$_Hash@V?$_Hmap_traits@KPAXV?$hash_compare@KU?$less@K@std@@@stdext@@V?$allocator@U?$pair@$$CBKPAX@std@@@std@@$0A@@stdext@@@stdext@@@std@@@std@@IAE@V?$allocator@U_List_position@?$_Hash@V?$_Hmap_traits@KPAXV?$hash_compare@KU?$less@K@std@@@stdext@@V?$allocator@U?$pair@$$CBKPAX@std@@@std@@$0A@@stdext@@@stdext@@@1@@Z 1003bcfc f i BaseManager.obj
 0001:0003acfc       ??0?$_Container_base_aux_alloc_real@V?$allocator@U?$pair@$$CBKV?$basic_string@DU?$char_traits@D@std@@V?$allocator@D@2@@std@@@std@@@std@@@std@@IAE@V?$allocator@U?$pair@$$CBKV?$basic_string@DU?$char_traits@D@std@@V?$allocator@D@2@@std@@@std@@@1@@Z 1003bcfc f i StringManager.obj
 0001:0003ad7a       ?clear@?$list@U?$pair@$$CBKPAX@std@@V?$allocator@U?$pair@$$CBKPAX@std@@@2@@std@@QAEXXZ 1003bd7a f i BaseManager.obj
 0001:0003ad7a       ?clear@?$list@PAVCControlWZ@@V?$allocator@PAVCControlWZ@@@std@@@std@@QAEXXZ 1003bd7a f i DialogWZ.obj
 0001:0003ad7a       ?clear@?$list@UtagRECT@@V?$allocator@UtagRECT@@@std@@@std@@QAEXXZ 1003bd7a f i DialogWZ.obj
 0001:0003ad7a       ?clear@?$list@PAXV?$allocator@PAX@std@@@std@@QAEXXZ 1003bd7a f i CtrlListWZ.obj
 0001:0003ad7a       ?clear@?$list@KV?$allocator@K@std@@@std@@QAEXXZ 1003bd7a f i BaseManager.obj
 0001:0003ade6       ??0CDlgBaseWZ@@QAE@XZ      1003bde6 f   DlgBaseWZ.obj
 0001:0003ae1a       ??1CDlgBaseWZ@@UAE@XZ      1003be1a f   DlgBaseWZ.obj
 0001:0003ae2c       ?ShowWindowWZ@CDlgBaseWZ@@UAEXW4ENUM_STATEWZ@@@Z 1003be2c f i DlgBaseWZ.obj
 0001:0003ae40       ??_ECDlgBaseWZ@@UAEPAXI@Z  1003be40 f i DlgBaseWZ.obj
 0001:0003ae40       ??_GCDlgBaseWZ@@UAEPAXI@Z  1003be40 f i DlgBaseWZ.obj
 0001:0003ae67       ?GetNameFromIndex@CColor@@SAPBDH@Z 1003be67 f   Color.obj
 0001:0003ae76       ?GetColorFromIndex@CColor@@SA?AV1@H@Z 1003be76 f   Color.obj
 0001:0003ae90       ??0CColor@@QAE@K@Z         1003be90 f   Color.obj
 0001:0003aeb4       ??BCColor@@QBEKXZ          1003beb4 f   Color.obj
 0001:0003aeca       ?SetRed@CColor@@QAEXH@Z    1003beca f   Color.obj
 0001:0003aeec       ?SetGreen@CColor@@QAEXH@Z  1003beec f   Color.obj
 0001:0003af0f       ?SetBlue@CColor@@QAEXH@Z   1003bf0f f   Color.obj
 0001:0003af32       ?SetRGB@CColor@@QAEXHHH@Z  1003bf32 f   Color.obj
 0001:0003af65       ?GetRed@CColor@@QBEHXZ     1003bf65 f   Color.obj
 0001:0003af7c       ?GetGreen@CColor@@QBEHXZ   1003bf7c f   Color.obj
 0001:0003af94       ?GetBlue@CColor@@QBEHXZ    1003bf94 f   Color.obj
 0001:0003afac       ?SetHue@CColor@@QAEXM@Z    1003bfac f   Color.obj
 0001:0003afd3       ?SetSaturation@CColor@@QAEXM@Z 1003bfd3 f   Color.obj
 0001:0003affa       ?SetLuminance@CColor@@QAEXM@Z 1003bffa f   Color.obj
 0001:0003b021       ?SetHLS@CColor@@QAEXMMM@Z  1003c021 f   Color.obj
 0001:0003b061       ?GetHue@CColor@@QBEMXZ     1003c061 f   Color.obj
 0001:0003b078       ?GetSaturation@CColor@@QBEMXZ 1003c078 f   Color.obj
 0001:0003b08f       ?GetLuminance@CColor@@QBEMXZ 1003c08f f   Color.obj
 0001:0003b0a6       ?ToHLS@CColor@@AAEXXZ      1003c0a6 f   Color.obj
 0001:0003b32c       ?ToRGB@CColor@@AAEXXZ      1003c32c f   Color.obj
 0001:0003b473       ?ToRGB1@CColor@@CAEMMM@Z   1003c473 f   Color.obj
 0001:0003b527       ??0CDialogManager@@QAE@XZ  1003c527 f   DialogManager.obj
 0001:0003b6c6       ??1CDialogManager@@UAE@XZ  1003c6c6 f   DialogManager.obj
 0001:0003b803       ?OnCreate@CDialogManager@@UAE_NPADPAUHWND__@@PAUHINSTANCE__@@PAX_N@Z 1003c803 f   DialogManager.obj
 0001:0003b85e       ?SetResourceFolderPath@CDialogManager@@UAEXPAD@Z 1003c85e f   DialogManager.obj
 0001:0003b877       ?EnableImeSystem@CDialogManager@@UAEX_N@Z 1003c877 f   DialogManager.obj
 0001:0003b88b       ?SetDiscAccess@CDialogManager@@UAEXPAX@Z 1003c88b f   DialogManager.obj
 0001:0003b8a4       ?CreateDialogWZ@CDialogManager@@UAEPAVCDialogWZ@@KK@Z 1003c8a4 f   DialogManager.obj
 0001:0003b9ba       ?CreateControlWZ@CDialogManager@@UAEPAVCControlWZ@@KKKKPAUtagRECT@@@Z 1003c9ba f   DialogManager.obj
 0001:0003ba1a       ?OnDestroy@CDialogManager@@UAEXXZ 1003ca1a f   DialogManager.obj
 0001:0003ba53       ?OnRelease@CDialogManager@@UAEXXZ 1003ca53 f   DialogManager.obj
 0001:0003baed       ?RemoveDialogWZ@CDialogManager@@UAE_NK@Z 1003caed f   DialogManager.obj
 0001:0003bb6c       ?RemoveControlWZ@CDialogManager@@UAE_NKK@Z 1003cb6c f   DialogManager.obj
 0001:0003bb9c       ?OnLoad@CDialogManager@@UAEKPAXPAKPAU_SYSTEMTIME@@@Z 1003cb9c f   DialogManager.obj
 0001:0003bd82       ?OnSave@CDialogManager@@UAEXPAXPAU_SYSTEMTIME@@@Z 1003cd82 f   DialogManager.obj
 0001:0003be61       ?ChangeDrawClassPtr@CDialogManager@@UAEXPAXPAUHWND__@@@Z 1003ce61 f   DialogManager.obj
 0001:0003bed3       ?GetDialogWZ@CDialogManager@@UAEPAVCDialogWZ@@K@Z 1003ced3 f   DialogManager.obj
 0001:0003befd       ?GetClientRectWZ@CDialogManager@@UAEXKPAUtagRECT@@@Z 1003cefd f   DialogManager.obj
 0001:0003bf31       ?GetDialogWZSizeRect@CDialogManager@@UAE_NKPAUtagRECT@@@Z 1003cf31 f   DialogManager.obj
 0001:0003bf6b       ?GetControlSizeRect@CDialogManager@@UAE_NKKPAUtagRECT@@@Z 1003cf6b f   DialogManager.obj
 0001:0003bfa8       ?OnDoAction@CDialogManager@@UAEXXZ 1003cfa8 f   DialogManager.obj
 0001:0003bffe       ?OnDraw@CDialogManager@@UAEXXZ 1003cffe f   DialogManager.obj
 0001:0003c056       ?OnDrawDialog@CDialogManager@@UAEXK@Z 1003d056 f   DialogManager.obj
 0001:0003c086       ?SetDialogImageFormat@CDialogManager@@UAEXKPAUSI_TFORMAT@@@Z 1003d086 f   DialogManager.obj
 0001:0003c0b7       ?SetControlImageFormat@CDialogManager@@UAEXKKPAUSI_TFORMAT@@@Z 1003d0b7 f   DialogManager.obj
 0001:0003c0eb       ?GetDialogIDToIndex@CDialogManager@@UAEKH@Z 1003d0eb f   DialogManager.obj
 0001:0003c11d       ?MoveTail@CDialogManager@@UAEXH@Z 1003d11d f   DialogManager.obj
 0001:0003c136       ?MoveHead@CDialogManager@@UAEXH@Z 1003d136 f   DialogManager.obj
 0001:0003c14f       ?PickDialog@CDialogManager@@UAEKHH@Z 1003d14f f   DialogManager.obj
 0001:0003c20e       ?MoveDialogWZ@CDialogManager@@UAEXKKUtagRECT@@@Z 1003d20e f   DialogManager.obj
 0001:0003c2ad       ?GetDlgCnt@CDialogManager@@UAEKXZ 1003d2ad f   DialogManager.obj
 0001:0003c2c1       ?GetCountStringTable@CDialogManager@@UAEHXZ 1003d2c1 f   DialogManager.obj
 0001:0003c2da       ?FindStringTableA@CDialogManager@@UAE_NKPADH@Z 1003d2da f   DialogManager.obj
 0001:0003c2f6       ?AddStringTableA@CDialogManager@@UAE_NKPAD@Z 1003d2f6 f   DialogManager.obj
 0001:0003c312       ?RemoveStringTable@CDialogManager@@UAE_NK@Z 1003d312 f   DialogManager.obj
 0001:0003c32b       ?GetStringTableIndexValueA@CDialogManager@@UAE_NHPAKPADH@Z 1003d32b f   DialogManager.obj
 0001:0003c34a       ?SaveStringTable@CDialogManager@@UAE_NPAD@Z 1003d34a f   DialogManager.obj
 0001:0003c48e       ?LoadStringTable@CDialogManager@@UAE_NPADW4ENUM_LOAD_UITYPE@@@Z 1003d48e f   DialogManager.obj
 0001:0003c5d5       ?FindStringTableW@CDialogManager@@UAE_NKPA_WH@Z 1003d5d5 f   DialogManager.obj
 0001:0003c687       ?AddStringTableW@CDialogManager@@UAE_NKPA_W@Z 1003d687 f   DialogManager.obj
 0001:0003c6e8       ?GetStringTableIndexValueW@CDialogManager@@UAE_NHPAKPA_WH@Z 1003d6e8 f   DialogManager.obj
 0001:0003c79d       ?SetDefaultFontID@CDialogManager@@UAEXK@Z 1003d79d f   DialogManager.obj
 0001:0003c7b6       ?GetDefaultFontID@CDialogManager@@UAEKXZ 1003d7b6 f   DialogManager.obj
 0001:0003c7ca       ?GetNumberOfDefaultFont@CDialogManager@@UAEHXZ 1003d7ca f   DialogManager.obj
 0001:0003c7de       ?GetDefaultFontInfo@CDialogManager@@UAEHHPAKPAUtagLOGFONTA@@@Z 1003d7de f   DialogManager.obj
 0001:0003c7fd       ?AddExtendedFont@CDialogManager@@UAEHKPAUtagLOGFONTA@@@Z 1003d7fd f   DialogManager.obj
 0001:0003c819       ?DeleteExtendedFont@CDialogManager@@UAEXK@Z 1003d819 f   DialogManager.obj
 0001:0003c832       ?DeleteAllExtendedFont@CDialogManager@@UAEXXZ 1003d832 f   DialogManager.obj
 0001:0003c846       ?GetNumberOfExtendedFont@CDialogManager@@UAEHXZ 1003d846 f   DialogManager.obj
 0001:0003c85a       ?GetExtendedFontInfo@CDialogManager@@UAEHHPAKPAUtagLOGFONTA@@@Z 1003d85a f   DialogManager.obj
 0001:0003c879       ?LoadExtendedFontInfo@CDialogManager@@UAEHPAD@Z 1003d879 f   DialogManager.obj
 0001:0003c892       ?SaveExtendedFontInfo@CDialogManager@@UAEHPAD@Z 1003d892 f   DialogManager.obj
 0001:0003c8ab       ?FirstDialogID@CDialogManager@@UAEXK@Z 1003d8ab f   DialogManager.obj
 0001:0003c902       ?DeAttachFirstDialogID@CDialogManager@@UAEXK@Z 1003d902 f   DialogManager.obj
 0001:0003c921       ?ApplyAttachDialog@CDialogManager@@UAEXXZ 1003d921 f   DialogManager.obj
 0001:0003c9aa       ?RequestFocus@CDialogManager@@UAEXPAVCDialogWZ@@@Z 1003d9aa f   DialogManager.obj
 0001:0003ca10       ?LockMessageDialogID@CDialogManager@@UAEXK@Z 1003da10 f   DialogManager.obj
 0001:0003ca58       ?GetActiveEditCount@CDialogManager@@UAEHXZ 1003da58 f   DialogManager.obj
 0001:0003cafa       ?SetExePath@CDialogManager@@UAEXPBD@Z 1003dafa f   DialogManager.obj
 0001:0003cb13       ?WindowProc@CDialogManager@@UAE_NPAUHWND__@@IIJPAUSI_MESSAGE@@@Z 1003db13 f   DialogManager.obj
 0001:0003d01e       ?GetLockDlgID@CDialogManager@@UAEKXZ 1003e01e f   DialogManager.obj
 0001:0003d02c       ?GetStringManager@CDialogManager@@UAEPAVCStringManager@@XZ 1003e02c f i DialogManager.obj
 0001:0003d03b       ?GetDlgManager@CDialogManager@@UAEPAVCBaseManager@@XZ 1003e03b f i DialogManager.obj
 0001:0003d04a       ??_GCDialogManager@@UAEPAXI@Z 1003e04a f i DialogManager.obj
 0001:0003d04a       ??_ECDialogManager@@UAEPAXI@Z 1003e04a f i DialogManager.obj
 0001:0003d071       ??0CDrawCtrl@@QAE@XZ       1003e071 f   DrawCtrl.obj
 0001:0003d0de       ??1CDrawCtrl@@UAE@XZ       1003e0de f   DrawCtrl.obj
 0001:0003d0f7       ?SetDiscAccess@CDrawCtrl@@QAEXPAX@Z 1003e0f7 f   DrawCtrl.obj
 0001:0003d10b       ?FileRead@CDrawCtrl@@QAEKPAX0K@Z 1003e10b f   DrawCtrl.obj
 0001:0003d13e       ?FileWrite@CDrawCtrl@@QAEKPAX0K@Z 1003e13e f   DrawCtrl.obj
 0001:0003d171       ?FileOpen@CDrawCtrl@@QAEPAXPBDKKPAU_SECURITY_ATTRIBUTES@@K@Z 1003e171 f   DrawCtrl.obj
 0001:0003d1cf       ?FileClose@CDrawCtrl@@QAEXPAX@Z 1003e1cf f   DrawCtrl.obj
 0001:0003d1e8       ?GetFileSize@CDrawCtrl@@QAEKPAX@Z 1003e1e8 f   DrawCtrl.obj
 0001:0003d201       ?OnRelease@CDrawCtrl@@QAEXPAX@Z 1003e201 f   DrawCtrl.obj
 0001:0003d245       ?BeginUseFont@CDrawCtrl@@QAE_NK@Z 1003e245 f   DrawCtrl.obj
 0001:0003d2eb       ?EndUseFont@CDrawCtrl@@QAEXXZ 1003e2eb f   DrawCtrl.obj
 0001:0003d310       ?BegineTransparency@CDrawCtrl@@QAEXM@Z 1003e310 f   DrawCtrl.obj
 0001:0003d343       ?EndTransparency@CDrawCtrl@@QAEXXZ 1003e343 f   DrawCtrl.obj
 0001:0003d35f       ?TextOutWZ@CDrawCtrl@@QAEXPBDMMK@Z 1003e35f f   DrawCtrl.obj
 0001:0003d40a       ?DrawTextA@CDrawCtrl@@QAEXPBDPAUtagRECT@@KKW4ENUM_TEXT_KIND@@K@Z 1003e40a f   DrawCtrl.obj
 0001:0003d5dc       ?DrawText_Depth@CDrawCtrl@@QAEXPBDPAUtagRECT@@KKW4ENUM_TEXT_KIND@@KM@Z 1003e5dc f   DrawCtrl.obj
 0001:0003d642       ?DrawTextW@CDrawCtrl@@QAEXPB_WPAUtagRECT@@KKW4ENUM_TEXT_KIND@@K@Z 1003e642 f   DrawCtrl.obj
 0001:0003d7d4       ?GetTextExtentPointA@CDrawCtrl@@QAEXPBDHPAUtagSIZE@@@Z 1003e7d4 f   DrawCtrl.obj
 0001:0003d7fa       ?GetTextExtentPointW@CDrawCtrl@@QAEXPB_WHPAUtagSIZE@@@Z 1003e7fa f   DrawCtrl.obj
 0001:0003d820       ?SetDefaultFontID@CDrawCtrl@@QAEXK@Z 1003e820 f   DrawCtrl.obj
 0001:0003d83f       ?GetDefaultFontID@CDrawCtrl@@QAEKXZ 1003e83f f   DrawCtrl.obj
 0001:0003d851       ?GetFontDC@CDrawCtrl@@QAEPAUHDC__@@K@Z 1003e851 f   DrawCtrl.obj
 0001:0003d871       ?GetFontLogFont@CDrawCtrl@@QAEHKPAUtagLOGFONTA@@@Z 1003e871 f   DrawCtrl.obj
 0001:0003d912       ?GetNumberOfDefaultFont@CDrawCtrl@@QAEHXZ 1003e912 f   DrawCtrl.obj
 0001:0003d92d       ?GetDefaultFontInfo@CDrawCtrl@@QAEHHPAKPAUtagLOGFONTA@@@Z 1003e92d f   DrawCtrl.obj
 0001:0003d9d6       ?AddExtendedFont@CDrawCtrl@@QAEHKPAUtagLOGFONTA@@@Z 1003e9d6 f   DrawCtrl.obj
 0001:0003da2d       ?DeleteExtendedFont@CDrawCtrl@@QAEXK@Z 1003ea2d f   DrawCtrl.obj
 0001:0003da4d       ?DeleteAllExtendedFont@CDrawCtrl@@QAEXXZ 1003ea4d f   DrawCtrl.obj
 0001:0003da68       ?GetNumberOfExtendedFont@CDrawCtrl@@QAEHXZ 1003ea68 f   DrawCtrl.obj
 0001:0003da83       ?GetExtendedFontInfo@CDrawCtrl@@QAEHHPAKPAUtagLOGFONTA@@@Z 1003ea83 f   DrawCtrl.obj
 0001:0003db14       ?LoadExtendedFontInfo@CDrawCtrl@@QAEHPBD@Z 1003eb14 f   DrawCtrl.obj
 0001:0003db36       ?SaveExtendedFontInfo@CDrawCtrl@@QAEHPBD@Z 1003eb36 f   DrawCtrl.obj
 0001:0003db56       ?LoadImageA@CDrawCtrl@@QAEPAXPBD@Z 1003eb56 f   DrawCtrl.obj
 0001:0003dcc7       ?GenerateEmptyTexture@CDrawCtrl@@QAEPAXHHH@Z 1003ecc7 f   DrawCtrl.obj
 0001:0003dcfd       ?LockTexture@CDrawCtrl@@QAEPAXPAXPAJPAH@Z 1003ecfd f   DrawCtrl.obj
 0001:0003dd2e       ?UnlockTexture@CDrawCtrl@@QAEXPAX@Z 1003ed2e f   DrawCtrl.obj
 0001:0003dd59       ?SetDrawClass@CDrawCtrl@@QAEXPAX@Z 1003ed59 f   DrawCtrl.obj
 0001:0003dd6d       ?ChangeStrToDWORD@CDrawCtrl@@QAEKPBD@Z 1003ed6d f   DrawCtrl.obj
 0001:0003dda2       ?SetBackGroundColor@CDrawCtrl@@QAEXK@Z 1003eda2 f   DrawCtrl.obj
 0001:0003de44       ?GetRealX@CDrawCtrl@@QAEMM@Z 1003ee44 f   DrawCtrl.obj
 0001:0003de61       ?GetRealY@CDrawCtrl@@QAEMM@Z 1003ee61 f   DrawCtrl.obj
 0001:0003de7e       ?GetStdX@CDrawCtrl@@QAEMM@Z 1003ee7e f   DrawCtrl.obj
 0001:0003de9b       ?GetStdY@CDrawCtrl@@QAEMM@Z 1003ee9b f   DrawCtrl.obj
 0001:0003deb8       ?SetExePath@CDrawCtrl@@QAEXPBD@Z 1003eeb8 f   DrawCtrl.obj
 0001:0003defe       ?DrawTexture@CDrawCtrl@@QAEXPAXABUSt_FRect@@1@Z 1003eefe f   DrawCtrl.obj
 0001:0003dfb3       ?DrawTexture@CDrawCtrl@@QAEXPAXABUSt_FRect@@1M@Z 1003efb3 f   DrawCtrl.obj
 0001:0003e069       ?DrawTexture@CDrawCtrl@@QAEXPAXABUSt_FRect@@@Z 1003f069 f   DrawCtrl.obj
 0001:0003e0de       ?DrawRectangle@CDrawCtrl@@QAEXABUtagRECT@@KH@Z 1003f0de f   DrawCtrl.obj
 0001:0003e2c6       ?DrawFillRectangle@CDrawCtrl@@QAEXABUtagRECT@@KPBUSI_Gradation@@@Z 1003f2c6 f   DrawCtrl.obj
 0001:0003e605       ?DrawRectangle@CDrawCtrl@@QAEXABUSt_FRect@@KH@Z 1003f605 f   DrawCtrl.obj
 0001:0003e7ba       ?DrawFillRectangle@CDrawCtrl@@QAEXABUSt_FRect@@KPBUSI_Gradation@@@Z 1003f7ba f   DrawCtrl.obj
 0001:0003ead9       ?DrawLine@CDrawCtrl@@QAEXABUSt_FRect@@K@Z 1003fad9 f   DrawCtrl.obj
 0001:0003ebaf       ?DrawShadowConvex@CDrawCtrl@@QAEXABUSt_FRect@@H@Z 1003fbaf f   DrawCtrl.obj
 0001:0003ef5b       ?DrawShadowConcave@CDrawCtrl@@QAEXABUSt_FRect@@H@Z 1003ff5b f   DrawCtrl.obj
 0001:0003f1dd       ?Draw3dShapeConvex@CDrawCtrl@@QAEXABUtagRECT@@K@Z 100401dd f   DrawCtrl.obj
 0001:0003f204       ?Draw3dShapeConvex@CDrawCtrl@@QAEXABUSt_FRect@@K@Z 10040204 f   DrawCtrl.obj
 0001:0003f93e       ?Draw3dShapeConcave@CDrawCtrl@@QAEXABUtagRECT@@K@Z 1004093e f   DrawCtrl.obj
 0001:0003f965       ?Draw3dShapeConcave@CDrawCtrl@@QAEXABUSt_FRect@@K@Z 10040965 f   DrawCtrl.obj
 0001:00040059       ?GetTextWidth@CDrawCtrl@@QAEHPBDK@Z 10041059 f   DrawCtrl.obj
 0001:000400e3       ?MakeReduceText@CDrawCtrl@@QAE_NPAV?$basic_string@DU?$char_traits@D@std@@V?$allocator@D@2@@std@@PBDABUtagRECT@@K@Z 100410e3 f   DrawCtrl.obj
 0001:000402b9       ??_GCDrawCtrl@@UAEPAXI@Z   100412b9 f i DrawCtrl.obj
 0001:000402b9       ??_ECDrawCtrl@@UAEPAXI@Z   100412b9 f i DrawCtrl.obj
 0001:000402e0       ?RealXToStdX@CDrawBase@@QAEMM@Z 100412e0 f i DrawCtrl.obj
 0001:00040325       ?RealYToStdY@CDrawBase@@QAEMM@Z 10041325 f i DrawCtrl.obj
 0001:0004036a       ?StdXToRealX@CDrawBase@@QAEMM@Z 1004136a f i DrawCtrl.obj
 0001:000403a9       ?StdYToRealY@CDrawBase@@QAEMM@Z 100413a9 f i DrawCtrl.obj
 0001:000403e8       ??0St_FRect@@QAE@ABUtagRECT@@@Z 100413e8 f i DrawCtrl.obj
 0001:00040434       ?append@?$basic_string@DU?$char_traits@D@std@@V?$allocator@D@2@@std@@QAEAAV12@ID@Z 10041434 f i DrawCtrl.obj
 0001:000404c6       ?append@?$basic_string@DU?$char_traits@D@std@@V?$allocator@D@2@@std@@QAEAAV12@PBDI@Z 100414c6 f i DrawCtrl.obj
 0001:000405f8       ?_Chassign@?$basic_string@DU?$char_traits@D@std@@V?$allocator@D@2@@std@@IAEXIID@Z 100415f8 f i DrawCtrl.obj
 0001:0004066f       ?append@?$basic_string@DU?$char_traits@D@std@@V?$allocator@D@2@@std@@QAEAAV12@ABV12@II@Z 1004166f f i DrawCtrl.obj
 0001:000407af       ?IsCPUID@FastMath@@YA_NXZ  100417af f   common:wzfastmath.obj
 0001:00040823       ?IsCPUSupport@FastMath@@YA_NW4SlIntrinsic@1@@Z 10041823 f   common:wzfastmath.obj
 0001:000408fd       ?IsOSSupport@FastMath@@YA_NW4SlIntrinsic@1@@Z 100418fd f   common:wzfastmath.obj
 0001:000409b8       ?GetCPUCaps@FastMath@@YAXPAUCPUCaps@1@@Z 100419b8 f   common:wzfastmath.obj
 0001:00040adc       ?Startup@FastMath@@YAXXZ   10041adc f   common:wzfastmath.obj
 0001:00040b75       ?MatrixRotationX_Scalar@@YAPAUWzMatrix@@PAU1@M@Z 10041b75 f i common:wzmath.obj
 0001:00040c89       ?MatrixRotationY_Scalar@@YAPAUWzMatrix@@PAU1@M@Z 10041c89 f i common:wzmath.obj
 0001:00040d9c       ?MatrixRotationZ_Scalar@@YAPAUWzMatrix@@PAU1@M@Z 10041d9c f i common:wzmath.obj
 0001:00040eb0       ?QuaternionMultiply_Scalar@@YAPAUWzQuaternion@@PAU1@PBU1@1@Z 10041eb0 f i common:wzmath.obj
 0001:00040f9f       ?MatrixInverse@@YAPAUWzMatrix@@PAU1@PBU1@@Z 10041f9f f   common:wzmath.obj
 0001:0004184d       ?MatrixRotationZYX@@YAPAUWzMatrix@@PAU1@PBUWzVector@@@Z 1004284d f   common:wzmath.obj
 0001:00041a19       ?MatrixRotationZXY@@YAPAUWzMatrix@@PAU1@PBUWzVector@@@Z 10042a19 f   common:wzmath.obj
 0001:00041be2       ?MatrixMultiply_Scalar@@YAPAUWzMatrix@@PAU1@PBU1@1@Z 10042be2 f   common:wzmath.obj
 0001:00041fa1       ?MatrixMultiply4x3_Scalar@@YAPAUWzMatrix@@PAU1@PBU1@1@Z 10042fa1 f   common:wzmath.obj
 0001:0004221b       ?MatrixRotationX_SSE@@YAPAUWzMatrix@@PAU1@M@Z 1004321b f   common:wzmath.obj
 0001:00042252       ?MatrixRotationY_SSE@@YAPAUWzMatrix@@PAU1@M@Z 10043252 f   common:wzmath.obj
 0001:00042286       ?MatrixRotationZ_SSE@@YAPAUWzMatrix@@PAU1@M@Z 10043286 f   common:wzmath.obj
 0001:000422ba       ?MatrixMultiply_SSE@@YAPAUWzMatrix@@PAU1@PBU1@1@Z 100432ba f   common:wzmath.obj
 0001:000423d5       ?MatrixRotationX_3DNOW@@YAPAUWzMatrix@@PAU1@M@Z 100433d5 f   common:wzmath.obj
 0001:00042420       ?MatrixRotationY_3DNOW@@YAPAUWzMatrix@@PAU1@M@Z 10043420 f   common:wzmath.obj
 0001:00042468       ?MatrixRotationZ_3DNOW@@YAPAUWzMatrix@@PAU1@M@Z 10043468 f   common:wzmath.obj
 0001:000424b0       ?MatrixMultiply_3DNOW@@YAPAUWzMatrix@@PAU1@PBU1@1@Z 100434b0 f   common:wzmath.obj
 0001:00042674       ?RotationToQuaternion@@YAPAUWzQuaternion@@PAU1@PBUWzVector@@@Z 10043674 f   common:wzmath.obj
 0001:00042778       ?GetQuaternionToConvertVector@@YAPAUWzQuaternion@@PAU1@PBUWzVector@@1@Z 10043778 f   common:wzmath.obj
 0001:000428c1       ?MatrixToQuaternion@@YAPAUWzQuaternion@@PAU1@PBUWzMatrix@@@Z 100438c1 f   common:wzmath.obj
 0001:00042aa2       ?QuaternionToAxisAngle@@YAXPAUWzVector@@PAMPBUWzQuaternion@@@Z 10043aa2 f   common:wzmath.obj
 0001:00042b98       ?QuaternionSlerp@@YAPAUWzQuaternion@@PAU1@PBU1@1M@Z 10043b98 f   common:wzmath.obj
 0001:00042d0e       ?QuaternionMultiply_SSE@@YAPAUWzQuaternion@@PAU1@PBU1@1@Z 10043d0e f   common:wzmath.obj
 0001:00042d80       ?QuaternionMultiply_3DNOWEXT@@YAPAUWzQuaternion@@PAU1@PBU1@1@Z 10043d80 f   common:wzmath.obj
 0001:00042e29       ?MatrixSetZero@@YAPAUWzMatrix@@PAU1@@Z 10043e29 f i common:wzmath.obj
 0001:00042f30       ?VectorDotProduct@@YAMPBUWzVector@@0@Z 10043f30 f i common:wzmath.obj
 0001:00042f62       ?VectorCrossProduct@@YAPAUWzVector@@PAU1@PBU1@1@Z 10043f62 f i common:wzmath.obj
 0001:00042fc5       ?VectorNormalize@@YAPAUWzVector@@PAU1@PBU1@@Z 10043fc5 f i common:wzmath.obj
 0001:00043020       ?VectorLength@@YAMPBUWzVector@@@Z 10044020 f i common:wzmath.obj
 0001:00043041       ?VectorLength2@@YAMPBUWzVector@@@Z 10044041 f i common:wzmath.obj
 0001:00043073       ?QuaternionRotation@@YAPAUWzQuaternion@@PAU1@PBUWzVector@@M@Z 10044073 f i common:wzmath.obj
 0001:000430f6       ?GetModuleTitle@?A0x5958724f@WzLog@@YAPBDXZ 100440f6 f   programcommonlibforengine:wzlogsystem.obj
 0001:000431b5       ??0WzLogSystem@WzLog@@QAE@XZ 100441b5 f   programcommonlibforengine:wzlogsystem.obj
 0001:00043203       ??1WzLogSystem@WzLog@@UAE@XZ 10044203 f   programcommonlibforengine:wzlogsystem.obj
 0001:00043225       ?AddLogHandler@WzLogSystem@WzLog@@QAEXPAVWzLogHandler@2@@Z 10044225 f   programcommonlibforengine:wzlogsystem.obj
 0001:0004326a       ?Initialize@WzLogSystem@WzLog@@QAEXXZ 1004426a f   programcommonlibforengine:wzlogsystem.obj
 0001:000432ca       ?Release@WzLogSystem@WzLog@@QAEXXZ 100442ca f   programcommonlibforengine:wzlogsystem.obj
 0001:000432f6       ?WriteLog@WzLogSystem@WzLog@@QAEXW4WZLOG_TYPE@WzLogType@@PBD@Z 100442f6 f   programcommonlibforengine:wzlogsystem.obj
 0001:0004333f       ?InitializeWzLogSystem@@YAXXZ 1004433f f   programcommonlibforengine:wzlogsystem.obj
 0001:000433ba       ?ReleaseWzLogSystem@@YAXXZ 100443ba f   programcommonlibforengine:wzlogsystem.obj
 0001:000433ff       ?AddWzLogHandler@@YAXPAVWzLogHandler@WzLog@@@Z 100443ff f   programcommonlibforengine:wzlogsystem.obj
 0001:0004341e       ?OutputWzLog@@YAXW4WZLOG_TYPE@WzLogType@@PBDZZ 1004441e f   programcommonlibforengine:wzlogsystem.obj
 0001:0004346d       ??_GWzLogSystem@WzLog@@UAEPAXI@Z 1004446d f i programcommonlibforengine:wzlogsystem.obj
 0001:0004346d       ??_EWzLogSystem@WzLog@@UAEPAXI@Z 1004446d f i programcommonlibforengine:wzlogsystem.obj
 0001:00043494       ??_E?$CWzSingleton@VWzLogSystem@WzLog@@@@UAEPAXI@Z 10044494 f i programcommonlibforengine:wzlogsystem.obj
 0001:00043494       ??_G?$CWzSingleton@VWzLogSystem@WzLog@@@@UAEPAXI@Z 10044494 f i programcommonlibforengine:wzlogsystem.obj
 0001:000434c3       ??0CDiscAccess@@QAE@XZ     100444c3 f   programcommonlibforengine:discaccess.obj
 0001:0004354c       ??1CDiscAccess@@QAE@XZ     1004454c f   programcommonlibforengine:discaccess.obj
 0001:000435c2       ?Create@CDiscAccess@@QAEHXZ 100445c2 f   programcommonlibforengine:discaccess.obj
 0001:000435f4       ?Destroy@CDiscAccess@@QAEXXZ 100445f4 f   programcommonlibforengine:discaccess.obj
 0001:0004362b       ?OpenDisc_Hard@CDiscAccess@@QAEHKPBD@Z 1004462b f   programcommonlibforengine:discaccess.obj
 0001:00043740       ?OpenDisc_Packer@CDiscAccess@@QAEHKPBD0W4ENUM_OPEN_PACKER_TYPE@@@Z 10044740 f   programcommonlibforengine:discaccess.obj
 0001:000439b8       ?CloseDisc@CDiscAccess@@QAEXK@Z 100449b8 f   programcommonlibforengine:discaccess.obj
 0001:00043ad9       ?SetActiveDisc@CDiscAccess@@QAEHK@Z 10044ad9 f   programcommonlibforengine:discaccess.obj
 0001:00043b87       ?GetActiveDisc@CDiscAccess@@QAEKXZ 10044b87 f   programcommonlibforengine:discaccess.obj
 0001:00043bd2       ?FixFileName@CDiscAccess@@AAEXPADPBD@Z 10044bd2 f   programcommonlibforengine:discaccess.obj
 0001:00043c83       ?OpenFile@CDiscAccess@@QAEPAXKPBDKKW4ENUM_OPEN_DISPOSITION@@@Z 10044c83 f   programcommonlibforengine:discaccess.obj
 0001:00044086       ?CloseFile@CDiscAccess@@QAEHPAX@Z 10045086 f   programcommonlibforengine:discaccess.obj
 0001:000441ec       ?SeekFile@CDiscAccess@@QAEKPAXJW4ENUM_SEEK_ORIGIN@@@Z 100451ec f   programcommonlibforengine:discaccess.obj
 0001:000443a1       ?ReadFile@CDiscAccess@@QAEKPAX0K@Z 100453a1 f   programcommonlibforengine:discaccess.obj
 0001:00044532       ?WriteFile@CDiscAccess@@QAEKPAXPBXK@Z 10045532 f   programcommonlibforengine:discaccess.obj
 0001:000446c3       ?FileExists@CDiscAccess@@QAEHKPBD@Z 100456c3 f   programcommonlibforengine:discaccess.obj
 0001:00044a42       ?GetFileSize@CDiscAccess@@QAEKPAX@Z 10045a42 f   programcommonlibforengine:discaccess.obj
 0001:00044b97       ?GetFileInformationByHandle@CDiscAccess@@QAEHPAXPAUSt_FileInformation@@@Z 10045b97 f   programcommonlibforengine:discaccess.obj
 0001:00044e48       ?CopyFileA@CDiscAccess@@QAEHKPBD0@Z 10045e48 f   programcommonlibforengine:discaccess.obj
 0001:000450f0       ?DeleteFileA@CDiscAccess@@QAEHKPBD@Z 100460f0 f   programcommonlibforengine:discaccess.obj
 0001:00045390       ?CreateDirectoryA@CDiscAccess@@QAEHKPBD@Z 10046390 f   programcommonlibforengine:discaccess.obj
 0001:00045632       ?RemoveDirectoryA@CDiscAccess@@QAEHKPBD@Z 10046632 f   programcommonlibforengine:discaccess.obj
 0001:000458d2       ??1CWzCriticalSection@@QAE@XZ 100468d2 f i programcommonlibforengine:discaccess.obj
 0001:000458ed       ??1CWzSync@@QAE@XZ         100468ed f i programcommonlibforengine:discaccess.obj
 0001:00045910       ??0?$CWzHandleManager@USt_DAFileInfo@@@@QAE@XZ 10046910 f i programcommonlibforengine:discaccess.obj
 0001:0004599c       ??1?$CWzHandleManager@USt_DAFileInfo@@@@UAE@XZ 1004699c f i programcommonlibforengine:discaccess.obj
 0001:00045a08       ?Add@?$CWzHandleManager@USt_DAFileInfo@@@@QAEPAXABUSt_DAFileInfo@@@Z 10046a08 f i programcommonlibforengine:discaccess.obj
 0001:00045adc       ?Release@?$CWzHandleManager@USt_DAFileInfo@@@@QAEHPAX@Z 10046adc f i programcommonlibforengine:discaccess.obj
 0001:00045b88       ?GetData@?$CWzHandleManager@USt_DAFileInfo@@@@QBEABUSt_DAFileInfo@@PAX@Z 10046b88 f i programcommonlibforengine:discaccess.obj
 0001:00045bc0       ?IsValidHandle@?$CWzHandleManager@USt_DAFileInfo@@@@QBEHPAX@Z 10046bc0 f i programcommonlibforengine:discaccess.obj
 0001:00045c0f       ??_G?$CWzHandleManager@USt_DAFileInfo@@@@UAEPAXI@Z 10046c0f f i programcommonlibforengine:discaccess.obj
 0001:00045c0f       ??_E?$CWzHandleManager@USt_DAFileInfo@@@@UAEPAXI@Z 10046c0f f i programcommonlibforengine:discaccess.obj
 0001:00045c36       ?Clear@?$CWzHandleManager@USt_DAFileInfo@@@@QAEXXZ 10046c36 f i programcommonlibforengine:discaccess.obj
 0001:00045c7c       ??0?$CWzArray@USt_DAFileInfo@@@@QAE@XZ 10046c7c f i programcommonlibforengine:discaccess.obj
 0001:00045ce5       ?Set@?$CWzArray@USt_DAFileInfo@@@@QAEXHABUSt_DAFileInfo@@@Z 10046ce5 f i programcommonlibforengine:discaccess.obj
 0001:00045d3a       ?Get@?$CWzArray@USt_DAFileInfo@@@@QBEAAUSt_DAFileInfo@@H@Z 10046d3a f i programcommonlibforengine:discaccess.obj
 0001:00045d69       ??0?$CWzArray@G@@QAE@XZ    10046d69 f i programcommonlibforengine:discaccess.obj
 0001:00045dd1       ??1?$CWzArray@USt_DAFileInfo@@@@QAE@XZ 10046dd1 f i programcommonlibforengine:discaccess.obj
 0001:00045dd1       ??1?$CWzArray@G@@QAE@XZ    10046dd1 f i programcommonlibforengine:discaccess.obj
 0001:00045de2       ?Set@?$CWzArray@G@@QAEXHABG@Z 10046de2 f i programcommonlibforengine:discaccess.obj
 0001:00045e30       ?Get@?$CWzArray@G@@QBEAAGH@Z 10046e30 f i programcommonlibforengine:discaccess.obj
 0001:00045e5f       ?Clear@?$CWzArray@USt_DAFileInfo@@@@QAEXXZ 10046e5f f i programcommonlibforengine:discaccess.obj
 0001:00045e88       ?MakeSureDimensionSize@?$CWzArray@USt_DAFileInfo@@@@AAEXH@Z 10046e88 f i programcommonlibforengine:discaccess.obj
 0001:00045f56       ?Clear@?$CWzArray@G@@QAEXXZ 10046f56 f i programcommonlibforengine:discaccess.obj
 0001:00045f7e       ?MakeSureDimensionSize@?$CWzArray@G@@AAEXH@Z 10046f7e f i programcommonlibforengine:discaccess.obj
 0001:0004604a       ?Release@?$CWzArray@G@@AAEXXZ 1004704a f i programcommonlibforengine:discaccess.obj
 0001:0004604a       ?Release@?$CWzArray@USt_DAFileInfo@@@@AAEXXZ 1004704a f i programcommonlibforengine:discaccess.obj
 0001:00046083       ??0length_error@std@@QAE@ABV?$basic_string@DU?$char_traits@D@std@@V?$allocator@D@2@@1@@Z 10047083 f i libcpmt:string.obj
 0001:000460a0       ??0out_of_range@std@@QAE@ABV?$basic_string@DU?$char_traits@D@std@@V?$allocator@D@2@@1@@Z 100470a0 f i libcpmt:string.obj
 0001:000460bd       ?_Xlen@_String_base@std@@SAXXZ 100470bd f   libcpmt:string.obj
 0001:000460f5       ?_Xran@_String_base@std@@SAXXZ 100470f5 f   libcpmt:string.obj
 0001:0004612d       ??_U@YAPAXI@Z              1004712d f   libcpmt:newaop.obj
 0001:00046138       ??0bad_alloc@std@@QAE@XZ   10047138 f i LIBCMT:new.obj
 0001:00046153       ??2@YAPAXI@Z               10047153 f   LIBCMT:new.obj
 0001:000461b8       ?_JumpToContinuation@@YGXPAXPAUEHRegistrationNode@@@Z 100471b8 f   LIBCMT:_trnsctrl_.obj
 0001:000461ea       ?_CallMemberFunction1@@YGXPAX00@Z 100471ea f   LIBCMT:_trnsctrl_.obj
 0001:000461ea       ?_CallMemberFunction0@@YGXPAX0@Z 100471ea f   LIBCMT:_trnsctrl_.obj
 0001:000461ea       ?_CallMemberFunction2@@YGXPAX00H@Z 100471ea f   LIBCMT:_trnsctrl_.obj
 0001:000461f1       ?_UnwindNestedFrames@@YGXPAUEHRegistrationNode@@PAUEHExceptionRecord@@@Z 100471f1 f   LIBCMT:_trnsctrl_.obj
 0001:00046245       ___CxxFrameHandler3        10047245 f   LIBCMT:_trnsctrl_.obj
 0001:000462ae       ?_CallSETranslator@@YAHPAUEHExceptionRecord@@PAUEHRegistrationNode@@PAX2PBU_s_FuncInfo@@H1@Z 100472ae f   LIBCMT:_trnsctrl_.obj
 0001:00046424       ?_GetRangeOfTrysToCheck@@YAPBU_s_TryBlockMapEntry@@PBU_s_FuncInfo@@HHPAI1@Z 10047424 f   LIBCMT:_trnsctrl_.obj
 0001:00046499       __CreateFrameInfo          10047499 f   LIBCMT:_trnsctrl_.obj
 0001:000464c5       __IsExceptionObjectToBeDestroyed 100474c5 f   LIBCMT:_trnsctrl_.obj
 0001:000464ec       __FindAndUnlinkFrame       100474ec f   LIBCMT:_trnsctrl_.obj
 0001:0004653e       ?_CallCatchBlock2@@YAPAXPAUEHRegistrationNode@@PBU_s_FuncInfo@@PAXHK@Z 1004753e f   LIBCMT:_trnsctrl_.obj
 0001:0004659e       @__security_check_cookie@4 1004759e f   LIBCMT:secchk.obj
 0001:000465ad       __cfltcvt_init             100475ad f   LIBCMT:_fpinit_.obj
 0001:0004660d       __fpmath                   1004760d f   LIBCMT:_fpinit_.obj
 0001:00046630       ??1type_info@@UAE@XZ       10047630 f   LIBCMT:typinfo.obj
 0001:00046640       ??_Etype_info@@UAEPAXI@Z   10047640 f i LIBCMT:typinfo.obj
 0001:00046640       ??_Gtype_info@@UAEPAXI@Z   10047640 f i LIBCMT:typinfo.obj
 0001:00046661       ??8type_info@@QBE_NABV0@@Z 10047661 f   LIBCMT:typinfo.obj
 0001:00046681       ??3@YAXPAX@Z               10047681 f   LIBCMT:delete.obj
 0001:0004668c       __CxxThrowException@8      1004768c f   LIBCMT:throw.obj
 0001:000466d8       __initp_misc_invarg        100476d8 f   LIBCMT:invarg.obj
 0001:000466e7       __invoke_watson            100476e7 f   LIBCMT:invarg.obj
 0001:0004680f       __invalid_parameter        1004780f f   LIBCMT:invarg.obj
 0001:00046835       __invalid_parameter_noinfo 10047835 f   LIBCMT:invarg.obj
 0001:00046845       ??0exception@std@@QAE@XZ   10047845 f   LIBCMT:stdexcpt.obj
 0001:00046856       ??0exception@std@@QAE@ABQBD@Z 10047856 f   LIBCMT:stdexcpt.obj
 0001:000468a9       ??0exception@std@@QAE@ABQBDH@Z 100478a9 f   LIBCMT:stdexcpt.obj
 0001:000468c6       ??0exception@std@@QAE@ABV01@@Z 100478c6 f   LIBCMT:stdexcpt.obj
 0001:00046923       ??1exception@std@@UAE@XZ   10047923 f   LIBCMT:stdexcpt.obj
 0001:00046939       ?what@exception@std@@UBEPBDXZ 10047939 f   LIBCMT:stdexcpt.obj
 0001:00046946       ??_Eexception@std@@UAEPAXI@Z 10047946 f i LIBCMT:stdexcpt.obj
 0001:00046946       ??_Gexception@std@@UAEPAXI@Z 10047946 f i LIBCMT:stdexcpt.obj
 0001:00046967       _ldiv                      10047967 f   LIBCMT:ldiv.obj
 0001:00046975       _memcpy_s                  10047975 f   LIBCMT:memcpy_s.obj
 0001:000469f2       _memmove_s                 100479f2 f   LIBCMT:memmove_s.obj
 0001:00046a4f       ??_V@YAXPAX@Z              10047a4f f   LIBCMT:delete2.obj
 0001:00046a5a       _strncmp                   10047a5a f   LIBCMT:strncmp.obj
 0001:00046b20       _strncpy                   10047b20 f   LIBCMT:strncpy.obj
 0001:00046c44       _atol                      10047c44 f   LIBCMT:atox.obj
 0001:00046c5a       __atoi64                   10047c5a f   LIBCMT:atox.obj
 0001:00046c70       ??0_LocaleUpdate@@QAE@PAUlocaleinfo_struct@@@Z 10047c70 f i LIBCMT:stricmp.obj
 0001:00046cf7       ___ascii_stricmp           10047cf7 f   LIBCMT:stricmp.obj
 0001:00046d30       __stricmp_l                10047d30 f   LIBCMT:stricmp.obj
 0001:00046e05       __stricmp                  10047e05 f   LIBCMT:stricmp.obj
 0001:00046e05       _stricmp                   10047e05 f   LIBCMT:stricmp.obj
 0001:00046e60       _memset                    10047e60 f   LIBCMT:memset.obj
 0001:00046eda       __fclose_nolock            10047eda f   LIBCMT:fclose.obj
 0001:00046f51       _fclose                    10047f51 f   LIBCMT:fclose.obj
 0001:00046fcd       _fputs                     10047fcd f   LIBCMT:fputs.obj
 0001:000470dc       _sprintf                   100480dc f   LIBCMT:sprintf.obj
 0001:00047159       __fsopen                   10048159 f   LIBCMT:fopen.obj
 0001:0004721d       _fopen                     1004821d f   LIBCMT:fopen.obj
 0001:000472ee       ___onexitinit              100482ee f   LIBCMT:onexit.obj
 0001:0004731f       __onexit                   1004831f f   LIBCMT:onexit.obj
 0001:0004735b       _atexit                    1004835b f   LIBCMT:onexit.obj
 0001:00047372       __snprintf                 10048372 f   LIBCMT:snprintf.obj
 0001:00047421       ??_L@YGXPAXIHP6EX0@Z1@Z    10048421 f   LIBCMT:ehvecctr.obj
 0001:00047486       ?__ArrayUnwind@@YGXPAXIHP6EX0@Z@Z 10048486 f   LIBCMT:ehvecdtr.obj
 0001:000474e4       ??_M@YGXPAXIHP6EX0@Z@Z     100484e4 f   LIBCMT:ehvecdtr.obj
 0001:00047550       __ftol2_sse                10048550 f   LIBCMT:ftol2.obj
 0001:00047559       __ftol2_pentium4           10048559 f   LIBCMT:ftol2.obj
 0001:0004756c       __ftol2_sse_excpt          1004856c f   LIBCMT:ftol2.obj
 0001:00047586       __ftol2                    10048586 f   LIBCMT:ftol2.obj
 0001:000475fb       _wcsncpy                   100485fb f   LIBCMT:wcsncpy.obj
 0001:00047645       __wtoi64                   10048645 f   LIBCMT:wtox.obj
 0001:00047660       _memcpy                    10048660 f   LIBCMT:memcpy.obj
 0001:000479c5       __wcstod_l                 100489c5 f   LIBCMT:wcstod.obj
 0001:00047acc       _wcstod                    10048acc f   LIBCMT:wcstod.obj
 0001:00047ae3       __snwprintf                10048ae3 f   LIBCMT:snwprint.obj
 0001:00047bc0       _memmove                   10048bc0 f   LIBCMT:memmove.obj
 0001:00047f25       _wcsncat                   10048f25 f   LIBCMT:wcsncat.obj
 0001:00047f65       __towlower_l               10048f65 f   LIBCMT:towlower.obj
 0001:0004801a       _towlower                  1004901a f   LIBCMT:towlower.obj
 0001:0004802d       __vswprintf_helper         1004902d f   LIBCMT:vswprnc.obj
 0001:00048125       __vswprintf_c_l            10049125 f   LIBCMT:vswprnc.obj
 0001:00048349       _wcstoul                   10049349 f   LIBCMT:wcstol.obj
 0001:00048375       _realloc                   10049375 f   LIBCMT:realloc.obj
 0001:00048590       _free                      10049590 f   LIBCMT:free.obj
 0001:00048620       _cos                       10049620 f   LIBCMT:_cos_.obj
 0001:00048660       __CIcos                    10049660 f   LIBCMT:_cos_.obj
 0001:0004869b       __CIcos_default            1004969b f   LIBCMT:_cos_.obj
 0001:000486af       __cos_default              100496af     LIBCMT:_cos_.obj
 0001:0004879c       __ismbblead_l              1004979c f   LIBCMT:ismbbyte.obj
 0001:000487b5       __ismbblead                100497b5 f   LIBCMT:ismbbyte.obj
 0001:000487cd       __purecall                 100497cd f   LIBCMT:purevirt.obj
 0001:000487f7       _rand                      100497f7 f   LIBCMT:rand.obj
 0001:00048819       __CRT_INIT@12              10049819 f   LIBCMT:dllcrt0.obj
 0001:00048a44       __DllMainCRTStartup@12     10049a44 f   LIBCMT:dllcrt0.obj
 0001:00048a70       __except_handler4          10049a70 f   LIBCMT:chandler4.obj
 0001:00048c00       _sin                       10049c00 f   LIBCMT:_sin_.obj
 0001:00048c40       __CIsin                    10049c40 f   LIBCMT:_sin_.obj
 0001:00048c7b       __CIsin_default            10049c7b f   LIBCMT:_sin_.obj
 0001:00048c8f       __sin_default              10049c8f     LIBCMT:_sin_.obj
 0001:00048d30       _acos                      10049d30 f   LIBCMT:_acos_.obj
 0001:00048d70       __CIacos                   10049d70 f   LIBCMT:_acos_.obj
 0001:00048dab       __CIacos_default           10049dab f   LIBCMT:_acos_.obj
 0001:00048dbf       __acos_default             10049dbf     LIBCMT:_acos_.obj
 0001:00048e80       __CIsqrt                   10049e80 f   LIBCMT:_sqrt_.obj
 0001:00048e94       _sqrt                      10049e94     LIBCMT:_sqrt_.obj
 0001:00048f40       _strrchr                   10049f40 f   LIBCMT:strrchr.obj
 0001:00048f6d       __vsnprintf_l              10049f6d f   LIBCMT:vsnprint.obj
 0001:00049020       __vsnprintf                1004a020 f   LIBCMT:vsnprint.obj
 0001:00049040       _strlen                    1004a040 f   LIBCMT:strlen.obj
 0001:000490cb       __EH_prolog3               1004a0cb f   LIBCMT:ehprolg3.obj
 0001:000490fe       __EH_prolog3_catch         1004a0fe f   LIBCMT:ehprolg3.obj
 0001:00049134       _V6_HeapAlloc              1004a134 f   LIBCMT:malloc.obj
 0001:00049183       _malloc                    1004a183 f   LIBCMT:malloc.obj
 0001:0004924d       __initp_heap_handler       1004a24d f   LIBCMT:handler.obj
 0001:0004925c       __callnewh                 1004a25c f   LIBCMT:handler.obj
 0001:00049284       ??0bad_exception@std@@QAE@PBD@Z 1004a284 f i LIBCMT:frame.obj
 0001:000492a2       ??1bad_exception@std@@UAE@XZ 1004a2a2 f i LIBCMT:frame.obj
 0001:000492ad       ??_Gbad_exception@std@@UAEPAXI@Z 1004a2ad f i LIBCMT:frame.obj
 0001:000492ad       ??_Ebad_exception@std@@UAEPAXI@Z 1004a2ad f i LIBCMT:frame.obj
 0001:000492d4       ___TypeMatch               1004a2d4 f   LIBCMT:frame.obj
 0001:00049333       ___FrameUnwindFilter       1004a333 f   LIBCMT:frame.obj
 0001:0004937c       ___FrameUnwindToState      1004a37c f   LIBCMT:frame.obj
 0001:000494a2       ___DestructExceptionObject 1004a4a2 f   LIBCMT:frame.obj
 0001:000494f7       ___AdjustPointer           1004a4f7 f   LIBCMT:frame.obj
 0001:00049780       ___BuildCatchObjectHelper  1004a780 f   LIBCMT:frame.obj
 0001:000498ff       ___BuildCatchObject        1004a8ff f   LIBCMT:frame.obj
 0001:00049e3a       ??0bad_exception@std@@QAE@ABV01@@Z 1004ae3a f i LIBCMT:frame.obj
 0001:00049e57       ___InternalCxxFrameHandler 1004ae57 f   LIBCMT:frame.obj
 0001:00049f3d       __encode_pointer           1004af3d f   LIBCMT:tidtable.obj
 0001:00049faf       __encoded_null             1004afaf f   LIBCMT:tidtable.obj
 0001:00049fb8       __decode_pointer           1004afb8 f   LIBCMT:tidtable.obj
 0001:0004a02a       ___crtTlsAlloc@4           1004b02a f   LIBCMT:tidtable.obj
 0001:0004a033       ___set_flsgetvalue         1004b033 f   LIBCMT:tidtable.obj
 0001:0004a067       __mtterm                   1004b067 f   LIBCMT:tidtable.obj
 0001:0004a0a4       __initptd                  1004b0a4 f   LIBCMT:tidtable.obj
 0001:0004a18b       __getptd_noexit            1004b18b f   LIBCMT:tidtable.obj
 0001:0004a204       __getptd                   1004b204 f   LIBCMT:tidtable.obj
 0001:0004a21e       __freefls@4                1004b21e f   LIBCMT:tidtable.obj
 0001:0004a34d       __freeptd                  1004b34d f   LIBCMT:tidtable.obj
 0001:0004a3bb       __mtinit                   1004b3bb f   LIBCMT:tidtable.obj
 0001:0004a548       ?terminate@@YAXXZ          1004b548 f   LIBCMT:hooks.obj
 0001:0004a581       ?unexpected@@YAXXZ         1004b581 f   LIBCMT:hooks.obj
 0001:0004a594       ?_inconsistency@@YAXXZ     1004b594 f   LIBCMT:hooks.obj
 0001:0004a5cc       __initp_eh_hooks           1004b5cc f   LIBCMT:hooks.obj
 0001:0004a5e0       __CallSettingFrame@12      1004b5e0 f   LIBCMT:lowhelpr.obj
 0001:0004a607       __NLG_Return               1004b607     LIBCMT:lowhelpr.obj
 0001:0004a62c       ___report_gsfailure        1004b62c f   LIBCMT:gs_report.obj
 0001:0004a732       __forcdecpt_l              1004b732 f   LIBCMT:cvt.obj
 0001:0004a7a5       __cropzeros_l              1004b7a5 f   LIBCMT:cvt.obj
 0001:0004a827       __positive                 1004b827 f   LIBCMT:cvt.obj
 0001:0004a843       __fassign_l                1004b843 f   LIBCMT:cvt.obj
 0001:0004a885       __fassign                  1004b885 f   LIBCMT:cvt.obj
 0001:0004a8be       __forcdecpt                1004b8be f   LIBCMT:cvt.obj
 0001:0004a8d1       __cropzeros                1004b8d1 f   LIBCMT:cvt.obj
 0001:0004aa53       __cftoe_l                  1004ba53 f   LIBCMT:cvt.obj
 0001:0004ab23       __cftoe                    1004bb23 f   LIBCMT:cvt.obj
 0001:0004ab43       __cftoa_l                  1004bb43 f   LIBCMT:cvt.obj
 0001:0004afad       __cftof_l                  1004bfad f   LIBCMT:cvt.obj
 0001:0004b068       __cftog_l                  1004c068 f   LIBCMT:cvt.obj
 0001:0004b162       __cfltcvt_l                1004c162 f   LIBCMT:cvt.obj
 0001:0004b1ea       __cfltcvt                  1004c1ea f   LIBCMT:cvt.obj
 0001:0004b20d       __initp_misc_cfltcvt_tab   1004c20d f   LIBCMT:cmiscdat.obj
 0001:0004b22e       __setdefaultprecision      1004c22e f   LIBCMT:fp8.obj
 0001:0004b259       __ms_p5_test_fdiv          1004c259 f   LIBCMT:_testfdiv_.obj
 0001:0004b297       __ms_p5_mp_test_fdiv       1004c297 f   LIBCMT:_testfdiv_.obj
 0001:0004b2c0       ?_Type_info_dtor@type_info@@CAXPAV1@@Z 1004c2c0 f   LIBCMT:typname.obj
 0001:0004b330       _strcmp                    1004c330 f   LIBCMT:strcmp.obj
 0001:0004b3b8       __crt_debugger_hook        1004c3b8 f   LIBCMT:dbghook.obj
 0001:0004b3c0       _strcpy_s                  1004c3c0 f   LIBCMT:strcpy_s.obj
 0001:0004b428       __get_errno_from_oserr     1004c428 f   LIBCMT:dosmap.obj
 0001:0004b46a       __errno                    1004c46a f   LIBCMT:dosmap.obj
 0001:0004b47d       ___doserrno                1004c47d f   LIBCMT:dosmap.obj
 0001:0004b490       __dosmaperr                1004c490 f   LIBCMT:dosmap.obj
 0001:0004b6e2       _strtol                    1004c6e2 f   LIBCMT:strtol.obj
 0001:0004b9a4       __strtoi64                 1004c9a4 f   LIBCMT:strtoq.obj
 0001:0004bbf5       ___updatetmbcinfo          1004cbf5 f   LIBCMT:mbctype.obj
 0001:0004bd15       __setmbcp_nolock           1004cd15 f   LIBCMT:mbctype.obj
 0001:0004befa       __setmbcp                  1004cefa f   LIBCMT:mbctype.obj
 0001:0004c094       ___initmbctable            1004d094 f   LIBCMT:mbctype.obj
 0001:0004c0b2       ___freetlocinfo            1004d0b2 f   LIBCMT:setlocal.obj
 0001:0004c1fb       ___addlocaleref            1004d1fb f   LIBCMT:setlocal.obj
 0001:0004c28a       ___removelocaleref         1004d28a f   LIBCMT:setlocal.obj
 0001:0004c361       ___updatetlocinfo          1004d361 f   LIBCMT:setlocal.obj
 0001:0004c3d7       __tolower_l                1004d3d7 f   LIBCMT:tolower.obj
 0001:0004c4ec       _tolower                   1004d4ec f   LIBCMT:tolower.obj
 0001:0004c56f       __VEC_memzero              1004d56f f   LIBCMT:p4_memset.obj
 0001:0004c64e       __get_sse2_info            1004d64e f   LIBCMT:cpu_disp.obj
 0001:0004c6b0       ___sse2_available_init     1004d6b0 f   LIBCMT:cpu_disp.obj
 0001:0004c6bd       __close_nolock             1004d6bd f   LIBCMT:close.obj
 0001:0004c759       __close                    1004d759 f   LIBCMT:close.obj
 0001:0004c826       __fileno                   1004d826 f   LIBCMT:fileno.obj
 0001:0004c858       __freebuf                  1004d858 f   LIBCMT:_freebuf.obj
 0001:0004c889       __flush                    1004d889 f   LIBCMT:fflush.obj
 0001:0004c8f1       __fflush_nolock            1004d8f1 f   LIBCMT:fflush.obj
 0001:0004ca13       __flushall                 1004da13 f   LIBCMT:fflush.obj
 0001:0004ca1c       ___iob_func                1004da1c f   LIBCMT:_file.obj
 0001:0004ca22       ___initstdio               1004da22 f   LIBCMT:_file.obj
 0001:0004cad3       ___endstdio                1004dad3 f   LIBCMT:_file.obj
 0001:0004caf3       __lock_file                1004daf3 f   LIBCMT:_file.obj
 0001:0004cb34       __lock_file2               1004db34 f   LIBCMT:_file.obj
 0001:0004cb66       __unlock_file              1004db66 f   LIBCMT:_file.obj
 0001:0004cba2       __unlock_file2             1004dba2 f   LIBCMT:_file.obj
 0001:0004cbd4       __SEH_prolog4              1004dbd4 f   LIBCMT:sehprolg4.obj
 0001:0004cc19       __SEH_epilog4              1004dc19 f   LIBCMT:sehprolg4.obj
 0001:0004cc2d       __stbuf                    1004dc2d f   LIBCMT:_sftbuf.obj
 0001:0004ccc9       __ftbuf                    1004dcc9 f   LIBCMT:_sftbuf.obj
 0001:0004ccfd       __fwrite_nolock            1004dcfd f   LIBCMT:fwrite.obj
 0001:0004ce5f       __ioinit                   1004de5f f   LIBCMT:ioinit.obj
 0001:0004d0b3       __ioterm                   1004e0b3 f   LIBCMT:ioinit.obj
 0001:0004d101       __flsbuf                   1004e101 f   LIBCMT:_flsbuf.obj
 0001:0004d30b       __output_l                 1004e30b f   LIBCMT:output.obj
 0001:0004dea3       __openfile                 1004eea3 f   LIBCMT:_open.obj
 0001:0004e16c       __getstream                1004f16c f   LIBCMT:stream.obj
 0001:0004e2a4       __local_unwind4            1004f2a4 f   LIBCMT:exsup4.obj
 0001:0004e37a       __seh_longjmp_unwind4@4    1004f37a f   LIBCMT:exsup4.obj
 0001:0004e396       @_EH4_CallFilterFunc@8     1004f396 f   LIBCMT:exsup4.obj
 0001:0004e3ad       @_EH4_TransferToHandler@8  1004f3ad f   LIBCMT:exsup4.obj
 0001:0004e3c6       @_EH4_GlobalUnwind@4       1004f3c6 f   LIBCMT:exsup4.obj
 0001:0004e3e0       @_EH4_LocalUnwind@16       1004f3e0 f   LIBCMT:exsup4.obj
 0001:0004e3f7       __malloc_crt               1004f3f7 f   LIBCMT:crtheap.obj
 0001:0004e43c       __calloc_crt               1004f43c f   LIBCMT:crtheap.obj
 0001:0004e488       __realloc_crt              1004f488 f   LIBCMT:crtheap.obj
 0001:0004e4d6       __msize                    1004f4d6 f   LIBCMT:msize.obj
 0001:0004e579       __crt_waiting_on_module_handle 1004f579 f   LIBCMT:crt0dat.obj
 0001:0004e5a9       __amsg_exit                1004f5a9 f   LIBCMT:crt0dat.obj
 0001:0004e5d2       ___crtCorExitProcess       1004f5d2 f   LIBCMT:crt0dat.obj
 0001:0004e5fd       ___crtExitProcess          1004f5fd f   LIBCMT:crt0dat.obj
 0001:0004e615       __lockexit                 1004f615 f   LIBCMT:crt0dat.obj
 0001:0004e61e       __unlockexit               1004f61e f   LIBCMT:crt0dat.obj
 0001:0004e644       __initterm_e               1004f644 f   LIBCMT:crt0dat.obj
 0001:0004e668       __cinit                    1004f668 f   LIBCMT:crt0dat.obj
 0001:0004e819       __exit                     1004f819 f   LIBCMT:crt0dat.obj
 0001:0004e82f       __cexit                    1004f82f f   LIBCMT:crt0dat.obj
 0001:0004e83e       __init_pointers            1004f83e f   LIBCMT:crt0dat.obj
 0001:0004eb40       __wcstoi64                 1004fb40 f   LIBCMT:wcstoq.obj
 0001:0004ebf2       __VEC_memcpy               1004fbf2 f   LIBCMT:p4_memcpy.obj
 0001:0004ece0       __wfltin2                  1004fce0 f   LIBCMT:_wcfin_.obj
 0001:0004ed89       _wcslen                    1004fd89 f   LIBCMT:wcslen.obj
 0001:0004eda3       __iswctype_l               1004fda3 f   LIBCMT:iswctype.obj
 0001:0004eed5       __woutput_l                1004fed5 f   LIBCMT:woutput.obj
 0001:0004fa6d       ___crtLCMapStringW         10050a6d f   LIBCMT:w_map.obj
 0001:0004fac4       __wchartodigit             10050ac4 f   LIBCMT:wchtodig.obj
 0001:0004fc9f       __mtinitlocks              10050c9f f   LIBCMT:mlock.obj
 0001:0004fcea       __mtdeletelocks            10050cea f   LIBCMT:mlock.obj
 0001:0004fd41       __unlock                   10050d41 f   LIBCMT:mlock.obj
 0001:0004fd58       __mtinitlocknum            10050d58 f   LIBCMT:mlock.obj
 0001:0004fe1b       __lock                     10050e1b f   LIBCMT:mlock.obj
 0001:0004fe4e       __heap_init                10050e4e f   LIBCMT:heapinit.obj
 0001:0004fe7e       __heap_term                10050e7e f   LIBCMT:heapinit.obj
 0001:0004fef2       ___sbh_find_block          10050ef2 f   LIBCMT:sbheap.obj
 0001:0004ff22       ___sbh_free_block          10050f22 f   LIBCMT:sbheap.obj
 0001:00050238       ___sbh_alloc_new_region    10051238 f   LIBCMT:sbheap.obj
 0001:000502e8       ___sbh_alloc_new_group     100512e8 f   LIBCMT:sbheap.obj
 0001:000503f0       ___sbh_resize_block        100513f0 f   LIBCMT:sbheap.obj
 0001:000506d1       ___sbh_alloc_block         100516d1 f   LIBCMT:sbheap.obj
 0001:000509b6       __sse2_mathfcns_init       100519b6 f   LIBCMT:_mathfcns_.obj
 0001:000509d0       __CIcos_pentium4           100519d0 f   LIBCMT:_cos_pentium4_.obj
 0001:000509e8       __cos_pentium4             100519e8     LIBCMT:_cos_pentium4_.obj
 0001:00050b80       __trandisp1                10051b80 f   LIBCMT:_87disp_.obj
 0001:00050be7       __trandisp2                10051be7 f   LIBCMT:_87disp_.obj
 0001:00050c73       __rttospopde               10051c73     LIBCMT:_87disp_.obj
 0001:00050c78       __rttospop                 10051c78     LIBCMT:_87disp_.obj
 0001:00050c7a       __rtnospop                 10051c7a     LIBCMT:_87disp_.obj
 0001:00050c7c       __rttosnpop                10051c7c     LIBCMT:_87disp_.obj
 0001:00050c7d       __rtnospopde               10051c7d     LIBCMT:_87disp_.obj
 0001:00050c84       __rtzeropop                10051c84     LIBCMT:_87disp_.obj
 0001:00050c86       __rtzeronpop               10051c86     LIBCMT:_87disp_.obj
 0001:00050c8b       __rtonepop                 10051c8b     LIBCMT:_87disp_.obj
 0001:00050c8d       __rtonenpop                10051c8d     LIBCMT:_87disp_.obj
 0001:00050c92       __tosnan1                  10051c92     LIBCMT:_87disp_.obj
 0001:00050cbd       __nosnan2                  10051cbd     LIBCMT:_87disp_.obj
 0001:00050cbf       __tosnan2                  10051cbf     LIBCMT:_87disp_.obj
 0001:00050ce7       __nan2                     10051ce7     LIBCMT:_87disp_.obj
 0001:00050d26       __rtindfpop                10051d26     LIBCMT:_87disp_.obj
 0001:00050d28       __rtindfnpop               10051d28     LIBCMT:_87disp_.obj
 0001:00050d39       __rttosnpopde              10051d39     LIBCMT:_87disp_.obj
 0001:00050d43       __rtchsifneg               10051d43     LIBCMT:_87disp_.obj
 0001:00050d50       __twoToTOS                 10051d50 f   LIBCMT:_common_.obj
 0001:00050d65       __load_CW                  10051d65 f   LIBCMT:_common_.obj
 0001:00050d7c       __convertTOStoQNaN         10051d7c f   LIBCMT:_common_.obj
 0001:00050d95       __fload_withFB             10051d95 f   LIBCMT:_common_.obj
 0001:00050dd8       __checkTOS_withFB          10051dd8 f   LIBCMT:_common_.obj
 0001:00050dee       __fast_exit                10051dee f   LIBCMT:_common_.obj
 0001:00050dfb       __math_exit                10051dfb f   LIBCMT:_common_.obj
 0001:00050e25       __check_overflow_exit      10051e25 f   LIBCMT:_common_.obj
 0001:00050e39       __check_range_exit         10051e39 f   LIBCMT:_common_.obj
 0001:00050ee0       __startTwoArgErrorHandling 10051ee0 f   LIBCMT:_genexcep_.obj
 0001:00050ef7       __startOneArgErrorHandling 10051ef7 f   LIBCMT:_genexcep_.obj
 0001:00050f33       _abort                     10051f33 f   LIBCMT:abort.obj
 0001:0005104a       __set_abort_behavior       1005204a f   LIBCMT:abort.obj
 0001:0005106b       __NMSG_WRITE               1005206b f   LIBCMT:crt0msg.obj
 0001:00051216       __FF_MSGBANNER             10052216 f   LIBCMT:crt0msg.obj
 0001:0005124f       __initp_misc_purevirt      1005224f f   LIBCMT:inithelp.obj
 0001:0005125e       __setenvp                  1005225e f   LIBCMT:stdenvp.obj
 0001:000514d6       __setargv                  100524d6 f   LIBCMT:stdargv.obj
 0001:00051591       ___crtGetEnvironmentStringsA 10052591 f   LIBCMT:a_env.obj
 0001:000516c8       __RTC_Initialize           100526c8 f   LIBCMT:_initsect_.obj
 0001:000516ee       __RTC_Terminate            100526ee f   LIBCMT:_initsect_.obj
 0001:00051714       __initp_misc_winxfltr      10052714 f   LIBCMT:winxfltr.obj
 0001:00051714       __fpclear                  10052714 f   LIBCMT:_fpinit_.obj
 0001:00051715       __XcptFilter               10052715 f   LIBCMT:winxfltr.obj
 0001:00051875       ___CppXcptFilter           10052875 f   LIBCMT:winxfltr.obj
 0001:00051895       ___security_init_cookie    10052895 f   LIBCMT:gs_support.obj
 0001:00051930       __ValidateImageBase        10052930 f   LIBCMT:pesect.obj
 0001:00051970       __FindPESection            10052970 f   LIBCMT:pesect.obj
 0001:000519c0       __IsNonwritableInCurrentImage 100529c0 f   LIBCMT:pesect.obj
 0001:00051a80       __CIsin_pentium4           10052a80 f   LIBCMT:_sin_pentium4_.obj
 0001:00051a98       __sin_pentium4             10052a98     LIBCMT:_sin_pentium4_.obj
 0001:00051c50       __CIacos_pentium4          10052c50 f   LIBCMT:_acos_pentium4_.obj
 0001:00051c68       __acos_pentium4            10052c68     LIBCMT:_acos_pentium4_.obj
 0001:000521a4       ?_ValidateRead@@YAHPBXI@Z  100531a4 f   LIBCMT:validate.obj
 0001:000521a4       ?_ValidateWrite@@YAHPAXI@Z 100531a4 f   LIBCMT:validate.obj
 0001:000521a4       ?_ValidateExecute@@YAHP6GHXZ@Z 100531a4 f   LIBCMT:validate.obj
 0001:000521b8       __global_unwind2           100531b8 f   LIBCMT:exsup.obj
 0001:0005221d       __local_unwind2            1005321d f   LIBCMT:exsup.obj
 0001:000522a1       __abnormal_termination     100532a1 f   LIBCMT:exsup.obj
 0001:000522c4       __NLG_Notify1              100532c4 f   LIBCMT:exsup.obj
 0001:000522cd       __NLG_Notify               100532cd f   LIBCMT:exsup.obj
 0001:000522e4       __NLG_Dispatch             100532e4     LIBCMT:exsup.obj
 0001:000522e4       __NLG_Dispatch2            100532e4     LIBCMT:exsup.obj
 0001:000522ec       __NLG_Call                 100532ec f   LIBCMT:exsup.obj
 0001:000522ee       __NLG_Return2              100532ee     LIBCMT:exsup.obj
 0001:000522ef       __isdigit_l                100532ef f i LIBCMT:_ctype.obj
 0001:00052340       _isdigit                   10053340 f i LIBCMT:_ctype.obj
 0001:0005236e       __atodbl_l                 1005336e f   LIBCMT:atodbl.obj
 0001:00052416       __atoflt_l                 10053416 f   LIBCMT:atodbl.obj
 0001:000524be       __fptostr                  100534be f   LIBCMT:_fptostr.obj
 0001:0005257d       ___dtold                   1005357d f   LIBCMT:_cfout_.obj
 0001:0005263a       __fltout2                  1005363a f   LIBCMT:_cfout_.obj
 0001:000526d0       __alldvrm                  100536d0 f   LIBCMT:lldvrm.obj
 0001:000527b0       __aullshr                  100537b0 f   LIBCMT:ullshr.obj
 0001:000527cf       __fptrap                   100537cf f   LIBCMT:crt0fp.obj
 0001:000527d8       __controlfp_s              100537d8 f   LIBCMT:_contrlfp_.obj
 0001:00052844       __isctype_l                10053844 f   LIBCMT:isctype.obj
 0001:00052900       __allmul                   10053900 f   LIBCMT:llmul.obj
 0001:00052940       __aulldvrm                 10053940 f   LIBCMT:ulldvrm.obj
 0001:000529d5       __freea                    100539d5 f i LIBCMT:a_map.obj
 0001:00052d9a       ___crtLCMapStringA         10053d9a f   LIBCMT:a_map.obj
 0001:00052f99       ___crtGetStringTypeA       10053f99 f   LIBCMT:a_str.obj
 0001:00052fdb       ___free_lc_time            10053fdb f   LIBCMT:inittime.obj
 0001:00053170       ___free_lconv_num          10054170 f   LIBCMT:initnum.obj
 0001:000531b5       ___free_lconv_mon          100541b5 f   LIBCMT:initmon.obj
 0001:00053243       _strcat_s                  10054243 f   LIBCMT:strcat_s.obj
 0001:000532c0       _strcspn                   100542c0 f   LIBCMT:strcspn.obj
 0001:00053306       _strncpy_s                 10054306 f   LIBCMT:strncpy_s.obj
 0001:000533c0       _strpbrk                   100543c0 f   LIBCMT:strpbrk.obj
 0001:00053400       __isleadbyte_l             10054400 f i LIBCMT:_wctype.obj
 0001:00053438       _isleadbyte                10054438 f i LIBCMT:_wctype.obj
 0001:0005344b       __set_osfhnd               1005444b f   LIBCMT:osfinfo.obj
 0001:000534cc       __free_osfhnd              100544cc f   LIBCMT:osfinfo.obj
 0001:00053552       __get_osfhandle            10054552 f   LIBCMT:osfinfo.obj
 0001:000535c9       ___lock_fhandle            100545c9 f   LIBCMT:osfinfo.obj
 0001:00053669       __unlock_fhandle           10054669 f   LIBCMT:osfinfo.obj
 0001:00053690       __alloc_osfhnd             10054690 f   LIBCMT:osfinfo.obj
 0001:0005382a       __write_nolock             1005482a f   LIBCMT:write.obj
 0001:00053f5d       __write                    10054f5d f   LIBCMT:write.obj
 0001:00054039       __commit                   10055039 f   LIBCMT:commit.obj
 0001:0005411a       __fcloseall                1005511a f   LIBCMT:closeall.obj
 0001:000541b9       __isatty                   100551b9 f   LIBCMT:isatty.obj
 0001:0005421d       __initp_misc_initcrit      1005521d f   LIBCMT:initcrit.obj
 0001:0005422c       ___crtInitCritSecAndSpinCount 1005522c f   LIBCMT:initcrit.obj
 0001:0005428c       __lseeki64_nolock          1005528c f   LIBCMT:lseeki64.obj
 0001:00054311       __lseeki64                 10055311 f   LIBCMT:lseeki64.obj
 0001:0005442a       __getbuf                   1005542a f   LIBCMT:_getbuf.obj
 0001:00054473       __get_printf_count_output  10055473 f   LIBCMT:printf.obj
 0001:00054489       __wctomb_s_l               10055489 f   LIBCMT:wctomb.obj
 0001:000545f5       _wctomb_s                  100555f5 f   LIBCMT:wctomb.obj
 0001:00054d31       __sopen_helper             10055d31 f   LIBCMT:open.obj
 0001:00054dfd       __sopen_s                  10055dfd f   LIBCMT:open.obj
 0001:00054e1d       __mbsnbicmp_l              10055e1d f   LIBCMT:mbsnbicm.obj
 0001:00055048       __mbsnbicmp                10056048 f   LIBCMT:mbsnbicm.obj
 0001:00055062       __mbsnbcmp_l               10056062 f   LIBCMT:mbsnbcmp.obj
 0001:000551cc       __mbsnbcmp                 100561cc f   LIBCMT:mbsnbcmp.obj
 0001:000551e6       __calloc_impl              100561e6 f   LIBCMT:calloc_impl.obj
 0001:00055304       __initp_misc_winsig        10056304 f   LIBCMT:winsig.obj
 0001:00055359       ___get_sigabrt             10056359 f   LIBCMT:winsig.obj
 0001:00055366       _raise                     10056366 f   LIBCMT:winsig.obj
 0001:00055516       __initp_misc_rand_s        10056516 f   LIBCMT:rand_s.obj
 0001:00055525       __ld12tod                  10056525 f   LIBCMT:_intrncvt_.obj
 0001:00055a69       __ld12tof                  10056a69 f   LIBCMT:_intrncvt_.obj
 0001:00055fad       ___wstrgtold12_l           10056fad f   LIBCMT:_wstrgtold_.obj
 0001:00056709       ___crtGetStringTypeW       10057709 f   LIBCMT:w_str.obj
 0001:00056747       __fputwc_nolock            10057747 f   LIBCMT:fputwc.obj
 0001:000568ce       __mbtowc_l                 100578ce f   LIBCMT:mbtowc.obj
 0001:000569e5       _mbtowc                    100579e5 f   LIBCMT:mbtowc.obj
 0001:000569ff       __87except                 100579ff f   LIBCMT:_87except_.obj
 0001:00056b3e       ___crtMessageBoxA          10057b3e f   LIBCMT:crtmbox.obj
 0001:00056ca7       __set_error_mode           10057ca7 f   LIBCMT:errmode.obj
 0001:00056cf2       ___libm_error_support      10057cf2 f   LIBCMT:_libm_error_.obj
 0001:00056fa2       ___strgtold12_l            10057fa2 f   LIBCMT:_strgtold_.obj
 0001:0005769a       _$I10_OUTPUT               1005869a f   LIBCMT:_x10fout_.obj
 0001:000580ec       __control87                100590ec f i LIBCMT:_ieee87_.obj
 0001:000583fb       ___ansicp                  100593fb f   LIBCMT:convrtcp.obj
 0001:00058444       ___convertcp               10059444 f   LIBCMT:convrtcp.obj
 0001:00058600       __alloca_probe_16          10059600 f   LIBCMT:alloca16.obj
 0001:00058616       __alloca_probe_8           10059616     LIBCMT:alloca16.obj
 0001:0005862c       __strnicmp_l               1005962c f   LIBCMT:strnicmp.obj
 0001:0005871e       __strnicmp                 1005971e f   LIBCMT:strnicmp.obj
 0001:0005877c       __putwch_nolock            1005977c f   LIBCMT:putwch.obj
 0001:00058850       __chkstk                   10059850 f   LIBCMT:chkstk.obj
 0001:00058850       __alloca_probe             10059850     LIBCMT:chkstk.obj
 0001:0005887b       __chsize_nolock            1005987b f   LIBCMT:chsize.obj
 0001:00058a31       __read_nolock              10059a31 f   LIBCMT:read.obj
 0001:00058ff3       __lseek_nolock             10059ff3 f   LIBCMT:lseek.obj
 0001:00059068       __setmode_nolock           1005a068 f   LIBCMT:setmode.obj
 0001:00059124       __get_fmode                1005a124 f   LIBCMT:setmode.obj
 0001:0005915d       ___mtold12                 1005a15d f   LIBCMT:_mantold_.obj
 0001:0005932b       __flswbuf                  1005a32b f   LIBCMT:_flswbuf.obj
 0001:0005949f       __raise_exc_ex             1005a49f f   LIBCMT:_fpexcept_.obj
 0001:0005977b       __raise_exc                1005a77b f   LIBCMT:_fpexcept_.obj
 0001:0005979e       __handle_exc               1005a79e f   LIBCMT:_fpexcept_.obj
 0001:00059980       __set_errno_from_matherr   1005a980 f   LIBCMT:_fpexcept_.obj
 0001:000599ad       __matherr                  1005a9ad f   LIBCMT:_matherr_.obj
 0001:000599b0       __statfp                   1005a9b0 f   LIBCMT:_fpctrl_.obj
 0001:000599c0       __clrfp                    1005a9c0 f   LIBCMT:_fpctrl_.obj
 0001:000599d1       __ctrlfp                   1005a9d1 f   LIBCMT:_fpctrl_.obj
 0001:000599fa       __set_statfp               1005a9fa f   LIBCMT:_fpctrl_.obj
 0001:00059a52       ___set_fpsr_sse2           1005aa52 f   LIBCMT:_fpctrl_.obj
 0001:00059ad0       ___ascii_strnicmp          1005aad0 f   LIBCMT:_strnicm.obj
 0001:00059b31       ___initconout              1005ab31 f   LIBCMT:initcon.obj
 0001:00059b50       ___termcon                 1005ab50 f   LIBCMT:initcon.obj
 0001:00059b7d       __set_exp                  1005ab7d f   LIBCMT:_util_.obj
 0001:00059ba9       __decomp                   1005aba9 f   LIBCMT:_util_.obj
 0001:00059c80       _strchr                    1005ac80 f   LIBCMT:strchr.obj
 0001:00059c86       ___from_strstr_to_strchr   1005ac86     LIBCMT:strchr.obj
 0001:00059d40       ??1CAutoFree@@QAE@XZ       1005ad40 f   wzFilePacker_static:wzFilePacker.obj
 0001:00059d50       ?CONVERT_PATHCHAR@CPackFile@@CAXPAD@Z 1005ad50 f i wzFilePacker_static:wzFilePacker.obj
 0001:00059db0       ??0CPackFile@@QAE@XZ       1005adb0 f   wzFilePacker_static:wzFilePacker.obj
 0001:00059de0       ?Close@CPackFile@@QAEXXZ   1005ade0 f   wzFilePacker_static:wzFilePacker.obj
 0001:00059e00       ?OpenFile@CPackFile@@QAEPAXPBDK@Z 1005ae00 f   wzFilePacker_static:wzFilePacker.obj
 0001:00059e30       ?FileExists@CPackFile@@QAEHPBD@Z 1005ae30 f   wzFilePacker_static:wzFilePacker.obj
 0001:00059e50       ?DeleteFileA@CPackFile@@QAEHPBD@Z 1005ae50 f   wzFilePacker_static:wzFilePacker.obj
 0001:00059e50       ?RemoveDirectoryA@CPackFile@@QAEHPBD@Z 1005ae50 f   wzFilePacker_static:wzFilePacker.obj
 0001:00059e70       ?CreateDirectoryA@CPackFile@@QAEHPBD@Z 1005ae70 f   wzFilePacker_static:wzFilePacker.obj
 0001:00059ea0       ?CloseFile@CPackFile@@QAEXPAX@Z 1005aea0 f   wzFilePacker_static:wzFilePacker.obj
 0001:00059eb0       ?GetFileProperties@CPackFile@@QAEHPAXPAUFileProperties@@@Z 1005aeb0 f   wzFilePacker_static:wzFilePacker.obj
 0001:00059f60       ?ReadFile@CPackFile@@QAEHPAX0K@Z 1005af60 f   wzFilePacker_static:wzFilePacker.obj
 0001:00059f80       ?WriteFile@CPackFile@@QAEHPAXPBXK@Z 1005af80 f   wzFilePacker_static:wzFilePacker.obj
 0001:00059fa0       ?GetFileSize@CPackFile@@QAEHPAXPA_K@Z 1005afa0 f   wzFilePacker_static:wzFilePacker.obj
 0001:00059fb0       ?GetFilePointer@CPackFile@@QAEHPAXPA_K@Z 1005afb0 f   wzFilePacker_static:wzFilePacker.obj
 0001:00059fc0       ?SetFilePointer@CPackFile@@QAEHPAX_KK@Z 1005afc0 f   wzFilePacker_static:wzFilePacker.obj
 0001:00059fe0       ?AddFile@CPackFile@@QAEHPBD0@Z 1005afe0 f   wzFilePacker_static:wzFilePacker.obj
 0001:0005a0f0       ??1CPackFile@@QAE@XZ       1005b0f0 f   wzFilePacker_static:wzFilePacker.obj
 0001:0005a100       ?Open@CPackFile@@QAEPAXPBD0K@Z 1005b100 f   wzFilePacker_static:wzFilePacker.obj
 0001:0005a220       @geVFile_CloseAPI@0        1005b220 f   wzFilePacker_static:vfile.obj
 0001:0005a2e0       @geVFile_Open_Detail@20    1005b2e0 f   wzFilePacker_static:vfile.obj
 0001:0005a3d0       @geVFile_Open@12           1005b3d0 f   wzFilePacker_static:vfile.obj
 0001:0005a4c0       @geVFile_DeleteFile@8      1005b4c0 f   wzFilePacker_static:vfile.obj
 0001:0005a4d0       @geVFile_FileExists@8      1005b4d0 f   wzFilePacker_static:vfile.obj
 0001:0005a4e0       @geVFile_Close@4           1005b4e0 f   wzFilePacker_static:vfile.obj
 0001:0005a530       @geVFile_GetS@12           1005b530 f   wzFilePacker_static:vfile.obj
 0001:0005a550       @geVFile_Read@12           1005b550 f   wzFilePacker_static:vfile.obj
 0001:0005a580       @geVFile_Write@12          1005b580 f   wzFilePacker_static:vfile.obj
 0001:0005a5b0       @geVFile_Seek@16           1005b5b0 f   wzFilePacker_static:vfile.obj
 0001:0005a5d0       @geVFile_Tell@8            1005b5d0 f   wzFilePacker_static:vfile.obj
 0001:0005a5e0       @geVFile_Size@8            1005b5e0 f   wzFilePacker_static:vfile.obj
 0001:0005a5f0       @geVFile_GetProperties@8   1005b5f0 f   wzFilePacker_static:vfile.obj
 0001:0005a600       @geVFile_EnlargeDirectorySize@8 1005b600 f   wzFilePacker_static:vfile.obj
 0001:0005a610       @geVFile_SetVersion@8      1005b610 f   wzFilePacker_static:vfile.obj
 0001:0005a620       @geVFile_IsPrevVersion@4   1005b620 f   wzFilePacker_static:vfile.obj
 0001:0005a630       @geVFile_OpenNewSystem@20  1005b630 f   wzFilePacker_static:vfile.obj
 0001:0005a770       _CopyVFile                 1005b770 f   wzFilePacker_static:vFile_util.obj
 0001:0005a8e0       _CopyOneFile               1005b8e0 f   wzFilePacker_static:vFile_util.obj
 0001:0005a960       _MakeDirectory             1005b960 f   wzFilePacker_static:vFile_util.obj
 0001:0005aa50       _geRam_Allocate            1005ba50 f   wzFilePacker_static:Ram.obj
 0001:0005aa70       _geRam_Free_               1005ba70 f   wzFilePacker_static:Ram.obj
 0001:0005aa80       _geRam_Realloc             1005ba80 f   wzFilePacker_static:Ram.obj
 0001:0005aae0       _Encrypt                   1005bae0 f   wzFilePacker_static:fsvfs.obj
 0001:0005ab20       _Decrypt                   1005bb20 f   wzFilePacker_static:fsvfs.obj
 0001:0005c500       @FSVFS_GetAPIs@0           1005d500 f   wzFilePacker_static:fsvfs.obj
 0001:0005ccb0       @FSMemory_GetAPIs@0        1005dcb0 f   wzFilePacker_static:FSMEMORY.obj
 0001:0005d940       @FSDos_GetAPIs@0           1005e940 f   wzFilePacker_static:fsdos.obj
 0001:0005d950       _DirTree_Create            1005e950 f   wzFilePacker_static:dirtree.obj
 0001:0005d9a0       _DirTree_Destroy           1005e9a0 f   wzFilePacker_static:dirtree.obj
 0001:0005dc40       _DirTree_SetFileSize       1005ec40 f   wzFilePacker_static:dirtree.obj
 0001:0005dc60       _DirTree_GetFileSize       1005ec60 f   wzFilePacker_static:dirtree.obj
 0001:0005dc80       _DirTree_WriteToFile       1005ec80 f   wzFilePacker_static:dirtree.obj
 0001:0005dcb0       _DirTree_GetSize           1005ecb0 f   wzFilePacker_static:dirtree.obj
 0001:0005e0d0       _DirTree_CreateFromFile    1005f0d0 f   wzFilePacker_static:dirtree.obj
 0001:0005e450       _DirTree_FindExact         1005f450 f   wzFilePacker_static:dirtree.obj
 0001:0005e4b0       _DirTree_FindPartial       1005f4b0 f   wzFilePacker_static:dirtree.obj
 0001:0005e530       _DirTree_AddFile           1005f530 f   wzFilePacker_static:dirtree.obj
 0001:0005e600       _DirTree_Remove            1005f600 f   wzFilePacker_static:dirtree.obj
 0001:0005e690       _DirTree_SetFileAttributes 1005f690 f   wzFilePacker_static:dirtree.obj
 0001:0005e6b0       _DirTree_GetFileAttributes 1005f6b0 f   wzFilePacker_static:dirtree.obj
 0001:0005e6c0       _DirTree_SetFileOffset     1005f6c0 f   wzFilePacker_static:dirtree.obj
 0001:0005e6e0       _DirTree_GetFileOffset     1005f6e0 f   wzFilePacker_static:dirtree.obj
 0001:0005e700       _DirTree_SetFileTime       1005f700 f   wzFilePacker_static:dirtree.obj
 0001:0005e720       _DirTree_GetFileTime       1005f720 f   wzFilePacker_static:dirtree.obj
 0001:0005e740       _DirTree_SetFileHints      1005f740 f   wzFilePacker_static:dirtree.obj
 0001:0005e7b0       _DirTree_GetFileHints      1005f7b0 f   wzFilePacker_static:dirtree.obj
 0001:0005e7d0       _DirTree_GetName           1005f7d0 f   wzFilePacker_static:dirtree.obj
 0001:0005e810       _DirTree_FileExists        1005f810 f   wzFilePacker_static:dirtree.obj
 0001:0005e830       _DirTree_CreateFinder      1005f830 f   wzFilePacker_static:dirtree.obj
 0001:0005e960       _DirTree_DestroyFinder     1005f960 f   wzFilePacker_static:dirtree.obj
 0001:0005e9a0       _DirTree_FinderGetNextFile 1005f9a0 f   wzFilePacker_static:dirtree.obj
 0001:0005ea60       _DirTree_SetAllFileOffset  1005fa60 f   wzFilePacker_static:dirtree.obj
 0001:0005eb10       _DuplicateString           1005fb10 f   wzFilePacker_static:dirtree-common.obj
 0001:0005eb50       _GetNextDir                1005fb50 f   wzFilePacker_static:dirtree-common.obj
 0001:0005eb80       _MatchPattern              1005fb80 f   wzFilePacker_static:dirtree-common.obj
 0001:0005ebe0       _PathHasDir                1005fbe0 f   wzFilePacker_static:dirtree-common.obj
 0001:0005ec00       ?_com_issue_error@@YGXJ@Z  1005fc00 f   comsuppw:comsupp.obj
 0001:0005ec20       ?_com_issue_errorex@@YGXJPAUIUnknown@@ABU_GUID@@@Z 1005fc20 f   comsuppw:comsupp.obj
 0001:0005eca0       ??1_com_error@@UAE@XZ      1005fca0 f i comsuppw:comraise.obj
 0001:0005ece0       ?_com_raise_error@@YGXJPAUIErrorInfo@@@Z 1005fce0 f   comsuppw:comraise.obj
 0001:0005ed20       ??0_com_error@@QAE@ABV0@@Z 1005fd20 f i comsuppw:comraise.obj
 0001:0005ed60       ??_G_com_error@@UAEPAXI@Z  1005fd60 f i comsuppw:comraise.obj
 0001:0005ed60       ??_E_com_error@@UAEPAXI@Z  1005fd60 f i comsuppw:comraise.obj
 0001:0005edb0       _RtlUnwind@16              1005fdb0 f   kernel32:KERNEL32.dll
 0001:0005edb6       __mbsstr_l                 1005fdb6 f   LIBCMT:mbsstr.obj
 0001:0005eef7       __mbsstr                   1005fef7 f   LIBCMT:mbsstr.obj
 0001:0005ef10       _memchr                    1005ff10 f   LIBCMT:memchr.obj
 0001:0005f1af       __splitpath                100601af f   LIBCMT:splitpat.obj
 0001:0005f200       _strstr                    10060200 f   LIBCMT:strstr.obj
 0001:0005f286       __mbsnbcpy_s               10060286 f   LIBCMT:mbsnbcpy_s.obj
 0001:0005f2a3       __mbsnbcpy_s_l             100602a3 f   LIBCMT:mbsnbcpy_s_l.obj
 0002:00000000       __imp_?GetNumberOfDefaultFont@CManagerText@@QAEHXZ 10062000     3drendererd3d:3DRendererD3D.dll
 0002:00000004       __imp_?SaveExtendedFontInfo@CManagerText@@QAEHPBD@Z 10062004     3drendererd3d:3DRendererD3D.dll
 0002:00000008       __imp_?LoadExtendedFontInfo@CManagerText@@QAEHPBDE@Z 10062008     3drendererd3d:3DRendererD3D.dll
 0002:0000000c       __imp_?GetExtendedFontInfo@CManagerText@@QAEHHPAUSt_FontMake@@@Z 1006200c     3drendererd3d:3DRendererD3D.dll
 0002:00000010       __imp_?GetNumberOfExtendedFont@CManagerText@@QAEHXZ 10062010     3drendererd3d:3DRendererD3D.dll
 0002:00000014       __imp_?DeleteAllExtendedFont@CManagerText@@QAEXXZ 10062014     3drendererd3d:3DRendererD3D.dll
 0002:00000018       __imp_?DeleteExtendedFont@CManagerText@@QAEHK@Z 10062018     3drendererd3d:3DRendererD3D.dll
 0002:0000001c       __imp_?AddExtendedFont@CManagerText@@QAEHKHHPBDEEEPAUtagLOGFONTA@@@Z 1006201c     3drendererd3d:3DRendererD3D.dll
 0002:00000020       __imp_?GetFontInfo@CManagerText@@QAEHHPAUSt_FontMake@@@Z 10062020     3drendererd3d:3DRendererD3D.dll
 0002:00000024       __imp_?GetFontInfoWzID@CManagerText@@QAEHKPAUSt_FontMake@@@Z 10062024     3drendererd3d:3DRendererD3D.dll
 0002:00000028       __imp_?GetFontDCByWzID@CManagerText@@QAEPAUHDC__@@K@Z 10062028     3drendererd3d:3DRendererD3D.dll
 0002:0000002c       __imp_?GetTextExtentPointW@CManagerText@@QAEXPB_WHPAUtagSIZE@@@Z 1006202c     3drendererd3d:3DRendererD3D.dll
 0002:00000030       __imp_?GetTextExtentPointA@CManagerText@@QAEXPBDHPAUtagSIZE@@@Z 10062030     3drendererd3d:3DRendererD3D.dll
 0002:00000034       __imp_?DrawTextA@CManagerText@@QAEXPBDHHKKKH@Z 10062034     3drendererd3d:3DRendererD3D.dll
 0002:00000038       __imp_?EndUseFont@CManagerText@@QAEXXZ 10062038     3drendererd3d:3DRendererD3D.dll
 0002:0000003c       __imp_?StartToUseFont@CManagerText@@QAEHK@Z 1006203c     3drendererd3d:3DRendererD3D.dll
 0002:00000040       \1773DRendererD3D_NULL_THUNK_DATA 10062040     3drendererd3d:3DRendererD3D.dll
 0002:00000044       __imp__RegQueryValueExA@24 10062044     advapi32:ADVAPI32.dll
 0002:00000048       __imp__RegOpenKeyExW@20    10062048     advapi32:ADVAPI32.dll
 0002:0000004c       __imp__RegQueryValueExW@24 1006204c     advapi32:ADVAPI32.dll
 0002:00000050       __imp__RegCloseKey@4       10062050     advapi32:ADVAPI32.dll
 0002:00000054       __imp__RegOpenKeyExA@20    10062054     advapi32:ADVAPI32.dll
 0002:00000058       \177ADVAPI32_NULL_THUNK_DATA 10062058     advapi32:ADVAPI32.dll
 0002:0000005c       __imp__GetTextExtentPoint32A@16 1006205c     gdi32:GDI32.dll
 0002:00000060       __imp__GetPixel@12         10062060     gdi32:GDI32.dll
 0002:00000064       __imp__SetPixel@16         10062064     gdi32:GDI32.dll
 0002:00000068       __imp__CreateCompatibleDC@4 10062068     gdi32:GDI32.dll
 0002:0000006c       __imp__CreateDIBSection@24 1006206c     gdi32:GDI32.dll
 0002:00000070       __imp__GetBkMode@4         10062070     gdi32:GDI32.dll
 0002:00000074       __imp__SetBkMode@8         10062074     gdi32:GDI32.dll
 0002:00000078       __imp__DeleteDC@4          10062078     gdi32:GDI32.dll
 0002:0000007c       __imp__SelectObject@8      1006207c     gdi32:GDI32.dll
 0002:00000080       __imp__DeleteObject@4      10062080     gdi32:GDI32.dll
 0002:00000084       __imp__CreateFontIndirectA@4 10062084     gdi32:GDI32.dll
 0002:00000088       \177GDI32_NULL_THUNK_DATA  10062088     gdi32:GDI32.dll
 0002:0000008c       __imp__GetFileSizeEx@8     1006208c     kernel32:KERNEL32.dll
 0002:00000090       __imp__SetFilePointerEx@20 10062090     kernel32:KERNEL32.dll
 0002:00000094       __imp__FindNextFileA@8     10062094     kernel32:KERNEL32.dll
 0002:00000098       __imp__lstrcpyA@8          10062098     kernel32:KERNEL32.dll
 0002:0000009c       __imp__lstrlenA@4          1006209c     kernel32:KERNEL32.dll
 0002:000000a0       __imp__SetEndOfFile@4      100620a0     kernel32:KERNEL32.dll
 0002:000000a4       __imp__WriteConsoleW@20    100620a4     kernel32:KERNEL32.dll
 0002:000000a8       __imp__GetConsoleOutputCP@0 100620a8     kernel32:KERNEL32.dll
 0002:000000ac       __imp__WriteConsoleA@20    100620ac     kernel32:KERNEL32.dll
 0002:000000b0       __imp__InitializeCriticalSectionAndSpinCount@8 100620b0     kernel32:KERNEL32.dll
 0002:000000b4       __imp__FlushFileBuffers@4  100620b4     kernel32:KERNEL32.dll
 0002:000000b8       __imp__GetConsoleMode@8    100620b8     kernel32:KERNEL32.dll
 0002:000000bc       __imp__GetConsoleCP@0      100620bc     kernel32:KERNEL32.dll
 0002:000000c0       __imp__SetStdHandle@8      100620c0     kernel32:KERNEL32.dll
 0002:000000c4       __imp__SetFileAttributesA@8 100620c4     kernel32:KERNEL32.dll
 0002:000000c8       __imp__GetStringTypeW@16   100620c8     kernel32:KERNEL32.dll
 0002:000000cc       __imp__HeapAlloc@12        100620cc     kernel32:KERNEL32.dll
 0002:000000d0       __imp__LCMapStringA@24     100620d0     kernel32:KERNEL32.dll
 0002:000000d4       __imp__GetSystemTimeAsFileTime@4 100620d4     kernel32:KERNEL32.dll
 0002:000000d8       __imp__GetCurrentProcessId@0 100620d8     kernel32:KERNEL32.dll
 0002:000000dc       __imp__QueryPerformanceCounter@4 100620dc     kernel32:KERNEL32.dll
 0002:000000e0       __imp__GetEnvironmentStringsW@0 100620e0     kernel32:KERNEL32.dll
 0002:000000e4       __imp__FreeEnvironmentStringsW@4 100620e4     kernel32:KERNEL32.dll
 0002:000000e8       __imp__GetEnvironmentStrings@0 100620e8     kernel32:KERNEL32.dll
 0002:000000ec       __imp__FreeEnvironmentStringsA@4 100620ec     kernel32:KERNEL32.dll
 0002:000000f0       __imp__VirtualAlloc@16     100620f0     kernel32:KERNEL32.dll
 0002:000000f4       __imp__VirtualFree@12      100620f4     kernel32:KERNEL32.dll
 0002:000000f8       __imp__HeapDestroy@4       100620f8     kernel32:KERNEL32.dll
 0002:000000fc       __imp__HeapCreate@12       100620fc     kernel32:KERNEL32.dll
 0002:00000100       __imp__LCMapStringW@24     10062100     kernel32:KERNEL32.dll
 0002:00000104       __imp__ExitProcess@4       10062104     kernel32:KERNEL32.dll
 0002:00000108       __imp__HeapSize@12         10062108     kernel32:KERNEL32.dll
 0002:0000010c       __imp__Sleep@4             1006210c     kernel32:KERNEL32.dll
 0002:00000110       __imp__SetFileTime@16      10062110     kernel32:KERNEL32.dll
 0002:00000114       __imp__GetFileAttributesA@4 10062114     kernel32:KERNEL32.dll
 0002:00000118       __imp__MoveFileA@8         10062118     kernel32:KERNEL32.dll
 0002:0000011c       __imp__GetLocalTime@4      1006211c     kernel32:KERNEL32.dll
 0002:00000120       __imp__InterlockedDecrement@4 10062120     kernel32:KERNEL32.dll
 0002:00000124       __imp__WinExec@8           10062124     kernel32:KERNEL32.dll
 0002:00000128       __imp__GetVersionExA@4     10062128     kernel32:KERNEL32.dll
 0002:0000012c       __imp__lstrcmpiA@8         1006212c     kernel32:KERNEL32.dll
 0002:00000130       __imp__IsDBCSLeadByteEx@8  10062130     kernel32:KERNEL32.dll
 0002:00000134       __imp__GetVersionExW@4     10062134     kernel32:KERNEL32.dll
 0002:00000138       __imp__LoadLibraryA@4      10062138     kernel32:KERNEL32.dll
 0002:0000013c       __imp__CompareStringA@24   1006213c     kernel32:KERNEL32.dll
 0002:00000140       __imp__lstrcpyW@8          10062140     kernel32:KERNEL32.dll
 0002:00000144       __imp__GetLocaleInfoW@16   10062144     kernel32:KERNEL32.dll
 0002:00000148       __imp__GetLocaleInfoA@16   10062148     kernel32:KERNEL32.dll
 0002:0000014c       __imp__GetProcessHeap@0    1006214c     kernel32:KERNEL32.dll
 0002:00000150       __imp__GetStartupInfoA@4   10062150     kernel32:KERNEL32.dll
 0002:00000154       __imp__GetFileType@4       10062154     kernel32:KERNEL32.dll
 0002:00000158       __imp__GetStdHandle@4      10062158     kernel32:KERNEL32.dll
 0002:0000015c       __imp__SetHandleCount@4    1006215c     kernel32:KERNEL32.dll
 0002:00000160       __imp__IsValidCodePage@4   10062160     kernel32:KERNEL32.dll
 0002:00000164       __imp__GetOEMCP@0          10062164     kernel32:KERNEL32.dll
 0002:00000168       __imp__GetACP@0            10062168     kernel32:KERNEL32.dll
 0002:0000016c       __imp__GetCPInfo@8         1006216c     kernel32:KERNEL32.dll
 0002:00000170       __imp__GetModuleHandleA@4  10062170     kernel32:KERNEL32.dll
 0002:00000174       __imp__HeapFree@12         10062174     kernel32:KERNEL32.dll
 0002:00000178       __imp__lstrcatW@8          10062178     kernel32:KERNEL32.dll
 0002:0000017c       __imp__FreeLibrary@4       1006217c     kernel32:KERNEL32.dll
 0002:00000180       __imp__GetSystemDirectoryW@8 10062180     kernel32:KERNEL32.dll
 0002:00000184       __imp__LoadLibraryExW@12   10062184     kernel32:KERNEL32.dll
 0002:00000188       __imp__GetProcAddress@8    10062188     kernel32:KERNEL32.dll
 0002:0000018c       __imp__lstrlenW@4          1006218c     kernel32:KERNEL32.dll
 0002:00000190       __imp__GetNumberFormatA@24 10062190     kernel32:KERNEL32.dll
 0002:00000194       __imp__GlobalAlloc@8       10062194     kernel32:KERNEL32.dll
 0002:00000198       __imp__GlobalLock@4        10062198     kernel32:KERNEL32.dll
 0002:0000019c       __imp__GlobalUnlock@4      1006219c     kernel32:KERNEL32.dll
 0002:000001a0       __imp__GlobalFree@4        100621a0     kernel32:KERNEL32.dll
 0002:000001a4       __imp__GetTickCount@0      100621a4     kernel32:KERNEL32.dll
 0002:000001a8       __imp__WideCharToMultiByte@32 100621a8     kernel32:KERNEL32.dll
 0002:000001ac       __imp__MultiByteToWideChar@24 100621ac     kernel32:KERNEL32.dll
 0002:000001b0       __imp__OutputDebugStringA@4 100621b0     kernel32:KERNEL32.dll
 0002:000001b4       __imp__GetStringTypeA@20   100621b4     kernel32:KERNEL32.dll
 0002:000001b8       __imp__SetLastError@4      100621b8     kernel32:KERNEL32.dll
 0002:000001bc       __imp__GetModuleFileNameA@12 100621bc     kernel32:KERNEL32.dll
 0002:000001c0       __imp__InitializeCriticalSection@4 100621c0     kernel32:KERNEL32.dll
 0002:000001c4       __imp__DeleteCriticalSection@4 100621c4     kernel32:KERNEL32.dll
 0002:000001c8       __imp__EnterCriticalSection@4 100621c8     kernel32:KERNEL32.dll
 0002:000001cc       __imp__LeaveCriticalSection@4 100621cc     kernel32:KERNEL32.dll
 0002:000001d0       __imp__CreateFileA@28      100621d0     kernel32:KERNEL32.dll
 0002:000001d4       __imp__CloseHandle@4       100621d4     kernel32:KERNEL32.dll
 0002:000001d8       __imp__SetFilePointer@16   100621d8     kernel32:KERNEL32.dll
 0002:000001dc       __imp__ReadFile@20         100621dc     kernel32:KERNEL32.dll
 0002:000001e0       __imp__WriteFile@20        100621e0     kernel32:KERNEL32.dll
 0002:000001e4       __imp__FindClose@4         100621e4     kernel32:KERNEL32.dll
 0002:000001e8       __imp__FindFirstFileA@8    100621e8     kernel32:KERNEL32.dll
 0002:000001ec       __imp__GetFileSize@8       100621ec     kernel32:KERNEL32.dll
 0002:000001f0       __imp__GetFileInformationByHandle@8 100621f0     kernel32:KERNEL32.dll
 0002:000001f4       __imp__CopyFileA@12        100621f4     kernel32:KERNEL32.dll
 0002:000001f8       __imp__DeleteFileA@4       100621f8     kernel32:KERNEL32.dll
 0002:000001fc       __imp__CreateDirectoryA@8  100621fc     kernel32:KERNEL32.dll
 0002:00000200       __imp__RemoveDirectoryA@4  10062200     kernel32:KERNEL32.dll
 0002:00000204       __imp__RtlUnwind@16        10062204     kernel32:KERNEL32.dll
 0002:00000208       __imp__RaiseException@16   10062208     kernel32:KERNEL32.dll
 0002:0000020c       __imp__TerminateProcess@8  1006220c     kernel32:KERNEL32.dll
 0002:00000210       __imp__GetCurrentProcess@0 10062210     kernel32:KERNEL32.dll
 0002:00000214       __imp__UnhandledExceptionFilter@4 10062214     kernel32:KERNEL32.dll
 0002:00000218       __imp__SetUnhandledExceptionFilter@4 10062218     kernel32:KERNEL32.dll
 0002:0000021c       __imp__IsDebuggerPresent@0 1006221c     kernel32:KERNEL32.dll
 0002:00000220       __imp__GetLastError@0      10062220     kernel32:KERNEL32.dll
 0002:00000224       __imp__HeapReAlloc@16      10062224     kernel32:KERNEL32.dll
 0002:00000228       __imp__GetCurrentThreadId@0 10062228     kernel32:KERNEL32.dll
 0002:0000022c       __imp__GetCommandLineA@0   1006222c     kernel32:KERNEL32.dll
 0002:00000230       __imp__GetModuleHandleW@4  10062230     kernel32:KERNEL32.dll
 0002:00000234       __imp__TlsGetValue@4       10062234     kernel32:KERNEL32.dll
 0002:00000238       __imp__TlsAlloc@0          10062238     kernel32:KERNEL32.dll
 0002:0000023c       __imp__TlsSetValue@8       1006223c     kernel32:KERNEL32.dll
 0002:00000240       __imp__TlsFree@4           10062240     kernel32:KERNEL32.dll
 0002:00000244       __imp__InterlockedIncrement@4 10062244     kernel32:KERNEL32.dll
 0002:00000248       \177KERNEL32_NULL_THUNK_DATA 10062248     kernel32:KERNEL32.dll
 0002:0000024c       __imp__SysAllocString@4    1006224c     oleaut32:OLEAUT32.dll
 0002:00000250       __imp__VariantInit@4       10062250     oleaut32:OLEAUT32.dll
 0002:00000254       __imp__SysFreeString@4     10062254     oleaut32:OLEAUT32.dll
 0002:00000258       __imp__VariantClear@4      10062258     oleaut32:OLEAUT32.dll
 0002:0000025c       __imp__GetErrorInfo@8      1006225c     oleaut32:OLEAUT32.dll
 0002:00000260       \177OLEAUT32_NULL_THUNK_DATA 10062260     oleaut32:OLEAUT32.dll
 0002:00000264       __imp__OffsetRect@12       10062264     user32:USER32.dll
 0002:00000268       __imp__ClientToScreen@8    10062268     user32:USER32.dll
 0002:0000026c       __imp__GetWindowRect@8     1006226c     user32:USER32.dll
 0002:00000270       __imp__UpdateWindow@4      10062270     user32:USER32.dll
 0002:00000274       __imp__ShowWindow@8        10062274     user32:USER32.dll
 0002:00000278       __imp__GetCursor@0         10062278     user32:USER32.dll
 0002:0000027c       __imp__LoadCursorA@8       1006227c     user32:USER32.dll
 0002:00000280       __imp__SetCursor@4         10062280     user32:USER32.dll
 0002:00000284       __imp__GetWindowTextLengthA@4 10062284     user32:USER32.dll
 0002:00000288       __imp__GetParent@4         10062288     user32:USER32.dll
 0002:0000028c       __imp__ReleaseCapture@0    1006228c     user32:USER32.dll
 0002:00000290       __imp__SetFocus@4          10062290     user32:USER32.dll
 0002:00000294       __imp__SetWindowTextA@8    10062294     user32:USER32.dll
 0002:00000298       __imp__GetWindowTextA@12   10062298     user32:USER32.dll
 0002:0000029c       __imp__PostMessageA@16     1006229c     user32:USER32.dll
 0002:000002a0       __imp__IsWindowEnabled@4   100622a0     user32:USER32.dll
 0002:000002a4       __imp__CallWindowProcA@20  100622a4     user32:USER32.dll
 0002:000002a8       __imp__GetCaretPos@4       100622a8     user32:USER32.dll
 0002:000002ac       __imp__DestroyWindow@4     100622ac     user32:USER32.dll
 0002:000002b0       __imp__MoveWindow@24       100622b0     user32:USER32.dll
 0002:000002b4       __imp__GetSysColor@4       100622b4     user32:USER32.dll
 0002:000002b8       __imp__GetClientRect@8     100622b8     user32:USER32.dll
 0002:000002bc       __imp__CreateWindowExA@48  100622bc     user32:USER32.dll
 0002:000002c0       __imp__SendMessageA@16     100622c0     user32:USER32.dll
 0002:000002c4       __imp__SetWindowLongA@12   100622c4     user32:USER32.dll
 0002:000002c8       __imp__GetDC@4             100622c8     user32:USER32.dll
 0002:000002cc       __imp__ReleaseDC@8         100622cc     user32:USER32.dll
 0002:000002d0       __imp__GetWindowLongA@8    100622d0     user32:USER32.dll
 0002:000002d4       __imp__PeekMessageW@20     100622d4     user32:USER32.dll
 0002:000002d8       __imp__GetMessageW@16      100622d8     user32:USER32.dll
 0002:000002dc       __imp__PostQuitMessage@4   100622dc     user32:USER32.dll
 0002:000002e0       __imp__TranslateMessage@4  100622e0     user32:USER32.dll
 0002:000002e4       __imp__DispatchMessageA@4  100622e4     user32:USER32.dll
 0002:000002e8       __imp__GetKeyboardLayout@4 100622e8     user32:USER32.dll
 0002:000002ec       __imp__keybd_event@16      100622ec     user32:USER32.dll
 0002:000002f0       __imp__PtInRect@12         100622f0     user32:USER32.dll
 0002:000002f4       __imp__GetKeyboardLayoutList@8 100622f4     user32:USER32.dll
 0002:000002f8       __imp__SendMessageW@16     100622f8     user32:USER32.dll
 0002:000002fc       __imp__GetAsyncKeyState@4  100622fc     user32:USER32.dll
 0002:00000300       __imp__GetFocus@0          10062300     user32:USER32.dll
 0002:00000304       __imp__PostMessageW@16     10062304     user32:USER32.dll
 0002:00000308       __imp__GetKeyState@4       10062308     user32:USER32.dll
 0002:0000030c       __imp__GetClipboardData@4  1006230c     user32:USER32.dll
 0002:00000310       __imp__OpenClipboard@4     10062310     user32:USER32.dll
 0002:00000314       __imp__EmptyClipboard@0    10062314     user32:USER32.dll
 0002:00000318       __imp__SetClipboardData@8  10062318     user32:USER32.dll
 0002:0000031c       __imp__CloseClipboard@0    1006231c     user32:USER32.dll
 0002:00000320       __imp__SetRect@20          10062320     user32:USER32.dll
 0002:00000324       __imp__IntersectRect@12    10062324     user32:USER32.dll
 0002:00000328       __imp__wsprintfA           10062328     user32:USER32.dll
 0002:0000032c       \177USER32_NULL_THUNK_DATA 1006232c     user32:USER32.dll
 0002:00000330       __imp__CoUninitialize@0    10062330     ole32:ole32.dll
 0002:00000334       __imp__CoInitialize@4      10062334     ole32:ole32.dll
 0002:00000338       __imp__CoCreateInstance@20 10062338     ole32:ole32.dll
 0002:0000033c       \177ole32_NULL_THUNK_DATA  1006233c     ole32:ole32.dll
 0002:00000340       ___xc_a                    10062340     LIBCMT:crt0init.obj
 0002:00000358       ___xc_z                    10062358     LIBCMT:crt0init.obj
 0002:0000035c       ___xi_a                    1006235c     LIBCMT:crt0init.obj
 0002:00000374       ___xi_z                    10062374     LIBCMT:crt0init.obj
 0002:00000378       ___xp_a                    10062378     LIBCMT:crt0init.obj
 0002:00000384       ___xp_z                    10062384     LIBCMT:crt0init.obj
 0002:00000388       ___xt_a                    10062388     LIBCMT:crt0init.obj
 0002:0000038c       ___xt_z                    1006238c     LIBCMT:crt0init.obj
 0002:000003ac       ??_C@_0P@GHFPNOJB@bad?5allocation?$AA@ 100623ac     stdafx.obj
 0002:000003c0       ??_7CBaseManager@@6B@      100623c0     BaseManager.obj
 0002:000003d4       __real@40800000            100623d4     BaseManager.obj
 0002:000003dc       ??_7length_error@std@@6B@  100623dc     BaseManager.obj
 0002:000003e4       ??_C@_0BB@MOGOBHAF@list?$DMT?$DO?5too?5long?$AA@ 100623e4     BaseManager.obj
 0002:000003f8       ??_C@_0BD@OLBABOEK@vector?$DMT?$DO?5too?5long?$AA@ 100623f8     BaseManager.obj
 0002:00000410       ??_7bad_alloc@std@@6B@     10062410     BaseManager.obj
 0002:00000418       ?npos@?$basic_string@DU?$char_traits@D@std@@V?$allocator@D@2@@std@@2IB 10062418     BaseManager.obj
 0002:00000420       ??_7logic_error@std@@6B@   10062420     BaseManager.obj
 0002:00000428       ??_C@_03JBJLGPFL@end?$AA@  10062428     StringManager.obj
 0002:0000042c       ??_C@_05FAGFPHJG@start?$AA@ 1006242c     StringManager.obj
 0002:00000434       ??_C@_06FKNHHIAI@?$CFd?7?$CFs?6?$AA@ 10062434     StringManager.obj
 0002:0000043c       ??_C@_06ODNDLLAM@start?6?$AA@ 1006243c     StringManager.obj
 0002:00000444       ??_C@_02BKFDOEMK@wt?$AA@   10062444     StringManager.obj
 0002:00000447       ??_C@_00CNPNBAHC@?$AA@     10062447     StringManager.obj
 0002:00000448       ??_C@_05OINFJHGD@?$CFI64u?$AA@ 10062448     ControlWZ.obj
 0002:00000450       ??_C@_01LFCBOECM@?4?$AA@   10062450     ControlWZ.obj
 0002:00000454       ??_C@_01IHBHIGKO@?0?$AA@   10062454     ControlWZ.obj
 0002:00000458       __real@3f800000            10062458     ControlWZ.obj
 0002:00000464       ??_7CControlWZ@@6B@        10062464     ControlWZ.obj
 0002:000005d8       __real@3f847ae140000000    100625d8     ControlWZ.obj
 0002:000005e0       __real@0000000000000000    100625e0     ControlWZ.obj
 0002:000005e8       __real@4008000000000000    100625e8     ControlWZ.obj
 0002:000005f0       __real@3ff0000000000000    100625f0     ControlWZ.obj
 0002:000005f8       ??_C@_08FLJNNHMK@ver?4r2?43?$AA@ 100625f8     ControlWZ.obj
 0002:00000604       ??_C@_08ECIGOGIL@ver?4r2?42?$AA@ 10062604     ControlWZ.obj
 0002:00000610       ??_C@_08BPHCNPKC@ver?4r1?45?$AA@ 10062610     ControlWZ.obj
 0002:0000061c       ??_C@_08HLBOBKKG@ver?4r1?41?$AA@ 1006261c     ControlWZ.obj
 0002:00000628       ??_C@_08LONFIJIG@ver?4r0?44?$AA@ 10062628     ControlWZ.obj
 0002:00000634       ??_C@_08GJKLLFEI@ver?4r2?41?$AA@ 10062634     ControlWZ.obj
 0002:00000640       ??_C@_08LHLPHML@ver?4r0?49?$AA@ 10062640     ControlWZ.obj
 0002:0000064c       ??_C@_08BCGAMGIK@ver?4r0?48?$AA@ 1006264c     ControlWZ.obj
 0002:00000658       ??_C@_08FADDEJGF@ver?4r1?42?$AA@ 10062658     ControlWZ.obj
 0002:00000664       ??_C@_0BL@NEHNAACP@HANDLE?5?$CL?5?$CFd?5?0?5FILE?5NAME?5?$DN?5?$AA@ 10062664     ControlWZ.obj
 0002:00000680       ??_C@_05OKCMKDO@?$CFI64i?$AA@ 10062680     ControlWZ.obj
 0002:0000068c       ??_7CCtrlButtonCheckWZ@@6B@ 1006268c     CtrlButtonCheckWZ.obj
 0002:00000814       ??_7CCtrlButtonWZ@@6B@     10062814     CtrlButtonWZ.obj
 0002:0000098c       ??_C@_08GGJOOOD@ver?4r1?44?$AA@ 1006298c     CtrlButtonWZ.obj
 0002:00000998       ??_C@_08DEFPIMGB@ver?4r1?46?$AA@ 10062998     CtrlButtonWZ.obj
 0002:000009a4       ??_C@_08EJCIHICE@ver?4r1?43?$AA@ 100629a4     CtrlButtonWZ.obj
 0002:000009b4       ??_7CCtrlClientWZ@@6B@     100629b4     CtrlClientWZ.obj
 0002:00000b24       __real@43c80000            10062b24     CtrlClientWZ.obj
 0002:00000b2c       ??_7CCtrlComboBoxWZ@@6B@   10062b2c     CtrlComboBox.obj
 0002:00000ca4       ??_7CCtrlDxEditBox@@6B@    10062ca4     CtrlDxEdit.obj
 0002:00000ebc       ??_7CCtrlBaseEdit@@6B@     10062ebc     CtrlDxEdit.obj
 0002:000010b0       ??_C@_1M@CKDELIOF@?$AA?$CF?$AA?4?$AA4?$AAf?$AA?5?$AA?$AA@ 100630b0     CtrlDxEdit.obj
 0002:000010bc       ??_C@_0BI@NIMEAFDJ@ScriptString_pcOutChars?$AA@ 100630bc     CtrlDxEdit.obj
 0002:000010d4       ??_C@_0BG@ENNDDIIO@ScriptString_pLogAttr?$AA@ 100630d4     CtrlDxEdit.obj
 0002:000010ec       ??_C@_0BB@KPJJNIOI@ScriptStringFree?$AA@ 100630ec     CtrlDxEdit.obj
 0002:00001100       ??_C@_0BC@PBCEOCLL@ScriptStringXtoCP?$AA@ 10063100     CtrlDxEdit.obj
 0002:00001114       ??_C@_0BC@NCOCHMDF@ScriptStringCPtoX?$AA@ 10063114     CtrlDxEdit.obj
 0002:00001128       ??_C@_0BE@DPDJMHJ@ScriptStringAnalyse?$AA@ 10063128     CtrlDxEdit.obj
 0002:0000113c       ??_C@_0BN@GIMDAPPD@ScriptApplyDigitSubstitution?$AA@ 1006313c     CtrlDxEdit.obj
 0002:0000115c       ??_C@_1BG@OAEOGKPD@?$AA?2?$AAu?$AAs?$AAp?$AA1?$AA0?$AA?4?$AAd?$AAl?$AAl?$AA?$AA@ 1006315c     CtrlDxEdit.obj
 0002:00001174       ??_C@_0BI@FKDAHLLJ@GetFileVersionInfoSizeA?$AA@ 10063174     CtrlDxEdit.obj
 0002:0000118c       ??_C@_0BE@JIHADGJK@GetFileVersionInfoA?$AA@ 1006318c     CtrlDxEdit.obj
 0002:000011a0       ??_C@_0P@EGBPEC@VerQueryValueA?$AA@ 100631a0     CtrlDxEdit.obj
 0002:000011b0       ??_C@_1BK@INCDNACE@?$AA?2?$AAv?$AAe?$AAr?$AAs?$AAi?$AAo?$AAn?$AA?4?$AAd?$AAl?$AAl?$AA?$AA@ 100631b0     CtrlDxEdit.obj
 0002:000011cc       ??_C@_0BI@LCGEKKLJ@ImmSetCompositionWindow?$AA@ 100631cc     CtrlDxEdit.obj
 0002:000011e4       ??_C@_0P@KLJNOAPA@ImmGetProperty?$AA@ 100631e4     CtrlDxEdit.obj
 0002:000011f4       ??_C@_08EPDNLFJN@ImmIsIME?$AA@ 100631f4     CtrlDxEdit.obj
 0002:00001200       ??_C@_0BC@OMCMFCHK@ImmSimulateHotKey?$AA@ 10063200     CtrlDxEdit.obj
 0002:00001214       ??_C@_0BH@MCPHEKIJ@ImmSetConversionStatus?$AA@ 10063214     CtrlDxEdit.obj
 0002:0000122c       ??_C@_0N@OLIMKHEA@ImmNotifyIME?$AA@ 1006322c     CtrlDxEdit.obj
 0002:0000123c       ??_C@_0BB@CEHHIDO@ImmGetVirtualKey?$AA@ 1006323c     CtrlDxEdit.obj
 0002:00001250       ??_C@_0BD@GDCNBOJF@ImmGetIMEFileNameA?$AA@ 10063250     CtrlDxEdit.obj
 0002:00001264       ??_C@_0BE@LPNAGBML@ImmGetDefaultIMEWnd?$AA@ 10063264     CtrlDxEdit.obj
 0002:00001278       ??_C@_0BH@GMNMAKPF@ImmGetConversionStatus?$AA@ 10063278     CtrlDxEdit.obj
 0002:00001290       ??_C@_0BB@BPOEGBEM@ImmSetOpenStatus?$AA@ 10063290     CtrlDxEdit.obj
 0002:000012a4       ??_C@_0BB@GAPKNCDL@ImmGetOpenStatus?$AA@ 100632a4     CtrlDxEdit.obj
 0002:000012b8       ??_C@_0BE@BDEIBNIK@ImmAssociateContext?$AA@ 100632b8     CtrlDxEdit.obj
 0002:000012cc       ??_C@_0BC@OCDKEPCD@ImmReleaseContext?$AA@ 100632cc     CtrlDxEdit.obj
 0002:000012e0       ??_C@_0O@KCHCFLMC@ImmGetContext?$AA@ 100632e0     CtrlDxEdit.obj
 0002:000012f0       ??_C@_0BF@INEDHPDK@ImmGetCandidateListW?$AA@ 100632f0     CtrlDxEdit.obj
 0002:00001308       ??_C@_0BJ@BIPOEMOA@ImmGetCompositionStringW?$AA@ 10063308     CtrlDxEdit.obj
 0002:00001324       ??_C@_0BL@MBEANDFB@ImmDisableTextFrameService?$AA@ 10063324     CtrlDxEdit.obj
 0002:00001340       ??_C@_0O@GKKOACL@ImmUnlockIMCC?$AA@ 10063340     CtrlDxEdit.obj
 0002:00001350       ??_C@_0M@OKKMJOGM@ImmLockIMCC?$AA@ 10063350     CtrlDxEdit.obj
 0002:0000135c       ??_C@_0N@PDIACEGP@ImmUnlockIMC?$AA@ 1006335c     CtrlDxEdit.obj
 0002:0000136c       ??_C@_0L@JGAMEFKO@ImmLockIMC?$AA@ 1006336c     CtrlDxEdit.obj
 0002:00001378       ??_C@_1BG@GAIJEFJ@?$AA?2?$AAi?$AAm?$AAm?$AA3?$AA2?$AA?4?$AAd?$AAl?$AAl?$AA?$AA@ 10063378     CtrlDxEdit.obj
 0002:00001394       ??_7CCtrlDxIMEEditBox@@6B@ 10063394     CtrlDxEdit.obj
 0002:000015b8       ??_C@_17GMPJMPF@?$AA?$CF?$AAs?$AA?5?$AA?$AA@ 100635b8     CtrlDxEdit.obj
 0002:000015c0       ??_C@_0L@GDMMIPKL@WINABC?4IME?$AA@ 100635c0     CtrlDxEdit.obj
 0002:000015cc       ??_C@_11LOCGONAA@?$AA?$AA@ 100635cc     CtrlDxEdit.obj
 0002:000015d0       ??_C@_01KICIPPFI@?2?$AA@   100635d0     CtrlDxEdit.obj
 0002:000015d4       ??_C@_0M@FEMOABAL@IMSC40W?4IME?$AA@ 100635d4     CtrlDxEdit.obj
 0002:000015e0       ??_C@_0N@ONOBNHOE@MSSCIPYA?4IME?$AA@ 100635e0     CtrlDxEdit.obj
 0002:000015f0       ??_C@_0N@JFHOELJF@PINTLGNT?4IME?$AA@ 100635f0     CtrlDxEdit.obj
 0002:00001600       ??_C@_0N@FHDFFBN@MSTCIPHA?4IME?$AA@ 10063600     CtrlDxEdit.obj
 0002:00001610       ??_C@_0N@JMLDIBIB@CINTLGNT?4IME?$AA@ 10063610     CtrlDxEdit.obj
 0002:00001620       ??_C@_0N@FFMHCBAD@TINTLGNT?4IME?$AA@ 10063620     CtrlDxEdit.obj
 0002:00001630       ??_C@_0BC@MEELNKEC@ShowReadingWindow?$AA@ 10063630     CtrlDxEdit.obj
 0002:00001644       ??_C@_0BB@EOIFCLLM@GetReadingString?$AA@ 10063644     CtrlDxEdit.obj
 0002:00001658       ??_C@_1CC@HJCBBEFJ@?$AAK?$AAe?$AAy?$AAb?$AAo?$AAa?$AAr?$AAd?$AA?5?$AAM?$AAa?$AAp?$AAp?$AAi?$AAn?$AAg?$AA?$AA@ 10063658     CtrlDxEdit.obj
 0002:0000167c       ??_C@_1BC@JHNLCPNJ@?$AAT?$AAI?$AAN?$AAT?$AAL?$AAG?$AAN?$AAT?$AA?$AA@ 1006367c     CtrlDxEdit.obj
 0002:00001690       ??_C@_1BA@EBBGJCHM@?$AAM?$AAS?$AAT?$AAC?$AAI?$AAP?$AAH?$AA?$AA@ 10063690     CtrlDxEdit.obj
 0002:000016a0       ??_C@_1FG@NAFBOIDA@?$AAs?$AAo?$AAf?$AAt?$AAw?$AAa?$AAr?$AAe?$AA?2?$AAm?$AAi?$AAc?$AAr?$AAo?$AAs?$AAo?$AAf?$AAt?$AA?2?$AAw?$AAi?$AAn?$AAd?$AAo?$AAw?$AAs?$AA?2?$AAc?$AAu?$AAr?$AAr?$AAe@ 100636a0     CtrlDxEdit.obj
 0002:000016fc       ??_7CCtrlMultilineEditWZ@@6B@ 100636fc     CtrlDxEdit.obj
 0002:00001984       __real@41a00000            10063984     CtrlDxEdit.obj
 0002:00001988       ??_C@_0BC@FMIJHMEI@Microsoft?5Win32s?6?$AA@ 10063988     CtrlEditWZ.obj
 0002:0000199c       ??_C@_0CG@EFLJMGJD@Microsoft?5Windows?5Millennium?5Edi@ 1006399c     CtrlEditWZ.obj
 0002:000019c4       ??_C@_03OENGOLCG@SE?5?$AA@ 100639c4     CtrlEditWZ.obj
 0002:000019c8       ??_C@_0BG@HILLGFCM@Microsoft?5Windows?598?5?$AA@ 100639c8     CtrlEditWZ.obj
 0002:000019e0       ??_C@_05BMOPIBIL@OSR2?5?$AA@ 100639e0     CtrlEditWZ.obj
 0002:000019e8       ??_C@_0BG@HAGDPGHP@Microsoft?5Windows?595?5?$AA@ 100639e8     CtrlEditWZ.obj
 0002:00001a00       ??_C@_08IANGBJF@SERVERNT?$AA@ 10063a00     CtrlEditWZ.obj
 0002:00001a0c       ??_C@_08NJBOKIMK@LANMANNT?$AA@ 10063a0c     CtrlEditWZ.obj
 0002:00001a18       ??_C@_0N@CNBBDHIF@Workstation?5?$AA@ 10063a18     CtrlEditWZ.obj
 0002:00001a28       ??_C@_05NFENELLP@WINNT?$AA@ 10063a28     CtrlEditWZ.obj
 0002:00001a30       ??_C@_0M@GGPOPAAP@ProductType?$AA@ 10063a30     CtrlEditWZ.obj
 0002:00001a3c       ??_C@_0DA@NKLICLFP@SYSTEM?2CurrentControlSet?2Control@ 10063a3c     CtrlEditWZ.obj
 0002:00001a6c       ??_C@_0M@NOLKAJHO@Server?54?40?5?$AA@ 10063a6c     CtrlEditWZ.obj
 0002:00001a78       ??_C@_0CA@CPILAOML@Server?54?40?0?5Enterprise?5Edition?5?$AA@ 10063a78     CtrlEditWZ.obj
 0002:00001a98       ??_C@_07GGILJBPJ@Server?5?$AA@ 10063a98     CtrlEditWZ.obj
 0002:00001aa0       ??_C@_0BB@BIAFMEFO@Advanced?5Server?5?$AA@ 10063aa0     CtrlEditWZ.obj
 0002:00001ab4       ??_C@_0BD@CMGHKCOJ@Datacenter?5Server?5?$AA@ 10063ab4     CtrlEditWZ.obj
 0002:00001ac8       ??_C@_0BC@IGDCANHF@Standard?5Edition?5?$AA@ 10063ac8     CtrlEditWZ.obj
 0002:00001adc       ??_C@_0N@BNPFCBGM@Web?5Edition?5?$AA@ 10063adc     CtrlEditWZ.obj
 0002:00001aec       ??_C@_0BE@NLEGHPDC@Enterprise?5Edition?5?$AA@ 10063aec     CtrlEditWZ.obj
 0002:00001b00       ??_C@_0BE@GKJIIJAP@Datacenter?5Edition?5?$AA@ 10063b00     CtrlEditWZ.obj
 0002:00001b14       ??_C@_0O@HLCCHGCK@Professional?5?$AA@ 10063b14     CtrlEditWZ.obj
 0002:00001b24       ??_C@_0O@MDJHKKNB@Home?5Edition?5?$AA@ 10063b24     CtrlEditWZ.obj
 0002:00001b34       ??_C@_0BB@EIAGMNAA@Workstation?54?40?5?$AA@ 10063b34     CtrlEditWZ.obj
 0002:00001b48       ??_C@_0BG@MPJOMPEN@Microsoft?5Windows?5NT?5?$AA@ 10063b48     CtrlEditWZ.obj
 0002:00001b60       ??_C@_0BI@LPKIKLGN@Microsoft?5Windows?52000?5?$AA@ 10063b60     CtrlEditWZ.obj
 0002:00001b78       ??_C@_0BG@LNOFGPNC@Microsoft?5Windows?5XP?5?$AA@ 10063b78     CtrlEditWZ.obj
 0002:00001b90       ??_C@_0CL@JEJIPKKK@Microsoft?5Windows?5Server?$CGnbsp?$DL20@ 10063b90     CtrlEditWZ.obj
 0002:00001bbc       ??_C@_06JIODDOFH@System?$AA@ 10063bbc     CtrlEditWZ.obj
 0002:00001bcc       ??_7CCtrlEditWZ@@6B@       10063bcc     CtrlEditWZ.obj
 0002:00001dc4       ??_C@_0BF@DCGMNAMN@Microsoft?5Windows?595?$AA@ 10063dc4     CtrlEditWZ.obj
 0002:00001ddc       ??_C@_04BBNPPDNC@Edit?$AA@ 10063ddc     CtrlEditWZ.obj
 0002:00001dec       ??_7CCtrlHScrollWZ@@6B@    10063dec     CtrlHScrollWZ.obj
 0002:00001fe0       __real@4059000000000000    10063fe0     CtrlHScrollWZ.obj
 0002:00001fec       ??_7CCtrlListWZ@@6B@       10063fec     CtrlListWZ.obj
 0002:00002248       __real@4014000000000000    10064248     CtrlListWZ.obj
 0002:00002250       ??_C@_02DPKJAMEF@?$CFd?$AA@ 10064250     CtrlListWZ.obj
 0002:00002258       ??_7out_of_range@std@@6B@  10064258     CtrlListWZ.obj
 0002:00002260       ??_C@_0BM@PAPJHAGI@invalid?5map?1set?$DMT?$DO?5iterator?$AA@ 10064260     CtrlListWZ.obj
 0002:0000227c       ??_C@_0BE@JONHPENG@map?1set?$DMT?$DO?5too?5long?$AA@ 1006427c     CtrlListWZ.obj
 0002:00002294       ??_7CCtrlPictureWZ@@6B@    10064294     CtrlPictureWZ.obj
 0002:00002420       __real@3fe0000000000000    10064420     CtrlPictureWZ.obj
 0002:00002428       __real@409f400000000000    10064428     CtrlPictureWZ.obj
 0002:00002430       __real@400921fb60000000    10064430     CtrlPictureWZ.obj
 0002:0000243c       ??_7CCtrlRectangleWZ@@6B@  1006443c     CtrlRectangleWZ.obj
 0002:000025cc       ??_7CCtrlStaticWZ@@6B@     100645cc     CtrlStaticWZ.obj
 0002:00002744       ??_C@_04CIENKOH@SMAL?$AA@  10064744     CtrlStaticWZ.obj
 0002:00002754       ??_7CCtrlImageStaticWZ@@6B@ 10064754     CtrlStaticWZ.obj
 0002:000028cc       __real@3f400000            100648cc     CtrlTabWZ.obj
 0002:000028d4       ??_7CCtrlTabWZ@@6B@        100648d4     CtrlTabWZ.obj
 0002:00002a98       __real@4000000000000000    10064a98     CtrlTabWZ.obj
 0002:00002aa0       __real@40400000            10064aa0     CtrlTabWZ.obj
 0002:00002aa4       __real@40a00000            10064aa4     CtrlTabWZ.obj
 0002:00002aa8       __real@40000000            10064aa8     CtrlTabWZ.obj
 0002:00002ab0       __real@4010000000000000    10064ab0     CtrlTabWZ.obj
 0002:00002ac0       __mask@@NegFloat@          10064ac0     CtrlTabWZ.obj
 0002:00002ad0       __real@3f4ccccd            10064ad0     CtrlTabWZ.obj
 0002:00002ad4       __real@3f2aaaab            10064ad4     CtrlTabWZ.obj
 0002:00002ad8       __real@3f000000            10064ad8     CtrlTabWZ.obj
 0002:00002ae4       ??_7CCtrlVScrollWZ@@6B@    10064ae4     CtrlVScrollWZ.obj
 0002:00002cd4       ??_C@_06JBKGCNBB@Delete?$AA@ 10064cd4     CtrlWebBrowserWZ.obj
 0002:00002cdc       ??_C@_08KAAPDIAN@NoRemove?$AA@ 10064cdc     CtrlWebBrowserWZ.obj
 0002:00002ce8       ??_C@_0M@DBGDLGLL@ForceRemove?$AA@ 10064ce8     CtrlWebBrowserWZ.obj
 0002:00002cf4       ??_C@_03LAIAPFCB@Val?$AA@  10064cf4     CtrlWebBrowserWZ.obj
 0002:00002cf8       ??_C@_01HMGJMAIH@B?$AA@    10064cf8     CtrlWebBrowserWZ.obj
 0002:00002cfc       ??_C@_01CKDDGHAB@D?$AA@    10064cfc     CtrlWebBrowserWZ.obj
 0002:00002d00       ??_C@_01PLPBNMEI@M?$AA@    10064d00     CtrlWebBrowserWZ.obj
 0002:00002d04       ??_C@_01CPLAODJH@S?$AA@    10064d04     CtrlWebBrowserWZ.obj
 0002:00002d28       _CLSID_CWithWebDialog      10064d28     CtrlWebBrowserWZ.obj
 0002:00002d38       _IID_IWithWebDialog        10064d38     CtrlWebBrowserWZ.obj
 0002:00002d4c       ??_7CCtrlWebBrowserWZ@@6B@ 10064d4c     CtrlWebBrowserWZ.obj
 0002:00002ed4       ??_C@_0BG@LIILJHBG@regsvr32?5?1s?5dlgwb?4dll?$AA@ 10064ed4     CtrlWebBrowserWZ.obj
 0002:00002eec       ??_C@_0BJ@OFMHLPBK@regsvr32?5?1u?5?1s?5dlgwb?4dll?$AA@ 10064eec     CtrlWebBrowserWZ.obj
 0002:00002f08       __GUID_0581a268_ebe1_4b95_8cee_c81a44f99a8f 10064f08     CtrlWebBrowserWZ.obj
 0002:00002f1c       ??_7CDialogWZ@@6B@         10064f1c     DialogWZ.obj
 0002:00002fd8       __real@43f00000            10064fd8     DialogWZ.obj
 0002:00002fdc       __real@43a10000            10064fdc     DialogWZ.obj
 0002:00002fe0       ??_C@_08HALAIEAJ@ver?4r2?40?$AA@ 10064fe0     DialogWZ.obj
 0002:00002ff0       ??_7CDlgBaseWZ@@6B@        10064ff0     DlgBaseWZ.obj
 0002:00003004       ??_C@_0M@GCLLLGON@yellowgreen?$AA@ 10065004     Color.obj
 0002:00003010       ??_C@_06ENJNJKEL@yellow?$AA@ 10065010     Color.obj
 0002:00003018       ??_C@_0L@FDFMBGNF@whitesmoke?$AA@ 10065018     Color.obj
 0002:00003024       ??_C@_05PMAELIEO@white?$AA@ 10065024     Color.obj
 0002:0000302c       ??_C@_05PPOGEFHN@wheat?$AA@ 1006502c     Color.obj
 0002:00003034       ??_C@_06KNANIGBM@violet?$AA@ 10065034     Color.obj
 0002:0000303c       ??_C@_09LFBHPEAP@turquoise?$AA@ 1006503c     Color.obj
 0002:00003048       ??_C@_06NALDPNEI@tomato?$AA@ 10065048     Color.obj
 0002:00003050       ??_C@_07CGANODJO@thistle?$AA@ 10065050     Color.obj
 0002:00003058       ??_C@_04LJCKMMGA@teal?$AA@ 10065058     Color.obj
 0002:00003060       ??_C@_03IIINPABG@tan?$AA@  10065060     Color.obj
 0002:00003064       ??_C@_09EKEFGALI@steelblue?$AA@ 10065064     Color.obj
 0002:00003070       ??_C@_0M@IPKJFOEB@springgreen?$AA@ 10065070     Color.obj
 0002:0000307c       ??_C@_04HPKDHBOB@snow?$AA@ 1006507c     Color.obj
 0002:00003084       ??_C@_09LKMPLBLE@slategray?$AA@ 10065084     Color.obj
 0002:00003090       ??_C@_09DPLBEIJJ@slateblue?$AA@ 10065090     Color.obj
 0002:0000309c       ??_C@_07MFCMKLDM@skyblue?$AA@ 1006509c     Color.obj
 0002:000030a4       ??_C@_06NBGLMDBG@silver?$AA@ 100650a4     Color.obj
 0002:000030ac       ??_C@_06CEGMHAGE@sienna?$AA@ 100650ac     Color.obj
 0002:000030b4       ??_C@_08MFJLKPPC@seashell?$AA@ 100650b4     Color.obj
 0002:000030c0       ??_C@_08EKGLDJFB@seagreen?$AA@ 100650c0     Color.obj
 0002:000030cc       ??_C@_0L@HLMGLGHH@sandybrown?$AA@ 100650cc     Color.obj
 0002:000030d8       ??_C@_06FBMAEJGO@salmon?$AA@ 100650d8     Color.obj
 0002:000030e0       ??_C@_0M@MOEGEDCP@saddlebrown?$AA@ 100650e0     Color.obj
 0002:000030ec       ??_C@_09FEEJNHFN@royalblue?$AA@ 100650ec     Color.obj
 0002:000030f8       ??_C@_09DJJHENIF@rosybrown?$AA@ 100650f8     Color.obj
 0002:00003104       ??_C@_03FAAAOPJM@red?$AA@  10065104     Color.obj
 0002:00003108       ??_C@_06GEHONCEN@purple?$AA@ 10065108     Color.obj
 0002:00003110       ??_C@_0L@MNADNFAH@powderblue?$AA@ 10065110     Color.obj
 0002:0000311c       ??_C@_04DDJGBPMH@plum?$AA@ 1006511c     Color.obj
 0002:00003124       ??_C@_04ECGBAEOC@pink?$AA@ 10065124     Color.obj
 0002:0000312c       ??_C@_04MJMKNOJB@peru?$AA@ 1006512c     Color.obj
 0002:00003134       ??_C@_09GELOGGEC@peachpuff?$AA@ 10065134     Color.obj
 0002:00003140       ??_C@_0L@NPJMDDDD@papayawhip?$AA@ 10065140     Color.obj
 0002:0000314c       ??_C@_0O@IPAPGMGK@palevioletred?$AA@ 1006514c     Color.obj
 0002:0000315c       ??_C@_0O@LCPHEOND@paleturquoise?$AA@ 1006515c     Color.obj
 0002:0000316c       ??_C@_09NAJHJFNO@palegreen?$AA@ 1006516c     Color.obj
 0002:00003178       ??_C@_0O@KONOLMEH@palegoldenrod?$AA@ 10065178     Color.obj
 0002:00003188       ??_C@_06DPBADMDK@orchid?$AA@ 10065188     Color.obj
 0002:00003190       ??_C@_09OPJMLMBK@orangered?$AA@ 10065190     Color.obj
 0002:0000319c       ??_C@_06HDDOCMMN@orange?$AA@ 1006519c     Color.obj
 0002:000031a4       ??_C@_09CNLBGLAE@olivedrab?$AA@ 100651a4     Color.obj
 0002:000031b0       ??_C@_05OFIFEKBG@olive?$AA@ 100651b0     Color.obj
 0002:000031b8       ??_C@_07MBCGBJON@oldlace?$AA@ 100651b8     Color.obj
 0002:000031c0       ??_C@_04DCMEIHPF@navy?$AA@ 100651c0     Color.obj
 0002:000031c8       ??_C@_0M@OKLAMJCL@navajowhite?$AA@ 100651c8     Color.obj
 0002:000031d4       ??_C@_08OIIPPDDA@moccasin?$AA@ 100651d4     Color.obj
 0002:000031e0       ??_C@_09HABDAMOF@mistyrose?$AA@ 100651e0     Color.obj
 0002:000031ec       ??_C@_09INCGBEJA@mintcream?$AA@ 100651ec     Color.obj
 0002:000031f8       ??_C@_0N@PJDKAOHK@midnightblue?$AA@ 100651f8     Color.obj
 0002:00003208       ??_C@_0BA@PNNCDMHM@mediumvioletred?$AA@ 10065208     Color.obj
 0002:00003218       ??_C@_0BA@MACKBOMF@mediumturquoise?$AA@ 10065218     Color.obj
 0002:00003228       ??_C@_0BC@POGDBPNO@mediumspringgreen?$AA@ 10065228     Color.obj
 0002:0000323c       ??_C@_0BA@EKIMKCFD@mediumslateblue?$AA@ 1006523c     Color.obj
 0002:0000324c       ??_C@_0P@BNCCGPJD@mediumseagreen?$AA@ 1006524c     Color.obj
 0002:0000325c       ??_C@_0N@DDGNBDHJ@mediumpurple?$AA@ 1006525c     Color.obj
 0002:0000326c       ??_C@_0N@GIADPNAO@mediumorchid?$AA@ 1006526c     Color.obj
 0002:0000327c       ??_C@_0L@CEFFILOH@mediumblue?$AA@ 1006527c     Color.obj
 0002:00003288       ??_C@_0BB@HHCOFKIC@mediumaquamarine?$AA@ 10065288     Color.obj
 0002:0000329c       ??_C@_06BDPIEPJF@maroon?$AA@ 1006529c     Color.obj
 0002:000032a4       ??_C@_07EMDGAPCI@magenta?$AA@ 100652a4     Color.obj
 0002:000032ac       ??_C@_05MLLCELJD@linen?$AA@ 100652ac     Color.obj
 0002:000032b4       ??_C@_09JKHHFGDO@limegreen?$AA@ 100652b4     Color.obj
 0002:000032c0       ??_C@_04HLLEONLG@lime?$AA@ 100652c0     Color.obj
 0002:000032c8       ??_C@_0M@FBHPKJLB@lightyellow?$AA@ 100652c8     Color.obj
 0002:000032d4       ??_C@_0P@EIHJHAMG@lightsteelblue?$AA@ 100652d4     Color.obj
 0002:000032e4       ??_C@_0P@LIPDKBMK@lightslategray?$AA@ 100652e4     Color.obj
 0002:000032f4       ??_C@_0N@JIFIFCAN@lightskyblue?$AA@ 100652f4     Color.obj
 0002:00003304       ??_C@_0O@BLOIENJC@lightseagreen?$AA@ 10065304     Color.obj
 0002:00003314       ??_C@_0M@ENCCHKJE@lightsalmon?$AA@ 10065314     Color.obj
 0002:00003320       ??_C@_09KOBGKMHP@lightpink?$AA@ 10065320     Color.obj
 0002:0000332c       ??_C@_09IPGPKIEB@lightgrey?$AA@ 1006532c     Color.obj
 0002:00003338       ??_C@_0L@OPBGACJD@lightgreen?$AA@ 10065338     Color.obj
 0002:00003344       ??_C@_0BF@PJADCIND@lightgoldenrodyellow?$AA@ 10065344     Color.obj
 0002:0000335c       ??_C@_09KPGEKFMK@lightcyan?$AA@ 1006535c     Color.obj
 0002:00003368       ??_C@_0L@BEAGLGMO@lightcoral?$AA@ 10065368     Color.obj
 0002:00003374       ??_C@_09NBIPJLA@lightblue?$AA@ 10065374     Color.obj
 0002:00003380       ??_C@_0N@ICDCAEHK@lemonchiffon?$AA@ 10065380     Color.obj
 0002:00003390       ??_C@_09MONDINDP@lawngreen?$AA@ 10065390     Color.obj
 0002:0000339c       ??_C@_0O@CCCMFNCK@lavenderblush?$AA@ 1006539c     Color.obj
 0002:000033ac       ??_C@_08KJDCPJPL@lavender?$AA@ 100653ac     Color.obj
 0002:000033b8       ??_C@_05PGGLPJAA@khaki?$AA@ 100653b8     Color.obj
 0002:000033c0       ??_C@_05NNJJIMHF@ivory?$AA@ 100653c0     Color.obj
 0002:000033c8       ??_C@_06MLCCIEFE@indigo?$AA@ 100653c8     Color.obj
 0002:000033d0       ??_C@_09IELIJPNO@indianred?$AA@ 100653d0     Color.obj
 0002:000033dc       ??_C@_07PCCOEED@hotpink?$AA@ 100653dc     Color.obj
 0002:000033e4       ??_C@_08BKNCNHLL@honeydew?$AA@ 100653e4     Color.obj
 0002:000033f0       ??_C@_0M@LFPLFELJ@greenyellow?$AA@ 100653f0     Color.obj
 0002:000033fc       ??_C@_05GBEEJKMC@green?$AA@ 100653fc     Color.obj
 0002:00003404       ??_C@_04GEBBKIAA@gray?$AA@ 10065404     Color.obj
 0002:0000340c       ??_C@_09KJDOAGJL@goldenrod?$AA@ 1006540c     Color.obj
 0002:00003418       ??_C@_04DBNGNIAN@gold?$AA@ 10065418     Color.obj
 0002:00003420       ??_C@_0L@CELMEDAA@ghostwhite?$AA@ 10065420     Color.obj
 0002:0000342c       ??_C@_09MIGKOGAO@gainsboro?$AA@ 1006542c     Color.obj
 0002:00003438       ??_C@_07FHEBJCGF@fuchsia?$AA@ 10065438     Color.obj
 0002:00003440       ??_C@_0M@HBKAKFBN@forestgreen?$AA@ 10065440     Color.obj
 0002:0000344c       ??_C@_0M@FFMCAIP@floralwhite?$AA@ 1006544c     Color.obj
 0002:00003458       ??_C@_09ELCPEDIM@firebrick?$AA@ 10065458     Color.obj
 0002:00003464       ??_C@_0L@MIOOBLBJ@dodgerblue?$AA@ 10065464     Color.obj
 0002:00003470       ??_C@_07DJPEDLIH@dimgray?$AA@ 10065470     Color.obj
 0002:00003478       ??_C@_0M@BGGBNDNG@deepskyblue?$AA@ 10065478     Color.obj
 0002:00003484       ??_C@_08CJGCPHKF@deeppink?$AA@ 10065484     Color.obj
 0002:00003490       ??_C@_0L@NGBKDFME@darkviolet?$AA@ 10065490     Color.obj
 0002:0000349c       ??_C@_0O@HKLGOIEA@darkturquoise?$AA@ 1006549c     Color.obj
 0002:000034ac       ??_C@_0O@HFGOKNPL@darkslategray?$AA@ 100654ac     Color.obj
 0002:000034bc       ??_C@_0O@PABAFENG@darkslateblue?$AA@ 100654bc     Color.obj
 0002:000034cc       ??_C@_0N@FBOCOPGH@darkseagreen?$AA@ 100654cc     Color.obj
 0002:000034dc       ??_C@_0L@CKNHPKLG@darksalmon?$AA@ 100654dc     Color.obj
 0002:000034e8       ??_C@_07MFAOOMGP@darkred?$AA@ 100654e8     Color.obj
 0002:000034f0       ??_C@_0L@EEAHIPOC@darkorchid?$AA@ 100654f0     Color.obj
 0002:000034fc       ??_C@_0L@ICJJPBF@darkorange?$AA@ 100654fc     Color.obj
 0002:00003508       ??_C@_0P@BGCLDNDK@darkolivegreen?$AA@ 10065508     Color.obj
 0002:00003518       ??_C@_0M@MEEFECHN@darkmagenta?$AA@ 10065518     Color.obj
 0002:00003524       ??_C@_09FAPDIPMK@darkkhaki?$AA@ 10065524     Color.obj
 0002:00003530       ??_C@_09MHNMOMAI@darkgreen?$AA@ 10065530     Color.obj
 0002:0000353c       ??_C@_08EADAAFKF@darkgray?$AA@ 1006553c     Color.obj
 0002:00003548       ??_C@_0O@GGJPBKNE@darkgoldenrod?$AA@ 10065548     Color.obj
 0002:00003558       ??_C@_08GHDCKAPC@darkcyan?$AA@ 10065558     Color.obj
 0002:00003564       ??_C@_08MFEOPMII@darkblue?$AA@ 10065564     Color.obj
 0002:00003570       ??_C@_04EDBDANFH@cyan?$AA@ 10065570     Color.obj
 0002:00003578       ??_C@_07DAGIGOOE@crimson?$AA@ 10065578     Color.obj
 0002:00003580       ??_C@_08DECOJLB@cornsilk?$AA@ 10065580     Color.obj
 0002:0000358c       ??_C@_0L@EPFJGEPF@cornflower?$AA@ 1006558c     Color.obj
 0002:00003598       ??_C@_05JKFECOJP@coral?$AA@ 10065598     Color.obj
 0002:000035a0       ??_C@_09BPADAHOC@chocolate?$AA@ 100655a0     Color.obj
 0002:000035ac       ??_C@_0L@CHNAEACO@chartreuse?$AA@ 100655ac     Color.obj
 0002:000035b8       ??_C@_09KIJDGGAG@cadetblue?$AA@ 100655b8     Color.obj
 0002:000035c4       ??_C@_09JHLANABP@burlywood?$AA@ 100655c4     Color.obj
 0002:000035d0       ??_C@_05EBJGJMAL@brown?$AA@ 100655d0     Color.obj
 0002:000035d8       ??_C@_0L@LKLKALMM@blueviolet?$AA@ 100655d8     Color.obj
 0002:000035e4       ??_C@_04OBGPFBCN@blue?$AA@ 100655e4     Color.obj
 0002:000035ec       ??_C@_0P@CMCBOAOE@blanchedalmond?$AA@ 100655ec     Color.obj
 0002:000035fc       ??_C@_05BIMBDNDC@black?$AA@ 100655fc     Color.obj
 0002:00003604       ??_C@_06HGAAELGA@bisque?$AA@ 10065604     Color.obj
 0002:0000360c       ??_C@_05EJOPPCPO@beige?$AA@ 1006560c     Color.obj
 0002:00003614       ??_C@_05CNOJAJLP@azure?$AA@ 10065614     Color.obj
 0002:0000361c       ??_C@_0L@MOKEMMG@aquamarine?$AA@ 1006561c     Color.obj
 0002:00003628       ??_C@_04GANAGBLL@aqua?$AA@ 10065628     Color.obj
 0002:00003630       ??_C@_0N@OJFLMGEJ@antiquewhite?$AA@ 10065630     Color.obj
 0002:00003640       ??_C@_09GNHGKALJ@aliceblue?$AA@ 10065640     Color.obj
 0002:00003650       ?m_namedColor@CColor@@0QBUDNamedColor@1@B 10065650     Color.obj
 0002:00003ab0       __real@4076800000000000    10065ab0     Color.obj
 0002:00003ab8       __real@404e000000000000    10065ab8     Color.obj
 0002:00003ac0       __real@4018000000000000    10065ac0     Color.obj
 0002:00003ac8       __real@407fe00000000000    10065ac8     Color.obj
 0002:00003ad0       __real@405e000000000000    10065ad0     Color.obj
 0002:00003ad8       __real@406fe00000000000    10065ad8     Color.obj
 0002:00003ae0       __real@406e000000000000    10065ae0     Color.obj
 0002:00003ae8       __real@4066800000000000    10065ae8     Color.obj
 0002:00003af4       ??_7CDialogManager@@6B@    10065af4     DialogManager.obj
 0002:00003be8       ??_C@_08KKNMKBOP@ver?4r1?48?$AA@ 10065be8     DialogManager.obj
 0002:00003bf4       ??_C@_08GCAFCLOH@ver?4r1?40?$AA@ 10065bf4     DialogManager.obj
 0002:00003c00       ??_C@_07CKKODHCP@ver?4r10?$AA@ 10065c00     DialogManager.obj
 0002:00003c08       ??_C@_04INIGBNHO@DFLT?$AA@ 10065c08     DrawCtrl.obj
 0002:00003c14       ??_7CDrawCtrl@@6B@         10065c14     DrawCtrl.obj
 0002:00003c18       __real@bf800000            10065c18     DrawCtrl.obj
 0002:00003c20       __real@3f50624de0000000    10065c20     DrawCtrl.obj
 0002:00003c28       __real@406a400000000000    10065c28     DrawCtrl.obj
 0002:00003c30       __real@4060000000000000    10065c30     DrawCtrl.obj
 0002:00003c38       __real@3f9cac0840000000    10065c38     DrawCtrl.obj
 0002:00003c40       __real@3fb70a3d80000000    10065c40     DrawCtrl.obj
 0002:00003c48       __real@3fc3333340000000    10065c48     DrawCtrl.obj
 0002:00003c50       __real@3fd147ae20000000    10065c50     DrawCtrl.obj
 0002:00003c58       __real@3fd0000000000000    10065c58     DrawCtrl.obj
 0002:00003c60       __real@3fa99999a0000000    10065c60     DrawCtrl.obj
 0002:00003c68       __real@3fb99999a0000000    10065c68     DrawCtrl.obj
 0002:00003c70       __real@3fd3333340000000    10065c70     DrawCtrl.obj
 0002:00003c78       ??_C@_04IBCFJNCN@?5?4?4?4?$AA@ 10065c78     DrawCtrl.obj
 0002:00003c80       __real@3a83126f            10065c80     common:wzmath.obj
 0002:00003c88       __real@3ee4f8b580000000    10065c88     common:wzmath.obj
 0002:00003c94       ??_7WzLogSystem@WzLog@@6B@ 10065c94     programcommonlibforengine:wzlogsystem.obj
 0002:00003c9c       ??_7?$CWzSingleton@VWzLogSystem@WzLog@@@@6B@ 10065c9c     programcommonlibforengine:wzlogsystem.obj
 0002:00003ca0       ??_C@_0N@PKIBJLNA@WzFilePacker?$AA@ 10065ca0     programcommonlibforengine:discaccess.obj
 0002:00003cb0       ??_C@_09LGACLDHG@Hard?5disk?$AA@ 10065cb0     programcommonlibforengine:discaccess.obj
 0002:00003cbc       ??_C@_04OHJIHAFH@None?$AA@ 10065cbc     programcommonlibforengine:discaccess.obj
 0002:00003ce8       ??_7?$CWzHandleManager@USt_DAFileInfo@@@@6B@ 10065ce8     programcommonlibforengine:discaccess.obj
 0002:00003cec       ??_C@_0BA@JFNIOLAK@string?5too?5long?$AA@ 10065cec     libcpmt:string.obj
 0002:00003cfc       ??_C@_0BI@CFPLBAOH@invalid?5string?5position?$AA@ 10065cfc     libcpmt:string.obj
 0002:00003d14       __FPinit                   10065d14     LIBCMT:_fpinit_.obj
 0002:00003d18       __FPmtinit                 10065d18     LIBCMT:_fpinit_.obj
 0002:00003d1c       __FPmtterm                 10065d1c     LIBCMT:_fpinit_.obj
 0002:00003d24       ??_7type_info@@6B@         10065d24     LIBCMT:typinfo.obj
 0002:00003d4c       ??_7exception@std@@6B@     10065d4c     LIBCMT:stdexcpt.obj
 0002:00003d54       ??_C@_0BC@EOODALEL@Unknown?5exception?$AA@ 10065d54     LIBCMT:stdexcpt.obj
 0002:00003d68       __pRawDllMain              10065d68     LIBCMT:dllcrt0.obj
 0002:00003d68       __pDefaultRawDllMain       10065d68     LIBCMT:dllcrt0.obj
 0002:00003d6c       __pDestructExceptionObject 10065d6c     LIBCMT:frame.obj
 0002:00003d74       ??_7bad_exception@std@@6B@ 10065d74     LIBCMT:frame.obj
 0002:00003d7c       ??_C@_0O@DPKOEFFH@bad?5exception?$AA@ 10065d7c     LIBCMT:frame.obj
 0002:00003d8c       ??_C@_0O@NLDKAIKN@EncodePointer?$AA@ 10065d8c     LIBCMT:tidtable.obj
 0002:00003d9c       ??_C@_1BK@DBDEIDLH@?$AAK?$AAE?$AAR?$AAN?$AAE?$AAL?$AA3?$AA2?$AA?4?$AAD?$AAL?$AAL?$AA?$AA@ 10065d9c     LIBCMT:tidtable.obj
 0002:00003db8       ??_C@_0O@KBPMFGHI@DecodePointer?$AA@ 10065db8     LIBCMT:tidtable.obj
 0002:00003dc8       ??_C@_07PEJMOBNF@FlsFree?$AA@ 10065dc8     LIBCMT:tidtable.obj
 0002:00003dd0       ??_C@_0M@JCPCPOEF@FlsSetValue?$AA@ 10065dd0     LIBCMT:tidtable.obj
 0002:00003ddc       ??_C@_0M@GDNOONDI@FlsGetValue?$AA@ 10065ddc     LIBCMT:tidtable.obj
 0002:00003de8       ??_C@_08KNHFBNJ@FlsAlloc?$AA@ 10065de8     LIBCMT:tidtable.obj
 0002:00003dfc       ??_C@_05KLBDPFGC@e?$CL000?$AA@ 10065dfc     LIBCMT:cvt.obj
 0002:00003e08       __real@4150017ec0000000    10065e08     LIBCMT:_testfdiv_.obj
 0002:00003e10       __real@4147ffff80000000    10065e10     LIBCMT:_testfdiv_.obj
 0002:00003e18       ??_C@_0BK@NHEOCAHP@IsProcessorFeaturePresent?$AA@ 10065e18     LIBCMT:_testfdiv_.obj
 0002:00003e34       ??_C@_08CPNIBGIE@KERNEL32?$AA@ 10065e34     LIBCMT:_testfdiv_.obj
 0002:00003ec0       ??_C@_01NEMOKFLO@?$DN?$AA@ 10065ec0     LIBCMT:setlocal.obj
 0002:00003ec4       ??_C@_1O@CEDCILHN@?$AA?$CI?$AAn?$AAu?$AAl?$AAl?$AA?$CJ?$AA?$AA@ 10065ec4     LIBCMT:output.obj
 0002:00003ed4       ??_C@_06OJHGLDPL@?$CInull?$CJ?$AA@ 10065ed4     LIBCMT:output.obj
 0002:00003ee0       ___lookuptable             10065ee0     LIBCMT:output.obj
 0002:00003f5c       ??_C@_0P@MIGLKIOC@CorExitProcess?$AA@ 10065f5c     LIBCMT:crt0dat.obj
 0002:00003f6c       ??_C@_1BI@BGOHAHKC@?$AAm?$AAs?$AAc?$AAo?$AAr?$AAe?$AAe?$AA?4?$AAd?$AAl?$AAl?$AA?$AA@ 10065f6c     LIBCMT:crt0dat.obj
 0002:00004848       __DEFAULT_CW_in_mem        10066848     LIBCMT:_common_.obj
 0002:0000484a       __pi_by_2_to_61            1006684a     LIBCMT:_common_.obj
 0002:00004884       ??_C@_0P@GGKDKEEG@runtime?5error?5?$AA@ 10066884     LIBCMT:crt0msg.obj
 0002:00004894       ??_C@_02PCIJFNDE@?$AN?6?$AA@ 10066894     LIBCMT:crt0msg.obj
 0002:00004898       ??_C@_0O@MJNIPGOH@TLOSS?5error?$AN?6?$AA@ 10066898     LIBCMT:crt0msg.obj
 0002:000048a8       ??_C@_0N@BONNPDHF@SING?5error?$AN?6?$AA@ 100668a8     LIBCMT:crt0msg.obj
 0002:000048b8       ??_C@_0P@MBDAJNE@DOMAIN?5error?$AN?6?$AA@ 100668b8     LIBCMT:crt0msg.obj
 0002:000048c8       ??_C@_0JL@DFDOOABL@R6034?$AN?6An?5application?5has?5made?5a@ 100668c8     LIBCMT:crt0msg.obj
 0002:00004968       ??_C@_0PH@EPAFIJ@R6033?$AN?6?9?5Attempt?5to?5use?5MSIL?5cod@ 10066968     LIBCMT:crt0msg.obj
 0002:00004a60       ??_C@_0DD@BKEEABMM@R6032?$AN?6?9?5not?5enough?5space?5for?5lo@ 10066a60     LIBCMT:crt0msg.obj
 0002:00004a98       ??_C@_0GD@OFKILIED@R6031?$AN?6?9?5Attempt?5to?5initialize?5t@ 10066a98     LIBCMT:crt0msg.obj
 0002:00004afc       ??_C@_0BP@LPMHJOKI@R6030?$AN?6?9?5CRT?5not?5initialized?$AN?6?$AA@ 10066afc     LIBCMT:crt0msg.obj
 0002:00004b1c       ??_C@_0CF@KJDAIALP@R6028?$AN?6?9?5unable?5to?5initialize?5he@ 10066b1c     LIBCMT:crt0msg.obj
 0002:00004b44       ??_C@_0DF@GAKBPDFP@R6027?$AN?6?9?5not?5enough?5space?5for?5lo@ 10066b44     LIBCMT:crt0msg.obj
 0002:00004b7c       ??_C@_0DF@IBLNNAIG@R6026?$AN?6?9?5not?5enough?5space?5for?5st@ 10066b7c     LIBCMT:crt0msg.obj
 0002:00004bb4       ??_C@_0CG@IOHKGFNJ@R6025?$AN?6?9?5pure?5virtual?5function?5c@ 10066bb4     LIBCMT:crt0msg.obj
 0002:00004bdc       ??_C@_0DF@JIJJFJDC@R6024?$AN?6?9?5not?5enough?5space?5for?5_o@ 10066bdc     LIBCMT:crt0msg.obj
 0002:00004c14       ??_C@_0CJ@EGEJHFME@R6019?$AN?6?9?5unable?5to?5open?5console?5@ 10066c14     LIBCMT:crt0msg.obj
 0002:00004c40       ??_C@_0CB@GNHNIELH@R6018?$AN?6?9?5unexpected?5heap?5error?$AN?6@ 10066c40     LIBCMT:crt0msg.obj
 0002:00004c64       ??_C@_0CN@FOLDKNG@R6017?$AN?6?9?5unexpected?5multithread?5@ 10066c64     LIBCMT:crt0msg.obj
 0002:00004c94       ??_C@_0CM@FAHFJNHO@R6016?$AN?6?9?5not?5enough?5space?5for?5th@ 10066c94     LIBCMT:crt0msg.obj
 0002:00004cc0       ??_C@_0JG@LBKMGKLD@?$AN?6This?5application?5has?5requested@ 10066cc0     LIBCMT:crt0msg.obj
 0002:00004d58       ??_C@_0CM@FLCNIPKK@R6009?$AN?6?9?5not?5enough?5space?5for?5en@ 10066d58     LIBCMT:crt0msg.obj
 0002:00004d84       ??_C@_0CK@KMMJOAPP@R6008?$AN?6?9?5not?5enough?5space?5for?5ar@ 10066d84     LIBCMT:crt0msg.obj
 0002:00004db0       ??_C@_0CN@LEKKICBM@R6002?$AN?6?9?5floating?5point?5support?5@ 10066db0     LIBCMT:crt0msg.obj
 0002:00004de0       ??_C@_0CF@GOGNBNAK@Microsoft?5Visual?5C?$CL?$CL?5Runtime?5Lib@ 10066de0     LIBCMT:crt0msg.obj
 0002:00004e08       ??_C@_02PHMGELLB@?6?6?$AA@ 10066e08     LIBCMT:crt0msg.obj
 0002:00004e0c       ??_C@_03KHICJKCI@?4?4?4?$AA@ 10066e0c     LIBCMT:crt0msg.obj
 0002:00004e10       ??_C@_0BH@DNAGHKFM@?$DMprogram?5name?5unknown?$DO?$AA@ 10066e10     LIBCMT:crt0msg.obj
 0002:00004e28       ??_C@_0BK@OFGJDLJJ@Runtime?5Error?$CB?6?6Program?3?5?$AA@ 10066e28     LIBCMT:crt0msg.obj
 0002:00004e48       __XcptActTab               10066e48     LIBCMT:winxfltr.obj
 0002:00006f80       ??_C@_0BK@CFCOFLF@?5Complete?5Object?5Locator?8?$AA@ 10068f80     LIBCMT:undname.obj
 0002:00006f9c       ??_C@_0BN@MECKDCOJ@?5Class?5Hierarchy?5Descriptor?8?$AA@ 10068f9c     LIBCMT:undname.obj
 0002:00006fbc       ??_C@_0BD@LGICGFMM@?5Base?5Class?5Array?8?$AA@ 10068fbc     LIBCMT:undname.obj
 0002:00006fd0       ??_C@_0BM@LDKODKLH@?5Base?5Class?5Descriptor?5at?5?$CI?$AA@ 10068fd0     LIBCMT:undname.obj
 0002:00006fec       ??_C@_0BC@DAFEJGAK@?5Type?5Descriptor?8?$AA@ 10068fec     LIBCMT:undname.obj
 0002:00007000       ??_C@_0BM@PMGGMLDN@?$GAlocal?5static?5thread?5guard?8?$AA@ 10069000     LIBCMT:undname.obj
 0002:0000701c       ??_C@_0CL@FGIJHLCE@?$GAmanaged?5vector?5copy?5constructor@ 1006901c     LIBCMT:undname.obj
 0002:00007048       ??_C@_0CJ@GJELGAMM@?$GAvector?5vbase?5copy?5constructor?5i@ 10069048     LIBCMT:undname.obj
 0002:00007074       ??_C@_0CD@CGAJBKEJ@?$GAvector?5copy?5constructor?5iterato@ 10069074     LIBCMT:undname.obj
 0002:00007098       ??_C@_0CB@PDBIFEP@?$GAdynamic?5atexit?5destructor?5for?5?8@ 10069098     LIBCMT:undname.obj
 0002:000070bc       ??_C@_0BL@CLIPGLGB@?$GAdynamic?5initializer?5for?5?8?$AA@ 100690bc     LIBCMT:undname.obj
 0002:000070d8       ??_C@_0CM@FCBBDIGB@?$GAeh?5vector?5vbase?5copy?5constructo@ 100690d8     LIBCMT:undname.obj
 0002:00007104       ??_C@_0CG@HLDDJMAG@?$GAeh?5vector?5copy?5constructor?5iter@ 10069104     LIBCMT:undname.obj
 0002:0000712c       ??_C@_0CF@IMGKMJNO@?$GAmanaged?5vector?5destructor?5itera@ 1006912c     LIBCMT:undname.obj
 0002:00007154       ??_C@_0CG@CFDHKGGD@?$GAmanaged?5vector?5constructor?5iter@ 10069154     LIBCMT:undname.obj
 0002:0000717c       ??_C@_0BN@CKNJLHMB@?$GAplacement?5delete?$FL?$FN?5closure?8?$AA@ 1006917c     LIBCMT:undname.obj
 0002:0000719c       ??_C@_0BL@CNOONJFP@?$GAplacement?5delete?5closure?8?$AA@ 1006919c     LIBCMT:undname.obj
 0002:000071b8       ??_C@_0P@HJKNJFNN@?$GAomni?5callsig?8?$AA@ 100691b8     LIBCMT:undname.obj
 0002:000071c8       ??_C@_09LBNFPBCA@?5delete?$FL?$FN?$AA@ 100691c8     LIBCMT:undname.obj
 0002:000071d4       ??_C@_06FHBGPFGH@?5new?$FL?$FN?$AA@ 100691d4     LIBCMT:undname.obj
 0002:000071dc       ??_C@_0CE@IIHCMGGL@?$GAlocal?5vftable?5constructor?5closu@ 100691dc     LIBCMT:undname.obj
 0002:00007200       ??_C@_0BA@KKLDJDLB@?$GAlocal?5vftable?8?$AA@ 10069200     LIBCMT:undname.obj
 0002:00007210       ??_C@_05KHLCHHI@?$GARTTI?$AA@ 10069210     LIBCMT:undname.obj
 0002:00007218       ??_C@_03KLGMFNMG@?$GAEH?$AA@ 10069218     LIBCMT:undname.obj
 0002:0000721c       ??_C@_0BA@KBCDOMBN@?$GAudt?5returning?8?$AA@ 1006921c     LIBCMT:undname.obj
 0002:0000722c       ??_C@_0BL@LLKPOHJI@?$GAcopy?5constructor?5closure?8?$AA@ 1006922c     LIBCMT:undname.obj
 0002:00007248       ??_C@_0CH@OOJPLCPH@?$GAeh?5vector?5vbase?5constructor?5ite@ 10069248     LIBCMT:undname.obj
 0002:00007270       ??_C@_0CA@GCEOPDGL@?$GAeh?5vector?5destructor?5iterator?8?$AA@ 10069270     LIBCMT:undname.obj
 0002:00007290       ??_C@_0CB@JONCMFFK@?$GAeh?5vector?5constructor?5iterator?8@ 10069290     LIBCMT:undname.obj
 0002:000072b4       ??_C@_0BL@NILFHHPC@?$GAvirtual?5displacement?5map?8?$AA@ 100692b4     LIBCMT:undname.obj
 0002:000072d0       ??_C@_0CE@IKBNEHA@?$GAvector?5vbase?5constructor?5iterat@ 100692d0     LIBCMT:undname.obj
 0002:000072f4       ??_C@_0BN@LFPFMEDL@?$GAvector?5destructor?5iterator?8?$AA@ 100692f4     LIBCMT:undname.obj
 0002:00007314       ??_C@_0BO@PFGOCPJJ@?$GAvector?5constructor?5iterator?8?$AA@ 10069314     LIBCMT:undname.obj
 0002:00007334       ??_C@_0BN@IMDCHIKM@?$GAscalar?5deleting?5destructor?8?$AA@ 10069334     LIBCMT:undname.obj
 0002:00007354       ??_C@_0BO@OBMKPJIG@?$GAdefault?5constructor?5closure?8?$AA@ 10069354     LIBCMT:undname.obj
 0002:00007374       ??_C@_0BN@DEGPLNFK@?$GAvector?5deleting?5destructor?8?$AA@ 10069374     LIBCMT:undname.obj
 0002:00007394       ??_C@_0BD@JDLKDPAB@?$GAvbase?5destructor?8?$AA@ 10069394     LIBCMT:undname.obj
 0002:000073a8       ??_C@_08OBABFOLI@?$GAstring?8?$AA@ 100693a8     LIBCMT:undname.obj
 0002:000073b4       ??_C@_0BF@KDPPACIK@?$GAlocal?5static?5guard?8?$AA@ 100693b4     LIBCMT:undname.obj
 0002:000073cc       ??_C@_08LLFFHHDJ@?$GAtypeof?8?$AA@ 100693cc     LIBCMT:undname.obj
 0002:000073d8       ??_C@_07FEEIOKP@?$GAvcall?8?$AA@ 100693d8     LIBCMT:undname.obj
 0002:000073e0       ??_C@_09BLBHBJP@?$GAvbtable?8?$AA@ 100693e0     LIBCMT:undname.obj
 0002:000073ec       ??_C@_09IFPLHPGF@?$GAvftable?8?$AA@ 100693ec     LIBCMT:undname.obj
 0002:000073f8       ??_C@_02MHEGNOJ@?$FO?$DN?$AA@ 100693f8     LIBCMT:undname.obj
 0002:000073fc       ??_C@_02DHLNPPGH@?$HM?$DN?$AA@ 100693fc     LIBCMT:undname.obj
 0002:00007400       ??_C@_02FGJGFEAB@?$CG?$DN?$AA@ 10069400     LIBCMT:undname.obj
 0002:00007404       ??_C@_03CDNPDDLA@?$DM?$DM?$DN?$AA@ 10069404     LIBCMT:undname.obj
 0002:00007408       ??_C@_03IKFCCPFF@?$DO?$DO?$DN?$AA@ 10069408     LIBCMT:undname.obj
 0002:0000740c       ??_C@_02FENAOKFI@?$CF?$DN?$AA@ 1006940c     LIBCMT:undname.obj
 0002:00007410       ??_C@_02FJEHGPIO@?1?$DN?$AA@ 10069410     LIBCMT:undname.obj
 0002:00007414       ??_C@_02FKMDLLOA@?9?$DN?$AA@ 10069414     LIBCMT:undname.obj
 0002:00007418       ??_C@_02FOEOMHFC@?$CL?$DN?$AA@ 10069418     LIBCMT:undname.obj
 0002:0000741c       ??_C@_02FPIMKNGF@?$CK?$DN?$AA@ 1006941c     LIBCMT:undname.obj
 0002:00007420       ??_C@_02NONPIBCD@?$HM?$HM?$AA@ 10069420     LIBCMT:undname.obj
 0002:00007424       ??_C@_02PPKAJPJL@?$CG?$CG?$AA@ 10069424     LIBCMT:undname.obj
 0002:00007428       ??_C@_01DNKMNLPK@?$HM?$AA@ 10069428     LIBCMT:undname.obj
 0002:0000742c       ??_C@_01JKBOJNNK@?$FO?$AA@ 1006942c     LIBCMT:undname.obj
 0002:00007430       ??_C@_01PJKLJHI@?$HO?$AA@  10069430     LIBCMT:undname.obj
 0002:00007434       ??_C@_02HCKGKOFO@?$CI?$CJ?$AA@ 10069434     LIBCMT:undname.obj
 0002:00007438       ??_C@_02EEKDKGMJ@?$DO?$DN?$AA@ 10069438     LIBCMT:undname.obj
 0002:0000743c       ??_C@_01PPODPGHN@?$DO?$AA@ 1006943c     LIBCMT:undname.obj
 0002:00007440       ??_C@_02EHCHHCKH@?$DM?$DN?$AA@ 10069440     LIBCMT:undname.obj
 0002:00007444       ??_C@_01MNNFJEPP@?$DM?$AA@ 10069444     LIBCMT:undname.obj
 0002:00007448       ??_C@_01FGNFDNOH@?$CF?$AA@ 10069448     LIBCMT:undname.obj
 0002:0000744c       ??_C@_01KMDKNFGN@?1?$AA@   1006944c     LIBCMT:undname.obj
 0002:00007450       ??_C@_03MNHNFDLC@?9?$DO?$CK?$AA@ 10069450     LIBCMT:undname.obj
 0002:00007454       ??_C@_01HNPIGOCE@?$CG?$AA@ 10069454     LIBCMT:undname.obj
 0002:00007458       ??_C@_01MIFGBAGJ@?$CL?$AA@ 10069458     LIBCMT:undname.obj
 0002:0000745c       ??_C@_01JOAMLHOP@?9?$AA@   1006945c     LIBCMT:undname.obj
 0002:00007460       ??_C@_02BAABKJLB@?9?9?$AA@ 10069460     LIBCMT:undname.obj
 0002:00007464       ??_C@_02ECNGHCIF@?$CL?$CL?$AA@ 10069464     LIBCMT:undname.obj
 0002:00007468       ??_C@_01NBENCBCI@?$CK?$AA@ 10069468     LIBCMT:undname.obj
 0002:0000746c       ??_C@_02HBOOOICD@?9?$DO?$AA@ 1006946c     LIBCMT:undname.obj
 0002:00007470       ??_C@_08LHJFAFGD@operator?$AA@ 10069470     LIBCMT:undname.obj
 0002:0000747c       ??_C@_02GPECMEKF@?$FL?$FN?$AA@ 1006947c     LIBCMT:undname.obj
 0002:00007480       ??_C@_02FDNJECIE@?$CB?$DN?$AA@ 10069480     LIBCMT:undname.obj
 0002:00007484       ??_C@_02EGOFBIJA@?$DN?$DN?$AA@ 10069484     LIBCMT:undname.obj
 0002:00007488       ??_C@_01DCLJPIOD@?$CB?$AA@ 10069488     LIBCMT:undname.obj
 0002:0000748c       ??_C@_02FODMEDOG@?$DM?$DM?$AA@ 1006948c     LIBCMT:undname.obj
 0002:00007490       ??_C@_02GPIOPFAK@?$DO?$DO?$AA@ 10069490     LIBCMT:undname.obj
 0002:00007494       ??_C@_07FPCDHGMM@?5delete?$AA@ 10069494     LIBCMT:undname.obj
 0002:0000749c       ??_C@_04NIHEBCM@?5new?$AA@ 1006949c     LIBCMT:undname.obj
 0002:000074a4       ??_C@_0M@GFIIJFMG@__unaligned?$AA@ 100694a4     LIBCMT:undname.obj
 0002:000074b0       ??_C@_0L@PILCLIHE@__restrict?$AA@ 100694b0     LIBCMT:undname.obj
 0002:000074bc       ??_C@_07JOMMBBKO@__ptr64?$AA@ 100694bc     LIBCMT:undname.obj
 0002:000074c4       ??_C@_09HIJEGCPM@__clrcall?$AA@ 100694c4     LIBCMT:undname.obj
 0002:000074d0       ??_C@_0L@JMKHOMEK@__fastcall?$AA@ 100694d0     LIBCMT:undname.obj
 0002:000074dc       ??_C@_0L@NPHFGOKO@__thiscall?$AA@ 100694dc     LIBCMT:undname.obj
 0002:000074e8       ??_C@_09IFJBGAPI@__stdcall?$AA@ 100694e8     LIBCMT:undname.obj
 0002:000074f4       ??_C@_08GHMPAG@__pascal?$AA@ 100694f4     LIBCMT:undname.obj
 0002:00007500       ??_C@_07KOLFKCDI@__cdecl?$AA@ 10069500     LIBCMT:undname.obj
 0002:00007508       ??_C@_08EHJDFFNH@__based?$CI?$AA@ 10069508     LIBCMT:undname.obj
 0002:00007698       ??_C@_13NOLLCAOD@?$AA?$AA?$AA?$AA@ 10069698     LIBCMT:a_map.obj
 0002:00007698       __real@00000000            10069698     ControlWZ.obj
 0002:000076a0       ___newctype                100696a0     LIBCMT:ctype.obj
 0002:000079a0       __wctype                   100699a0     LIBCMT:ctype.obj
 0002:00007ba8       ___newclmap                10069ba8     LIBCMT:ctype.obj
 0002:00007d28       ___newcumap                10069d28     LIBCMT:ctype.obj
 0002:00007ea8       ??_C@_08JCCMCCIL@HH?3mm?3ss?$AA@ 10069ea8     LIBCMT:strftime.obj
 0002:00007eb4       ??_C@_0BE@CKGJFCPC@dddd?0?5MMMM?5dd?0?5yyyy?$AA@ 10069eb4     LIBCMT:strftime.obj
 0002:00007ec8       ??_C@_08BPBNCDIB@MM?1dd?1yy?$AA@ 10069ec8     LIBCMT:strftime.obj
 0002:00007ed4       ??_C@_02CJNFDJBF@PM?$AA@   10069ed4     LIBCMT:strftime.obj
 0002:00007ed8       ??_C@_02DEDBPAFC@AM?$AA@   10069ed8     LIBCMT:strftime.obj
 0002:00007edc       ??_C@_08EDHMEBNP@December?$AA@ 10069edc     LIBCMT:strftime.obj
 0002:00007ee8       ??_C@_08HCHEGEOA@November?$AA@ 10069ee8     LIBCMT:strftime.obj
 0002:00007ef4       ??_C@_07JJNFCEND@October?$AA@ 10069ef4     LIBCMT:strftime.obj
 0002:00007efc       ??_C@_09BHHEALKD@September?$AA@ 10069efc     LIBCMT:strftime.obj
 0002:00007f08       ??_C@_06LBBHFDDG@August?$AA@ 10069f08     LIBCMT:strftime.obj
 0002:00007f10       ??_C@_04MIEPOIFP@July?$AA@ 10069f10     LIBCMT:strftime.obj
 0002:00007f18       ??_C@_04CNLMGBGM@June?$AA@ 10069f18     LIBCMT:strftime.obj
 0002:00007f20       ??_C@_05DMJDNLEJ@April?$AA@ 10069f20     LIBCMT:strftime.obj
 0002:00007f28       ??_C@_05HPCKOFNC@March?$AA@ 10069f28     LIBCMT:strftime.obj
 0002:00007f30       ??_C@_08GNJGEPFN@February?$AA@ 10069f30     LIBCMT:strftime.obj
 0002:00007f3c       ??_C@_07CGJPFGJA@January?$AA@ 10069f3c     LIBCMT:strftime.obj
 0002:00007f44       ??_C@_03MKABNOCG@Dec?$AA@  10069f44     LIBCMT:strftime.obj
 0002:00007f48       ??_C@_03JPJOFNIA@Nov?$AA@  10069f48     LIBCMT:strftime.obj
 0002:00007f4c       ??_C@_03BMAOKBAD@Oct?$AA@  10069f4c     LIBCMT:strftime.obj
 0002:00007f50       ??_C@_03GGCAPAJC@Sep?$AA@  10069f50     LIBCMT:strftime.obj
 0002:00007f54       ??_C@_03IFJFEIGA@Aug?$AA@  10069f54     LIBCMT:strftime.obj
 0002:00007f58       ??_C@_03LBGABGKK@Jul?$AA@  10069f58     LIBCMT:strftime.obj
 0002:00007f5c       ??_C@_03IDFGHECI@Jun?$AA@  10069f5c     LIBCMT:strftime.obj
 0002:00007f60       ??_C@_03CNMDKL@May?$AA@    10069f60     LIBCMT:strftime.obj
 0002:00007f64       ??_C@_03LEOLGMJP@Apr?$AA@  10069f64     LIBCMT:strftime.obj
 0002:00007f68       ??_C@_03ODNJBKGA@Mar?$AA@  10069f68     LIBCMT:strftime.obj
 0002:00007f6c       ??_C@_03HJBDCHOM@Feb?$AA@  10069f6c     LIBCMT:strftime.obj
 0002:00007f70       ??_C@_03JIHJHPIE@Jan?$AA@  10069f70     LIBCMT:strftime.obj
 0002:00007f74       ??_C@_08INBOOONO@Saturday?$AA@ 10069f74     LIBCMT:strftime.obj
 0002:00007f80       ??_C@_06JECMNKMI@Friday?$AA@ 10069f80     LIBCMT:strftime.obj
 0002:00007f88       ??_C@_08HACCIKIA@Thursday?$AA@ 10069f88     LIBCMT:strftime.obj
 0002:00007f94       ??_C@_09DLIGFAKA@Wednesday?$AA@ 10069f94     LIBCMT:strftime.obj
 0002:00007fa0       ??_C@_07BAAGCFCM@Tuesday?$AA@ 10069fa0     LIBCMT:strftime.obj
 0002:00007fa8       ??_C@_06JLEDEDGH@Monday?$AA@ 10069fa8     LIBCMT:strftime.obj
 0002:00007fb0       ??_C@_06OOPIFAJ@Sunday?$AA@ 10069fb0     LIBCMT:strftime.obj
 0002:00007fb8       ??_C@_03FEFJNEK@Sat?$AA@   10069fb8     LIBCMT:strftime.obj
 0002:00007fbc       ??_C@_03IDIOELNC@Fri?$AA@  10069fbc     LIBCMT:strftime.obj
 0002:00007fc0       ??_C@_03IOFIKPDN@Thu?$AA@  10069fc0     LIBCMT:strftime.obj
 0002:00007fc4       ??_C@_03MHOMLAJA@Wed?$AA@  10069fc4     LIBCMT:strftime.obj
 0002:00007fc8       ??_C@_03NAGEINEP@Tue?$AA@  10069fc8     LIBCMT:strftime.obj
 0002:00007fcc       ??_C@_03PDAGKDH@Mon?$AA@   10069fcc     LIBCMT:strftime.obj
 0002:00007fd0       ??_C@_03KOEHGMDN@Sun?$AA@  10069fd0     LIBCMT:strftime.obj
 0002:00007fd8       ___lookuptable_s           10069fd8     LIBCMT:outputs.obj
 0002:00008034       ??_C@_0BI@DFKBFLJE@GetProcessWindowStation?$AA@ 1006a034     LIBCMT:crtmbox.obj
 0002:0000804c       ??_C@_0BK@CIDNPOGP@GetUserObjectInformationA?$AA@ 1006a04c     LIBCMT:crtmbox.obj
 0002:00008068       ??_C@_0BD@HHGDFDBJ@GetLastActivePopup?$AA@ 1006a068     LIBCMT:crtmbox.obj
 0002:0000807c       ??_C@_0BA@HNOPNCHB@GetActiveWindow?$AA@ 1006a07c     LIBCMT:crtmbox.obj
 0002:0000808c       ??_C@_0M@CHKKJDAI@MessageBoxA?$AA@ 1006a08c     LIBCMT:crtmbox.obj
 0002:00008098       ??_C@_0L@NDEGIDAG@USER32?4DLL?$AA@ 1006a098     LIBCMT:crtmbox.obj
 0002:00008110       ??_C@_03LALBNOCG@cos?$AA@  1006a110     LIBCMT:_libm_error_.obj
 0002:00008114       ??_C@_03BLEJJJBH@sin?$AA@  1006a114     LIBCMT:_libm_error_.obj
 0002:00008118       ??_C@_04EHEDPDJG@modf?$AA@ 1006a118     LIBCMT:_libm_error_.obj
 0002:00008120       ??_C@_05PBJFFIGL@floor?$AA@ 1006a120     LIBCMT:_libm_error_.obj
 0002:00008128       ??_C@_04GFPJNGEK@ceil?$AA@ 1006a128     LIBCMT:_libm_error_.obj
 0002:00008130       ??_C@_04MLLJIGOK@atan?$AA@ 1006a130     LIBCMT:_libm_error_.obj
 0002:00008138       ??_C@_05EOHGHCHD@exp10?$AA@ 1006a138     LIBCMT:_libm_error_.obj
 0002:00008140       ??_C@_04PDIFKINK@acos?$AA@ 1006a140     LIBCMT:_libm_error_.obj
 0002:00008148       ??_C@_04FIHNOPOL@asin?$AA@ 1006a148     LIBCMT:_libm_error_.obj
 0002:00008150       ??_C@_03MGHMBJCF@log?$AA@  1006a150     LIBCMT:_libm_error_.obj
 0002:00008154       ??_C@_05HGHHAHAP@log10?$AA@ 1006a154     LIBCMT:_libm_error_.obj
 0002:0000815c       ??_C@_03KHJOGHMM@exp?$AA@  1006a15c     LIBCMT:_libm_error_.obj
 0002:00008160       ??_C@_03JGHBODFD@pow?$AA@  1006a160     LIBCMT:_libm_error_.obj
 0002:00008164       ??_C@_06IMKFLFPG@1?$CDQNAN?$AA@ 1006a164     LIBCMT:_x10fout_.obj
 0002:0000816c       ??_C@_05DNEBIAHO@1?$CDINF?$AA@ 1006a16c     LIBCMT:_x10fout_.obj
 0002:00008174       ??_C@_05PHHOCPM@1?$CDIND?$AA@ 1006a174     LIBCMT:_x10fout_.obj
 0002:0000817c       ??_C@_06PGGFOGJG@1?$CDSNAN?$AA@ 1006a17c     LIBCMT:_x10fout_.obj
 0002:00008184       ___dnames                  1006a184     LIBCMT:timeset.obj
 0002:0000819c       ___mnames                  1006a19c     LIBCMT:timeset.obj
 0002:000081c4       ??_C@_0L@KDOEJCKC@_nextafter?$AA@ 1006a1c4     LIBCMT:_fpexcept_.obj
 0002:000081d0       ??_C@_05JGDBENOH@_logb?$AA@ 1006a1d0     LIBCMT:_fpexcept_.obj
 0002:000081d8       ??_C@_03ONILCKOB@_yn?$AA@  1006a1d8     LIBCMT:_fpexcept_.obj
 0002:000081dc       ??_C@_03NAKIGLHK@_y1?$AA@  1006a1dc     LIBCMT:_fpexcept_.obj
 0002:000081e0       ??_C@_03MJLDFKDL@_y0?$AA@  1006a1e0     LIBCMT:_fpexcept_.obj
 0002:000081e4       ??_C@_05GKKHEGJL@frexp?$AA@ 1006a1e4     LIBCMT:_fpexcept_.obj
 0002:000081ec       ??_C@_04KEPJIHGP@fmod?$AA@ 1006a1ec     LIBCMT:_fpexcept_.obj
 0002:000081f4       ??_C@_06MEIMCGCF@_hypot?$AA@ 1006a1f4     LIBCMT:_fpexcept_.obj
 0002:000081fc       ??_C@_05KBKMEMPO@_cabs?$AA@ 1006a1fc     LIBCMT:_fpexcept_.obj
 0002:00008204       ??_C@_05CEJMAHNP@ldexp?$AA@ 1006a204     LIBCMT:_fpexcept_.obj
 0002:0000820c       ??_C@_04ODHECPBC@fabs?$AA@ 1006a20c     LIBCMT:_fpexcept_.obj
 0002:00008214       ??_C@_04EIAKFFMI@sqrt?$AA@ 1006a214     LIBCMT:_fpexcept_.obj
 0002:0000821c       ??_C@_05KNGEOGJB@atan2?$AA@ 1006a21c     LIBCMT:_fpexcept_.obj
 0002:00008224       ??_C@_04FJHINJAO@tanh?$AA@ 1006a224     LIBCMT:_fpexcept_.obj
 0002:0000822c       ??_C@_04HPJJNFIM@cosh?$AA@ 1006a22c     LIBCMT:_fpexcept_.obj
 0002:00008234       ??_C@_04COOMCNPB@sinh?$AA@ 1006a234     LIBCMT:_fpexcept_.obj
 0002:0000823c       ??_C@_07GPDNMNG@CONOUT$?$AA@ 1006a23c     LIBCMT:initcon.obj
 0002:00008460       __real@4f800000            1006a460     wzFilePacker_static:wzFilePacker.obj
 0002:00008cc8       ??_C@_0BI@LCBABOGN@header?5is?5Final?5Version?$AA@ 1006acc8     wzFilePacker_static:fsvfs.obj
 0002:00008ce0       ??_C@_0P@FOHJAHFG@header?5invalid?$AA@ 1006ace0     wzFilePacker_static:fsvfs.obj
 0002:00008cf0       ??_C@_0DM@MLIJDPNB@Now?5Packing?5File?5Version?5?3?5?$CFd?0?5P@ 1006acf0     wzFilePacker_static:fsvfs.obj
 0002:00008d2c       ??_C@_0DA@JPDHOIDD@?$CK?$CK?$CK?$CK?$CK?$CK?$CK?$CK?$CK?$CK?$CK?$CK?$CK?$CK?$CK?$CK?5N2_UpdateFilePo@ 1006ad2c     wzFilePacker_static:fsvfs.obj
 0002:00008d5c       ??_C@_0CO@LGMGIONK@?$CK?$CK?$CK?$CK?$CK?$CK?$CK?$CK?$CK?$CK?$CK?$CK?$CK?$CK?$CK?$CK?5N2_SetFilePoint@ 1006ad5c     wzFilePacker_static:fsvfs.obj
 0002:00008d8c       ??_C@_0DF@IHAPMOPK@?$CL?$CL?$CL?$CL?$CL?$CL?$CL?$CL?$CL?$CL?5ReadFail_4_Error?5?3?5?G?O@ 1006ad8c     wzFilePacker_static:fsvfs.obj
 0002:00008dc4       ??_C@_0DH@HABJGGNC@?$CL?$CL?$CL?$CL?$CL?$CL?$CL?$CL?$CL?$CL?5ReadFail_3_Error?5?3?5?$MA?P@ 1006adc4     wzFilePacker_static:fsvfs.obj
 0002:00008dfc       ??_C@_0DG@LCJJILDN@?$CL?$CL?$CL?$CL?$CL?$CL?$CL?$CL?$CL?$CL?5ReadFail_2_Error?5?3?5?$LP?$MA@ 1006adfc     wzFilePacker_static:fsvfs.obj
 0002:00008e34       ??_C@_0CG@GENKINJN@?$CL?$CL?$CL?$CL?$CL?$CL?$CL?$CL?$CL?$CL?5ReadFail_1_ErrorCode?5@ 1006ae34     wzFilePacker_static:fsvfs.obj
 0002:00008e5c       ??_C@_0BH@MMBDGEON@Remove?5Fsvfs?5Tree?5Fail?$AA@ 1006ae5c     wzFilePacker_static:fsvfs.obj
 0002:00008e74       ??_C@_0BK@PKGCLKLI@Remove?5Fsvfs?5Tree?5SUCCESS?$AA@ 1006ae74     wzFilePacker_static:fsvfs.obj
 0002:00008e90       ??_C@_0BM@OPDJPMGP@Not?5File?5SameName?5Tree?9Node?$AA@ 1006ae90     wzFilePacker_static:fsvfs.obj
 0002:000092e0       ??_C@_02CEGDFPFP@?4?2?$AA@ 1006b2e0     wzFilePacker_static:fsdos.obj
 0002:000092e4       ??_C@_0BP@PFJFMKGH@Win32_SetFilePointer_Error?3?$CFd?6?$AA@ 1006b2e4     wzFilePacker_static:fsdos.obj
 0002:00009738       __GUID_df0b3d60_548f_101b_8e65_08002b2bd119 1006b738     comsuppw:comsupp.obj
 0002:00009748       ??_7_com_error@@6B@        1006b748     comsuppw:comraise.obj
 0002:00009750       __load_config_used         1006b750     LIBCMT:loadcfg.obj
 0002:0000980c       ??_R4CBaseManager@@6B@     1006b80c     BaseManager.obj
 0002:00009820       ??_R3CBaseManager@@8       1006b820     BaseManager.obj
 0002:00009830       ??_R2CBaseManager@@8       1006b830     BaseManager.obj
 0002:00009838       ??_R1A@?0A@EA@CBaseManager@@8 1006b838     BaseManager.obj
 0002:00009854       ??_R4length_error@std@@6B@ 1006b854     BaseManager.obj
 0002:00009868       ??_R3length_error@std@@8   1006b868     BaseManager.obj
 0002:00009878       ??_R2length_error@std@@8   1006b878     BaseManager.obj
 0002:00009888       ??_R1A@?0A@EA@length_error@std@@8 1006b888     BaseManager.obj
 0002:000098a4       ??_R1A@?0A@EA@logic_error@std@@8 1006b8a4     BaseManager.obj
 0002:000098c0       ??_R3logic_error@std@@8    1006b8c0     BaseManager.obj
 0002:000098d0       ??_R2logic_error@std@@8    1006b8d0     BaseManager.obj
 0002:000098dc       ??_R1A@?0A@EA@exception@std@@8 1006b8dc     BaseManager.obj
 0002:000098f8       ??_R3exception@std@@8      1006b8f8     BaseManager.obj
 0002:00009908       ??_R2exception@std@@8      1006b908     BaseManager.obj
 0002:00009910       ??_R4bad_alloc@std@@6B@    1006b910     BaseManager.obj
 0002:00009924       ??_R3bad_alloc@std@@8      1006b924     BaseManager.obj
 0002:00009934       ??_R2bad_alloc@std@@8      1006b934     BaseManager.obj
 0002:00009940       ??_R1A@?0A@EA@bad_alloc@std@@8 1006b940     BaseManager.obj
 0002:0000995c       ??_R4logic_error@std@@6B@  1006b95c     BaseManager.obj
 0002:00009970       ??_R4CControlWZ@@6B@       1006b970     ControlWZ.obj
 0002:00009984       ??_R3CControlWZ@@8         1006b984     ControlWZ.obj
 0002:00009994       ??_R2CControlWZ@@8         1006b994     ControlWZ.obj
 0002:0000999c       ??_R1A@?0A@EA@CControlWZ@@8 1006b99c     ControlWZ.obj
 0002:000099b8       ??_R4CCtrlButtonCheckWZ@@6B@ 1006b9b8     CtrlButtonCheckWZ.obj
 0002:000099cc       ??_R3CCtrlButtonCheckWZ@@8 1006b9cc     CtrlButtonCheckWZ.obj
 0002:000099dc       ??_R2CCtrlButtonCheckWZ@@8 1006b9dc     CtrlButtonCheckWZ.obj
 0002:000099ec       ??_R1A@?0A@EA@CCtrlButtonCheckWZ@@8 1006b9ec     CtrlButtonCheckWZ.obj
 0002:00009a08       ??_R1A@?0A@EA@CCtrlButtonWZ@@8 1006ba08     CtrlButtonCheckWZ.obj
 0002:00009a24       ??_R3CCtrlButtonWZ@@8      1006ba24     CtrlButtonCheckWZ.obj
 0002:00009a34       ??_R2CCtrlButtonWZ@@8      1006ba34     CtrlButtonCheckWZ.obj
 0002:00009a40       ??_R4CCtrlButtonWZ@@6B@    1006ba40     CtrlButtonWZ.obj
 0002:00009a54       ??_R4CCtrlClientWZ@@6B@    1006ba54     CtrlClientWZ.obj
 0002:00009a68       ??_R3CCtrlClientWZ@@8      1006ba68     CtrlClientWZ.obj
 0002:00009a78       ??_R2CCtrlClientWZ@@8      1006ba78     CtrlClientWZ.obj
 0002:00009a84       ??_R1A@?0A@EA@CCtrlClientWZ@@8 1006ba84     CtrlClientWZ.obj
 0002:00009aa0       ??_R4CCtrlComboBoxWZ@@6B@  1006baa0     CtrlComboBox.obj
 0002:00009ab4       ??_R3CCtrlComboBoxWZ@@8    1006bab4     CtrlComboBox.obj
 0002:00009ac4       ??_R2CCtrlComboBoxWZ@@8    1006bac4     CtrlComboBox.obj
 0002:00009ad0       ??_R1A@?0A@EA@CCtrlComboBoxWZ@@8 1006bad0     CtrlComboBox.obj
 0002:00009aec       ??_R4CCtrlBaseEdit@@6B@    1006baec     CtrlDxEdit.obj
 0002:00009b00       ??_R3CCtrlBaseEdit@@8      1006bb00     CtrlDxEdit.obj
 0002:00009b10       ??_R2CCtrlBaseEdit@@8      1006bb10     CtrlDxEdit.obj
 0002:00009b1c       ??_R1A@?0A@EA@CCtrlBaseEdit@@8 1006bb1c     CtrlDxEdit.obj
 0002:00009b38       ??_R4CCtrlDxEditBox@@6B@   1006bb38     CtrlDxEdit.obj
 0002:00009b4c       ??_R3CCtrlDxEditBox@@8     1006bb4c     CtrlDxEdit.obj
 0002:00009b5c       ??_R2CCtrlDxEditBox@@8     1006bb5c     CtrlDxEdit.obj
 0002:00009b6c       ??_R1A@?0A@EA@CCtrlDxEditBox@@8 1006bb6c     CtrlDxEdit.obj
 0002:00009b88       ??_R4CCtrlDxIMEEditBox@@6B@ 1006bb88     CtrlDxEdit.obj
 0002:00009b9c       ??_R3CCtrlDxIMEEditBox@@8  1006bb9c     CtrlDxEdit.obj
 0002:00009bac       ??_R2CCtrlDxIMEEditBox@@8  1006bbac     CtrlDxEdit.obj
 0002:00009bc0       ??_R1A@?0A@EA@CCtrlDxIMEEditBox@@8 1006bbc0     CtrlDxEdit.obj
 0002:00009bdc       ??_R4CCtrlMultilineEditWZ@@6B@ 1006bbdc     CtrlDxEdit.obj
 0002:00009bf0       ??_R3CCtrlMultilineEditWZ@@8 1006bbf0     CtrlDxEdit.obj
 0002:00009c00       ??_R2CCtrlMultilineEditWZ@@8 1006bc00     CtrlDxEdit.obj
 0002:00009c18       ??_R1A@?0A@EA@CCtrlMultilineEditWZ@@8 1006bc18     CtrlDxEdit.obj
 0002:00009c34       ??_R4CCtrlEditWZ@@6B@      1006bc34     CtrlEditWZ.obj
 0002:00009c48       ??_R3CCtrlEditWZ@@8        1006bc48     CtrlEditWZ.obj
 0002:00009c58       ??_R2CCtrlEditWZ@@8        1006bc58     CtrlEditWZ.obj
 0002:00009c68       ??_R1A@?0A@EA@CCtrlEditWZ@@8 1006bc68     CtrlEditWZ.obj
 0002:00009c84       ??_R4CCtrlHScrollWZ@@6B@   1006bc84     CtrlHScrollWZ.obj
 0002:00009c98       ??_R3CCtrlHScrollWZ@@8     1006bc98     CtrlHScrollWZ.obj
 0002:00009ca8       ??_R2CCtrlHScrollWZ@@8     1006bca8     CtrlHScrollWZ.obj
 0002:00009cb4       ??_R1A@?0A@EA@CCtrlHScrollWZ@@8 1006bcb4     CtrlHScrollWZ.obj
 0002:00009cd0       ??_R4CCtrlListWZ@@6B@      1006bcd0     CtrlListWZ.obj
 0002:00009ce4       ??_R3CCtrlListWZ@@8        1006bce4     CtrlListWZ.obj
 0002:00009cf4       ??_R2CCtrlListWZ@@8        1006bcf4     CtrlListWZ.obj
 0002:00009d00       ??_R1A@?0A@EA@CCtrlListWZ@@8 1006bd00     CtrlListWZ.obj
 0002:00009d1c       ??_R4out_of_range@std@@6B@ 1006bd1c     CtrlListWZ.obj
 0002:00009d30       ??_R3out_of_range@std@@8   1006bd30     CtrlListWZ.obj
 0002:00009d40       ??_R2out_of_range@std@@8   1006bd40     CtrlListWZ.obj
 0002:00009d50       ??_R1A@?0A@EA@out_of_range@std@@8 1006bd50     CtrlListWZ.obj
 0002:00009d6c       ??_R4CCtrlPictureWZ@@6B@   1006bd6c     CtrlPictureWZ.obj
 0002:00009d80       ??_R3CCtrlPictureWZ@@8     1006bd80     CtrlPictureWZ.obj
 0002:00009d90       ??_R2CCtrlPictureWZ@@8     1006bd90     CtrlPictureWZ.obj
 0002:00009d9c       ??_R1A@?0A@EA@CCtrlPictureWZ@@8 1006bd9c     CtrlPictureWZ.obj
 0002:00009db8       ??_R4CCtrlRectangleWZ@@6B@ 1006bdb8     CtrlRectangleWZ.obj
 0002:00009dcc       ??_R3CCtrlRectangleWZ@@8   1006bdcc     CtrlRectangleWZ.obj
 0002:00009ddc       ??_R2CCtrlRectangleWZ@@8   1006bddc     CtrlRectangleWZ.obj
 0002:00009de8       ??_R1A@?0A@EA@CCtrlRectangleWZ@@8 1006bde8     CtrlRectangleWZ.obj
 0002:00009e04       ??_R4CCtrlStaticWZ@@6B@    1006be04     CtrlStaticWZ.obj
 0002:00009e18       ??_R3CCtrlStaticWZ@@8      1006be18     CtrlStaticWZ.obj
 0002:00009e28       ??_R2CCtrlStaticWZ@@8      1006be28     CtrlStaticWZ.obj
 0002:00009e34       ??_R1A@?0A@EA@CCtrlStaticWZ@@8 1006be34     CtrlStaticWZ.obj
 0002:00009e50       ??_R4CCtrlImageStaticWZ@@6B@ 1006be50     CtrlStaticWZ.obj
 0002:00009e64       ??_R3CCtrlImageStaticWZ@@8 1006be64     CtrlStaticWZ.obj
 0002:00009e74       ??_R2CCtrlImageStaticWZ@@8 1006be74     CtrlStaticWZ.obj
 0002:00009e84       ??_R1A@?0A@EA@CCtrlImageStaticWZ@@8 1006be84     CtrlStaticWZ.obj
 0002:00009ea0       ??_R4CCtrlTabWZ@@6B@       1006bea0     CtrlTabWZ.obj
 0002:00009eb4       ??_R3CCtrlTabWZ@@8         1006beb4     CtrlTabWZ.obj
 0002:00009ec4       ??_R2CCtrlTabWZ@@8         1006bec4     CtrlTabWZ.obj
 0002:00009ed0       ??_R1A@?0A@EA@CCtrlTabWZ@@8 1006bed0     CtrlTabWZ.obj
 0002:00009eec       ??_R4CCtrlVScrollWZ@@6B@   1006beec     CtrlVScrollWZ.obj
 0002:00009f00       ??_R3CCtrlVScrollWZ@@8     1006bf00     CtrlVScrollWZ.obj
 0002:00009f10       ??_R2CCtrlVScrollWZ@@8     1006bf10     CtrlVScrollWZ.obj
 0002:00009f1c       ??_R1A@?0A@EA@CCtrlVScrollWZ@@8 1006bf1c     CtrlVScrollWZ.obj
 0002:00009f38       ??_R4CCtrlWebBrowserWZ@@6B@ 1006bf38     CtrlWebBrowserWZ.obj
 0002:00009f4c       ??_R3CCtrlWebBrowserWZ@@8  1006bf4c     CtrlWebBrowserWZ.obj
 0002:00009f5c       ??_R2CCtrlWebBrowserWZ@@8  1006bf5c     CtrlWebBrowserWZ.obj
 0002:00009f68       ??_R1A@?0A@EA@CCtrlWebBrowserWZ@@8 1006bf68     CtrlWebBrowserWZ.obj
 0002:00009f84       ??_R4CDialogWZ@@6B@        1006bf84     DialogWZ.obj
 0002:00009f98       ??_R3CDialogWZ@@8          1006bf98     DialogWZ.obj
 0002:00009fa8       ??_R2CDialogWZ@@8          1006bfa8     DialogWZ.obj
 0002:00009fb4       ??_R1A@?0A@EA@CDialogWZ@@8 1006bfb4     DialogWZ.obj
 0002:00009fd0       ??_R1A@?0A@EA@CDlgBaseWZ@@8 1006bfd0     DialogWZ.obj
 0002:00009fec       ??_R3CDlgBaseWZ@@8         1006bfec     DialogWZ.obj
 0002:00009ffc       ??_R2CDlgBaseWZ@@8         1006bffc     DialogWZ.obj
 0002:0000a004       ??_R4CDlgBaseWZ@@6B@       1006c004     DlgBaseWZ.obj
 0002:0000a018       ??_R4CDialogManager@@6B@   1006c018     DialogManager.obj
 0002:0000a02c       ??_R3CDialogManager@@8     1006c02c     DialogManager.obj
 0002:0000a03c       ??_R2CDialogManager@@8     1006c03c     DialogManager.obj
 0002:0000a044       ??_R1A@?0A@EA@CDialogManager@@8 1006c044     DialogManager.obj
 0002:0000a060       ??_R4CDrawCtrl@@6B@        1006c060     DrawCtrl.obj
 0002:0000a074       ??_R3CDrawCtrl@@8          1006c074     DrawCtrl.obj
 0002:0000a084       ??_R2CDrawCtrl@@8          1006c084     DrawCtrl.obj
 0002:0000a08c       ??_R1A@?0A@EA@CDrawCtrl@@8 1006c08c     DrawCtrl.obj
 0002:0000a0a8       ??_R4?$CWzSingleton@VWzLogSystem@WzLog@@@@6B@ 1006c0a8     programcommonlibforengine:wzlogsystem.obj
 0002:0000a0bc       ??_R3?$CWzSingleton@VWzLogSystem@WzLog@@@@8 1006c0bc     programcommonlibforengine:wzlogsystem.obj
 0002:0000a0cc       ??_R2?$CWzSingleton@VWzLogSystem@WzLog@@@@8 1006c0cc     programcommonlibforengine:wzlogsystem.obj
 0002:0000a0d4       ??_R1A@?0A@EA@?$CWzSingleton@VWzLogSystem@WzLog@@@@8 1006c0d4     programcommonlibforengine:wzlogsystem.obj
 0002:0000a0f0       ??_R4WzLogSystem@WzLog@@6B@ 1006c0f0     programcommonlibforengine:wzlogsystem.obj
 0002:0000a104       ??_R3WzLogSystem@WzLog@@8  1006c104     programcommonlibforengine:wzlogsystem.obj
 0002:0000a114       ??_R2WzLogSystem@WzLog@@8  1006c114     programcommonlibforengine:wzlogsystem.obj
 0002:0000a120       ??_R1A@?0A@EA@WzLogSystem@WzLog@@8 1006c120     programcommonlibforengine:wzlogsystem.obj
 0002:0000a13c       ??_R4?$CWzHandleManager@USt_DAFileInfo@@@@6B@ 1006c13c     programcommonlibforengine:discaccess.obj
 0002:0000a150       ??_R3?$CWzHandleManager@USt_DAFileInfo@@@@8 1006c150     programcommonlibforengine:discaccess.obj
 0002:0000a160       ??_R2?$CWzHandleManager@USt_DAFileInfo@@@@8 1006c160     programcommonlibforengine:discaccess.obj
 0002:0000a168       ??_R1A@?0A@EA@?$CWzHandleManager@USt_DAFileInfo@@@@8 1006c168     programcommonlibforengine:discaccess.obj
 0002:0000a184       ??_R4type_info@@6B@        1006c184     LIBCMT:typinfo.obj
 0002:0000a198       ??_R3type_info@@8          1006c198     LIBCMT:typinfo.obj
 0002:0000a1a8       ??_R2type_info@@8          1006c1a8     LIBCMT:typinfo.obj
 0002:0000a1b0       ??_R1A@?0A@EA@type_info@@8 1006c1b0     LIBCMT:typinfo.obj
 0002:0000a1cc       ??_R4exception@std@@6B@    1006c1cc     LIBCMT:stdexcpt.obj
 0002:0000a1e0       ??_R4bad_exception@std@@6B@ 1006c1e0     LIBCMT:frame.obj
 0002:0000a1f4       ??_R3bad_exception@std@@8  1006c1f4     LIBCMT:frame.obj
 0002:0000a204       ??_R2bad_exception@std@@8  1006c204     LIBCMT:frame.obj
 0002:0000a210       ??_R1A@?0A@EA@bad_exception@std@@8 1006c210     LIBCMT:frame.obj
 0002:0000a230       ___safe_se_handler_table   1006c230     <linker-defined>
 0002:0000a40c       ___rtc_iaa                 1006c40c     LIBCMT:_initsect_.obj
 0002:0000a410       ___rtc_izz                 1006c410     LIBCMT:_initsect_.obj
 0002:0000a414       ___rtc_taa                 1006c414     LIBCMT:_initsect_.obj
 0002:0000a418       ___rtc_tzz                 1006c418     LIBCMT:_initsect_.obj
 0002:0000a584       __TI3?AVlength_error@std@@ 1006c584     BaseManager.obj
 0002:0000a5c0       __CTA3?AVlength_error@std@@ 1006c5c0     BaseManager.obj
 0002:0000a5d0       __CT??_R0?AVlength_error@std@@@8??0length_error@std@@QAE@ABV01@@Z40 1006c5d0     BaseManager.obj
 0002:0000a5ec       __CT??_R0?AVlogic_error@std@@@8??0logic_error@std@@QAE@ABV01@@Z40 1006c5ec     BaseManager.obj
 0002:0000a608       __CT??_R0?AVexception@std@@@8??0exception@std@@QAE@ABV01@@Z12 1006c608     BaseManager.obj
 0002:0000a6d4       __TI2?AVbad_alloc@std@@    1006c6d4     BaseManager.obj
 0002:0000a6e4       __CTA2?AVbad_alloc@std@@   1006c6e4     BaseManager.obj
 0002:0000a6f0       __CT??_R0?AVbad_alloc@std@@@8??0bad_alloc@std@@QAE@ABV01@@Z12 1006c6f0     BaseManager.obj
 0002:0000b37c       __TI3?AVout_of_range@std@@ 1006d37c     CtrlListWZ.obj
 0002:0000b3b8       __CTA3?AVout_of_range@std@@ 1006d3b8     CtrlListWZ.obj
 0002:0000b3c8       __CT??_R0?AVout_of_range@std@@@8??0out_of_range@std@@QAE@ABV01@@Z40 1006d3c8     CtrlListWZ.obj
 0002:0000b7f4       __TI1?AVCAtlException@ATL@@ 1006d7f4     CtrlWebBrowserWZ.obj
 0002:0000b804       __CTA1?AVCAtlException@ATL@@ 1006d804     CtrlWebBrowserWZ.obj
 0002:0000b80c       __CT??_R0?AVCAtlException@ATL@@@84 1006d80c     CtrlWebBrowserWZ.obj
 0002:0000c194       __TI2?AVbad_exception@std@@ 1006e194     LIBCMT:frame.obj
 0002:0000c1a4       __CTA2?AVbad_exception@std@@ 1006e1a4     LIBCMT:frame.obj
 0002:0000c1b0       __CT??_R0?AVbad_exception@std@@@8??0bad_exception@std@@QAE@ABV01@@Z12 1006e1b0     LIBCMT:frame.obj
 0002:0000c56c       __TI1?AV_com_error@@       1006e56c     comsuppw:comraise.obj
 0002:0000c57c       __CTA1?AV_com_error@@      1006e57c     comsuppw:comraise.obj
 0002:0000c584       __CT??_R0?AV_com_error@@@8??0_com_error@@QAE@ABV0@@Z16 1006e584     comsuppw:comraise.obj
 0002:0000c5a0       __IMPORT_DESCRIPTOR_KERNEL32 1006e5a0     kernel32:KERNEL32.dll
 0002:0000c5b4       __IMPORT_DESCRIPTOR_USER32 1006e5b4     user32:USER32.dll
 0002:0000c5c8       __IMPORT_DESCRIPTOR_GDI32  1006e5c8     gdi32:GDI32.dll
 0002:0000c5dc       __IMPORT_DESCRIPTOR_ADVAPI32 1006e5dc     advapi32:ADVAPI32.dll
 0002:0000c5f0       __IMPORT_DESCRIPTOR_ole32  1006e5f0     ole32:ole32.dll
 0002:0000c604       __IMPORT_DESCRIPTOR_OLEAUT32 1006e604     oleaut32:OLEAUT32.dll
 0002:0000c618       __IMPORT_DESCRIPTOR_3DRendererD3D 1006e618     3drendererd3d:3DRendererD3D.dll
 0002:0000c62c       __NULL_IMPORT_DESCRIPTOR   1006e62c     kernel32:KERNEL32.dll
 0003:00000004       ??_R0?AVCBaseManager@@@8   10070004     BaseManager.obj
 0003:00000020       ??_R0?AVlength_error@std@@@8 10070020     BaseManager.obj
 0003:00000040       ??_R0?AVlogic_error@std@@@8 10070040     BaseManager.obj
 0003:00000060       ??_R0?AVexception@std@@@8  10070060     BaseManager.obj
 0003:0000007c       ??_R0?AVbad_alloc@std@@@8  1007007c     BaseManager.obj
 0003:000000b0       ??_R0?AVCControlWZ@@@8     100700b0     ControlWZ.obj
 0003:000000e4       ??_R0?AVCCtrlButtonCheckWZ@@@8 100700e4     CtrlButtonCheckWZ.obj
 0003:00000108       ??_R0?AVCCtrlButtonWZ@@@8  10070108     CtrlButtonCheckWZ.obj
 0003:00000124       ??_R0?AVCCtrlClientWZ@@@8  10070124     CtrlClientWZ.obj
 0003:00000140       ??_R0?AVCCtrlComboBoxWZ@@@8 10070140     CtrlComboBox.obj
 0003:00000164       ?_ScriptApplyDigitSubstitution@CUniBuffer@CCtrlDxEditBox@@0P6GJPBUtag_SCRIPT_DIGITSUBSTITUTE@@PAUtag_SCRIPT_CONTROL@@PAUtag_SCRIPT_STATE@@@ZA 10070164     CtrlDxEdit.obj
 0003:00000168       ?_ScriptStringAnalyse@CUniBuffer@CCtrlDxEditBox@@0P6GJPAUHDC__@@PBXHHHKHPAUtag_SCRIPT_CONTROL@@PAUtag_SCRIPT_STATE@@PBHPAUtag_SCRIPT_TABDEF@@PBEPAPAX@ZA 10070168     CtrlDxEdit.obj
 0003:0000016c       ?_ScriptStringCPtoX@CUniBuffer@CCtrlDxEditBox@@0P6GJPAXHHPAH@ZA 1007016c     CtrlDxEdit.obj
 0003:00000170       ?_ScriptStringXtoCP@CUniBuffer@CCtrlDxEditBox@@0P6GJPAXHPAH1@ZA 10070170     CtrlDxEdit.obj
 0003:00000174       ?_ScriptStringFree@CUniBuffer@CCtrlDxEditBox@@0P6GJPAPAX@ZA 10070174     CtrlDxEdit.obj
 0003:00000178       ?_ScriptString_pLogAttr@CUniBuffer@CCtrlDxEditBox@@0P6GPBUtag_SCRIPT_LOGATTR@@PAX@ZA 10070178     CtrlDxEdit.obj
 0003:0000017c       ?_ScriptString_pcOutChars@CUniBuffer@CCtrlDxEditBox@@0P6GPBHPAX@ZA 1007017c     CtrlDxEdit.obj
 0003:00000180       ?_ImmLockIMC@CCtrlDxIMEEditBox@@1P6GPAU__MIDL___MIDL_itf_dimm_0000_0000_0012@@PAUHIMC__@@@ZA 10070180     CtrlDxEdit.obj
 0003:00000184       ?_ImmUnlockIMC@CCtrlDxIMEEditBox@@1P6GHPAUHIMC__@@@ZA 10070184     CtrlDxEdit.obj
 0003:00000188       ?_ImmLockIMCC@CCtrlDxIMEEditBox@@1P6GPAXPAUHIMCC__@@@ZA 10070188     CtrlDxEdit.obj
 0003:0000018c       ?_ImmUnlockIMCC@CCtrlDxIMEEditBox@@1P6GHPAUHIMCC__@@@ZA 1007018c     CtrlDxEdit.obj
 0003:00000190       ?_ImmDisableTextFrameService@CCtrlDxIMEEditBox@@1P6GHK@ZA 10070190     CtrlDxEdit.obj
 0003:00000194       ?_ImmGetCompositionStringW@CCtrlDxIMEEditBox@@1P6GJPAUHIMC__@@KPAXK@ZA 10070194     CtrlDxEdit.obj
 0003:00000198       ?_ImmGetCandidateListW@CCtrlDxIMEEditBox@@1P6GKPAUHIMC__@@KPAUtagCANDIDATELIST@@K@ZA 10070198     CtrlDxEdit.obj
 0003:0000019c       ?_ImmGetContext@CCtrlDxIMEEditBox@@1P6GPAUHIMC__@@PAUHWND__@@@ZA 1007019c     CtrlDxEdit.obj
 0003:000001a0       ?_ImmReleaseContext@CCtrlDxIMEEditBox@@1P6GHPAUHWND__@@PAUHIMC__@@@ZA 100701a0     CtrlDxEdit.obj
 0003:000001a4       ?_ImmAssociateContext@CCtrlDxIMEEditBox@@1P6GPAUHIMC__@@PAUHWND__@@PAU2@@ZA 100701a4     CtrlDxEdit.obj
 0003:000001a8       ?_ImmGetOpenStatus@CCtrlDxIMEEditBox@@1P6GHPAUHIMC__@@@ZA 100701a8     CtrlDxEdit.obj
 0003:000001ac       ?_ImmSetOpenStatus@CCtrlDxIMEEditBox@@1P6GHPAUHIMC__@@H@ZA 100701ac     CtrlDxEdit.obj
 0003:000001b0       ?_ImmGetConversionStatus@CCtrlDxIMEEditBox@@1P6GHPAUHIMC__@@PAK1@ZA 100701b0     CtrlDxEdit.obj
 0003:000001b4       ?_ImmGetDefaultIMEWnd@CCtrlDxIMEEditBox@@1P6GPAUHWND__@@PAU2@@ZA 100701b4     CtrlDxEdit.obj
 0003:000001b8       ?_ImmGetIMEFileNameA@CCtrlDxIMEEditBox@@1P6GIPAUHKL__@@PADI@ZA 100701b8     CtrlDxEdit.obj
 0003:000001bc       ?_ImmGetVirtualKey@CCtrlDxIMEEditBox@@1P6GIPAUHWND__@@@ZA 100701bc     CtrlDxEdit.obj
 0003:000001c0       ?_ImmNotifyIME@CCtrlDxIMEEditBox@@1P6GHPAUHIMC__@@KKK@ZA 100701c0     CtrlDxEdit.obj
 0003:000001c4       ?_ImmSetConversionStatus@CCtrlDxIMEEditBox@@1P6GHPAUHIMC__@@KK@ZA 100701c4     CtrlDxEdit.obj
 0003:000001c8       ?_ImmSimulateHotKey@CCtrlDxIMEEditBox@@1P6GHPAUHWND__@@K@ZA 100701c8     CtrlDxEdit.obj
 0003:000001cc       ?_ImmIsIME@CCtrlDxIMEEditBox@@1P6GHPAUHKL__@@@ZA 100701cc     CtrlDxEdit.obj
 0003:000001d0       ?_ImmGetProperty@CCtrlDxIMEEditBox@@1P6GKPAUHKL__@@K@ZA 100701d0     CtrlDxEdit.obj
 0003:000001d4       ?_ImmSetCompositionWindow@CCtrlDxIMEEditBox@@1P6GHPAUHIMC__@@PAUtagCOMPOSITIONFORM@@@ZA 100701d4     CtrlDxEdit.obj
 0003:000001d8       ?_GetReadingString@CCtrlDxIMEEditBox@@1P6GIPAUHIMC__@@IPA_WPAH2PAI@ZA 100701d8     CtrlDxEdit.obj
 0003:000001dc       ?_ShowReadingWindow@CCtrlDxIMEEditBox@@1P6GHPAUHIMC__@@H@ZA 100701dc     CtrlDxEdit.obj
 0003:000001e0       ?_VerQueryValueA@CCtrlDxIMEEditBox@@1P6GHQAXPADPAPAXPAI@ZA 100701e0     CtrlDxEdit.obj
 0003:000001e4       ?_GetFileVersionInfoA@CCtrlDxIMEEditBox@@1P6GHPADKKPAX@ZA 100701e4     CtrlDxEdit.obj
 0003:000001e8       ?_GetFileVersionInfoSizeA@CCtrlDxIMEEditBox@@1P6GKPADPAK@ZA 100701e8     CtrlDxEdit.obj
 0003:000001ec       ?s_aszIndicator@CCtrlDxIMEEditBox@@1PAY02_WA 100701ec     CtrlDxEdit.obj
 0003:0000020a       ?s_bEnableImeSystem@CCtrlDxIMEEditBox@@1_NA 1007020a     CtrlDxEdit.obj
 0003:0000020c       ?s_wszCurrIndicator@CCtrlDxIMEEditBox@@1PA_WA 1007020c     CtrlDxEdit.obj
 0003:00000210       ??_R0?AVCCtrlBaseEdit@@@8  10070210     CtrlDxEdit.obj
 0003:0000022c       ??_R0?AVCCtrlDxEditBox@@@8 1007022c     CtrlDxEdit.obj
 0003:0000024c       ??_R0?AVCCtrlDxIMEEditBox@@@8 1007024c     CtrlDxEdit.obj
 0003:00000278       ??_R0?AVCCtrlMultilineEditWZ@@@8 10070278     CtrlDxEdit.obj
 0003:000002a8       ??_R0?AVCCtrlEditWZ@@@8    100702a8     CtrlEditWZ.obj
 0003:000002c4       ??_R0?AVCCtrlHScrollWZ@@@8 100702c4     CtrlHScrollWZ.obj
 0003:000002e4       ??_R0?AVCCtrlListWZ@@@8    100702e4     CtrlListWZ.obj
 0003:00000300       ??_R0?AVout_of_range@std@@@8 10070300     CtrlListWZ.obj
 0003:00000320       ??_R0?AVCCtrlPictureWZ@@@8 10070320     CtrlPictureWZ.obj
 0003:00000340       ??_R0?AVCCtrlRectangleWZ@@@8 10070340     CtrlRectangleWZ.obj
 0003:00000360       ??_R0?AVCCtrlStaticWZ@@@8  10070360     CtrlStaticWZ.obj
 0003:0000037c       ??_R0?AVCCtrlImageStaticWZ@@@8 1007037c     CtrlStaticWZ.obj
 0003:000003a0       ??_R0?AVCCtrlTabWZ@@@8     100703a0     CtrlTabWZ.obj
 0003:000003bc       ??_R0?AVCCtrlVScrollWZ@@@8 100703bc     CtrlVScrollWZ.obj
 0003:000003dc       ??_R0?AVCCtrlWebBrowserWZ@@@8 100703dc     CtrlWebBrowserWZ.obj
 0003:000003fc       ??_R0?AVCAtlException@ATL@@@8 100703fc     CtrlWebBrowserWZ.obj
 0003:0000041c       ??_R0?AVCDialogWZ@@@8      1007041c     DialogWZ.obj
 0003:00000434       ??_R0?AVCDlgBaseWZ@@@8     10070434     DialogWZ.obj
 0003:00000450       ??_R0?AVCDialogManager@@@8 10070450     DialogManager.obj
 0003:00000470       ??_R0?AVCDrawCtrl@@@8      10070470     DrawCtrl.obj
 0003:00000490       ?g_MatMulFunc@@3P6APAUWzMatrix@@PAU1@PBU1@1@ZA 10070490     common:wzmath.obj
 0003:00000494       ?g_MatMul4x3Func@@3P6APAUWzMatrix@@PAU1@PBU1@1@ZA 10070494     common:wzmath.obj
 0003:00000498       ?g_MatRotXFunc@@3P6APAUWzMatrix@@PAU1@M@ZA 10070498     common:wzmath.obj
 0003:0000049c       ?g_MatRotYFunc@@3P6APAUWzMatrix@@PAU1@M@ZA 1007049c     common:wzmath.obj
 0003:000004a0       ?g_MatRotZFunc@@3P6APAUWzMatrix@@PAU1@M@ZA 100704a0     common:wzmath.obj
 0003:000004a4       ?g_QuatMulFunc@@3P6APAUWzQuaternion@@PAU1@PBU1@1@ZA 100704a4     common:wzmath.obj
 0003:000004b0       ?_PMPM@@3PAIA              100704b0     common:wzmath.obj
 0003:000004c0       ?_PPMM@@3PAIA              100704c0     common:wzmath.obj
 0003:000004d0       ?_MPPM@@3PAIA              100704d0     common:wzmath.obj
 0003:000004e0       ?_PM@@3PAIA                100704e0     common:wzmath.obj
 0003:000004f0       ?_MP@@3PAIA                100704f0     common:wzmath.obj
 0003:000004f8       ??_R0?AV?$CWzSingleton@VWzLogSystem@WzLog@@@@@8 100704f8     programcommonlibforengine:wzlogsystem.obj
 0003:0000052c       ??_R0?AVWzLogSystem@WzLog@@@8 1007052c     programcommonlibforengine:wzlogsystem.obj
 0003:00000550       ?g_lpszDiscType@@3PAPBDA   10070550     programcommonlibforengine:discaccess.obj
 0003:0000055c       ??_R0?AV?$CWzHandleManager@USt_DAFileInfo@@@@@8 1007055c     programcommonlibforengine:discaccess.obj
 0003:0000059c       ___security_cookie         1007059c     LIBCMT:gs_cookie.obj
 0003:000005a0       ___security_cookie_complement 100705a0     LIBCMT:gs_cookie.obj
 0003:000005a4       __fltused                  100705a4     LIBCMT:_fpinit_.obj
 0003:000005a8       __ldused                   100705a8     LIBCMT:_fpinit_.obj
 0003:000005b0       ??_R0?AVtype_info@@@8      100705b0     LIBCMT:typinfo.obj
 0003:00000614       ??_R0?AVbad_exception@std@@@8 10070614     LIBCMT:frame.obj
 0003:00000634       ___flsindex                10070634     LIBCMT:tidtable.obj
 0003:00000638       ___getvalueindex           10070638     LIBCMT:tidtable.obj
 0003:00000640       __cfltcvt_tab              10070640     LIBCMT:cmiscdat.obj
 0003:000007e0       ___initialmbcinfo          100707e0     LIBCMT:mbctype.obj
 0003:00000a00       __mbctype                  10070a00     LIBCMT:mbctype.obj
 0003:00000b08       __mbcasemap                10070b08     LIBCMT:mbctype.obj
 0003:00000c08       ___ptmbcinfo               10070c08     LIBCMT:mbctype.obj
 0003:00000d04       ___globallocalestatus      10070d04     LIBCMT:glstatus.obj
 0003:00000d08       ___clocalestr              10070d08     LIBCMT:nlsdata2.obj
 0003:00000d10       ___initiallocinfo          10070d10     LIBCMT:nlsdata2.obj
 0003:00000de8       ___ptlocinfo               10070de8     LIBCMT:nlsdata2.obj
 0003:00000dec       ___lc_clike                10070dec     LIBCMT:nlsdata2.obj
 0003:00000df0       ___initiallocalestructinfo 10070df0     LIBCMT:nlsdata2.obj
 0003:00000df8       __iob                      10070df8     LIBCMT:_file.obj
 0003:00001078       ___badioinfo               10071078     LIBCMT:ioinit.obj
 0003:000010b8       ___nullstring              100710b8     LIBCMT:output.obj
 0003:000010bc       ___wnullstring             100710bc     LIBCMT:output.obj
 0003:000010c0       __aexit_rtn                100710c0     LIBCMT:crt0dat.obj
 0003:000010d0       __HUGE                     100710d0     LIBCMT:_huge_.obj
 0003:000011f8       __amblksiz                 100711f8     LIBCMT:heapinit.obj
 0003:00001200       __indefinite               10071200     LIBCMT:_87disp_.obj
 0003:0000120a       __piby2                    1007120a     LIBCMT:_87disp_.obj
 0003:00001230       ___abort_behavior          10071230     LIBCMT:abort.obj
 0003:000012f0       __First_FPE_Indx           100712f0     LIBCMT:winxfltr.obj
 0003:000012f4       __Num_FPE                  100712f4     LIBCMT:winxfltr.obj
 0003:000012f8       __XcptActTabSize           100712f8     LIBCMT:winxfltr.obj
 0003:000012fc       __XcptActTabCount          100712fc     LIBCMT:winxfltr.obj
 0003:00001300       __NLG_Destination          10071300     LIBCMT:exsup.obj
 0003:00001310       __pctype                   10071310     LIBCMT:ctype.obj
 0003:00001314       __pwctype                  10071314     LIBCMT:ctype.obj
 0003:00001318       ___lc_time_c               10071318     LIBCMT:strftime.obj
 0003:000013d0       ___lc_time_curr            100713d0     LIBCMT:strftime.obj
 0003:000013d4       ___lconv_static_decimal    100713d4     LIBCMT:lconv.obj
 0003:000013d8       ___lconv_c                 100713d8     LIBCMT:lconv.obj
 0003:00001408       ___lconv                   10071408     LIBCMT:lconv.obj
 0003:0000140c       ___mb_cur_max              1007140c     LIBCMT:nlsdata1.obj
 0003:00001410       ___decimal_point           10071410     LIBCMT:nlsdata1.obj
 0003:00001414       ___decimal_point_length    10071414     LIBCMT:nlsdata1.obj
 0003:00001450       __timezone                 10071450     LIBCMT:timeset.obj
 0003:00001454       __daylight                 10071454     LIBCMT:timeset.obj
 0003:00001458       __dstbias                  10071458     LIBCMT:timeset.obj
 0003:000014e0       __tzname                   100714e0     LIBCMT:timeset.obj
 0003:00001510       __lookuptrailbytes         10071510     LIBCMT:read.obj
 0003:00001610       __pow10pos                 10071610     LIBCMT:_constpow_.obj
 0003:00001770       __pow10neg                 10071770     LIBCMT:_constpow_.obj
 0003:000019b8       __matherr_flag             100719b8     LIBCMT:_matherr_.obj
 0003:000019d8       __lpdays                   100719d8     LIBCMT:days.obj
 0003:00001a0c       __days                     10071a0c     LIBCMT:days.obj
 0003:00001a40       __coninpfh                 10071a40     LIBCMT:initcon.obj
 0003:00001a44       __confh                    10071a44     LIBCMT:initcon.obj
 0003:00001a48       __d_inf                    10071a48     LIBCMT:_util_.obj
 0003:00001a50       __d_ind                    10071a50     LIBCMT:_util_.obj
 0003:00001a58       __d_max                    10071a58     LIBCMT:_util_.obj
 0003:00001a60       __d_min                    10071a60     LIBCMT:_util_.obj
 0003:00001a68       __d_mzero                  10071a68     LIBCMT:_util_.obj
 0003:00001a84       _cchCurDir                 10071a84     wzFilePacker_static:vFile_util.obj
 0003:00001bcc       ?__errorPfn@@3P6GXJPAUIErrorInfo@@@ZA 10071bcc     comsuppw:comsupp.obj
 0003:00001bd0       ??_R0?AV_com_error@@@8     10071bd0     comsuppw:comraise.obj
 0003:00001c00       ?s_instance@?$CWzSingleton@VWzLogSystem@WzLog@@@@0PAVWzLogSystem@WzLog@@A 10071c00     dllaccess.obj
 0003:00003c28       ?s_hklCurrent@CCtrlDxIMEEditBox@@1PAUHKL__@@A 10073c28     CtrlDxEdit.obj
 0003:00003c2c       ?s_hDllIme@CCtrlDxIMEEditBox@@1PAUHINSTANCE__@@A 10073c2c     CtrlDxEdit.obj
 0003:00003c30       ?s_adwCompStringClause@CCtrlDxIMEEditBox@@1PAKA 10073c30     CtrlDxEdit.obj
 0003:00004030       ?s_wszReadingString@CCtrlDxIMEEditBox@@1PA_WA 10074030     CtrlDxEdit.obj
 0003:00004070       ?s_hDllImm32@CCtrlDxIMEEditBox@@0PAUHINSTANCE__@@A 10074070     CtrlDxEdit.obj
 0003:00004074       ?s_bVerticalCand@CCtrlDxIMEEditBox@@1_NA 10074074     CtrlDxEdit.obj
 0003:00004075       ?s_bHorizontalReading@CCtrlDxIMEEditBox@@1_NA 10074075     CtrlDxEdit.obj
 0003:00004076       ?s_bInsertOnType@CCtrlDxIMEEditBox@@1_NA 10074076     CtrlDxEdit.obj
 0003:00004077       ?s_bUseDefWindowCandidate@CCtrlDxIMEEditBox@@1_NA 10074077     CtrlDxEdit.obj
 0003:00004078       ?s_abCompStringAttr@CCtrlDxIMEEditBox@@1PAEA 10074078     CtrlDxEdit.obj
 0003:00004178       ?s_nCompCaret@CCtrlDxIMEEditBox@@1HA 10074178     CtrlDxEdit.obj
 0003:0000417c       ?s_dwProperty@CCtrlDxIMEEditBox@@1KA 1007417c     CtrlDxEdit.obj
 0003:00004180       ?s_hDllVer@CCtrlDxIMEEditBox@@0PAUHINSTANCE__@@A 10074180     CtrlDxEdit.obj
 0003:00004184       ?s_nFirstTargetConv@CCtrlDxIMEEditBox@@1HA 10074184     CtrlDxEdit.obj
 0003:00004188       ?s_bHideCaret@CCtrlDxEditBox@@1_NA 10074188     CtrlDxEdit.obj
 0003:00004189       ?s_bChineseIME@CCtrlDxIMEEditBox@@1_NA 10074189     CtrlDxEdit.obj
 0003:0000418a       ?s_bShowReadingWindow@CCtrlDxIMEEditBox@@1_NA 1007418a     CtrlDxEdit.obj
 0003:0000418c       ?s_ptCompString@CCtrlDxIMEEditBox@@1UtagPOINT@@A 1007418c     CtrlDxEdit.obj
 0003:00004194       ?s_hImcDef@CCtrlDxIMEEditBox@@0PAUHIMC__@@A 10074194     CtrlDxEdit.obj
 0003:00004198       ?s_hWnd@CCtrlDxIMEEditBox@@2PAUHWND__@@A 10074198     CtrlDxEdit.obj
 0003:0000419c       ?s_hDll@CUniBuffer@CCtrlDxEditBox@@0PAUHINSTANCE__@@A 1007419c     CtrlDxEdit.obj
 0003:000041a0       ?s_ImeState@CCtrlDxIMEEditBox@@1W4IMESTATE@1@A 100741a0     CtrlDxEdit.obj
 0003:000041a4       ?EXTERNAL_API_INITIALIZER@@3VCExternalApiInitializer@@A 100741a4     CtrlDxEdit.obj
 0003:000041a8       ?s_Locale@CCtrlDxIMEEditBox@@1V?$CGrowableArray@UCInputLocale@CCtrlDxIMEEditBox@@@@A 100741a8     CtrlDxEdit.obj
 0003:000041b8       ?s_CandList@CCtrlDxIMEEditBox@@1UCCandList@1@A 100741b8     CtrlDxEdit.obj
 0003:00005614       ?m_spWebBW@CCtrlWebBrowserWZ@@2PAXA 10075614     CtrlWebBrowserWZ.obj
 0003:00005618       ?m_hWebDlg@CCtrlWebBrowserWZ@@1PAUHWND__@@A 10075618     CtrlWebBrowserWZ.obj
 0003:00005624       ?static_mousecursor_pos@CDialogWZ@@2UtagPOINT@@A 10075624     DialogWZ.obj
 0003:0000562c       ?static_stdListEditPtr@CDialogWZ@@2V?$list@PAVCControlWZ@@V?$allocator@PAVCControlWZ@@@std@@@std@@A 1007562c     DialogWZ.obj
 0003:00005648       ?m_sLockDlgID@CDialogManager@@2KA 10075648     DialogManager.obj
 0003:00005c64       ?m_dummyData@?$CWzHandleManager@USt_DAFileInfo@@@@1USt_DAFileInfo@@A 10075c64     programcommonlibforengine:discaccess.obj
 0003:00005c6c       ?m_nullData@?$CWzHandleManager@USt_DAFileInfo@@@@1USt_DAFileInfo@@A 10075c6c     programcommonlibforengine:discaccess.obj
 0003:00005c74       ?m_dummyData@?$CWzArray@USt_DAFileInfo@@@@0USt_DAFileInfo@@A 10075c74     programcommonlibforengine:discaccess.obj
 0003:00005c7c       ?m_dummyData@?$CWzArray@G@@0GA 10075c7c     programcommonlibforengine:discaccess.obj
 0003:00005c90       ___fastflag                10075c90     LIBCMT:_fpinit_.obj
 0003:00005c94       __adjust_fdiv              10075c94     LIBCMT:_fpinit_.obj
 0003:00005c98       ___pInvalidArgHandler      10075c98     LIBCMT:invarg.obj
 0003:00005ca0       __aenvptr                  10075ca0     LIBCMT:dllcrt0.obj
 0003:00005ca4       __wenvptr                  10075ca4     LIBCMT:dllcrt0.obj
 0003:00005ca8       ___error_mode              10075ca8     LIBCMT:dllcrt0.obj
 0003:00005cac       ___app_type                10075cac     LIBCMT:dllcrt0.obj
 0003:00005cb0       ?_pnhHeap@@3P6AHI@ZA       10075cb0     LIBCMT:handler.obj
 0003:00005cb4       _gpFlsAlloc                10075cb4     LIBCMT:tidtable.obj
 0003:00005cb8       _gpFlsGetValue             10075cb8     LIBCMT:tidtable.obj
 0003:00005cbc       _gpFlsSetValue             10075cbc     LIBCMT:tidtable.obj
 0003:00005cc0       _gpFlsFree                 10075cc0     LIBCMT:tidtable.obj
 0003:00005cc4       ?__pInconsistency@@3P6AXXZA 10075cc4     LIBCMT:hooks.obj
 0003:00005ff8       ___mbulinfo                10075ff8     LIBCMT:mbctype.obj
 0003:00006004       ___mbcodepage              10076004     LIBCMT:mbctype.obj
 0003:00006008       ___ismbcodepage            10076008     LIBCMT:mbctype.obj
 0003:0000600c       ___mblcid                  1007600c     LIBCMT:mbctype.obj
 0003:00006010       ___locale_changed          10076010     LIBCMT:setlocal.obj
 0003:00006014       ___lc_handle               10076014     LIBCMT:nlsdata2.obj
 0003:0000602c       ___lc_codepage             1007602c     LIBCMT:nlsdata2.obj
 0003:00006030       ___lc_collate_cp           10076030     LIBCMT:nlsdata2.obj
 0003:00006034       __cflush                   10076034     LIBCMT:_file.obj
 0003:00006038       __stdbuf                   10076038     LIBCMT:_sftbuf.obj
 0003:00006040       __maxwait                  10076040     LIBCMT:crtheap.obj
 0003:00006044       __umaskval                 10076044     LIBCMT:crt0dat.obj
 0003:00006048       ___argc                    10076048     LIBCMT:crt0dat.obj
 0003:0000604c       ___argv                    1007604c     LIBCMT:crt0dat.obj
 0003:00006050       ___wargv                   10076050     LIBCMT:crt0dat.obj
 0003:00006054       __environ                  10076054     LIBCMT:crt0dat.obj
 0003:00006058       ___initenv                 10076058     LIBCMT:crt0dat.obj
 0003:0000605c       __wenviron                 1007605c     LIBCMT:crt0dat.obj
 0003:00006060       ___winitenv                10076060     LIBCMT:crt0dat.obj
 0003:00006064       __pgmptr                   10076064     LIBCMT:crt0dat.obj
 0003:00006068       __wpgmptr                  10076068     LIBCMT:crt0dat.obj
 0003:0000606c       __exitflag                 1007606c     LIBCMT:crt0dat.obj
 0003:00006070       __C_Termination_Done       10076070     LIBCMT:crt0dat.obj
 0003:00006074       __C_Exit_Done              10076074     LIBCMT:crt0dat.obj
 0003:00006078       __newmode                  10076078     LIBCMT:_newmode.obj
 0003:000061d0       __crtheap                  100761d0     LIBCMT:heapinit.obj
 0003:000061d4       ___sbh_pHeaderDefer        100761d4     LIBCMT:sbheap.obj
 0003:000064f4       ___pPurecall               100764f4     LIBCMT:inithelp.obj
 0003:00006604       __outputformat             10076604     LIBCMT:outputformat.obj
 0003:0000661c       ?pArgList@UnDecorator@@0PAVReplicator@@A 1007661c     LIBCMT:undname.obj
 0003:00006620       ?pZNameList@UnDecorator@@0PAVReplicator@@A 10076620     LIBCMT:undname.obj
 0003:00006624       ?pTemplateArgList@UnDecorator@@0PAVReplicator@@A 10076624     LIBCMT:undname.obj
 0003:00006628       ?gName@UnDecorator@@0PBDB  10076628     LIBCMT:undname.obj
 0003:0000662c       ?name@UnDecorator@@0PBDB   1007662c     LIBCMT:undname.obj
 0003:00006630       ?outputString@UnDecorator@@0PADA 10076630     LIBCMT:undname.obj
 0003:00006634       ?maxStringLength@UnDecorator@@0HA 10076634     LIBCMT:undname.obj
 0003:00006638       ?disableFlags@UnDecorator@@0KA 10076638     LIBCMT:undname.obj
 0003:0000663c       ?m_pGetParameter@UnDecorator@@0P6APADJ@ZA 1007663c     LIBCMT:undname.obj
 0003:00006640       ?fExplicitTemplateParams@UnDecorator@@0_NA 10076640     LIBCMT:undname.obj
 0003:00006641       ?fGetTemplateArgumentList@UnDecorator@@0_NA 10076641     LIBCMT:undname.obj
 0003:0000664c       ___lconv_static_null       1007664c     LIBCMT:lconv.obj
 0003:00006658       __commode                  10076658     LIBCMT:ncommode.obj
 0003:00006748       __fmode                    10076748     LIBCMT:txtmode.obj
 0003:0000674c       ?autofree@@3VCAutoFree@@A  1007674c     wzFilePacker_static:wzFilePacker.obj
 0003:00006758       _dwTreeCount               10076758     wzFilePacker_static:vfile.obj
 0003:0000675c       _g_nTreeArrayCount         1007675c     wzFilePacker_static:vfile.obj
 0003:00006760       _g_ulStartBinaryOffset     10076760     wzFilePacker_static:vfile.obj
 0003:00006768       _g_ulTatalBinarySize       10076768     wzFilePacker_static:vfile.obj
 0003:00006774       _bCurDirCreated            10076774     wzFilePacker_static:vFile_util.obj
 0003:00007084       __pmatherr                 10077084     <common>
 0003:00007088       ___use_sse2_mathfcns       10077088     <common>
 0003:0000708c       ___sbh_cntHeaderList       1007708c     <common>
 0003:00007090       ___sbh_pHeaderList         10077090     <common>
 0003:00007094       ___sbh_threshold           10077094     <common>
 0003:00007098       ___sbh_pHeaderScan         10077098     <common>
 0003:0000709c       ___sbh_sizeHeaderList      1007709c     <common>
 0003:000070a0       ___sbh_indGroupDefer       100770a0     <common>
 0003:000070a4       ___active_heap             100770a4     <common>
 0003:000070a8       ___env_initialized         100770a8     <common>
 0003:000070ac       ___onexitend               100770ac     <common>
 0003:000070b0       ___onexitbegin             100770b0     <common>
 0003:000070b4       ___mbctype_initialized     100770b4     <common>
 0003:000070b8       ___dyn_tls_init_callback   100770b8     <common>
 0003:000070bc       __nhandle                  100770bc     <common>
 0003:000070c0       ___pioinfo                 100770c0     <common>
 0003:000071c0       ___piob                    100771c0     <common>
 0003:000071e0       __bufin                    100771e0     <common>
 0003:000081e0       __nstream                  100781e0     <common>
 0003:000081e4       ___sse2_available          100781e4     <common>
 0003:000081e8       __debugger_hook_dummy      100781e8     <common>
 0003:000081ec       __acmdln                   100781ec     <common>
 0003:000081f0       _StupidUnusedPointer       100781f0     <common>
 0003:00008200       _g_TreeList                10078200     <common>

 entry point at        0001:00048a44

 Static symbols

 0001:0000148d       __catch$?_Buynode@?$list@PAXV?$allocator@PAX@std@@@std@@IAEPAU_Node@?$_List_nod@PAXV?$allocator@PAX@std@@@2@PAU342@0ABQAX@Z$0 1000248d f i BaseManager.obj
 0001:0000148d       __catch$?_Buynode@?$list@PAVCControlWZ@@V?$allocator@PAVCControlWZ@@@std@@@std@@IAEPAU_Node@?$_List_nod@PAVCControlWZ@@V?$allocator@PAVCControlWZ@@@std@@@2@PAU342@0ABQAVCControlWZ@@@Z$0 1000248d f i BaseManager.obj
 0001:0000148d       __catch$?_Buynode@?$list@KV?$allocator@K@std@@@std@@IAEPAU_Node@?$_List_nod@KV?$allocator@K@std@@@2@PAU342@0ABK@Z$0 1000248d f i BaseManager.obj
 0001:00001f43       __catch$?_Buynode@?$list@U?$pair@$$CBKPAX@std@@V?$allocator@U?$pair@$$CBKPAX@std@@@2@@std@@IAEPAU_Node@?$_List_nod@U?$pair@$$CBKPAX@std@@V?$allocator@U?$pair@$$CBKPAX@std@@@2@@2@XZ$0 10002f43 f i BaseManager.obj
 0001:000023ba       __catch$?_Buynode@?$list@U?$pair@$$CBKPAX@std@@V?$allocator@U?$pair@$$CBKPAX@std@@@2@@std@@IAEPAU_Node@?$_List_nod@U?$pair@$$CBKPAX@std@@V?$allocator@U?$pair@$$CBKPAX@std@@@2@@2@PAU342@0ABU?$pair@$$CBKPAX@2@@Z$0 100033ba f i BaseManager.obj
 0001:00002798       __catch$??$_Insert@V?$_Const_iterator@$00@?$list@U?$pair@$$CBKPAX@std@@V?$allocator@U?$pair@$$CBKPAX@std@@@2@@std@@@?$list@U?$pair@$$CBKPAX@std@@V?$allocator@U?$pair@$$CBKPAX@std@@@2@@std@@QAEXV?$_Const_iterator@$00@01@00Uforward_iterator_tag@1@@Z$0 10003798 f i BaseManager.obj
 0001:00002ae6       __catch$??$_Uninit_copy@PAU_List_position@?$_Hash@V?$_Hmap_traits@KPAXV?$hash_compare@KU?$less@K@std@@@stdext@@V?$allocator@U?$pair@$$CBKPAX@std@@@std@@$0A@@stdext@@@stdext@@PAU123@V?$allocator@U_List_position@?$_Hash@V?$_Hmap_traits@KPAXV?$hash_compare@KU?$less@K@std@@@stdext@@V?$allocator@U?$pair@$$CBKPAX@std@@@std@@$0A@@stdext@@@stdext@@@std@@@std@@YAPAU_List_position@?$_Hash@V?$_Hmap_traits@KPAXV?$hash_compare@KU?$less@K@std@@@stdext@@V?$allocator@U?$pair@$$CBKPAX@std@@@std@@$0A@@stdext@@@stdext@@PAU123@00AAV?$allocator@U_List_position@?$_Hash@V?$_Hmap_traits@KPAXV?$hash_compare@KU?$less@K@std@@@stdext@@V?$allocator@U?$pair@$$CBKPAX@std@@@std@@$0A@@stdext@@@stdext@@@0@U_Nonscalar_ptr_iterator_tag@0@U_Range_checked_iterator_tag@0@@Z$0 10003ae6 f i BaseManager.obj
 0001:00002ae6       __catch$??$_Uninit_copy@PAU_List_position@?$_Hash@V?$_Hmap_traits@KV?$basic_string@DU?$char_traits@D@std@@V?$allocator@D@2@@std@@V?$hash_compare@KU?$less@K@std@@@stdext@@V?$allocator@U?$pair@$$CBKV?$basic_string@DU?$char_traits@D@std@@V?$allocator@D@2@@std@@@std@@@2@$0A@@stdext@@@stdext@@PAU123@V?$allocator@U_List_position@?$_Hash@V?$_Hmap_traits@KV?$basic_string@DU?$char_traits@D@std@@V?$allocator@D@2@@std@@V?$hash_compare@KU?$less@K@std@@@stdext@@V?$allocator@U?$pair@$$CBKV?$basic_string@DU?$char_traits@D@std@@V?$allocator@D@2@@std@@@std@@@2@$0A@@stdext@@@stdext@@@std@@@std@@YAPAU_List_position@?$_Hash@V?$_Hmap_traits@KV?$basic_string@DU?$char_traits@D@std@@V?$allocator@D@2@@std@@V?$hash_compare@KU?$less@K@std@@@stdext@@V?$allocator@U?$pair@$$CBKV?$basic_string@DU?$char_traits@D@std@@V?$allocator@D@2@@std@@@std@@@2@$0A@@stdext@@@stdext@@PAU123@00AAV?$allocator@U_List_position@?$_Hash@V?$_Hmap_traits@KV?$basic_string@DU?$char_traits@D@std@@V?$allocator@D@2@@std@@V?$hash_compare@KU?$less@K@std@@@stdext@@V?$allocator@U?$pair@$$CBKV?$basic_string@DU?$char_traits@D@std@@V?$allocator@D@2@@std@@@std@@@2@$0A@@stdext@@@stdext@@@0@U_Nonscalar_ptr_iterator_tag@0@U_Range_checked_iterator_tag@0@@Z$0 10003ae6 f i BaseManager.obj
 0001:000031a4       __catch$?_Copy@?$basic_string@DU?$char_traits@D@std@@V?$allocator@D@2@@std@@IAEXII@Z$0 100041a4 f i BaseManager.obj
 0001:000031d0       __catch$?_Copy@?$basic_string@DU?$char_traits@D@std@@V?$allocator@D@2@@std@@IAEXII@Z$1 100041d0 f i BaseManager.obj
 0001:00005503       __catch$?_Buynode@?$list@U?$pair@$$CBKV?$basic_string@DU?$char_traits@D@std@@V?$allocator@D@2@@std@@@std@@V?$allocator@U?$pair@$$CBKV?$basic_string@DU?$char_traits@D@std@@V?$allocator@D@2@@std@@@std@@@2@@std@@IAEPAU_Node@?$_List_nod@U?$pair@$$CBKV?$basic_string@DU?$char_traits@D@std@@V?$allocator@D@2@@std@@@std@@V?$allocator@U?$pair@$$CBKV?$basic_string@DU?$char_traits@D@std@@V?$allocator@D@2@@std@@@std@@@2@@2@XZ$0 10006503 f i StringManager.obj
 0001:00005bb6       __catch$?_Buynode@?$list@U?$pair@$$CBKV?$basic_string@DU?$char_traits@D@std@@V?$allocator@D@2@@std@@@std@@V?$allocator@U?$pair@$$CBKV?$basic_string@DU?$char_traits@D@std@@V?$allocator@D@2@@std@@@std@@@2@@std@@IAEPAU_Node@?$_List_nod@U?$pair@$$CBKV?$basic_string@DU?$char_traits@D@std@@V?$allocator@D@2@@std@@@std@@V?$allocator@U?$pair@$$CBKV?$basic_string@DU?$char_traits@D@std@@V?$allocator@D@2@@std@@@std@@@2@@2@PAU342@0ABU?$pair@$$CBKV?$basic_string@DU?$char_traits@D@std@@V?$allocator@D@2@@std@@@2@@Z$0 10006bb6 f i StringManager.obj
 0001:00005efd       __catch$?_Insert_n@?$vector@U_List_position@?$_Hash@V?$_Hmap_traits@KPAXV?$hash_compare@KU?$less@K@std@@@stdext@@V?$allocator@U?$pair@$$CBKPAX@std@@@std@@$0A@@stdext@@@stdext@@V?$allocator@U_List_position@?$_Hash@V?$_Hmap_traits@KPAXV?$hash_compare@KU?$less@K@std@@@stdext@@V?$allocator@U?$pair@$$CBKPAX@std@@@std@@$0A@@stdext@@@stdext@@@std@@@std@@IAEXV?$_Vector_const_iterator@U_List_position@?$_Hash@V?$_Hmap_traits@KPAXV?$hash_compare@KU?$less@K@std@@@stdext@@V?$allocator@U?$pair@$$CBKPAX@std@@@std@@$0A@@stdext@@@stdext@@V?$allocator@U_List_position@?$_Hash@V?$_Hmap_traits@KPAXV?$hash_compare@KU?$less@K@std@@@stdext@@V?$allocator@U?$pair@$$CBKPAX@std@@@std@@$0A@@stdext@@@stdext@@@std@@@2@IABU_List_position@?$_Hash@V?$_Hmap_traits@KPAXV?$hash_compare@KU?$less@K@std@@@stdext@@V?$allocator@U?$pair@$$CBKPAX@std@@@std@@$0A@@stdext@@@stdext@@@Z$0 10006efd f i StringManager.obj
 0001:00005efd       __catch$?_Insert_n@?$vector@U_List_position@?$_Hash@V?$_Hmap_traits@KV?$basic_string@DU?$char_traits@D@std@@V?$allocator@D@2@@std@@V?$hash_compare@KU?$less@K@std@@@stdext@@V?$allocator@U?$pair@$$CBKV?$basic_string@DU?$char_traits@D@std@@V?$allocator@D@2@@std@@@std@@@2@$0A@@stdext@@@stdext@@V?$allocator@U_List_position@?$_Hash@V?$_Hmap_traits@KV?$basic_string@DU?$char_traits@D@std@@V?$allocator@D@2@@std@@V?$hash_compare@KU?$less@K@std@@@stdext@@V?$allocator@U?$pair@$$CBKV?$basic_string@DU?$char_traits@D@std@@V?$allocator@D@2@@std@@@std@@@2@$0A@@stdext@@@stdext@@@std@@@std@@IAEXV?$_Vector_const_iterator@U_List_position@?$_Hash@V?$_Hmap_traits@KV?$basic_string@DU?$char_traits@D@std@@V?$allocator@D@2@@std@@V?$hash_compare@KU?$less@K@std@@@stdext@@V?$allocator@U?$pair@$$CBKV?$basic_string@DU?$char_traits@D@std@@V?$allocator@D@2@@std@@@std@@@2@$0A@@stdext@@@stdext@@V?$allocator@U_List_position@?$_Hash@V?$_Hmap_traits@KV?$basic_string@DU?$char_traits@D@std@@V?$allocator@D@2@@std@@V?$hash_compare@KU?$less@K@std@@@stdext@@V?$allocator@U?$pair@$$CBKV?$basic_string@DU?$char_traits@D@std@@V?$allocator@D@2@@std@@@std@@@2@$0A@@stdext@@@stdext@@@std@@@2@IABU_List_position@?$_Hash@V?$_Hmap_traits@KV?$basic_string@DU?$char_traits@D@std@@V?$allocator@D@2@@std@@V?$hash_compare@KU?$less@K@std@@@stdext@@V?$allocator@U?$pair@$$CBKV?$basic_string@DU?$char_traits@D@std@@V?$allocator@D@2@@std@@@std@@@2@$0A@@stdext@@@stdext@@@Z$0 10006efd f i StringManager.obj
 0001:000061b7       __catch$?_Insert_n@?$vector@U_List_position@?$_Hash@V?$_Hmap_traits@KPAXV?$hash_compare@KU?$less@K@std@@@stdext@@V?$allocator@U?$pair@$$CBKPAX@std@@@std@@$0A@@stdext@@@stdext@@V?$allocator@U_List_position@?$_Hash@V?$_Hmap_traits@KPAXV?$hash_compare@KU?$less@K@std@@@stdext@@V?$allocator@U?$pair@$$CBKPAX@std@@@std@@$0A@@stdext@@@stdext@@@std@@@std@@IAEXV?$_Vector_const_iterator@U_List_position@?$_Hash@V?$_Hmap_traits@KPAXV?$hash_compare@KU?$less@K@std@@@stdext@@V?$allocator@U?$pair@$$CBKPAX@std@@@std@@$0A@@stdext@@@stdext@@V?$allocator@U_List_position@?$_Hash@V?$_Hmap_traits@KPAXV?$hash_compare@KU?$less@K@std@@@stdext@@V?$allocator@U?$pair@$$CBKPAX@std@@@std@@$0A@@stdext@@@stdext@@@std@@@2@IABU_List_position@?$_Hash@V?$_Hmap_traits@KPAXV?$hash_compare@KU?$less@K@std@@@stdext@@V?$allocator@U?$pair@$$CBKPAX@std@@@std@@$0A@@stdext@@@stdext@@@Z$2 100071b7 f i StringManager.obj
 0001:000061b7       __catch$?_Insert_n@?$vector@U_List_position@?$_Hash@V?$_Hmap_traits@KV?$basic_string@DU?$char_traits@D@std@@V?$allocator@D@2@@std@@V?$hash_compare@KU?$less@K@std@@@stdext@@V?$allocator@U?$pair@$$CBKV?$basic_string@DU?$char_traits@D@std@@V?$allocator@D@2@@std@@@std@@@2@$0A@@stdext@@@stdext@@V?$allocator@U_List_position@?$_Hash@V?$_Hmap_traits@KV?$basic_string@DU?$char_traits@D@std@@V?$allocator@D@2@@std@@V?$hash_compare@KU?$less@K@std@@@stdext@@V?$allocator@U?$pair@$$CBKV?$basic_string@DU?$char_traits@D@std@@V?$allocator@D@2@@std@@@std@@@2@$0A@@stdext@@@stdext@@@std@@@std@@IAEXV?$_Vector_const_iterator@U_List_position@?$_Hash@V?$_Hmap_traits@KV?$basic_string@DU?$char_traits@D@std@@V?$allocator@D@2@@std@@V?$hash_compare@KU?$less@K@std@@@stdext@@V?$allocator@U?$pair@$$CBKV?$basic_string@DU?$char_traits@D@std@@V?$allocator@D@2@@std@@@std@@@2@$0A@@stdext@@@stdext@@V?$allocator@U_List_position@?$_Hash@V?$_Hmap_traits@KV?$basic_string@DU?$char_traits@D@std@@V?$allocator@D@2@@std@@V?$hash_compare@KU?$less@K@std@@@stdext@@V?$allocator@U?$pair@$$CBKV?$basic_string@DU?$char_traits@D@std@@V?$allocator@D@2@@std@@@std@@@2@$0A@@stdext@@@stdext@@@std@@@2@IABU_List_position@?$_Hash@V?$_Hmap_traits@KV?$basic_string@DU?$char_traits@D@std@@V?$allocator@D@2@@std@@V?$hash_compare@KU?$less@K@std@@@stdext@@V?$allocator@U?$pair@$$CBKV?$basic_string@DU?$char_traits@D@std@@V?$allocator@D@2@@std@@@std@@@2@$0A@@stdext@@@stdext@@@Z$2 100071b7 f i StringManager.obj
 0001:000065cd       __catch$??$_Insert@V?$_Const_iterator@$00@?$list@U?$pair@$$CBKV?$basic_string@DU?$char_traits@D@std@@V?$allocator@D@2@@std@@@std@@V?$allocator@U?$pair@$$CBKV?$basic_string@DU?$char_traits@D@std@@V?$allocator@D@2@@std@@@std@@@2@@std@@@?$list@U?$pair@$$CBKV?$basic_string@DU?$char_traits@D@std@@V?$allocator@D@2@@std@@@std@@V?$allocator@U?$pair@$$CBKV?$basic_string@DU?$char_traits@D@std@@V?$allocator@D@2@@std@@@std@@@2@@std@@QAEXV?$_Const_iterator@$00@01@00Uforward_iterator_tag@1@@Z$0 100075cd f i StringManager.obj
 0001:000066c5       __catch$??$_Uninit_fill_n@PAU_List_position@?$_Hash@V?$_Hmap_traits@KPAXV?$hash_compare@KU?$less@K@std@@@stdext@@V?$allocator@U?$pair@$$CBKPAX@std@@@std@@$0A@@stdext@@@stdext@@IU123@V?$allocator@U_List_position@?$_Hash@V?$_Hmap_traits@KPAXV?$hash_compare@KU?$less@K@std@@@stdext@@V?$allocator@U?$pair@$$CBKPAX@std@@@std@@$0A@@stdext@@@stdext@@@std@@@std@@YAXPAU_List_position@?$_Hash@V?$_Hmap_traits@KPAXV?$hash_compare@KU?$less@K@std@@@stdext@@V?$allocator@U?$pair@$$CBKPAX@std@@@std@@$0A@@stdext@@@stdext@@IABU123@AAV?$allocator@U_List_position@?$_Hash@V?$_Hmap_traits@KPAXV?$hash_compare@KU?$less@K@std@@@stdext@@V?$allocator@U?$pair@$$CBKPAX@std@@@std@@$0A@@stdext@@@stdext@@@0@U_Nonscalar_ptr_iterator_tag@0@U_Range_checked_iterator_tag@0@@Z$0 100076c5 f i StringManager.obj
 0001:000066c5       __catch$??$_Uninit_fill_n@PAU_List_position@?$_Hash@V?$_Hmap_traits@KV?$basic_string@DU?$char_traits@D@std@@V?$allocator@D@2@@std@@V?$hash_compare@KU?$less@K@std@@@stdext@@V?$allocator@U?$pair@$$CBKV?$basic_string@DU?$char_traits@D@std@@V?$allocator@D@2@@std@@@std@@@2@$0A@@stdext@@@stdext@@IU123@V?$allocator@U_List_position@?$_Hash@V?$_Hmap_traits@KV?$basic_string@DU?$char_traits@D@std@@V?$allocator@D@2@@std@@V?$hash_compare@KU?$less@K@std@@@stdext@@V?$allocator@U?$pair@$$CBKV?$basic_string@DU?$char_traits@D@std@@V?$allocator@D@2@@std@@@std@@@2@$0A@@stdext@@@stdext@@@std@@@std@@YAXPAU_List_position@?$_Hash@V?$_Hmap_traits@KV?$basic_string@DU?$char_traits@D@std@@V?$allocator@D@2@@std@@V?$hash_compare@KU?$less@K@std@@@stdext@@V?$allocator@U?$pair@$$CBKV?$basic_string@DU?$char_traits@D@std@@V?$allocator@D@2@@std@@@std@@@2@$0A@@stdext@@@stdext@@IABU123@AAV?$allocator@U_List_position@?$_Hash@V?$_Hmap_traits@KV?$basic_string@DU?$char_traits@D@std@@V?$allocator@D@2@@std@@V?$hash_compare@KU?$less@K@std@@@stdext@@V?$allocator@U?$pair@$$CBKV?$basic_string@DU?$char_traits@D@std@@V?$allocator@D@2@@std@@@std@@@2@$0A@@stdext@@@stdext@@@0@U_Nonscalar_ptr_iterator_tag@0@U_Range_checked_iterator_tag@0@@Z$0 100076c5 f i StringManager.obj
 0001:000150e5       _swprintf                  100160e5 f   CtrlDxEdit.obj
 0001:0001f91a       __catch$?_Insert_n@?$vector@KV?$allocator@K@std@@@std@@IAEXV?$_Vector_const_iterator@KV?$allocator@K@std@@@2@IABK@Z$0 1002091a f i CtrlDxEdit.obj
 0001:0001fb45       __catch$?_Insert_n@?$vector@KV?$allocator@K@std@@@std@@IAEXV?$_Vector_const_iterator@KV?$allocator@K@std@@@2@IABK@Z$2 10020b45 f i CtrlDxEdit.obj
 0001:0002d59e       __catch$?_Buynode@?$_Tree@V?$_Tmap_traits@V?$basic_string@DU?$char_traits@D@std@@V?$allocator@D@2@@std@@PAXU?$less@V?$basic_string@DU?$char_traits@D@std@@V?$allocator@D@2@@std@@@2@V?$allocator@U?$pair@$$CBV?$basic_string@DU?$char_traits@D@std@@V?$allocator@D@2@@std@@PAX@std@@@2@$00@std@@@std@@IAEPAU_Node@?$_Tree_nod@V?$_Tmap_traits@V?$basic_string@DU?$char_traits@D@std@@V?$allocator@D@2@@std@@PAXU?$less@V?$basic_string@DU?$char_traits@D@std@@V?$allocator@D@2@@std@@@2@V?$allocator@U?$pair@$$CBV?$basic_string@DU?$char_traits@D@std@@V?$allocator@D@2@@std@@PAX@std@@@2@$00@std@@@2@XZ$0 1002e59e f i CtrlListWZ.obj
 0001:0002d680       __catch$?_Buynode@?$_Tree@V?$_Tmap_traits@V?$basic_string@DU?$char_traits@D@std@@V?$allocator@D@2@@std@@PAXU?$less@V?$basic_string@DU?$char_traits@D@std@@V?$allocator@D@2@@std@@@2@V?$allocator@U?$pair@$$CBV?$basic_string@DU?$char_traits@D@std@@V?$allocator@D@2@@std@@PAX@std@@@2@$00@std@@@std@@IAEPAU_Node@?$_Tree_nod@V?$_Tmap_traits@V?$basic_string@DU?$char_traits@D@std@@V?$allocator@D@2@@std@@PAXU?$less@V?$basic_string@DU?$char_traits@D@std@@V?$allocator@D@2@@std@@@2@V?$allocator@U?$pair@$$CBV?$basic_string@DU?$char_traits@D@std@@V?$allocator@D@2@@std@@PAX@std@@@2@$00@std@@@2@PAU342@00ABU?$pair@$$CBV?$basic_string@DU?$char_traits@D@std@@V?$allocator@D@2@@std@@PAX@2@D@Z$0 1002e680 f i CtrlListWZ.obj
 0001:0003459e       __catch$?_Buynode@?$_Tree@V?$_Tmap_traits@KKU?$less@K@std@@V?$allocator@U?$pair@$$CBKK@std@@@2@$0A@@std@@@std@@IAEPAU_Node@?$_Tree_nod@V?$_Tmap_traits@KKU?$less@K@std@@V?$allocator@U?$pair@$$CBKK@std@@@2@$0A@@std@@@2@XZ$0 1003559e f i CtrlTabWZ.obj
 0001:0003459e       __catch$?_Buynode@?$_Tree@V?$_Tmap_traits@KPAUCListSellData@CCtrlListWZ@@U?$less@K@std@@V?$allocator@U?$pair@$$CBKPAUCListSellData@CCtrlListWZ@@@std@@@4@$0A@@std@@@std@@IAEPAU_Node@?$_Tree_nod@V?$_Tmap_traits@KPAUCListSellData@CCtrlListWZ@@U?$less@K@std@@V?$allocator@U?$pair@$$CBKPAUCListSellData@CCtrlListWZ@@@std@@@4@$0A@@std@@@2@XZ$0 1003559e f i CtrlTabWZ.obj
 0001:0003459e       __catch$?_Buynode@?$_Tree@V?$_Tmap_traits@KPAXU?$less@K@std@@V?$allocator@U?$pair@$$CBKPAX@std@@@2@$0A@@std@@@std@@IAEPAU_Node@?$_Tree_nod@V?$_Tmap_traits@KPAXU?$less@K@std@@V?$allocator@U?$pair@$$CBKPAX@std@@@2@$0A@@std@@@2@XZ$0 1003559e f i CtrlTabWZ.obj
 0001:0003467b       __catch$?_Buynode@?$_Tree@V?$_Tmap_traits@KPAUCListSellData@CCtrlListWZ@@U?$less@K@std@@V?$allocator@U?$pair@$$CBKPAUCListSellData@CCtrlListWZ@@@std@@@4@$0A@@std@@@std@@IAEPAU_Node@?$_Tree_nod@V?$_Tmap_traits@KPAUCListSellData@CCtrlListWZ@@U?$less@K@std@@V?$allocator@U?$pair@$$CBKPAUCListSellData@CCtrlListWZ@@@std@@@4@$0A@@std@@@2@PAU342@00ABU?$pair@$$CBKPAUCListSellData@CCtrlListWZ@@@2@D@Z$0 1003567b f i CtrlTabWZ.obj
 0001:0003467b       __catch$?_Buynode@?$_Tree@V?$_Tmap_traits@KPAXU?$less@K@std@@V?$allocator@U?$pair@$$CBKPAX@std@@@2@$0A@@std@@@std@@IAEPAU_Node@?$_Tree_nod@V?$_Tmap_traits@KPAXU?$less@K@std@@V?$allocator@U?$pair@$$CBKPAX@std@@@2@$0A@@std@@@2@PAU342@00ABU?$pair@$$CBKPAX@2@D@Z$0 1003567b f i CtrlTabWZ.obj
 0001:0003467b       __catch$?_Buynode@?$_Tree@V?$_Tmap_traits@KKU?$less@K@std@@V?$allocator@U?$pair@$$CBKK@std@@@2@$0A@@std@@@std@@IAEPAU_Node@?$_Tree_nod@V?$_Tmap_traits@KKU?$less@K@std@@V?$allocator@U?$pair@$$CBKK@std@@@2@$0A@@std@@@2@PAU342@00ABU?$pair@$$CBKK@2@D@Z$0 1003567b f i CtrlTabWZ.obj
 0001:0003a91b       __catch$?_Buynode@?$list@UtagRECT@@V?$allocator@UtagRECT@@@std@@@std@@IAEPAU_Node@?$_List_nod@UtagRECT@@V?$allocator@UtagRECT@@@std@@@2@XZ$0 1003b91b f i DialogWZ.obj
 0001:0003aa23       __catch$?_Buynode@?$list@UtagRECT@@V?$allocator@UtagRECT@@@std@@@std@@IAEPAU_Node@?$_List_nod@UtagRECT@@V?$allocator@UtagRECT@@@std@@@2@PAU342@0ABUtagRECT@@@Z$0 1003ba23 f i DialogWZ.obj
 0001:0003ac93       __catch$?_Buynode@?$list@PAXV?$allocator@PAX@std@@@std@@IAEPAU_Node@?$_List_nod@PAXV?$allocator@PAX@std@@@2@XZ$0 1003bc93 f i DialogWZ.obj
 0001:0003ac93       __catch$?_Buynode@?$list@KV?$allocator@K@std@@@std@@IAEPAU_Node@?$_List_nod@KV?$allocator@K@std@@@2@XZ$0 1003bc93 f i DialogWZ.obj
 0001:0003ac93       __catch$?_Buynode@?$list@PAVCControlWZ@@V?$allocator@PAVCControlWZ@@@std@@@std@@IAEPAU_Node@?$_List_nod@PAVCControlWZ@@V?$allocator@PAVCControlWZ@@@std@@@2@XZ$0 1003bc93 f i DialogWZ.obj
 0001:0004627b       ?CatchGuardHandler@@YA?AW4_EXCEPTION_DISPOSITION@@PAUEHExceptionRecord@@PAUCatchGuardRN@@PAX2@Z 1004727b f   LIBCMT:_trnsctrl_.obj
 0001:00046385       ?TranslatorGuardHandler@@YA?AW4_EXCEPTION_DISPOSITION@@PAUEHExceptionRecord@@PAUTranslatorGuardRN@@PAX2@Z 10047385 f   LIBCMT:_trnsctrl_.obj
 0001:00047234       __onexit_nolock            10048234 f   LIBCMT:onexit.obj
 0001:0004814f       ?wcstoxl@@YAKPAUlocaleinfo_struct@@PB_WPAPB_WHH@Z 1004914f f   LIBCMT:wcstol.obj
 0001:00048749       ?x_ismbbtype_l@@YAHPAUlocaleinfo_struct@@IHH@Z 10049749 f   LIBCMT:ismbbyte.obj
 0001:0004894e       ___DllMainCRTStartup       1004994e f   LIBCMT:dllcrt0.obj
 0001:0004945d       ?ExFilterRethrow@@YAHPAU_EXCEPTION_POINTERS@@@Z 1004a45d f   LIBCMT:frame.obj
 0001:00049520       ?IsInExceptionSpec@@YAEPAUEHExceptionRecord@@PBU_s_ESTypeList@@@Z 1004a520 f   LIBCMT:frame.obj
 0001:0004959b       ?CallUnexpected@@YAXPBU_s_ESTypeList@@@Z 1004a59b f   LIBCMT:frame.obj
 0001:000495cc       __catch$?CallUnexpected@@YAXPBU_s_ESTypeList@@@Z$0 1004a5cc f   LIBCMT:frame.obj
 0001:000495e4       ?CallCatchBlock@@YAPAXPAUEHExceptionRecord@@PAUEHRegistrationNode@@PAU_CONTEXT@@PBU_s_FuncInfo@@PAXHK@Z 1004a5e4 f   LIBCMT:frame.obj
 0001:00049991       ?CatchIt@@YAXPAUEHExceptionRecord@@PAUEHRegistrationNode@@PAU_CONTEXT@@PAXPBU_s_FuncInfo@@PBU_s_HandlerType@@PBU_s_CatchableType@@PBU_s_TryBlockMapEntry@@H1E@Z 1004a991 f   LIBCMT:frame.obj
 0001:000499ff       ?FindHandlerForForeignException@@YAXPAUEHExceptionRecord@@PAUEHRegistrationNode@@PAU_CONTEXT@@PAXPBU_s_FuncInfo@@HH1@Z 1004a9ff f   LIBCMT:frame.obj
 0001:00049af3       ?FindHandler@@YAXPAUEHExceptionRecord@@PAUEHRegistrationNode@@PAU_CONTEXT@@PAXPBU_s_FuncInfo@@EH1@Z 1004aaf3 f   LIBCMT:frame.obj
 0001:0004a89f       __shift                    1004b89f f   LIBCMT:cvt.obj
 0001:0004a8e4       __cftoe2_l                 1004b8e4 f   LIBCMT:cvt.obj
 0001:0004aeb6       __cftof2_l                 1004beb6 f   LIBCMT:cvt.obj
 0001:0004b4b3       ?strtoxl@@YAKPAUlocaleinfo_struct@@PBDPAPBDHH@Z 1004c4b3 f   LIBCMT:strtol.obj
 0001:0004b70d       ?strtoxq@@YA_KPAUlocaleinfo_struct@@PBDPAPBDHH@Z 1004c70d f   LIBCMT:strtoq.obj
 0001:0004b9cf       ?CPtoLCID@@YAHH@Z          1004c9cf f   LIBCMT:mbctype.obj
 0001:0004b9fe       ?setSBCS@@YAXPAUthreadmbcinfostruct@@@Z 1004c9fe f   LIBCMT:mbctype.obj
 0001:0004ba62       ?setSBUpLow@@YAXPAUthreadmbcinfostruct@@@Z 1004ca62 f   LIBCMT:mbctype.obj
 0001:0004bc99       ?getSystemCP@@YAHH@Z       1004cc99 f   LIBCMT:mbctype.obj
 0001:0004c323       __updatetlocinfoEx_nolock  1004d323 f   LIBCMT:setlocal.obj
 0001:0004c518       _fastzero_I                1004d518 f   LIBCMT:p4_memset.obj
 0001:0004c5fe       _has_osfxsr_set            1004d5fe f   LIBCMT:cpu_disp.obj
 0001:0004c939       _flsall                    1004d939 f   LIBCMT:fflush.obj
 0001:0004d265       _write_char                1004e265 f   LIBCMT:output.obj
 0001:0004d298       _write_multi_char          1004e298 f   LIBCMT:output.obj
 0001:0004d2be       _write_string              1004e2be f   LIBCMT:output.obj
 0001:0004e334       __unwind_handler4          1004f334 f   LIBCMT:exsup4.obj
 0001:0004e627       __initterm                 1004f627 f   LIBCMT:crt0dat.obj
 0001:0004e6ed       _doexit                    1004f6ed f   LIBCMT:crt0dat.obj
 0001:0004e88c       ?wcstoxq@@YA_KPAUlocaleinfo_struct@@PB_WPAPB_WHH@Z 1004f88c f   LIBCMT:wcstoq.obj
 0001:0004eb6b       _fastcopy_I                1004fb6b f   LIBCMT:p4_memcpy.obj
 0001:0004ee2d       _write_char                1004fe2d f   LIBCMT:woutput.obj
 0001:0004ee5c       _write_multi_char          1004fe5c f   LIBCMT:woutput.obj
 0001:0004ee83       _write_string              1004fe83 f   LIBCMT:woutput.obj
 0001:0005133c       _parse_cmdline             1005233c f   LIBCMT:stdargv.obj
 0001:000521d8       __unwind_handler           100531d8 f   LIBCMT:exsup.obj
 0001:000529f5       ?__crtLCMapStringA_stat@@YAHPAUlocaleinfo_struct@@KKPBDHPADHHH@Z 100539f5 f   LIBCMT:a_map.obj
 0001:00052ddf       ?__crtGetStringTypeA_stat@@YAHPAUlocaleinfo_struct@@KPBDHPAGHHH@Z 10053ddf f   LIBCMT:a_str.obj
 0001:00054612       __tsopen_nolock            10055612 f   LIBCMT:open.obj
 0001:00055322       _siglookup                 10056322 f   LIBCMT:winsig.obj
 0001:00057fbe       __hw_cw                    10058fbe f   LIBCMT:_ieee87_.obj
 0001:0005804c       ___hw_cw_sse2              1005904c f   LIBCMT:_ieee87_.obj
 0001:0005a1d0       @geVFile_RegisterFileSystemInternal@8 1005b1d0 f   wzFilePacker_static:vfile.obj
 0001:0005a240       _RegisterBuiltInAPIs       1005b240 f   wzFilePacker_static:vfile.obj
 0001:0005a2b0       @CheckOpenFlags@4          1005b2b0 f   wzFilePacker_static:vfile.obj
 0001:0005aa30       _geRam_DoCriticalCallback  1005ba30 f   wzFilePacker_static:Ram.obj
 0001:0005ab60       @FSVFS_FinderCreate@12     1005bb60 f   wzFilePacker_static:fsvfs.obj
 0001:0005abd0       @FSVFS_FinderGetNextFile@4 1005bbd0 f   wzFilePacker_static:fsvfs.obj
 0001:0005abf0       @FSVFS_FinderGetProperties@8 1005bbf0 f   wzFilePacker_static:fsvfs.obj
 0001:0005ac50       @FSVFS_FinderDestroy@4     1005bc50 f   wzFilePacker_static:fsvfs.obj
 0001:0005ac80       @FSVFS_OpenNewSystem@16    1005bc80 f   wzFilePacker_static:fsvfs.obj
 0001:0005b360       @FSVFS_MakeSpace@24        1005c360 f   wzFilePacker_static:fsvfs.obj
 0001:0005b600       @FSVFS_EnlargeDirectorySize@8 1005c600 f   wzFilePacker_static:fsvfs.obj
 0001:0005b6e0       @FSVFS_Close@4             1005c6e0 f   wzFilePacker_static:fsvfs.obj
 0001:0005b850       @ForceFilePos@4            1005c850 f   wzFilePacker_static:fsvfs.obj
 0001:0005b870       _ClampOperationSize        1005c870 f   wzFilePacker_static:fsvfs.obj
 0001:0005b8b0       @UpdateFilePos@4           1005c8b0 f   wzFilePacker_static:fsvfs.obj
 0001:0005b990       @FSVFS_GetS@12             1005c990 f   wzFilePacker_static:fsvfs.obj
 0001:0005b9e0       @FSVFS_Read@12             1005c9e0 f   wzFilePacker_static:fsvfs.obj
 0001:0005bb50       @FSVFS_Write@12            1005cb50 f   wzFilePacker_static:fsvfs.obj
 0001:0005bbb0       @FSVFS_Seek@16             1005cbb0 f   wzFilePacker_static:fsvfs.obj
 0001:0005bc40       @FSVFS_EOF@4               1005cc40 f   wzFilePacker_static:fsvfs.obj
 0001:0005bc60       @FSVFS_Tell@8              1005cc60 f   wzFilePacker_static:fsvfs.obj
 0001:0005bc80       @FSVFS_Size@8              1005cc80 f   wzFilePacker_static:fsvfs.obj
 0001:0005bca0       @FSVFS_GetProperties@8     1005cca0 f   wzFilePacker_static:fsvfs.obj
 0001:0005bcf0       @FSVFS_SetAttributes@8     1005ccf0 f   wzFilePacker_static:fsvfs.obj
 0001:0005bd10       @FSVFS_SetTime@8           1005cd10 f   wzFilePacker_static:fsvfs.obj
 0001:0005bd20       @FSVFS_SetHints@8          1005cd20 f   wzFilePacker_static:fsvfs.obj
 0001:0005bd30       @FSVFS_FileExists@12       1005cd30 f   wzFilePacker_static:fsvfs.obj
 0001:0005bd50       @FSVFS_Disperse@16         1005cd50 f   wzFilePacker_static:fsvfs.obj
 0001:0005bd50       @FSMemory_RenameFile@16    1005cd50 f   wzFilePacker_static:fsvfs.obj
 0001:0005bd50       @FSDos_UpdateContext@16    1005cd50 f   wzFilePacker_static:fsvfs.obj
 0001:0005bd50       @FSVFS_SetSize@12          1005cd50 f   wzFilePacker_static:fsvfs.obj
 0001:0005bd50       @FSDos_Disperse@16         1005cd50 f   wzFilePacker_static:fsvfs.obj
 0001:0005bd50       @FSVFS_UpdateContext@16    1005cd50 f   wzFilePacker_static:fsvfs.obj
 0001:0005bd50       @FSMemory_Disperse@16      1005cd50 f   wzFilePacker_static:fsvfs.obj
 0001:0005bd50       @FSVFS_RenameFile@16       1005cd50 f   wzFilePacker_static:fsvfs.obj
 0001:0005bd50       @FSMemory_SetSize@12       1005cd50 f   wzFilePacker_static:fsvfs.obj
 0001:0005bd60       _FSVFS_GetVoidSpace        1005cd60 f   wzFilePacker_static:fsvfs.obj
 0001:0005c1f0       _FSVFS_SetVoidSpace        1005d1f0 f   wzFilePacker_static:fsvfs.obj
 0001:0005c510       @FSVFS_Open@20             1005d510 f   wzFilePacker_static:fsvfs.obj
 0001:0005c6d0       @FSVFS_DeleteFile@12       1005d6d0 f   wzFilePacker_static:fsvfs.obj
 0001:0005c810       @FSMemory_FinderDestroy@4  1005d810 f   wzFilePacker_static:FSMEMORY.obj
 0001:0005c820       @FSMemory_Open@20          1005d820 f   wzFilePacker_static:FSMEMORY.obj
 0001:0005c830       @FSMemory_OpenNewSystem@16 1005d830 f   wzFilePacker_static:FSMEMORY.obj
 0001:0005c8f0       @FSMemory_UpdateContext@16 1005d8f0 f   wzFilePacker_static:FSMEMORY.obj
 0001:0005c920       @FSMemory_Close@4          1005d920 f   wzFilePacker_static:FSMEMORY.obj
 0001:0005c960       @ClampOperationSize@12     1005d960 f   wzFilePacker_static:FSMEMORY.obj
 0001:0005c9a0       @DataPtr@4                 1005d9a0 f   wzFilePacker_static:FSMEMORY.obj
 0001:0005c9b0       @FSMemory_GetS@12          1005d9b0 f   wzFilePacker_static:FSMEMORY.obj
 0001:0005ca10       @FSMemory_Read@12          1005da10 f   wzFilePacker_static:FSMEMORY.obj
 0001:0005ca70       @TestForExpansion@12       1005da70 f   wzFilePacker_static:FSMEMORY.obj
 0001:0005caf0       @FSMemory_Write@12         1005daf0 f   wzFilePacker_static:FSMEMORY.obj
 0001:0005cb70       @FSMemory_Seek@16          1005db70 f   wzFilePacker_static:FSMEMORY.obj
 0001:0005cc40       @FSMemory_EOF@4            1005dc40 f   wzFilePacker_static:FSMEMORY.obj
 0001:0005cc60       @FSMemory_Tell@8           1005dc60 f   wzFilePacker_static:FSMEMORY.obj
 0001:0005cc80       @FSMemory_Size@8           1005dc80 f   wzFilePacker_static:FSMEMORY.obj
 0001:0005cca0       @FSMemory_FinderCreate@12  1005dca0 f   wzFilePacker_static:FSMEMORY.obj
 0001:0005cca0       @FSMemory_FileExists@12    1005dca0 f   wzFilePacker_static:FSMEMORY.obj
 0001:0005cca0       @FSMemory_DeleteFile@12    1005dca0 f   wzFilePacker_static:FSMEMORY.obj
 0001:0005ccc0       _BuildFileName             1005dcc0 f   wzFilePacker_static:fsdos.obj
 0001:0005cd90       @FSDos_FinderCreate@12     1005dd90 f   wzFilePacker_static:fsdos.obj
 0001:0005ce60       @FSDos_FinderGetNextFile@4 1005de60 f   wzFilePacker_static:fsdos.obj
 0001:0005ced0       @FSDos_FinderGetProperties@8 1005ded0 f   wzFilePacker_static:fsdos.obj
 0001:0005cf50       @FSDos_FinderDestroy@4     1005df50 f   wzFilePacker_static:fsdos.obj
 0001:0005cf80       _IsRootDirectory           1005df80 f   wzFilePacker_static:fsdos.obj
 0001:0005cfd0       @FSDos_Open@20             1005dfd0 f   wzFilePacker_static:fsdos.obj
 0001:0005d1d0       @FSDos_OpenNewSystem@16    1005e1d0 f   wzFilePacker_static:fsdos.obj
 0001:0005d1f0       @FSDos_Close@4             1005e1f0 f   wzFilePacker_static:fsdos.obj
 0001:0005d240       @FSDos_GetS@12             1005e240 f   wzFilePacker_static:fsdos.obj
 0001:0005d320       @FSDos_Read@12             1005e320 f   wzFilePacker_static:fsdos.obj
 0001:0005d380       @FSDos_Write@12            1005e380 f   wzFilePacker_static:fsdos.obj
 0001:0005d3c0       @FSDos_Seek@16             1005e3c0 f   wzFilePacker_static:fsdos.obj
 0001:0005d480       @FSDos_EOF@4               1005e480 f   wzFilePacker_static:fsdos.obj
 0001:0005d510       @FSDos_Tell@8              1005e510 f   wzFilePacker_static:fsdos.obj
 0001:0005d580       @FSDos_Size@8              1005e580 f   wzFilePacker_static:fsdos.obj
 0001:0005d5f0       @FSDos_GetProperties@8     1005e5f0 f   wzFilePacker_static:fsdos.obj
 0001:0005d6b0       @FSDos_SetSize@12          1005e6b0 f   wzFilePacker_static:fsdos.obj
 0001:0005d700       @FSDos_SetAttributes@8     1005e700 f   wzFilePacker_static:fsdos.obj
 0001:0005d730       @FSDos_SetTime@8           1005e730 f   wzFilePacker_static:fsdos.obj
 0001:0005d760       @FSMemory_EnlargeDirectorySize@8 1005e760 f   wzFilePacker_static:fsdos.obj
 0001:0005d760       @FSDos_SetHints@8          1005e760 f   wzFilePacker_static:fsdos.obj
 0001:0005d760       @FSDos_EnlargeDirectorySize@8 1005e760 f   wzFilePacker_static:fsdos.obj
 0001:0005d760       @FSMemory_FinderGetNextFile@4 1005e760 f   wzFilePacker_static:fsdos.obj
 0001:0005d760       @FSMemory_FinderGetProperties@8 1005e760 f   wzFilePacker_static:fsdos.obj
 0001:0005d760       @FSMemory_GetProperties@8  1005e760 f   wzFilePacker_static:fsdos.obj
 0001:0005d760       @FSMemory_SetAttributes@8  1005e760 f   wzFilePacker_static:fsdos.obj
 0001:0005d760       @FSMemory_SetTime@8        1005e760 f   wzFilePacker_static:fsdos.obj
 0001:0005d760       @FSMemory_SetHints@8       1005e760 f   wzFilePacker_static:fsdos.obj
 0001:0005d770       @FSDos_FileExists@12       1005e770 f   wzFilePacker_static:fsdos.obj
 0001:0005d800       @FSDos_DeleteFile@12       1005e800 f   wzFilePacker_static:fsdos.obj
 0001:0005d890       @FSDos_RenameFile@16       1005e890 f   wzFilePacker_static:fsdos.obj
 0001:0005da00       _WriteTree                 1005ea00 f   wzFilePacker_static:dirtree.obj
 0001:0005db80       _DirTree_WriteToFile1      1005eb80 f   wzFilePacker_static:dirtree.obj
 0001:0005dd20       _ReadTree                  1005ed20 f   wzFilePacker_static:dirtree.obj
 0001:0005df70       _ReadTreeCount             1005ef70 f   wzFilePacker_static:dirtree.obj
 0001:0005efbd       __splitpath_helper         1005ffbd f   LIBCMT:splitpat.obj
 0001:0005f4c0       __unwindfunclet$??0CBaseManager@@QAE@XZ$0 100604c0 f   BaseManager.obj
 0001:0005f4cb       __ehhandler$??0CBaseManager@@QAE@XZ 100604cb f   BaseManager.obj
 0001:0005f4e6       __unwindfunclet$??1CBaseManager@@UAE@XZ$0 100604e6 f   BaseManager.obj
 0001:0005f4f1       __unwindfunclet$??1CBaseManager@@UAE@XZ$2 100604f1 f   BaseManager.obj
 0001:0005f4f9       __ehhandler$??1CBaseManager@@UAE@XZ 100604f9 f   BaseManager.obj
 0001:0005f514       __unwindfunclet$??1?$_Hash@V?$_Hmap_traits@KPAXV?$hash_compare@KU?$less@K@std@@@stdext@@V?$allocator@U?$pair@$$CBKPAX@std@@@std@@$0A@@stdext@@@stdext@@QAE@XZ$0 10060514 f   BaseManager.obj
 0001:0005f51c       __unwindfunclet$??1?$_Hash@V?$_Hmap_traits@KPAXV?$hash_compare@KU?$less@K@std@@@stdext@@V?$allocator@U?$pair@$$CBKPAX@std@@@std@@$0A@@stdext@@@stdext@@QAE@XZ$1 1006051c f   BaseManager.obj
 0001:0005f527       __unwindfunclet$??1?$_Hash@V?$_Hmap_traits@KPAXV?$hash_compare@KU?$less@K@std@@@stdext@@V?$allocator@U?$pair@$$CBKPAX@std@@@std@@$0A@@stdext@@@stdext@@QAE@XZ$3 10060527 f   BaseManager.obj
 0001:0005f52f       __unwindfunclet$??1?$_Hash@V?$_Hmap_traits@KPAXV?$hash_compare@KU?$less@K@std@@@stdext@@V?$allocator@U?$pair@$$CBKPAX@std@@@std@@$0A@@stdext@@@stdext@@QAE@XZ$6 1006052f f   BaseManager.obj
 0001:0005f537       __ehhandler$??1?$_Hash@V?$_Hmap_traits@KPAXV?$hash_compare@KU?$less@K@std@@@stdext@@V?$allocator@U?$pair@$$CBKPAX@std@@@std@@$0A@@stdext@@@stdext@@QAE@XZ 10060537 f   BaseManager.obj
 0001:0005f552       __unwindfunclet$??0?$_Hash@V?$_Hmap_traits@KPAXV?$hash_compare@KU?$less@K@std@@@stdext@@V?$allocator@U?$pair@$$CBKPAX@std@@@std@@$0A@@stdext@@@stdext@@QAE@ABV?$hash_compare@KU?$less@K@std@@@1@ABV?$allocator@U?$pair@$$CBKPAX@std@@@std@@@Z$0 10060552 f   BaseManager.obj
 0001:0005f55d       __unwindfunclet$??0?$_Hash@V?$_Hmap_traits@KPAXV?$hash_compare@KU?$less@K@std@@@stdext@@V?$allocator@U?$pair@$$CBKPAX@std@@@std@@$0A@@stdext@@@stdext@@QAE@ABV?$hash_compare@KU?$less@K@std@@@1@ABV?$allocator@U?$pair@$$CBKPAX@std@@@std@@@Z$1 1006055d f   BaseManager.obj
 0001:0005f56b       __unwindfunclet$??0?$_Hash@V?$_Hmap_traits@KPAXV?$hash_compare@KU?$less@K@std@@@stdext@@V?$allocator@U?$pair@$$CBKPAX@std@@@std@@$0A@@stdext@@@stdext@@QAE@ABV?$hash_compare@KU?$less@K@std@@@1@ABV?$allocator@U?$pair@$$CBKPAX@std@@@std@@@Z$2 1006056b f   BaseManager.obj
 0001:0005f579       __ehhandler$??0?$_Hash@V?$_Hmap_traits@KPAXV?$hash_compare@KU?$less@K@std@@@stdext@@V?$allocator@U?$pair@$$CBKPAX@std@@@std@@$0A@@stdext@@@stdext@@QAE@ABV?$hash_compare@KU?$less@K@std@@@1@ABV?$allocator@U?$pair@$$CBKPAX@std@@@std@@@Z 10060579 f   BaseManager.obj
 0001:0005f597       __unwindfunclet$??1?$list@KV?$allocator@K@std@@@std@@QAE@XZ$0 10060597 f   BaseManager.obj
 0001:0005f597       __unwindfunclet$??1?$list@UtagRECT@@V?$allocator@UtagRECT@@@std@@@std@@QAE@XZ$0 10060597 f   BaseManager.obj
 0001:0005f597       __unwindfunclet$??1?$list@U?$pair@$$CBKPAX@std@@V?$allocator@U?$pair@$$CBKPAX@std@@@2@@std@@QAE@XZ$0 10060597 f   BaseManager.obj
 0001:0005f59f       __ehhandler$??1?$list@U?$pair@$$CBKPAX@std@@V?$allocator@U?$pair@$$CBKPAX@std@@@2@@std@@QAE@XZ 1006059f f   BaseManager.obj
 0001:0005f59f       __ehhandler$??1?$list@UtagRECT@@V?$allocator@UtagRECT@@@std@@@std@@QAE@XZ 1006059f f   BaseManager.obj
 0001:0005f59f       __ehhandler$??1?$list@KV?$allocator@K@std@@@std@@QAE@XZ 1006059f f   BaseManager.obj
 0001:0005f5ba       __ehhandler$?_Buynode@?$list@PAVCControlWZ@@V?$allocator@PAVCControlWZ@@@std@@@std@@IAEPAU_Node@?$_List_nod@PAVCControlWZ@@V?$allocator@PAVCControlWZ@@@std@@@2@PAU342@0ABQAVCControlWZ@@@Z 100605ba f   BaseManager.obj
 0001:0005f5ba       __ehhandler$?_Buynode@?$list@KV?$allocator@K@std@@@std@@IAEPAU_Node@?$_List_nod@KV?$allocator@K@std@@@2@PAU342@0ABK@Z 100605ba f   BaseManager.obj
 0001:0005f5ba       __ehhandler$?_Buynode@?$list@PAXV?$allocator@PAX@std@@@std@@IAEPAU_Node@?$_List_nod@PAXV?$allocator@PAX@std@@@2@PAU342@0ABQAX@Z 100605ba f   BaseManager.obj
 0001:0005f5d5       __unwindfunclet$?_Incsize@?$list@U?$pair@$$CBKV?$basic_string@DU?$char_traits@D@std@@V?$allocator@D@2@@std@@@std@@V?$allocator@U?$pair@$$CBKV?$basic_string@DU?$char_traits@D@std@@V?$allocator@D@2@@std@@@std@@@2@@std@@IAEXI@Z$0 100605d5 f   BaseManager.obj
 0001:0005f5d5       __unwindfunclet$?_Incsize@?$list@PAVCControlWZ@@V?$allocator@PAVCControlWZ@@@std@@@std@@IAEXI@Z$0 100605d5 f   BaseManager.obj
 0001:0005f5d5       __unwindfunclet$?_Incsize@?$list@U?$pair@$$CBKPAX@std@@V?$allocator@U?$pair@$$CBKPAX@std@@@2@@std@@IAEXI@Z$0 100605d5 f   BaseManager.obj
 0001:0005f5d5       __unwindfunclet$?_Incsize@?$list@KV?$allocator@K@std@@@std@@IAEXI@Z$0 100605d5 f   BaseManager.obj
 0001:0005f5d5       __unwindfunclet$?_Incsize@?$list@UtagRECT@@V?$allocator@UtagRECT@@@std@@@std@@IAEXI@Z$0 100605d5 f   BaseManager.obj
 0001:0005f5d5       __unwindfunclet$?_Incsize@?$list@PAXV?$allocator@PAX@std@@@std@@IAEXI@Z$0 100605d5 f   BaseManager.obj
 0001:0005f5dd       __ehhandler$?_Incsize@?$list@UtagRECT@@V?$allocator@UtagRECT@@@std@@@std@@IAEXI@Z 100605dd f   BaseManager.obj
 0001:0005f5dd       __ehhandler$?_Incsize@?$list@U?$pair@$$CBKV?$basic_string@DU?$char_traits@D@std@@V?$allocator@D@2@@std@@@std@@V?$allocator@U?$pair@$$CBKV?$basic_string@DU?$char_traits@D@std@@V?$allocator@D@2@@std@@@std@@@2@@std@@IAEXI@Z 100605dd f   BaseManager.obj
 0001:0005f5dd       __ehhandler$?_Incsize@?$list@PAXV?$allocator@PAX@std@@@std@@IAEXI@Z 100605dd f   BaseManager.obj
 0001:0005f5dd       __ehhandler$?_Incsize@?$list@KV?$allocator@K@std@@@std@@IAEXI@Z 100605dd f   BaseManager.obj
 0001:0005f5dd       __ehhandler$?_Incsize@?$list@U?$pair@$$CBKPAX@std@@V?$allocator@U?$pair@$$CBKPAX@std@@@2@@std@@IAEXI@Z 100605dd f   BaseManager.obj
 0001:0005f5dd       __ehhandler$?_Incsize@?$list@PAVCControlWZ@@V?$allocator@PAVCControlWZ@@@std@@@std@@IAEXI@Z 100605dd f   BaseManager.obj
 0001:0005f5fb       __ehhandler$?_Buynode@?$list@U?$pair@$$CBKPAX@std@@V?$allocator@U?$pair@$$CBKPAX@std@@@2@@std@@IAEPAU_Node@?$_List_nod@U?$pair@$$CBKPAX@std@@V?$allocator@U?$pair@$$CBKPAX@std@@@2@@2@XZ 100605fb f   BaseManager.obj
 0001:0005f616       __ehhandler$?_Buynode@?$list@U?$pair@$$CBKPAX@std@@V?$allocator@U?$pair@$$CBKPAX@std@@@2@@std@@IAEPAU_Node@?$_List_nod@U?$pair@$$CBKPAX@std@@V?$allocator@U?$pair@$$CBKPAX@std@@@2@@2@PAU342@0ABU?$pair@$$CBKPAX@2@@Z 10060616 f   BaseManager.obj
 0001:0005f631       __ehhandler$??$_Insert@V?$_Const_iterator@$00@?$list@U?$pair@$$CBKPAX@std@@V?$allocator@U?$pair@$$CBKPAX@std@@@2@@std@@@?$list@U?$pair@$$CBKPAX@std@@V?$allocator@U?$pair@$$CBKPAX@std@@@2@@std@@QAEXV?$_Const_iterator@$00@01@00Uforward_iterator_tag@1@@Z 10060631 f   BaseManager.obj
 0001:0005f64f       __ehhandler$??$_Uninit_copy@PAU_List_position@?$_Hash@V?$_Hmap_traits@KPAXV?$hash_compare@KU?$less@K@std@@@stdext@@V?$allocator@U?$pair@$$CBKPAX@std@@@std@@$0A@@stdext@@@stdext@@PAU123@V?$allocator@U_List_position@?$_Hash@V?$_Hmap_traits@KPAXV?$hash_compare@KU?$less@K@std@@@stdext@@V?$allocator@U?$pair@$$CBKPAX@std@@@std@@$0A@@stdext@@@stdext@@@std@@@std@@YAPAU_List_position@?$_Hash@V?$_Hmap_traits@KPAXV?$hash_compare@KU?$less@K@std@@@stdext@@V?$allocator@U?$pair@$$CBKPAX@std@@@std@@$0A@@stdext@@@stdext@@PAU123@00AAV?$allocator@U_List_position@?$_Hash@V?$_Hmap_traits@KPAXV?$hash_compare@KU?$less@K@std@@@stdext@@V?$allocator@U?$pair@$$CBKPAX@std@@@std@@$0A@@stdext@@@stdext@@@0@U_Nonscalar_ptr_iterator_tag@0@U_Range_checked_iterator_tag@0@@Z 1006064f f   BaseManager.obj
 0001:0005f64f       __ehhandler$??$_Uninit_copy@PAU_List_position@?$_Hash@V?$_Hmap_traits@KV?$basic_string@DU?$char_traits@D@std@@V?$allocator@D@2@@std@@V?$hash_compare@KU?$less@K@std@@@stdext@@V?$allocator@U?$pair@$$CBKV?$basic_string@DU?$char_traits@D@std@@V?$allocator@D@2@@std@@@std@@@2@$0A@@stdext@@@stdext@@PAU123@V?$allocator@U_List_position@?$_Hash@V?$_Hmap_traits@KV?$basic_string@DU?$char_traits@D@std@@V?$allocator@D@2@@std@@V?$hash_compare@KU?$less@K@std@@@stdext@@V?$allocator@U?$pair@$$CBKV?$basic_string@DU?$char_traits@D@std@@V?$allocator@D@2@@std@@@std@@@2@$0A@@stdext@@@stdext@@@std@@@std@@YAPAU_List_position@?$_Hash@V?$_Hmap_traits@KV?$basic_string@DU?$char_traits@D@std@@V?$allocator@D@2@@std@@V?$hash_compare@KU?$less@K@std@@@stdext@@V?$allocator@U?$pair@$$CBKV?$basic_string@DU?$char_traits@D@std@@V?$allocator@D@2@@std@@@std@@@2@$0A@@stdext@@@stdext@@PAU123@00AAV?$allocator@U_List_position@?$_Hash@V?$_Hmap_traits@KV?$basic_string@DU?$char_traits@D@std@@V?$allocator@D@2@@std@@V?$hash_compare@KU?$less@K@std@@@stdext@@V?$allocator@U?$pair@$$CBKV?$basic_string@DU?$char_traits@D@std@@V?$allocator@D@2@@std@@@std@@@2@$0A@@stdext@@@stdext@@@0@U_Nonscalar_ptr_iterator_tag@0@U_Range_checked_iterator_tag@0@@Z 1006064f f   BaseManager.obj
 0001:0005f66a       __unwindfunclet$??0logic_error@std@@QAE@ABV?$basic_string@DU?$char_traits@D@std@@V?$allocator@D@2@@1@@Z$0 1006066a f   BaseManager.obj
 0001:0005f66a       __unwindfunclet$??0logic_error@std@@QAE@ABV01@@Z$0 1006066a f   BaseManager.obj
 0001:0005f672       __ehhandler$??0logic_error@std@@QAE@ABV?$basic_string@DU?$char_traits@D@std@@V?$allocator@D@2@@1@@Z 10060672 f   BaseManager.obj
 0001:0005f672       __ehhandler$??0logic_error@std@@QAE@ABV01@@Z 10060672 f   BaseManager.obj
 0001:0005f68d       __ehhandler$?_Copy@?$basic_string@DU?$char_traits@D@std@@V?$allocator@D@2@@std@@IAEXII@Z 1006068d f   BaseManager.obj
 0001:0005f6ab       __unwindfunclet$??0CStringManager@@QAE@XZ$0 100606ab f   StringManager.obj
 0001:0005f6b6       __ehhandler$??0CStringManager@@QAE@XZ 100606b6 f   StringManager.obj
 0001:0005f6d4       __unwindfunclet$?FindString@CStringManager@@QAE_NKPAD@Z$0 100606d4 f   StringManager.obj
 0001:0005f6dc       __ehhandler$?FindString@CStringManager@@QAE_NKPAD@Z 100606dc f   StringManager.obj
 0001:0005f704       __unwindfunclet$?FindString@CStringManager@@QAEABV?$basic_string@DU?$char_traits@D@std@@V?$allocator@D@2@@std@@K@Z$0 10060704 f   StringManager.obj
 0001:0005f712       __ehhandler$?FindString@CStringManager@@QAEABV?$basic_string@DU?$char_traits@D@std@@V?$allocator@D@2@@std@@K@Z 10060712 f   StringManager.obj
 0001:0005f72d       __unwindfunclet$??A?$hash_map@KV?$basic_string@DU?$char_traits@D@std@@V?$allocator@D@2@@std@@V?$hash_compare@KU?$less@K@std@@@stdext@@V?$allocator@U?$pair@$$CBKV?$basic_string@DU?$char_traits@D@std@@V?$allocator@D@2@@std@@@std@@@2@@stdext@@QAEAAV?$basic_string@DU?$char_traits@D@std@@V?$allocator@D@2@@std@@ABK@Z$0 1006072d f   StringManager.obj
 0001:0005f735       __unwindfunclet$??A?$hash_map@KV?$basic_string@DU?$char_traits@D@std@@V?$allocator@D@2@@std@@V?$hash_compare@KU?$less@K@std@@@stdext@@V?$allocator@U?$pair@$$CBKV?$basic_string@DU?$char_traits@D@std@@V?$allocator@D@2@@std@@@std@@@2@@stdext@@QAEAAV?$basic_string@DU?$char_traits@D@std@@V?$allocator@D@2@@std@@ABK@Z$1 10060735 f   StringManager.obj
 0001:0005f73d       __ehhandler$??A?$hash_map@KV?$basic_string@DU?$char_traits@D@std@@V?$allocator@D@2@@std@@V?$hash_compare@KU?$less@K@std@@@stdext@@V?$allocator@U?$pair@$$CBKV?$basic_string@DU?$char_traits@D@std@@V?$allocator@D@2@@std@@@std@@@2@@stdext@@QAEAAV?$basic_string@DU?$char_traits@D@std@@V?$allocator@D@2@@std@@ABK@Z 1006073d f   StringManager.obj
 0001:0005f75b       __unwindfunclet$??1?$_Hash@V?$_Hmap_traits@KV?$basic_string@DU?$char_traits@D@std@@V?$allocator@D@2@@std@@V?$hash_compare@KU?$less@K@std@@@stdext@@V?$allocator@U?$pair@$$CBKV?$basic_string@DU?$char_traits@D@std@@V?$allocator@D@2@@std@@@std@@@2@$0A@@stdext@@@stdext@@QAE@XZ$0 1006075b f   StringManager.obj
 0001:0005f763       __unwindfunclet$??1?$_Hash@V?$_Hmap_traits@KV?$basic_string@DU?$char_traits@D@std@@V?$allocator@D@2@@std@@V?$hash_compare@KU?$less@K@std@@@stdext@@V?$allocator@U?$pair@$$CBKV?$basic_string@DU?$char_traits@D@std@@V?$allocator@D@2@@std@@@std@@@2@$0A@@stdext@@@stdext@@QAE@XZ$1 10060763 f   StringManager.obj
 0001:0005f76e       __unwindfunclet$??1?$_Hash@V?$_Hmap_traits@KV?$basic_string@DU?$char_traits@D@std@@V?$allocator@D@2@@std@@V?$hash_compare@KU?$less@K@std@@@stdext@@V?$allocator@U?$pair@$$CBKV?$basic_string@DU?$char_traits@D@std@@V?$allocator@D@2@@std@@@std@@@2@$0A@@stdext@@@stdext@@QAE@XZ$3 1006076e f   StringManager.obj
 0001:0005f776       __unwindfunclet$??1?$_Hash@V?$_Hmap_traits@KV?$basic_string@DU?$char_traits@D@std@@V?$allocator@D@2@@std@@V?$hash_compare@KU?$less@K@std@@@stdext@@V?$allocator@U?$pair@$$CBKV?$basic_string@DU?$char_traits@D@std@@V?$allocator@D@2@@std@@@std@@@2@$0A@@stdext@@@stdext@@QAE@XZ$6 10060776 f   StringManager.obj
 0001:0005f77e       __ehhandler$??1?$_Hash@V?$_Hmap_traits@KV?$basic_string@DU?$char_traits@D@std@@V?$allocator@D@2@@std@@V?$hash_compare@KU?$less@K@std@@@stdext@@V?$allocator@U?$pair@$$CBKV?$basic_string@DU?$char_traits@D@std@@V?$allocator@D@2@@std@@@std@@@2@$0A@@stdext@@@stdext@@QAE@XZ 1006077e f   StringManager.obj
 0001:0005f799       __unwindfunclet$??0?$_Hash@V?$_Hmap_traits@KV?$basic_string@DU?$char_traits@D@std@@V?$allocator@D@2@@std@@V?$hash_compare@KU?$less@K@std@@@stdext@@V?$allocator@U?$pair@$$CBKV?$basic_string@DU?$char_traits@D@std@@V?$allocator@D@2@@std@@@std@@@2@$0A@@stdext@@@stdext@@QAE@ABV?$hash_compare@KU?$less@K@std@@@1@ABV?$allocator@U?$pair@$$CBKV?$basic_string@DU?$char_traits@D@std@@V?$allocator@D@2@@std@@@std@@@std@@@Z$0 10060799 f   StringManager.obj
 0001:0005f7a4       __unwindfunclet$??0?$_Hash@V?$_Hmap_traits@KV?$basic_string@DU?$char_traits@D@std@@V?$allocator@D@2@@std@@V?$hash_compare@KU?$less@K@std@@@stdext@@V?$allocator@U?$pair@$$CBKV?$basic_string@DU?$char_traits@D@std@@V?$allocator@D@2@@std@@@std@@@2@$0A@@stdext@@@stdext@@QAE@ABV?$hash_compare@KU?$less@K@std@@@1@ABV?$allocator@U?$pair@$$CBKV?$basic_string@DU?$char_traits@D@std@@V?$allocator@D@2@@std@@@std@@@std@@@Z$1 100607a4 f   StringManager.obj
 0001:0005f7b2       __unwindfunclet$??0?$_Hash@V?$_Hmap_traits@KV?$basic_string@DU?$char_traits@D@std@@V?$allocator@D@2@@std@@V?$hash_compare@KU?$less@K@std@@@stdext@@V?$allocator@U?$pair@$$CBKV?$basic_string@DU?$char_traits@D@std@@V?$allocator@D@2@@std@@@std@@@2@$0A@@stdext@@@stdext@@QAE@ABV?$hash_compare@KU?$less@K@std@@@1@ABV?$allocator@U?$pair@$$CBKV?$basic_string@DU?$char_traits@D@std@@V?$allocator@D@2@@std@@@std@@@std@@@Z$2 100607b2 f   StringManager.obj
 0001:0005f7c0       __ehhandler$??0?$_Hash@V?$_Hmap_traits@KV?$basic_string@DU?$char_traits@D@std@@V?$allocator@D@2@@std@@V?$hash_compare@KU?$less@K@std@@@stdext@@V?$allocator@U?$pair@$$CBKV?$basic_string@DU?$char_traits@D@std@@V?$allocator@D@2@@std@@@std@@@2@$0A@@stdext@@@stdext@@QAE@ABV?$hash_compare@KU?$less@K@std@@@1@ABV?$allocator@U?$pair@$$CBKV?$basic_string@DU?$char_traits@D@std@@V?$allocator@D@2@@std@@@std@@@std@@@Z 100607c0 f   StringManager.obj
 0001:0005f7de       __unwindfunclet$??1?$vector@U_List_position@?$_Hash@V?$_Hmap_traits@KPAXV?$hash_compare@KU?$less@K@std@@@stdext@@V?$allocator@U?$pair@$$CBKPAX@std@@@std@@$0A@@stdext@@@stdext@@V?$allocator@U_List_position@?$_Hash@V?$_Hmap_traits@KPAXV?$hash_compare@KU?$less@K@std@@@stdext@@V?$allocator@U?$pair@$$CBKPAX@std@@@std@@$0A@@stdext@@@stdext@@@std@@@std@@QAE@XZ$0 100607de f   StringManager.obj
 0001:0005f7de       __unwindfunclet$??1?$vector@U_List_position@?$_Hash@V?$_Hmap_traits@KV?$basic_string@DU?$char_traits@D@std@@V?$allocator@D@2@@std@@V?$hash_compare@KU?$less@K@std@@@stdext@@V?$allocator@U?$pair@$$CBKV?$basic_string@DU?$char_traits@D@std@@V?$allocator@D@2@@std@@@std@@@2@$0A@@stdext@@@stdext@@V?$allocator@U_List_position@?$_Hash@V?$_Hmap_traits@KV?$basic_string@DU?$char_traits@D@std@@V?$allocator@D@2@@std@@V?$hash_compare@KU?$less@K@std@@@stdext@@V?$allocator@U?$pair@$$CBKV?$basic_string@DU?$char_traits@D@std@@V?$allocator@D@2@@std@@@std@@@2@$0A@@stdext@@@stdext@@@std@@@std@@QAE@XZ$0 100607de f   StringManager.obj
 0001:0005f7e6       __ehhandler$??1?$vector@U_List_position@?$_Hash@V?$_Hmap_traits@KPAXV?$hash_compare@KU?$less@K@std@@@stdext@@V?$allocator@U?$pair@$$CBKPAX@std@@@std@@$0A@@stdext@@@stdext@@V?$allocator@U_List_position@?$_Hash@V?$_Hmap_traits@KPAXV?$hash_compare@KU?$less@K@std@@@stdext@@V?$allocator@U?$pair@$$CBKPAX@std@@@std@@$0A@@stdext@@@stdext@@@std@@@std@@QAE@XZ 100607e6 f   StringManager.obj
 0001:0005f7e6       __ehhandler$??1?$vector@U_List_position@?$_Hash@V?$_Hmap_traits@KV?$basic_string@DU?$char_traits@D@std@@V?$allocator@D@2@@std@@V?$hash_compare@KU?$less@K@std@@@stdext@@V?$allocator@U?$pair@$$CBKV?$basic_string@DU?$char_traits@D@std@@V?$allocator@D@2@@std@@@std@@@2@$0A@@stdext@@@stdext@@V?$allocator@U_List_position@?$_Hash@V?$_Hmap_traits@KV?$basic_string@DU?$char_traits@D@std@@V?$allocator@D@2@@std@@V?$hash_compare@KU?$less@K@std@@@stdext@@V?$allocator@U?$pair@$$CBKV?$basic_string@DU?$char_traits@D@std@@V?$allocator@D@2@@std@@@std@@@2@$0A@@stdext@@@stdext@@@std@@@std@@QAE@XZ 100607e6 f   StringManager.obj
 0001:0005f801       __unwindfunclet$??0?$list@KV?$allocator@K@std@@@std@@QAE@XZ$0 10060801 f   StringManager.obj
 0001:0005f801       __unwindfunclet$??0?$list@PAXV?$allocator@PAX@std@@@std@@QAE@XZ$0 10060801 f   StringManager.obj
 0001:0005f801       __unwindfunclet$??0?$list@UtagRECT@@V?$allocator@UtagRECT@@@std@@@std@@QAE@XZ$0 10060801 f   StringManager.obj
 0001:0005f801       __unwindfunclet$??0?$list@PAVCControlWZ@@V?$allocator@PAVCControlWZ@@@std@@@std@@QAE@XZ$0 10060801 f   StringManager.obj
 0001:0005f801       __unwindfunclet$??0?$list@U?$pair@$$CBKV?$basic_string@DU?$char_traits@D@std@@V?$allocator@D@2@@std@@@std@@V?$allocator@U?$pair@$$CBKV?$basic_string@DU?$char_traits@D@std@@V?$allocator@D@2@@std@@@std@@@2@@std@@QAE@ABV?$allocator@U?$pair@$$CBKV?$basic_string@DU?$char_traits@D@std@@V?$allocator@D@2@@std@@@std@@@1@@Z$0 10060801 f   StringManager.obj
 0001:0005f801       __unwindfunclet$??0?$list@U?$pair@$$CBKPAX@std@@V?$allocator@U?$pair@$$CBKPAX@std@@@2@@std@@QAE@ABV?$allocator@U?$pair@$$CBKPAX@std@@@1@@Z$0 10060801 f   StringManager.obj
 0001:0005f809       __ehhandler$??0?$list@U?$pair@$$CBKPAX@std@@V?$allocator@U?$pair@$$CBKPAX@std@@@2@@std@@QAE@ABV?$allocator@U?$pair@$$CBKPAX@std@@@1@@Z 10060809 f   StringManager.obj
 0001:0005f809       __ehhandler$??0?$list@UtagRECT@@V?$allocator@UtagRECT@@@std@@@std@@QAE@XZ 10060809 f   StringManager.obj
 0001:0005f809       __ehhandler$??0?$list@U?$pair@$$CBKV?$basic_string@DU?$char_traits@D@std@@V?$allocator@D@2@@std@@@std@@V?$allocator@U?$pair@$$CBKV?$basic_string@DU?$char_traits@D@std@@V?$allocator@D@2@@std@@@std@@@2@@std@@QAE@ABV?$allocator@U?$pair@$$CBKV?$basic_string@DU?$char_traits@D@std@@V?$allocator@D@2@@std@@@std@@@1@@Z 10060809 f   StringManager.obj
 0001:0005f809       __ehhandler$??0?$list@PAXV?$allocator@PAX@std@@@std@@QAE@XZ 10060809 f   StringManager.obj
 0001:0005f809       __ehhandler$??0?$list@PAVCControlWZ@@V?$allocator@PAVCControlWZ@@@std@@@std@@QAE@XZ 10060809 f   StringManager.obj
 0001:0005f809       __ehhandler$??0?$list@KV?$allocator@K@std@@@std@@QAE@XZ 10060809 f   StringManager.obj
 0001:0005f824       __ehhandler$?_Buynode@?$list@U?$pair@$$CBKV?$basic_string@DU?$char_traits@D@std@@V?$allocator@D@2@@std@@@std@@V?$allocator@U?$pair@$$CBKV?$basic_string@DU?$char_traits@D@std@@V?$allocator@D@2@@std@@@std@@@2@@std@@IAEPAU_Node@?$_List_nod@U?$pair@$$CBKV?$basic_string@DU?$char_traits@D@std@@V?$allocator@D@2@@std@@@std@@V?$allocator@U?$pair@$$CBKV?$basic_string@DU?$char_traits@D@std@@V?$allocator@D@2@@std@@@std@@@2@@2@XZ 10060824 f   StringManager.obj
 0001:0005f83f       __ehhandler$?_Buynode@?$list@U?$pair@$$CBKV?$basic_string@DU?$char_traits@D@std@@V?$allocator@D@2@@std@@@std@@V?$allocator@U?$pair@$$CBKV?$basic_string@DU?$char_traits@D@std@@V?$allocator@D@2@@std@@@std@@@2@@std@@IAEPAU_Node@?$_List_nod@U?$pair@$$CBKV?$basic_string@DU?$char_traits@D@std@@V?$allocator@D@2@@std@@@std@@V?$allocator@U?$pair@$$CBKV?$basic_string@DU?$char_traits@D@std@@V?$allocator@D@2@@std@@@std@@@2@@2@PAU342@0ABU?$pair@$$CBKV?$basic_string@DU?$char_traits@D@std@@V?$allocator@D@2@@std@@@2@@Z 1006083f f   StringManager.obj
 0001:0005f85a       __ehhandler$?_Insert_n@?$vector@U_List_position@?$_Hash@V?$_Hmap_traits@KV?$basic_string@DU?$char_traits@D@std@@V?$allocator@D@2@@std@@V?$hash_compare@KU?$less@K@std@@@stdext@@V?$allocator@U?$pair@$$CBKV?$basic_string@DU?$char_traits@D@std@@V?$allocator@D@2@@std@@@std@@@2@$0A@@stdext@@@stdext@@V?$allocator@U_List_position@?$_Hash@V?$_Hmap_traits@KV?$basic_string@DU?$char_traits@D@std@@V?$allocator@D@2@@std@@V?$hash_compare@KU?$less@K@std@@@stdext@@V?$allocator@U?$pair@$$CBKV?$basic_string@DU?$char_traits@D@std@@V?$allocator@D@2@@std@@@std@@@2@$0A@@stdext@@@stdext@@@std@@@std@@IAEXV?$_Vector_const_iterator@U_List_position@?$_Hash@V?$_Hmap_traits@KV?$basic_string@DU?$char_traits@D@std@@V?$allocator@D@2@@std@@V?$hash_compare@KU?$less@K@std@@@stdext@@V?$allocator@U?$pair@$$CBKV?$basic_string@DU?$char_traits@D@std@@V?$allocator@D@2@@std@@@std@@@2@$0A@@stdext@@@stdext@@V?$allocator@U_List_position@?$_Hash@V?$_Hmap_traits@KV?$basic_string@DU?$char_traits@D@std@@V?$allocator@D@2@@std@@V?$hash_compare@KU?$less@K@std@@@stdext@@V?$allocator@U?$pair@$$CBKV?$basic_string@DU?$char_traits@D@std@@V?$allocator@D@2@@std@@@std@@@2@$0A@@stdext@@@stdext@@@std@@@2@IABU_List_position@?$_Hash@V?$_Hmap_traits@KV?$basic_string@DU?$char_traits@D@std@@V?$allocator@D@2@@std@@V?$hash_compare@KU?$less@K@std@@@stdext@@V?$allocator@U?$pair@$$CBKV?$basic_string@DU?$char_traits@D@std@@V?$allocator@D@2@@std@@@std@@@2@$0A@@stdext@@@stdext@@@Z 1006085a f   StringManager.obj
 0001:0005f85a       __ehhandler$?_Insert_n@?$vector@U_List_position@?$_Hash@V?$_Hmap_traits@KPAXV?$hash_compare@KU?$less@K@std@@@stdext@@V?$allocator@U?$pair@$$CBKPAX@std@@@std@@$0A@@stdext@@@stdext@@V?$allocator@U_List_position@?$_Hash@V?$_Hmap_traits@KPAXV?$hash_compare@KU?$less@K@std@@@stdext@@V?$allocator@U?$pair@$$CBKPAX@std@@@std@@$0A@@stdext@@@stdext@@@std@@@std@@IAEXV?$_Vector_const_iterator@U_List_position@?$_Hash@V?$_Hmap_traits@KPAXV?$hash_compare@KU?$less@K@std@@@stdext@@V?$allocator@U?$pair@$$CBKPAX@std@@@std@@$0A@@stdext@@@stdext@@V?$allocator@U_List_position@?$_Hash@V?$_Hmap_traits@KPAXV?$hash_compare@KU?$less@K@std@@@stdext@@V?$allocator@U?$pair@$$CBKPAX@std@@@std@@$0A@@stdext@@@stdext@@@std@@@2@IABU_List_position@?$_Hash@V?$_Hmap_traits@KPAXV?$hash_compare@KU?$less@K@std@@@stdext@@V?$allocator@U?$pair@$$CBKPAX@std@@@std@@$0A@@stdext@@@stdext@@@Z 1006085a f   StringManager.obj
 0001:0005f878       __unwindfunclet$??$_Construct@U?$pair@$$CBKV?$basic_string@DU?$char_traits@D@std@@V?$allocator@D@2@@std@@@std@@U12@@std@@YAXPAU?$pair@$$CBKV?$basic_string@DU?$char_traits@D@std@@V?$allocator@D@2@@std@@@0@ABU10@@Z$0 10060878 f   StringManager.obj
 0001:0005f886       __ehhandler$??$_Construct@U?$pair@$$CBKV?$basic_string@DU?$char_traits@D@std@@V?$allocator@D@2@@std@@@std@@U12@@std@@YAXPAU?$pair@$$CBKV?$basic_string@DU?$char_traits@D@std@@V?$allocator@D@2@@std@@@0@ABU10@@Z 10060886 f   StringManager.obj
 0001:0005f8a1       __ehhandler$??$_Insert@V?$_Const_iterator@$00@?$list@U?$pair@$$CBKV?$basic_string@DU?$char_traits@D@std@@V?$allocator@D@2@@std@@@std@@V?$allocator@U?$pair@$$CBKV?$basic_string@DU?$char_traits@D@std@@V?$allocator@D@2@@std@@@std@@@2@@std@@@?$list@U?$pair@$$CBKV?$basic_string@DU?$char_traits@D@std@@V?$allocator@D@2@@std@@@std@@V?$allocator@U?$pair@$$CBKV?$basic_string@DU?$char_traits@D@std@@V?$allocator@D@2@@std@@@std@@@2@@std@@QAEXV?$_Const_iterator@$00@01@00Uforward_iterator_tag@1@@Z 100608a1 f   StringManager.obj
 0001:0005f8bf       __ehhandler$??$_Uninit_fill_n@PAU_List_position@?$_Hash@V?$_Hmap_traits@KV?$basic_string@DU?$char_traits@D@std@@V?$allocator@D@2@@std@@V?$hash_compare@KU?$less@K@std@@@stdext@@V?$allocator@U?$pair@$$CBKV?$basic_string@DU?$char_traits@D@std@@V?$allocator@D@2@@std@@@std@@@2@$0A@@stdext@@@stdext@@IU123@V?$allocator@U_List_position@?$_Hash@V?$_Hmap_traits@KV?$basic_string@DU?$char_traits@D@std@@V?$allocator@D@2@@std@@V?$hash_compare@KU?$less@K@std@@@stdext@@V?$allocator@U?$pair@$$CBKV?$basic_string@DU?$char_traits@D@std@@V?$allocator@D@2@@std@@@std@@@2@$0A@@stdext@@@stdext@@@std@@@std@@YAXPAU_List_position@?$_Hash@V?$_Hmap_traits@KV?$basic_string@DU?$char_traits@D@std@@V?$allocator@D@2@@std@@V?$hash_compare@KU?$less@K@std@@@stdext@@V?$allocator@U?$pair@$$CBKV?$basic_string@DU?$char_traits@D@std@@V?$allocator@D@2@@std@@@std@@@2@$0A@@stdext@@@stdext@@IABU123@AAV?$allocator@U_List_position@?$_Hash@V?$_Hmap_traits@KV?$basic_string@DU?$char_traits@D@std@@V?$allocator@D@2@@std@@V?$hash_compare@KU?$less@K@std@@@stdext@@V?$allocator@U?$pair@$$CBKV?$basic_string@DU?$char_traits@D@std@@V?$allocator@D@2@@std@@@std@@@2@$0A@@stdext@@@stdext@@@0@U_Nonscalar_ptr_iterator_tag@0@U_Range_checked_iterator_tag@0@@Z 100608bf f   StringManager.obj
 0001:0005f8bf       __ehhandler$??$_Uninit_fill_n@PAU_List_position@?$_Hash@V?$_Hmap_traits@KPAXV?$hash_compare@KU?$less@K@std@@@stdext@@V?$allocator@U?$pair@$$CBKPAX@std@@@std@@$0A@@stdext@@@stdext@@IU123@V?$allocator@U_List_position@?$_Hash@V?$_Hmap_traits@KPAXV?$hash_compare@KU?$less@K@std@@@stdext@@V?$allocator@U?$pair@$$CBKPAX@std@@@std@@$0A@@stdext@@@stdext@@@std@@@std@@YAXPAU_List_position@?$_Hash@V?$_Hmap_traits@KPAXV?$hash_compare@KU?$less@K@std@@@stdext@@V?$allocator@U?$pair@$$CBKPAX@std@@@std@@$0A@@stdext@@@stdext@@IABU123@AAV?$allocator@U_List_position@?$_Hash@V?$_Hmap_traits@KPAXV?$hash_compare@KU?$less@K@std@@@stdext@@V?$allocator@U?$pair@$$CBKPAX@std@@@std@@$0A@@stdext@@@stdext@@@0@U_Nonscalar_ptr_iterator_tag@0@U_Range_checked_iterator_tag@0@@Z 100608bf f   StringManager.obj
 0001:0005f8da       __unwindfunclet$??0CControlWZ@@QAE@XZ$0 100608da f   ControlWZ.obj
 0001:0005f8e5       __unwindfunclet$??0CControlWZ@@QAE@XZ$1 100608e5 f   ControlWZ.obj
 0001:0005f8f3       __ehhandler$??0CControlWZ@@QAE@XZ 100608f3 f   ControlWZ.obj
 0001:0005f90e       __unwindfunclet$??1CControlWZ@@UAE@XZ$0 1006090e f   ControlWZ.obj
 0001:0005f919       __ehhandler$??1CControlWZ@@UAE@XZ 10060919 f   ControlWZ.obj
 0001:0005f934       __unwindfunclet$?SetMoney@CControlWZ@@UAEX_K@Z$0 10060934 f   ControlWZ.obj
 0001:0005f93c       __ehhandler$?SetMoney@CControlWZ@@UAEX_K@Z 1006093c f   ControlWZ.obj
 0001:0005f957       __unwindfunclet$?SetMoneyWithSymbol@CControlWZ@@UAEX_J@Z$0 10060957 f   ControlWZ.obj
 0001:0005f95f       __ehhandler$?SetMoneyWithSymbol@CControlWZ@@UAEX_J@Z 1006095f f   ControlWZ.obj
 0001:0005f97a       __unwindfunclet$??0SI_TSUBINFO@@QAE@XZ$0 1006097a f   ControlWZ.obj
 0001:0005f988       __ehhandler$??0SI_TSUBINFO@@QAE@XZ 10060988 f   ControlWZ.obj
 0001:0005f9a6       __unwindfunclet$?SetTextID@CCtrlButtonWZ@@UAEXK@Z$0 100609a6 f   CtrlButtonWZ.obj
 0001:0005f9ae       __ehhandler$?SetTextID@CCtrlButtonWZ@@UAEXK@Z 100609ae f   CtrlButtonWZ.obj
 0001:0005f9d3       __unwindfunclet$??0CCtrlDxEditBox@@QAE@XZ$0 100609d3 f   CtrlDxEdit.obj
 0001:0005f9db       __unwindfunclet$??0CCtrlDxEditBox@@QAE@XZ$1 100609db f   CtrlDxEdit.obj
 0001:0005f9e9       __unwindfunclet$??0CCtrlDxEditBox@@QAE@XZ$2 100609e9 f   CtrlDxEdit.obj
 0001:0005f9f7       __ehhandler$??0CCtrlDxEditBox@@QAE@XZ 100609f7 f   CtrlDxEdit.obj
 0001:0005fa12       __unwindfunclet$??1CCtrlDxEditBox@@UAE@XZ$0 10060a12 f   CtrlDxEdit.obj
 0001:0005fa1a       __unwindfunclet$??1CCtrlDxEditBox@@UAE@XZ$1 10060a1a f   CtrlDxEdit.obj
 0001:0005fa28       __ehhandler$??1CCtrlDxEditBox@@UAE@XZ 10060a28 f   CtrlDxEdit.obj
 0001:0005fa43       __unwindfunclet$?SetTextWZW@CCtrlDxEditBox@@UAEXPB_W_N@Z$0 10060a43 f   CtrlDxEdit.obj
 0001:0005fa4b       __ehhandler$?SetTextWZW@CCtrlDxEditBox@@UAEXPB_W_N@Z 10060a4b f   CtrlDxEdit.obj
 0001:0005fa73       __unwindfunclet$??0CCtrlDxIMEEditBox@@QAE@XZ$0 10060a73 f   CtrlDxEdit.obj
 0001:0005fa7b       __ehhandler$??0CCtrlDxIMEEditBox@@QAE@XZ 10060a7b f   CtrlDxEdit.obj
 0001:0005fa96       __unwindfunclet$??1CCtrlDxIMEEditBox@@UAE@XZ$0 10060a96 f   CtrlDxEdit.obj
 0001:0005fa9e       __ehhandler$??1CCtrlDxIMEEditBox@@UAE@XZ 10060a9e f   CtrlDxEdit.obj
 0001:0005fab9       __unwindfunclet$??0CCtrlMultilineEditWZ@@QAE@XZ$0 10060ab9 f   CtrlDxEdit.obj
 0001:0005fac4       __unwindfunclet$??0CCtrlMultilineEditWZ@@QAE@XZ$1 10060ac4 f   CtrlDxEdit.obj
 0001:0005fad5       __ehhandler$??0CCtrlMultilineEditWZ@@QAE@XZ 10060ad5 f   CtrlDxEdit.obj
 0001:0005faf0       __unwindfunclet$??1CCtrlMultilineEditWZ@@UAE@XZ$0 10060af0 f   CtrlDxEdit.obj
 0001:0005faf8       __unwindfunclet$??1CCtrlMultilineEditWZ@@UAE@XZ$1 10060af8 f   CtrlDxEdit.obj
 0001:0005fb06       __unwindfunclet$??1CCtrlMultilineEditWZ@@UAE@XZ$3 10060b06 f   CtrlDxEdit.obj
 0001:0005fb0e       __ehhandler$??1CCtrlMultilineEditWZ@@UAE@XZ 10060b0e f   CtrlDxEdit.obj
 0001:0005fb29       __unwindfunclet$??0?$vector@KV?$allocator@K@std@@@std@@QAE@XZ$0 10060b29 f   CtrlDxEdit.obj
 0001:0005fb29       __unwindfunclet$??0?$vector@U_List_position@?$_Hash@V?$_Hmap_traits@KPAXV?$hash_compare@KU?$less@K@std@@@stdext@@V?$allocator@U?$pair@$$CBKPAX@std@@@std@@$0A@@stdext@@@stdext@@V?$allocator@U_List_position@?$_Hash@V?$_Hmap_traits@KPAXV?$hash_compare@KU?$less@K@std@@@stdext@@V?$allocator@U?$pair@$$CBKPAX@std@@@std@@$0A@@stdext@@@stdext@@@std@@@std@@QAE@ABV?$allocator@U_List_position@?$_Hash@V?$_Hmap_traits@KPAXV?$hash_compare@KU?$less@K@std@@@stdext@@V?$allocator@U?$pair@$$CBKPAX@std@@@std@@$0A@@stdext@@@stdext@@@1@@Z$0 10060b29 f   CtrlDxEdit.obj
 0001:0005fb29       __unwindfunclet$??0?$vector@U_List_position@?$_Hash@V?$_Hmap_traits@KV?$basic_string@DU?$char_traits@D@std@@V?$allocator@D@2@@std@@V?$hash_compare@KU?$less@K@std@@@stdext@@V?$allocator@U?$pair@$$CBKV?$basic_string@DU?$char_traits@D@std@@V?$allocator@D@2@@std@@@std@@@2@$0A@@stdext@@@stdext@@V?$allocator@U_List_position@?$_Hash@V?$_Hmap_traits@KV?$basic_string@DU?$char_traits@D@std@@V?$allocator@D@2@@std@@V?$hash_compare@KU?$less@K@std@@@stdext@@V?$allocator@U?$pair@$$CBKV?$basic_string@DU?$char_traits@D@std@@V?$allocator@D@2@@std@@@std@@@2@$0A@@stdext@@@stdext@@@std@@@std@@QAE@ABV?$allocator@U_List_position@?$_Hash@V?$_Hmap_traits@KV?$basic_string@DU?$char_traits@D@std@@V?$allocator@D@2@@std@@V?$hash_compare@KU?$less@K@std@@@stdext@@V?$allocator@U?$pair@$$CBKV?$basic_string@DU?$char_traits@D@std@@V?$allocator@D@2@@std@@@std@@@2@$0A@@stdext@@@stdext@@@1@@Z$0 10060b29 f   CtrlDxEdit.obj
 0001:0005fb34       __ehhandler$??0?$vector@U_List_position@?$_Hash@V?$_Hmap_traits@KPAXV?$hash_compare@KU?$less@K@std@@@stdext@@V?$allocator@U?$pair@$$CBKPAX@std@@@std@@$0A@@stdext@@@stdext@@V?$allocator@U_List_position@?$_Hash@V?$_Hmap_traits@KPAXV?$hash_compare@KU?$less@K@std@@@stdext@@V?$allocator@U?$pair@$$CBKPAX@std@@@std@@$0A@@stdext@@@stdext@@@std@@@std@@QAE@ABV?$allocator@U_List_position@?$_Hash@V?$_Hmap_traits@KPAXV?$hash_compare@KU?$less@K@std@@@stdext@@V?$allocator@U?$pair@$$CBKPAX@std@@@std@@$0A@@stdext@@@stdext@@@1@@Z 10060b34 f   CtrlDxEdit.obj
 0001:0005fb34       __ehhandler$??0?$vector@U_List_position@?$_Hash@V?$_Hmap_traits@KV?$basic_string@DU?$char_traits@D@std@@V?$allocator@D@2@@std@@V?$hash_compare@KU?$less@K@std@@@stdext@@V?$allocator@U?$pair@$$CBKV?$basic_string@DU?$char_traits@D@std@@V?$allocator@D@2@@std@@@std@@@2@$0A@@stdext@@@stdext@@V?$allocator@U_List_position@?$_Hash@V?$_Hmap_traits@KV?$basic_string@DU?$char_traits@D@std@@V?$allocator@D@2@@std@@V?$hash_compare@KU?$less@K@std@@@stdext@@V?$allocator@U?$pair@$$CBKV?$basic_string@DU?$char_traits@D@std@@V?$allocator@D@2@@std@@@std@@@2@$0A@@stdext@@@stdext@@@std@@@std@@QAE@ABV?$allocator@U_List_position@?$_Hash@V?$_Hmap_traits@KV?$basic_string@DU?$char_traits@D@std@@V?$allocator@D@2@@std@@V?$hash_compare@KU?$less@K@std@@@stdext@@V?$allocator@U?$pair@$$CBKV?$basic_string@DU?$char_traits@D@std@@V?$allocator@D@2@@std@@@std@@@2@$0A@@stdext@@@stdext@@@1@@Z 10060b34 f   CtrlDxEdit.obj
 0001:0005fb34       __ehhandler$??0?$vector@KV?$allocator@K@std@@@std@@QAE@XZ 10060b34 f   CtrlDxEdit.obj
 0001:0005fb52       __unwindfunclet$??1?$vector@KV?$allocator@K@std@@@std@@QAE@XZ$0 10060b52 f   CtrlDxEdit.obj
 0001:0005fb52       __unwindfunclet$??1?$list@U?$pair@$$CBKV?$basic_string@DU?$char_traits@D@std@@V?$allocator@D@2@@std@@@std@@V?$allocator@U?$pair@$$CBKV?$basic_string@DU?$char_traits@D@std@@V?$allocator@D@2@@std@@@std@@@2@@std@@QAE@XZ$0 10060b52 f   CtrlDxEdit.obj
 0001:0005fb5a       __ehhandler$??1?$list@U?$pair@$$CBKV?$basic_string@DU?$char_traits@D@std@@V?$allocator@D@2@@std@@@std@@V?$allocator@U?$pair@$$CBKV?$basic_string@DU?$char_traits@D@std@@V?$allocator@D@2@@std@@@std@@@2@@std@@QAE@XZ 10060b5a f   CtrlDxEdit.obj
 0001:0005fb5a       __ehhandler$??1?$vector@KV?$allocator@K@std@@@std@@QAE@XZ 10060b5a f   CtrlDxEdit.obj
 0001:0005fb75       __ehhandler$?_Insert_n@?$vector@KV?$allocator@K@std@@@std@@IAEXV?$_Vector_const_iterator@KV?$allocator@K@std@@@2@IABK@Z 10060b75 f   CtrlDxEdit.obj
 0001:0005fb93       __unwindfunclet$?_Xlen@?$vector@KV?$allocator@K@std@@@std@@KAXXZ$0 10060b93 f   CtrlDxEdit.obj
 0001:0005fb93       __unwindfunclet$?_Xlen@?$vector@U_List_position@?$_Hash@V?$_Hmap_traits@KV?$basic_string@DU?$char_traits@D@std@@V?$allocator@D@2@@std@@V?$hash_compare@KU?$less@K@std@@@stdext@@V?$allocator@U?$pair@$$CBKV?$basic_string@DU?$char_traits@D@std@@V?$allocator@D@2@@std@@@std@@@2@$0A@@stdext@@@stdext@@V?$allocator@U_List_position@?$_Hash@V?$_Hmap_traits@KV?$basic_string@DU?$char_traits@D@std@@V?$allocator@D@2@@std@@V?$hash_compare@KU?$less@K@std@@@stdext@@V?$allocator@U?$pair@$$CBKV?$basic_string@DU?$char_traits@D@std@@V?$allocator@D@2@@std@@@std@@@2@$0A@@stdext@@@stdext@@@std@@@std@@KAXXZ$0 10060b93 f   CtrlDxEdit.obj
 0001:0005fb93       __unwindfunclet$?_Xlen@?$vector@U_List_position@?$_Hash@V?$_Hmap_traits@KPAXV?$hash_compare@KU?$less@K@std@@@stdext@@V?$allocator@U?$pair@$$CBKPAX@std@@@std@@$0A@@stdext@@@stdext@@V?$allocator@U_List_position@?$_Hash@V?$_Hmap_traits@KPAXV?$hash_compare@KU?$less@K@std@@@stdext@@V?$allocator@U?$pair@$$CBKPAX@std@@@std@@$0A@@stdext@@@stdext@@@std@@@std@@KAXXZ$0 10060b93 f   CtrlDxEdit.obj
 0001:0005fb9b       __ehhandler$?_Xlen@?$vector@U_List_position@?$_Hash@V?$_Hmap_traits@KV?$basic_string@DU?$char_traits@D@std@@V?$allocator@D@2@@std@@V?$hash_compare@KU?$less@K@std@@@stdext@@V?$allocator@U?$pair@$$CBKV?$basic_string@DU?$char_traits@D@std@@V?$allocator@D@2@@std@@@std@@@2@$0A@@stdext@@@stdext@@V?$allocator@U_List_position@?$_Hash@V?$_Hmap_traits@KV?$basic_string@DU?$char_traits@D@std@@V?$allocator@D@2@@std@@V?$hash_compare@KU?$less@K@std@@@stdext@@V?$allocator@U?$pair@$$CBKV?$basic_string@DU?$char_traits@D@std@@V?$allocator@D@2@@std@@@std@@@2@$0A@@stdext@@@stdext@@@std@@@std@@KAXXZ 10060b9b f   CtrlDxEdit.obj
 0001:0005fb9b       __ehhandler$?_Xlen@?$vector@U_List_position@?$_Hash@V?$_Hmap_traits@KPAXV?$hash_compare@KU?$less@K@std@@@stdext@@V?$allocator@U?$pair@$$CBKPAX@std@@@std@@$0A@@stdext@@@stdext@@V?$allocator@U_List_position@?$_Hash@V?$_Hmap_traits@KPAXV?$hash_compare@KU?$less@K@std@@@stdext@@V?$allocator@U?$pair@$$CBKPAX@std@@@std@@$0A@@stdext@@@stdext@@@std@@@std@@KAXXZ 10060b9b f   CtrlDxEdit.obj
 0001:0005fb9b       __ehhandler$?_Xlen@?$vector@KV?$allocator@K@std@@@std@@KAXXZ 10060b9b f   CtrlDxEdit.obj
 0001:0005fbb9       __unwindfunclet$??0CCtrlEditWZ@@QAE@XZ$0 10060bb9 f   CtrlEditWZ.obj
 0001:0005fbc1       __ehhandler$??0CCtrlEditWZ@@QAE@XZ 10060bc1 f   CtrlEditWZ.obj
 0001:0005fbdc       __unwindfunclet$??0CCtrlHScrollWZ@@QAE@XZ$0 10060bdc f   CtrlHScrollWZ.obj
 0001:0005fbe4       __unwindfunclet$??0CCtrlHScrollWZ@@QAE@XZ$1 10060be4 f   CtrlHScrollWZ.obj
 0001:0005fbf2       __unwindfunclet$??0CCtrlHScrollWZ@@QAE@XZ$2 10060bf2 f   CtrlHScrollWZ.obj
 0001:0005fc00       __ehhandler$??0CCtrlHScrollWZ@@QAE@XZ 10060c00 f   CtrlHScrollWZ.obj
 0001:0005fc1b       __unwindfunclet$??1CCtrlHScrollWZ@@UAE@XZ$0 10060c1b f   CtrlHScrollWZ.obj
 0001:0005fc23       __unwindfunclet$??1CCtrlHScrollWZ@@UAE@XZ$1 10060c23 f   CtrlHScrollWZ.obj
 0001:0005fc31       __unwindfunclet$??1CCtrlHScrollWZ@@UAE@XZ$2 10060c31 f   CtrlHScrollWZ.obj
 0001:0005fc3f       __ehhandler$??1CCtrlHScrollWZ@@UAE@XZ 10060c3f f   CtrlHScrollWZ.obj
 0001:0005fc5a       __unwindfunclet$??0CCtrlListWZ@@QAE@XZ$0 10060c5a f   CtrlListWZ.obj
 0001:0005fc62       __unwindfunclet$??0CCtrlListWZ@@QAE@XZ$1 10060c62 f   CtrlListWZ.obj
 0001:0005fc70       __unwindfunclet$??0CCtrlListWZ@@QAE@XZ$2 10060c70 f   CtrlListWZ.obj
 0001:0005fc7e       __ehhandler$??0CCtrlListWZ@@QAE@XZ 10060c7e f   CtrlListWZ.obj
 0001:0005fc99       __unwindfunclet$??1CCtrlListWZ@@UAE@XZ$0 10060c99 f   CtrlListWZ.obj
 0001:0005fca1       __unwindfunclet$??1CCtrlListWZ@@UAE@XZ$1 10060ca1 f   CtrlListWZ.obj
 0001:0005fcaf       __unwindfunclet$??1CCtrlListWZ@@UAE@XZ$2 10060caf f   CtrlListWZ.obj
 0001:0005fcbd       __unwindfunclet$??1CCtrlListWZ@@UAE@XZ$4 10060cbd f   CtrlListWZ.obj
 0001:0005fcc5       __unwindfunclet$??1CCtrlListWZ@@UAE@XZ$10 10060cc5 f   CtrlListWZ.obj
 0001:0005fccd       __unwindfunclet$??1CCtrlListWZ@@UAE@XZ$17 10060ccd f   CtrlListWZ.obj
 0001:0005fcd5       __ehhandler$??1CCtrlListWZ@@UAE@XZ 10060cd5 f   CtrlListWZ.obj
 0001:0005fcf0       __unwindfunclet$?OnLoad@CCtrlListWZ@@UAEXPAX@Z$0 10060cf0 f   CtrlListWZ.obj
 0001:0005fcfb       __ehhandler$?OnLoad@CCtrlListWZ@@UAEXPAX@Z 10060cfb f   CtrlListWZ.obj
 0001:0005fd23       __unwindfunclet$?SetReportUseCnt@CCtrlListWZ@@UAEXF@Z$0 10060d23 f   CtrlListWZ.obj
 0001:0005fd2d       __ehhandler$?SetReportUseCnt@CCtrlListWZ@@UAEXF@Z 10060d2d f   CtrlListWZ.obj
 0001:0005fd4b       __unwindfunclet$?InsertItemBack@CCtrlListWZ@@UAEHXZ$0 10060d4b f   CtrlListWZ.obj
 0001:0005fd55       __ehhandler$?InsertItemBack@CCtrlListWZ@@UAEHXZ 10060d55 f   CtrlListWZ.obj
 0001:0005fd73       __unwindfunclet$?InsertItemFront@CCtrlListWZ@@UAEHXZ$0 10060d73 f   CtrlListWZ.obj
 0001:0005fd7d       __ehhandler$?InsertItemFront@CCtrlListWZ@@UAEHXZ 10060d7d f   CtrlListWZ.obj
 0001:0005fd9b       __unwindfunclet$?UpdateListDate@CCtrlListWZ@@IAEHPAX@Z$0 10060d9b f   CtrlListWZ.obj
 0001:0005fda6       __unwindfunclet$?UpdateListDate@CCtrlListWZ@@IAEHPAX@Z$1 10060da6 f   CtrlListWZ.obj
 0001:0005fdb1       __unwindfunclet$?UpdateListDate@CCtrlListWZ@@IAEHPAX@Z$2 10060db1 f   CtrlListWZ.obj
 0001:0005fdb9       __unwindfunclet$?UpdateListDate@CCtrlListWZ@@IAEHPAX@Z$3 10060db9 f   CtrlListWZ.obj
 0001:0005fdc1       __ehhandler$?UpdateListDate@CCtrlListWZ@@IAEHPAX@Z 10060dc1 f   CtrlListWZ.obj
 0001:0005fde9       __unwindfunclet$?SetItemWZA@CCtrlListWZ@@UAE_NHPBDKKKKK@Z$0 10060de9 f   CtrlListWZ.obj
 0001:0005fdf1       __ehhandler$?SetItemWZA@CCtrlListWZ@@UAE_NHPBDKKKKK@Z 10060df1 f   CtrlListWZ.obj
 0001:0005fe19       __unwindfunclet$?SetItemWZA@CCtrlListWZ@@UAE_NHHPBDKKKKK@Z$0 10060e19 f   CtrlListWZ.obj
 0001:0005fe21       __ehhandler$?SetItemWZA@CCtrlListWZ@@UAE_NHHPBDKKKKK@Z 10060e21 f   CtrlListWZ.obj
 0001:0005fe49       __unwindfunclet$?SelectReportButton@CCtrlListWZ@@UAEXH@Z$0 10060e49 f   CtrlListWZ.obj
 0001:0005fe54       __unwindfunclet$?SelectReportButton@CCtrlListWZ@@UAEXH@Z$1 10060e54 f   CtrlListWZ.obj
 0001:0005fe5c       __unwindfunclet$?SelectReportButton@CCtrlListWZ@@UAEXH@Z$2 10060e5c f   CtrlListWZ.obj
 0001:0005fe67       __unwindfunclet$?SelectReportButton@CCtrlListWZ@@UAEXH@Z$3 10060e67 f   CtrlListWZ.obj
 0001:0005fe72       __unwindfunclet$?SelectReportButton@CCtrlListWZ@@UAEXH@Z$4 10060e72 f   CtrlListWZ.obj
 0001:0005fe7d       __ehhandler$?SelectReportButton@CCtrlListWZ@@UAEXH@Z 10060e7d f   CtrlListWZ.obj
 0001:0005fe9b       __unwindfunclet$??1CListData@CCtrlListWZ@@QAE@XZ$0 10060e9b f   CtrlListWZ.obj
 0001:0005fea6       __unwindfunclet$??1CListData@CCtrlListWZ@@QAE@XZ$3 10060ea6 f   CtrlListWZ.obj
 0001:0005feae       __ehhandler$??1CListData@CCtrlListWZ@@QAE@XZ 10060eae f   CtrlListWZ.obj
 0001:0005fec9       __unwindfunclet$??1?$map@KPAXU?$less@K@std@@V?$allocator@U?$pair@$$CBKPAX@std@@@2@@std@@QAE@XZ$1 10060ec9 f   CtrlListWZ.obj
 0001:0005fec9       __unwindfunclet$??1?$map@KPAUCListSellData@CCtrlListWZ@@U?$less@K@std@@V?$allocator@U?$pair@$$CBKPAUCListSellData@CCtrlListWZ@@@std@@@4@@std@@QAE@XZ$1 10060ec9 f   CtrlListWZ.obj
 0001:0005fec9       __unwindfunclet$??1?$multimap@V?$basic_string@DU?$char_traits@D@std@@V?$allocator@D@2@@std@@PAXU?$less@V?$basic_string@DU?$char_traits@D@std@@V?$allocator@D@2@@std@@@2@V?$allocator@U?$pair@$$CBV?$basic_string@DU?$char_traits@D@std@@V?$allocator@D@2@@std@@PAX@std@@@2@@std@@QAE@XZ$1 10060ec9 f   CtrlListWZ.obj
 0001:0005fed1       __ehhandler$??1?$map@KPAXU?$less@K@std@@V?$allocator@U?$pair@$$CBKPAX@std@@@2@@std@@QAE@XZ 10060ed1 f   CtrlListWZ.obj
 0001:0005fed1       __ehhandler$??1?$multimap@V?$basic_string@DU?$char_traits@D@std@@V?$allocator@D@2@@std@@PAXU?$less@V?$basic_string@DU?$char_traits@D@std@@V?$allocator@D@2@@std@@@2@V?$allocator@U?$pair@$$CBV?$basic_string@DU?$char_traits@D@std@@V?$allocator@D@2@@std@@PAX@std@@@2@@std@@QAE@XZ 10060ed1 f   CtrlListWZ.obj
 0001:0005fed1       __ehhandler$??1?$map@KPAUCListSellData@CCtrlListWZ@@U?$less@K@std@@V?$allocator@U?$pair@$$CBKPAUCListSellData@CCtrlListWZ@@@std@@@4@@std@@QAE@XZ 10060ed1 f   CtrlListWZ.obj
 0001:0005feec       __unwindfunclet$??1SBTData@@QAE@XZ$0 10060eec f   CtrlListWZ.obj
 0001:0005fef7       __ehhandler$??1SBTData@@QAE@XZ 10060ef7 f   CtrlListWZ.obj
 0001:0005ff12       __unwindfunclet$??0SBTData@@QAE@XZ$0 10060f12 f   CtrlListWZ.obj
 0001:0005ff1d       __ehhandler$??0SBTData@@QAE@XZ 10060f1d f   CtrlListWZ.obj
 0001:0005ff38       __unwindfunclet$?Add@CListData@CCtrlListWZ@@QAE_NPBDKKKKK@Z$0 10060f38 f   CtrlListWZ.obj
 0001:0005ff42       __ehhandler$?Add@CListData@CCtrlListWZ@@QAE_NPBDKKKKK@Z 10060f42 f   CtrlListWZ.obj
 0001:0005ff5d       __unwindfunclet$?Add@CListData@CCtrlListWZ@@QAE_NHPBDKKKKK@Z$0 10060f5d f   CtrlListWZ.obj
 0001:0005ff67       __ehhandler$?Add@CListData@CCtrlListWZ@@QAE_NHPBDKKKKK@Z 10060f67 f   CtrlListWZ.obj
 0001:0005ff85       __unwindfunclet$?erase@?$_Tree@V?$_Tmap_traits@V?$basic_string@DU?$char_traits@D@std@@V?$allocator@D@2@@std@@PAXU?$less@V?$basic_string@DU?$char_traits@D@std@@V?$allocator@D@2@@std@@@2@V?$allocator@U?$pair@$$CBV?$basic_string@DU?$char_traits@D@std@@V?$allocator@D@2@@std@@PAX@std@@@2@$00@std@@@std@@QAE?AViterator@12@Vconst_iterator@12@@Z$0 10060f85 f   CtrlListWZ.obj
 0001:0005ff8d       __ehhandler$?erase@?$_Tree@V?$_Tmap_traits@V?$basic_string@DU?$char_traits@D@std@@V?$allocator@D@2@@std@@PAXU?$less@V?$basic_string@DU?$char_traits@D@std@@V?$allocator@D@2@@std@@@2@V?$allocator@U?$pair@$$CBV?$basic_string@DU?$char_traits@D@std@@V?$allocator@D@2@@std@@PAX@std@@@2@$00@std@@@std@@QAE?AViterator@12@Vconst_iterator@12@@Z 10060f8d f   CtrlListWZ.obj
 0001:0005ffab       __unwindfunclet$?_Insert@?$_Tree@V?$_Tmap_traits@KKU?$less@K@std@@V?$allocator@U?$pair@$$CBKK@std@@@2@$0A@@std@@@std@@IAE?AViterator@12@_NPAU_Node@?$_Tree_nod@V?$_Tmap_traits@KKU?$less@K@std@@V?$allocator@U?$pair@$$CBKK@std@@@2@$0A@@std@@@2@ABU?$pair@$$CBKK@2@@Z$0 10060fab f   CtrlListWZ.obj
 0001:0005ffab       __unwindfunclet$?_Insert@?$_Tree@V?$_Tmap_traits@V?$basic_string@DU?$char_traits@D@std@@V?$allocator@D@2@@std@@PAXU?$less@V?$basic_string@DU?$char_traits@D@std@@V?$allocator@D@2@@std@@@2@V?$allocator@U?$pair@$$CBV?$basic_string@DU?$char_traits@D@std@@V?$allocator@D@2@@std@@PAX@std@@@2@$00@std@@@std@@IAE?AViterator@12@_NPAU_Node@?$_Tree_nod@V?$_Tmap_traits@V?$basic_string@DU?$char_traits@D@std@@V?$allocator@D@2@@std@@PAXU?$less@V?$basic_string@DU?$char_traits@D@std@@V?$allocator@D@2@@std@@@2@V?$allocator@U?$pair@$$CBV?$basic_string@DU?$char_traits@D@std@@V?$allocator@D@2@@std@@PAX@std@@@2@$00@std@@@2@ABU?$pair@$$CBV?$basic_string@DU?$char_traits@D@std@@V?$allocator@D@2@@std@@PAX@2@@Z$0 10060fab f   CtrlListWZ.obj
 0001:0005ffab       __unwindfunclet$?_Insert@?$_Tree@V?$_Tmap_traits@KPAXU?$less@K@std@@V?$allocator@U?$pair@$$CBKPAX@std@@@2@$0A@@std@@@std@@IAE?AViterator@12@_NPAU_Node@?$_Tree_nod@V?$_Tmap_traits@KPAXU?$less@K@std@@V?$allocator@U?$pair@$$CBKPAX@std@@@2@$0A@@std@@@2@ABU?$pair@$$CBKPAX@2@@Z$0 10060fab f   CtrlListWZ.obj
 0001:0005ffab       __unwindfunclet$?_Insert@?$_Tree@V?$_Tmap_traits@KPAUCListSellData@CCtrlListWZ@@U?$less@K@std@@V?$allocator@U?$pair@$$CBKPAUCListSellData@CCtrlListWZ@@@std@@@4@$0A@@std@@@std@@IAE?AViterator@12@_NPAU_Node@?$_Tree_nod@V?$_Tmap_traits@KPAUCListSellData@CCtrlListWZ@@U?$less@K@std@@V?$allocator@U?$pair@$$CBKPAUCListSellData@CCtrlListWZ@@@std@@@4@$0A@@std@@@2@ABU?$pair@$$CBKPAUCListSellData@CCtrlListWZ@@@2@@Z$0 10060fab f   CtrlListWZ.obj
 0001:0005ffb3       __ehhandler$?_Insert@?$_Tree@V?$_Tmap_traits@KPAXU?$less@K@std@@V?$allocator@U?$pair@$$CBKPAX@std@@@2@$0A@@std@@@std@@IAE?AViterator@12@_NPAU_Node@?$_Tree_nod@V?$_Tmap_traits@KPAXU?$less@K@std@@V?$allocator@U?$pair@$$CBKPAX@std@@@2@$0A@@std@@@2@ABU?$pair@$$CBKPAX@2@@Z 10060fb3 f   CtrlListWZ.obj
 0001:0005ffb3       __ehhandler$?_Insert@?$_Tree@V?$_Tmap_traits@KPAUCListSellData@CCtrlListWZ@@U?$less@K@std@@V?$allocator@U?$pair@$$CBKPAUCListSellData@CCtrlListWZ@@@std@@@4@$0A@@std@@@std@@IAE?AViterator@12@_NPAU_Node@?$_Tree_nod@V?$_Tmap_traits@KPAUCListSellData@CCtrlListWZ@@U?$less@K@std@@V?$allocator@U?$pair@$$CBKPAUCListSellData@CCtrlListWZ@@@std@@@4@$0A@@std@@@2@ABU?$pair@$$CBKPAUCListSellData@CCtrlListWZ@@@2@@Z 10060fb3 f   CtrlListWZ.obj
 0001:0005ffb3       __ehhandler$?_Insert@?$_Tree@V?$_Tmap_traits@KKU?$less@K@std@@V?$allocator@U?$pair@$$CBKK@std@@@2@$0A@@std@@@std@@IAE?AViterator@12@_NPAU_Node@?$_Tree_nod@V?$_Tmap_traits@KKU?$less@K@std@@V?$allocator@U?$pair@$$CBKK@std@@@2@$0A@@std@@@2@ABU?$pair@$$CBKK@2@@Z 10060fb3 f   CtrlListWZ.obj
 0001:0005ffb3       __ehhandler$?_Insert@?$_Tree@V?$_Tmap_traits@V?$basic_string@DU?$char_traits@D@std@@V?$allocator@D@2@@std@@PAXU?$less@V?$basic_string@DU?$char_traits@D@std@@V?$allocator@D@2@@std@@@2@V?$allocator@U?$pair@$$CBV?$basic_string@DU?$char_traits@D@std@@V?$allocator@D@2@@std@@PAX@std@@@2@$00@std@@@std@@IAE?AViterator@12@_NPAU_Node@?$_Tree_nod@V?$_Tmap_traits@V?$basic_string@DU?$char_traits@D@std@@V?$allocator@D@2@@std@@PAXU?$less@V?$basic_string@DU?$char_traits@D@std@@V?$allocator@D@2@@std@@@2@V?$allocator@U?$pair@$$CBV?$basic_string@DU?$char_traits@D@std@@V?$allocator@D@2@@std@@PAX@std@@@2@$00@std@@@2@ABU?$pair@$$CBV?$basic_string@DU?$char_traits@D@std@@V?$allocator@D@2@@std@@PAX@2@@Z 10060fb3 f   CtrlListWZ.obj
 0001:0005ffd1       __unwindfunclet$?erase@?$_Tree@V?$_Tmap_traits@KKU?$less@K@std@@V?$allocator@U?$pair@$$CBKK@std@@@2@$0A@@std@@@std@@QAE?AViterator@12@Vconst_iterator@12@@Z$0 10060fd1 f   CtrlListWZ.obj
 0001:0005ffd1       __unwindfunclet$?erase@?$_Tree@V?$_Tmap_traits@KPAUCListSellData@CCtrlListWZ@@U?$less@K@std@@V?$allocator@U?$pair@$$CBKPAUCListSellData@CCtrlListWZ@@@std@@@4@$0A@@std@@@std@@QAE?AViterator@12@Vconst_iterator@12@@Z$0 10060fd1 f   CtrlListWZ.obj
 0001:0005ffd1       __unwindfunclet$?erase@?$_Tree@V?$_Tmap_traits@KPAXU?$less@K@std@@V?$allocator@U?$pair@$$CBKPAX@std@@@2@$0A@@std@@@std@@QAE?AViterator@12@Vconst_iterator@12@@Z$0 10060fd1 f   CtrlListWZ.obj
 0001:0005ffd9       __ehhandler$?erase@?$_Tree@V?$_Tmap_traits@KKU?$less@K@std@@V?$allocator@U?$pair@$$CBKK@std@@@2@$0A@@std@@@std@@QAE?AViterator@12@Vconst_iterator@12@@Z 10060fd9 f   CtrlListWZ.obj
 0001:0005ffd9       __ehhandler$?erase@?$_Tree@V?$_Tmap_traits@KPAUCListSellData@CCtrlListWZ@@U?$less@K@std@@V?$allocator@U?$pair@$$CBKPAUCListSellData@CCtrlListWZ@@@std@@@4@$0A@@std@@@std@@QAE?AViterator@12@Vconst_iterator@12@@Z 10060fd9 f   CtrlListWZ.obj
 0001:0005ffd9       __ehhandler$?erase@?$_Tree@V?$_Tmap_traits@KPAXU?$less@K@std@@V?$allocator@U?$pair@$$CBKPAX@std@@@2@$0A@@std@@@std@@QAE?AViterator@12@Vconst_iterator@12@@Z 10060fd9 f   CtrlListWZ.obj
 0001:0005fff7       __ehhandler$?_Buynode@?$_Tree@V?$_Tmap_traits@V?$basic_string@DU?$char_traits@D@std@@V?$allocator@D@2@@std@@PAXU?$less@V?$basic_string@DU?$char_traits@D@std@@V?$allocator@D@2@@std@@@2@V?$allocator@U?$pair@$$CBV?$basic_string@DU?$char_traits@D@std@@V?$allocator@D@2@@std@@PAX@std@@@2@$00@std@@@std@@IAEPAU_Node@?$_Tree_nod@V?$_Tmap_traits@V?$basic_string@DU?$char_traits@D@std@@V?$allocator@D@2@@std@@PAXU?$less@V?$basic_string@DU?$char_traits@D@std@@V?$allocator@D@2@@std@@@2@V?$allocator@U?$pair@$$CBV?$basic_string@DU?$char_traits@D@std@@V?$allocator@D@2@@std@@PAX@std@@@2@$00@std@@@2@XZ 10060ff7 f   CtrlListWZ.obj
 0001:00060012       __unwindfunclet$?_Buynode@?$_Tree@V?$_Tmap_traits@V?$basic_string@DU?$char_traits@D@std@@V?$allocator@D@2@@std@@PAXU?$less@V?$basic_string@DU?$char_traits@D@std@@V?$allocator@D@2@@std@@@2@V?$allocator@U?$pair@$$CBV?$basic_string@DU?$char_traits@D@std@@V?$allocator@D@2@@std@@PAX@std@@@2@$00@std@@@std@@IAEPAU_Node@?$_Tree_nod@V?$_Tmap_traits@V?$basic_string@DU?$char_traits@D@std@@V?$allocator@D@2@@std@@PAXU?$less@V?$basic_string@DU?$char_traits@D@std@@V?$allocator@D@2@@std@@@2@V?$allocator@U?$pair@$$CBV?$basic_string@DU?$char_traits@D@std@@V?$allocator@D@2@@std@@PAX@std@@@2@$00@std@@@2@PAU342@00ABU?$pair@$$CBV?$basic_string@DU?$char_traits@D@std@@V?$allocator@D@2@@std@@PAX@2@D@Z$2 10061012 f   CtrlListWZ.obj
 0001:00060020       __ehhandler$?_Buynode@?$_Tree@V?$_Tmap_traits@V?$basic_string@DU?$char_traits@D@std@@V?$allocator@D@2@@std@@PAXU?$less@V?$basic_string@DU?$char_traits@D@std@@V?$allocator@D@2@@std@@@2@V?$allocator@U?$pair@$$CBV?$basic_string@DU?$char_traits@D@std@@V?$allocator@D@2@@std@@PAX@std@@@2@$00@std@@@std@@IAEPAU_Node@?$_Tree_nod@V?$_Tmap_traits@V?$basic_string@DU?$char_traits@D@std@@V?$allocator@D@2@@std@@PAXU?$less@V?$basic_string@DU?$char_traits@D@std@@V?$allocator@D@2@@std@@@2@V?$allocator@U?$pair@$$CBV?$basic_string@DU?$char_traits@D@std@@V?$allocator@D@2@@std@@PAX@std@@@2@$00@std@@@2@PAU342@00ABU?$pair@$$CBV?$basic_string@DU?$char_traits@D@std@@V?$allocator@D@2@@std@@PAX@2@D@Z 10061020 f   CtrlListWZ.obj
 0001:0006003b       __unwindfunclet$??0CCtrlStaticWZ@@QAE@XZ$0 1006103b f   CtrlStaticWZ.obj
 0001:00060043       __ehhandler$??0CCtrlStaticWZ@@QAE@XZ 10061043 f   CtrlStaticWZ.obj
 0001:0006005e       __unwindfunclet$??1CCtrlStaticWZ@@UAE@XZ$0 1006105e f   CtrlStaticWZ.obj
 0001:00060066       __ehhandler$??1CCtrlStaticWZ@@UAE@XZ 10061066 f   CtrlStaticWZ.obj
 0001:00060081       __unwindfunclet$?ChangeCaptionString@CCtrlStaticWZ@@UAEXXZ$0 10061081 f   CtrlStaticWZ.obj
 0001:00060089       __ehhandler$?ChangeCaptionString@CCtrlStaticWZ@@UAEXXZ 10061089 f   CtrlStaticWZ.obj
 0001:000600ae       __unwindfunclet$??0CCtrlTabWZ@@QAE@XZ$0 100610ae f   CtrlTabWZ.obj
 0001:000600b6       __ehhandler$??0CCtrlTabWZ@@QAE@XZ 100610b6 f   CtrlTabWZ.obj
 0001:000600d1       __unwindfunclet$??1CCtrlTabWZ@@UAE@XZ$0 100610d1 f   CtrlTabWZ.obj
 0001:000600d9       __unwindfunclet$??1CCtrlTabWZ@@UAE@XZ$3 100610d9 f   CtrlTabWZ.obj
 0001:000600e1       __ehhandler$??1CCtrlTabWZ@@UAE@XZ 100610e1 f   CtrlTabWZ.obj
 0001:000600fc       __unwindfunclet$?SetItemCount@CCtrlTabWZ@@UAE_NH@Z$0 100610fc f   CtrlTabWZ.obj
 0001:00060106       __ehhandler$?SetItemCount@CCtrlTabWZ@@UAE_NH@Z 10061106 f   CtrlTabWZ.obj
 0001:00060124       __unwindfunclet$??1STAB_INFO@@QAE@XZ$0 10061124 f   CtrlTabWZ.obj
 0001:0006012c       __unwindfunclet$??1STAB_INFO@@QAE@XZ$1 1006112c f   CtrlTabWZ.obj
 0001:00060134       __ehhandler$??1STAB_INFO@@QAE@XZ 10061134 f   CtrlTabWZ.obj
 0001:0006014f       __unwindfunclet$??0?$_Tree@V?$_Tmap_traits@V?$basic_string@DU?$char_traits@D@std@@V?$allocator@D@2@@std@@PAXU?$less@V?$basic_string@DU?$char_traits@D@std@@V?$allocator@D@2@@std@@@2@V?$allocator@U?$pair@$$CBV?$basic_string@DU?$char_traits@D@std@@V?$allocator@D@2@@std@@PAX@std@@@2@$00@std@@@std@@QAE@ABU?$less@V?$basic_string@DU?$char_traits@D@std@@V?$allocator@D@2@@std@@@1@ABV?$allocator@U?$pair@$$CBV?$basic_string@DU?$char_traits@D@std@@V?$allocator@D@2@@std@@PAX@std@@@1@@Z$0 1006114f f   CtrlTabWZ.obj
 0001:0006014f       __unwindfunclet$??0?$_Tree@V?$_Tmap_traits@KPAUCListSellData@CCtrlListWZ@@U?$less@K@std@@V?$allocator@U?$pair@$$CBKPAUCListSellData@CCtrlListWZ@@@std@@@4@$0A@@std@@@std@@QAE@ABU?$less@K@1@ABV?$allocator@U?$pair@$$CBKPAUCListSellData@CCtrlListWZ@@@std@@@1@@Z$0 1006114f f   CtrlTabWZ.obj
 0001:0006014f       __unwindfunclet$??0?$_Tree@V?$_Tmap_traits@KPAXU?$less@K@std@@V?$allocator@U?$pair@$$CBKPAX@std@@@2@$0A@@std@@@std@@QAE@ABU?$less@K@1@ABV?$allocator@U?$pair@$$CBKPAX@std@@@1@@Z$0 1006114f f   CtrlTabWZ.obj
 0001:0006014f       __unwindfunclet$??0?$_Tree@V?$_Tmap_traits@KKU?$less@K@std@@V?$allocator@U?$pair@$$CBKK@std@@@2@$0A@@std@@@std@@QAE@ABU?$less@K@1@ABV?$allocator@U?$pair@$$CBKK@std@@@1@@Z$0 1006114f f   CtrlTabWZ.obj
 0001:00060157       __ehhandler$??0?$_Tree@V?$_Tmap_traits@KKU?$less@K@std@@V?$allocator@U?$pair@$$CBKK@std@@@2@$0A@@std@@@std@@QAE@ABU?$less@K@1@ABV?$allocator@U?$pair@$$CBKK@std@@@1@@Z 10061157 f   CtrlTabWZ.obj
 0001:00060157       __ehhandler$??0?$_Tree@V?$_Tmap_traits@KPAUCListSellData@CCtrlListWZ@@U?$less@K@std@@V?$allocator@U?$pair@$$CBKPAUCListSellData@CCtrlListWZ@@@std@@@4@$0A@@std@@@std@@QAE@ABU?$less@K@1@ABV?$allocator@U?$pair@$$CBKPAUCListSellData@CCtrlListWZ@@@std@@@1@@Z 10061157 f   CtrlTabWZ.obj
 0001:00060157       __ehhandler$??0?$_Tree@V?$_Tmap_traits@KPAXU?$less@K@std@@V?$allocator@U?$pair@$$CBKPAX@std@@@2@$0A@@std@@@std@@QAE@ABU?$less@K@1@ABV?$allocator@U?$pair@$$CBKPAX@std@@@1@@Z 10061157 f   CtrlTabWZ.obj
 0001:00060157       __ehhandler$??0?$_Tree@V?$_Tmap_traits@V?$basic_string@DU?$char_traits@D@std@@V?$allocator@D@2@@std@@PAXU?$less@V?$basic_string@DU?$char_traits@D@std@@V?$allocator@D@2@@std@@@2@V?$allocator@U?$pair@$$CBV?$basic_string@DU?$char_traits@D@std@@V?$allocator@D@2@@std@@PAX@std@@@2@$00@std@@@std@@QAE@ABU?$less@V?$basic_string@DU?$char_traits@D@std@@V?$allocator@D@2@@std@@@1@ABV?$allocator@U?$pair@$$CBV?$basic_string@DU?$char_traits@D@std@@V?$allocator@D@2@@std@@PAX@std@@@1@@Z 10061157 f   CtrlTabWZ.obj
 0001:00060172       __ehhandler$?_Buynode@?$_Tree@V?$_Tmap_traits@KKU?$less@K@std@@V?$allocator@U?$pair@$$CBKK@std@@@2@$0A@@std@@@std@@IAEPAU_Node@?$_Tree_nod@V?$_Tmap_traits@KKU?$less@K@std@@V?$allocator@U?$pair@$$CBKK@std@@@2@$0A@@std@@@2@XZ 10061172 f   CtrlTabWZ.obj
 0001:00060172       __ehhandler$?_Buynode@?$_Tree@V?$_Tmap_traits@KPAXU?$less@K@std@@V?$allocator@U?$pair@$$CBKPAX@std@@@2@$0A@@std@@@std@@IAEPAU_Node@?$_Tree_nod@V?$_Tmap_traits@KPAXU?$less@K@std@@V?$allocator@U?$pair@$$CBKPAX@std@@@2@$0A@@std@@@2@XZ 10061172 f   CtrlTabWZ.obj
 0001:00060172       __ehhandler$?_Buynode@?$_Tree@V?$_Tmap_traits@KPAUCListSellData@CCtrlListWZ@@U?$less@K@std@@V?$allocator@U?$pair@$$CBKPAUCListSellData@CCtrlListWZ@@@std@@@4@$0A@@std@@@std@@IAEPAU_Node@?$_Tree_nod@V?$_Tmap_traits@KPAUCListSellData@CCtrlListWZ@@U?$less@K@std@@V?$allocator@U?$pair@$$CBKPAUCListSellData@CCtrlListWZ@@@std@@@4@$0A@@std@@@2@XZ 10061172 f   CtrlTabWZ.obj
 0001:0006018d       __ehhandler$?_Buynode@?$_Tree@V?$_Tmap_traits@KPAUCListSellData@CCtrlListWZ@@U?$less@K@std@@V?$allocator@U?$pair@$$CBKPAUCListSellData@CCtrlListWZ@@@std@@@4@$0A@@std@@@std@@IAEPAU_Node@?$_Tree_nod@V?$_Tmap_traits@KPAUCListSellData@CCtrlListWZ@@U?$less@K@std@@V?$allocator@U?$pair@$$CBKPAUCListSellData@CCtrlListWZ@@@std@@@4@$0A@@std@@@2@PAU342@00ABU?$pair@$$CBKPAUCListSellData@CCtrlListWZ@@@2@D@Z 1006118d f   CtrlTabWZ.obj
 0001:0006018d       __ehhandler$?_Buynode@?$_Tree@V?$_Tmap_traits@KKU?$less@K@std@@V?$allocator@U?$pair@$$CBKK@std@@@2@$0A@@std@@@std@@IAEPAU_Node@?$_Tree_nod@V?$_Tmap_traits@KKU?$less@K@std@@V?$allocator@U?$pair@$$CBKK@std@@@2@$0A@@std@@@2@PAU342@00ABU?$pair@$$CBKK@2@D@Z 1006118d f   CtrlTabWZ.obj
 0001:0006018d       __ehhandler$?_Buynode@?$_Tree@V?$_Tmap_traits@KPAXU?$less@K@std@@V?$allocator@U?$pair@$$CBKPAX@std@@@2@$0A@@std@@@std@@IAEPAU_Node@?$_Tree_nod@V?$_Tmap_traits@KPAXU?$less@K@std@@V?$allocator@U?$pair@$$CBKPAX@std@@@2@$0A@@std@@@2@PAU342@00ABU?$pair@$$CBKPAX@2@D@Z 1006118d f   CtrlTabWZ.obj
 0001:000601a8       __unwindfunclet$??0CCtrlVScrollWZ@@QAE@XZ$0 100611a8 f   CtrlVScrollWZ.obj
 0001:000601b0       __unwindfunclet$??0CCtrlVScrollWZ@@QAE@XZ$1 100611b0 f   CtrlVScrollWZ.obj
 0001:000601be       __unwindfunclet$??0CCtrlVScrollWZ@@QAE@XZ$2 100611be f   CtrlVScrollWZ.obj
 0001:000601cc       __ehhandler$??0CCtrlVScrollWZ@@QAE@XZ 100611cc f   CtrlVScrollWZ.obj
 0001:000601e7       __unwindfunclet$??1CCtrlVScrollWZ@@UAE@XZ$0 100611e7 f   CtrlVScrollWZ.obj
 0001:000601ef       __unwindfunclet$??1CCtrlVScrollWZ@@UAE@XZ$1 100611ef f   CtrlVScrollWZ.obj
 0001:000601fd       __unwindfunclet$??1CCtrlVScrollWZ@@UAE@XZ$2 100611fd f   CtrlVScrollWZ.obj
 0001:0006020b       __ehhandler$??1CCtrlVScrollWZ@@UAE@XZ 1006120b f   CtrlVScrollWZ.obj
 0001:00060226       __unwindfunclet$?Navigate@CCtrlWebBrowserWZ@@UAEXPB_W@Z$0 10061226 f   CtrlWebBrowserWZ.obj
 0001:0006022e       __unwindfunclet$?Navigate@CCtrlWebBrowserWZ@@UAEXPB_W@Z$1 1006122e f   CtrlWebBrowserWZ.obj
 0001:00060236       __unwindfunclet$?Navigate@CCtrlWebBrowserWZ@@UAEXPB_W@Z$4 10061236 f   CtrlWebBrowserWZ.obj
 0001:0006023e       __ehhandler$?Navigate@CCtrlWebBrowserWZ@@UAEXPB_W@Z 1006123e f   CtrlWebBrowserWZ.obj
 0001:00060259       __unwindfunclet$??0_bstr_t@@QAE@PB_W@Z$0 10061259 f   CtrlWebBrowserWZ.obj
 0001:00060263       __ehhandler$??0_bstr_t@@QAE@PB_W@Z 10061263 f   CtrlWebBrowserWZ.obj
 0001:0006027e       __unwindfunclet$??0CDialogWZ@@QAE@XZ$0 1006127e f   DialogWZ.obj
 0001:00060286       __unwindfunclet$??0CDialogWZ@@QAE@XZ$1 10061286 f   DialogWZ.obj
 0001:00060291       __unwindfunclet$??0CDialogWZ@@QAE@XZ$2 10061291 f   DialogWZ.obj
 0001:0006029c       __unwindfunclet$??0CDialogWZ@@QAE@XZ$3 1006129c f   DialogWZ.obj
 0001:000602a6       __ehhandler$??0CDialogWZ@@QAE@XZ 100612a6 f   DialogWZ.obj
 0001:000602c1       __unwindfunclet$??1CDialogWZ@@UAE@XZ$0 100612c1 f   DialogWZ.obj
 0001:000602c9       __unwindfunclet$??1CDialogWZ@@UAE@XZ$1 100612c9 f   DialogWZ.obj
 0001:000602d4       __unwindfunclet$??1CDialogWZ@@UAE@XZ$2 100612d4 f   DialogWZ.obj
 0001:000602df       __unwindfunclet$??1CDialogWZ@@UAE@XZ$3 100612df f   DialogWZ.obj
 0001:000602e7       __ehhandler$??1CDialogWZ@@UAE@XZ 100612e7 f   DialogWZ.obj
 0001:00060302       __unwindfunclet$?CreateControllWZ@CDialogWZ@@QAEPAVCControlWZ@@KKKPAUHWND__@@PAUHINSTANCE__@@PAUtagRECT@@PAX@Z$0 10061302 f   DialogWZ.obj
 0001:0006030c       __unwindfunclet$?CreateControllWZ@CDialogWZ@@QAEPAVCControlWZ@@KKKPAUHWND__@@PAUHINSTANCE__@@PAUtagRECT@@PAX@Z$1 1006130c f   DialogWZ.obj
 0001:00060316       __unwindfunclet$?CreateControllWZ@CDialogWZ@@QAEPAVCControlWZ@@KKKPAUHWND__@@PAUHINSTANCE__@@PAUtagRECT@@PAX@Z$2 10061316 f   DialogWZ.obj
 0001:00060320       __unwindfunclet$?CreateControllWZ@CDialogWZ@@QAEPAVCControlWZ@@KKKPAUHWND__@@PAUHINSTANCE__@@PAUtagRECT@@PAX@Z$3 10061320 f   DialogWZ.obj
 0001:0006032a       __unwindfunclet$?CreateControllWZ@CDialogWZ@@QAEPAVCControlWZ@@KKKPAUHWND__@@PAUHINSTANCE__@@PAUtagRECT@@PAX@Z$4 1006132a f   DialogWZ.obj
 0001:00060334       __unwindfunclet$?CreateControllWZ@CDialogWZ@@QAEPAVCControlWZ@@KKKPAUHWND__@@PAUHINSTANCE__@@PAUtagRECT@@PAX@Z$5 10061334 f   DialogWZ.obj
 0001:0006033e       __unwindfunclet$?CreateControllWZ@CDialogWZ@@QAEPAVCControlWZ@@KKKPAUHWND__@@PAUHINSTANCE__@@PAUtagRECT@@PAX@Z$6 1006133e f   DialogWZ.obj
 0001:00060348       __unwindfunclet$?CreateControllWZ@CDialogWZ@@QAEPAVCControlWZ@@KKKPAUHWND__@@PAUHINSTANCE__@@PAUtagRECT@@PAX@Z$7 10061348 f   DialogWZ.obj
 0001:00060352       __unwindfunclet$?CreateControllWZ@CDialogWZ@@QAEPAVCControlWZ@@KKKPAUHWND__@@PAUHINSTANCE__@@PAUtagRECT@@PAX@Z$8 10061352 f   DialogWZ.obj
 0001:0006035c       __unwindfunclet$?CreateControllWZ@CDialogWZ@@QAEPAVCControlWZ@@KKKPAUHWND__@@PAUHINSTANCE__@@PAUtagRECT@@PAX@Z$9 1006135c f   DialogWZ.obj
 0001:00060366       __unwindfunclet$?CreateControllWZ@CDialogWZ@@QAEPAVCControlWZ@@KKKPAUHWND__@@PAUHINSTANCE__@@PAUtagRECT@@PAX@Z$10 10061366 f   DialogWZ.obj
 0001:00060370       __unwindfunclet$?CreateControllWZ@CDialogWZ@@QAEPAVCControlWZ@@KKKPAUHWND__@@PAUHINSTANCE__@@PAUtagRECT@@PAX@Z$11 10061370 f   DialogWZ.obj
 0001:0006037a       __unwindfunclet$?CreateControllWZ@CDialogWZ@@QAEPAVCControlWZ@@KKKPAUHWND__@@PAUHINSTANCE__@@PAUtagRECT@@PAX@Z$12 1006137a f   DialogWZ.obj
 0001:00060384       __unwindfunclet$?CreateControllWZ@CDialogWZ@@QAEPAVCControlWZ@@KKKPAUHWND__@@PAUHINSTANCE__@@PAUtagRECT@@PAX@Z$13 10061384 f   DialogWZ.obj
 0001:0006038e       __unwindfunclet$?CreateControllWZ@CDialogWZ@@QAEPAVCControlWZ@@KKKPAUHWND__@@PAUHINSTANCE__@@PAUtagRECT@@PAX@Z$14 1006138e f   DialogWZ.obj
 0001:0006039b       __ehhandler$?CreateControllWZ@CDialogWZ@@QAEPAVCControlWZ@@KKKPAUHWND__@@PAUHINSTANCE__@@PAUtagRECT@@PAX@Z 1006139b f   DialogWZ.obj
 0001:000603b9       __ehhandler$?_Buynode@?$list@UtagRECT@@V?$allocator@UtagRECT@@@std@@@std@@IAEPAU_Node@?$_List_nod@UtagRECT@@V?$allocator@UtagRECT@@@std@@@2@XZ 100613b9 f   DialogWZ.obj
 0001:000603d4       __ehhandler$?_Buynode@?$list@UtagRECT@@V?$allocator@UtagRECT@@@std@@@std@@IAEPAU_Node@?$_List_nod@UtagRECT@@V?$allocator@UtagRECT@@@std@@@2@PAU342@0ABUtagRECT@@@Z 100613d4 f   DialogWZ.obj
 0001:000603ef       __ehhandler$?_Buynode@?$list@KV?$allocator@K@std@@@std@@IAEPAU_Node@?$_List_nod@KV?$allocator@K@std@@@2@XZ 100613ef f   DialogWZ.obj
 0001:000603ef       __ehhandler$?_Buynode@?$list@PAVCControlWZ@@V?$allocator@PAVCControlWZ@@@std@@@std@@IAEPAU_Node@?$_List_nod@PAVCControlWZ@@V?$allocator@PAVCControlWZ@@@std@@@2@XZ 100613ef f   DialogWZ.obj
 0001:000603ef       __ehhandler$?_Buynode@?$list@PAXV?$allocator@PAX@std@@@std@@IAEPAU_Node@?$_List_nod@PAXV?$allocator@PAX@std@@@2@XZ 100613ef f   DialogWZ.obj
 0001:0006040a       __unwindfunclet$??0?$_Container_base_aux_alloc_real@V?$allocator@PAVCControlWZ@@@std@@@std@@IAE@V?$allocator@PAVCControlWZ@@@1@@Z$0 1006140a f   DialogWZ.obj
 0001:0006040a       __unwindfunclet$??0?$_Container_base_aux_alloc_real@V?$allocator@U?$pair@$$CBKPAX@std@@@std@@@std@@IAE@V?$allocator@U?$pair@$$CBKPAX@std@@@1@@Z$0 1006140a f   DialogWZ.obj
 0001:0006040a       __unwindfunclet$??0?$_Container_base_aux_alloc_real@V?$allocator@U_List_position@?$_Hash@V?$_Hmap_traits@KPAXV?$hash_compare@KU?$less@K@std@@@stdext@@V?$allocator@U?$pair@$$CBKPAX@std@@@std@@$0A@@stdext@@@stdext@@@std@@@std@@IAE@V?$allocator@U_List_position@?$_Hash@V?$_Hmap_traits@KPAXV?$hash_compare@KU?$less@K@std@@@stdext@@V?$allocator@U?$pair@$$CBKPAX@std@@@std@@$0A@@stdext@@@stdext@@@1@@Z$0 1006140a f   DialogWZ.obj
 0001:0006040a       __unwindfunclet$??0?$_Container_base_aux_alloc_real@V?$allocator@PAX@std@@@std@@IAE@V?$allocator@PAX@1@@Z$0 1006140a f   DialogWZ.obj
 0001:0006040a       __unwindfunclet$??0?$_Container_base_aux_alloc_real@V?$allocator@U?$pair@$$CBKV?$basic_string@DU?$char_traits@D@std@@V?$allocator@D@2@@std@@@std@@@std@@@std@@IAE@V?$allocator@U?$pair@$$CBKV?$basic_string@DU?$char_traits@D@std@@V?$allocator@D@2@@std@@@std@@@1@@Z$0 1006140a f   DialogWZ.obj
 0001:0006040a       __unwindfunclet$??0?$_Container_base_aux_alloc_real@V?$allocator@K@std@@@std@@IAE@V?$allocator@K@1@@Z$0 1006140a f   DialogWZ.obj
 0001:0006040a       __unwindfunclet$??0?$_Container_base_aux_alloc_real@V?$allocator@U_List_position@?$_Hash@V?$_Hmap_traits@KV?$basic_string@DU?$char_traits@D@std@@V?$allocator@D@2@@std@@V?$hash_compare@KU?$less@K@std@@@stdext@@V?$allocator@U?$pair@$$CBKV?$basic_string@DU?$char_traits@D@std@@V?$allocator@D@2@@std@@@std@@@2@$0A@@stdext@@@stdext@@@std@@@std@@IAE@V?$allocator@U_List_position@?$_Hash@V?$_Hmap_traits@KV?$basic_string@DU?$char_traits@D@std@@V?$allocator@D@2@@std@@V?$hash_compare@KU?$less@K@std@@@stdext@@V?$allocator@U?$pair@$$CBKV?$basic_string@DU?$char_traits@D@std@@V?$allocator@D@2@@std@@@std@@@2@$0A@@stdext@@@stdext@@@1@@Z$0 1006140a f   DialogWZ.obj
 0001:0006040a       __unwindfunclet$??0?$_Container_base_aux_alloc_real@V?$allocator@U?$pair@$$CBKPAUCListSellData@CCtrlListWZ@@@std@@@std@@@std@@IAE@V?$allocator@U?$pair@$$CBKPAUCListSellData@CCtrlListWZ@@@std@@@1@@Z$0 1006140a f   DialogWZ.obj
 0001:0006040a       __unwindfunclet$??0?$_Container_base_aux_alloc_real@V?$allocator@U?$pair@$$CBV?$basic_string@DU?$char_traits@D@std@@V?$allocator@D@2@@std@@PAX@std@@@std@@@std@@IAE@V?$allocator@U?$pair@$$CBV?$basic_string@DU?$char_traits@D@std@@V?$allocator@D@2@@std@@PAX@std@@@1@@Z$0 1006140a f   DialogWZ.obj
 0001:0006040a       __unwindfunclet$??0?$_Container_base_aux_alloc_real@V?$allocator@UtagRECT@@@std@@@std@@IAE@V?$allocator@UtagRECT@@@1@@Z$0 1006140a f   DialogWZ.obj
 0001:0006040a       __unwindfunclet$??0?$_Container_base_aux_alloc_real@V?$allocator@U?$pair@$$CBKK@std@@@std@@@std@@IAE@V?$allocator@U?$pair@$$CBKK@std@@@1@@Z$0 1006140a f   DialogWZ.obj
 0001:00060412       __ehhandler$??0?$_Container_base_aux_alloc_real@V?$allocator@U?$pair@$$CBKK@std@@@std@@@std@@IAE@V?$allocator@U?$pair@$$CBKK@std@@@1@@Z 10061412 f   DialogWZ.obj
 0001:00060412       __ehhandler$??0?$_Container_base_aux_alloc_real@V?$allocator@U?$pair@$$CBKPAUCListSellData@CCtrlListWZ@@@std@@@std@@@std@@IAE@V?$allocator@U?$pair@$$CBKPAUCListSellData@CCtrlListWZ@@@std@@@1@@Z 10061412 f   DialogWZ.obj
 0001:00060412       __ehhandler$??0?$_Container_base_aux_alloc_real@V?$allocator@UtagRECT@@@std@@@std@@IAE@V?$allocator@UtagRECT@@@1@@Z 10061412 f   DialogWZ.obj
 0001:00060412       __ehhandler$??0?$_Container_base_aux_alloc_real@V?$allocator@U?$pair@$$CBV?$basic_string@DU?$char_traits@D@std@@V?$allocator@D@2@@std@@PAX@std@@@std@@@std@@IAE@V?$allocator@U?$pair@$$CBV?$basic_string@DU?$char_traits@D@std@@V?$allocator@D@2@@std@@PAX@std@@@1@@Z 10061412 f   DialogWZ.obj
 0001:00060412       __ehhandler$??0?$_Container_base_aux_alloc_real@V?$allocator@U?$pair@$$CBKV?$basic_string@DU?$char_traits@D@std@@V?$allocator@D@2@@std@@@std@@@std@@@std@@IAE@V?$allocator@U?$pair@$$CBKV?$basic_string@DU?$char_traits@D@std@@V?$allocator@D@2@@std@@@std@@@1@@Z 10061412 f   DialogWZ.obj
 0001:00060412       __ehhandler$??0?$_Container_base_aux_alloc_real@V?$allocator@PAX@std@@@std@@IAE@V?$allocator@PAX@1@@Z 10061412 f   DialogWZ.obj
 0001:00060412       __ehhandler$??0?$_Container_base_aux_alloc_real@V?$allocator@U_List_position@?$_Hash@V?$_Hmap_traits@KV?$basic_string@DU?$char_traits@D@std@@V?$allocator@D@2@@std@@V?$hash_compare@KU?$less@K@std@@@stdext@@V?$allocator@U?$pair@$$CBKV?$basic_string@DU?$char_traits@D@std@@V?$allocator@D@2@@std@@@std@@@2@$0A@@stdext@@@stdext@@@std@@@std@@IAE@V?$allocator@U_List_position@?$_Hash@V?$_Hmap_traits@KV?$basic_string@DU?$char_traits@D@std@@V?$allocator@D@2@@std@@V?$hash_compare@KU?$less@K@std@@@stdext@@V?$allocator@U?$pair@$$CBKV?$basic_string@DU?$char_traits@D@std@@V?$allocator@D@2@@std@@@std@@@2@$0A@@stdext@@@stdext@@@1@@Z 10061412 f   DialogWZ.obj
 0001:00060412       __ehhandler$??0?$_Container_base_aux_alloc_real@V?$allocator@K@std@@@std@@IAE@V?$allocator@K@1@@Z 10061412 f   DialogWZ.obj
 0001:00060412       __ehhandler$??0?$_Container_base_aux_alloc_real@V?$allocator@PAVCControlWZ@@@std@@@std@@IAE@V?$allocator@PAVCControlWZ@@@1@@Z 10061412 f   DialogWZ.obj
 0001:00060412       __ehhandler$??0?$_Container_base_aux_alloc_real@V?$allocator@U_List_position@?$_Hash@V?$_Hmap_traits@KPAXV?$hash_compare@KU?$less@K@std@@@stdext@@V?$allocator@U?$pair@$$CBKPAX@std@@@std@@$0A@@stdext@@@stdext@@@std@@@std@@IAE@V?$allocator@U_List_position@?$_Hash@V?$_Hmap_traits@KPAXV?$hash_compare@KU?$less@K@std@@@stdext@@V?$allocator@U?$pair@$$CBKPAX@std@@@std@@$0A@@stdext@@@stdext@@@1@@Z 10061412 f   DialogWZ.obj
 0001:00060412       __ehhandler$??0?$_Container_base_aux_alloc_real@V?$allocator@U?$pair@$$CBKPAX@std@@@std@@@std@@IAE@V?$allocator@U?$pair@$$CBKPAX@std@@@1@@Z 10061412 f   DialogWZ.obj
 0001:0006042d       __unwindfunclet$??__F?static_stdListEditPtr@CDialogWZ@@2V?$list@PAVCControlWZ@@V?$allocator@PAVCControlWZ@@@std@@@std@@A@@YAXXZ$0 1006142d f   DialogWZ.obj
 0001:00060437       __ehhandler$??__F?static_stdListEditPtr@CDialogWZ@@2V?$list@PAVCControlWZ@@V?$allocator@PAVCControlWZ@@@std@@@std@@A@@YAXXZ 10061437 f   DialogWZ.obj
 0001:00060452       __unwindfunclet$??0CDialogManager@@QAE@XZ$0 10061452 f   DialogManager.obj
 0001:00060460       __unwindfunclet$??0CDialogManager@@QAE@XZ$1 10061460 f   DialogManager.obj
 0001:0006046a       __unwindfunclet$??0CDialogManager@@QAE@XZ$2 1006146a f   DialogManager.obj
 0001:00060474       __unwindfunclet$??0CDialogManager@@QAE@XZ$3 10061474 f   DialogManager.obj
 0001:0006047e       __ehhandler$??0CDialogManager@@QAE@XZ 1006147e f   DialogManager.obj
 0001:00060499       __unwindfunclet$??1CDialogManager@@UAE@XZ$0 10061499 f   DialogManager.obj
 0001:000604a7       __unwindfunclet$??1CDialogManager@@UAE@XZ$1 100614a7 f   DialogManager.obj
 0001:000604af       __ehhandler$??1CDialogManager@@UAE@XZ 100614af f   DialogManager.obj
 0001:000604ca       __unwindfunclet$?CreateDialogWZ@CDialogManager@@UAEPAVCDialogWZ@@KK@Z$0 100614ca f   DialogManager.obj
 0001:000604d4       __ehhandler$?CreateDialogWZ@CDialogManager@@UAEPAVCDialogWZ@@KK@Z 100614d4 f   DialogManager.obj
 0001:000604ef       __unwindfunclet$?InitializeWzLogSystem@@YAXXZ$0 100614ef f   programcommonlibforengine:wzlogsystem.obj
 0001:000604f9       __ehhandler$?InitializeWzLogSystem@@YAXXZ 100614f9 f   programcommonlibforengine:wzlogsystem.obj
 0001:00060514       __unwindfunclet$??0CDiscAccess@@QAE@XZ$0 10061514 f   programcommonlibforengine:discaccess.obj
 0001:00060522       __unwindfunclet$??0CDiscAccess@@QAE@XZ$1 10061522 f   programcommonlibforengine:discaccess.obj
 0001:00060530       __ehhandler$??0CDiscAccess@@QAE@XZ 10061530 f   programcommonlibforengine:discaccess.obj
 0001:0006054b       __unwindfunclet$??1CDiscAccess@@QAE@XZ$0 1006154b f   programcommonlibforengine:discaccess.obj
 0001:00060559       __unwindfunclet$??1CDiscAccess@@QAE@XZ$1 10061559 f   programcommonlibforengine:discaccess.obj
 0001:00060567       __ehhandler$??1CDiscAccess@@QAE@XZ 10061567 f   programcommonlibforengine:discaccess.obj
 0001:00060582       __unwindfunclet$?OpenDisc_Packer@CDiscAccess@@QAEHKPBD0W4ENUM_OPEN_PACKER_TYPE@@@Z$0 10061582 f   programcommonlibforengine:discaccess.obj
 0001:0006058a       __unwindfunclet$?OpenDisc_Packer@CDiscAccess@@QAEHKPBD0W4ENUM_OPEN_PACKER_TYPE@@@Z$1 1006158a f   programcommonlibforengine:discaccess.obj
 0001:00060594       __ehhandler$?OpenDisc_Packer@CDiscAccess@@QAEHKPBD0W4ENUM_OPEN_PACKER_TYPE@@@Z 10061594 f   programcommonlibforengine:discaccess.obj
 0001:000605af       __unwindfunclet$?CloseDisc@CDiscAccess@@QAEXK@Z$0 100615af f   programcommonlibforengine:discaccess.obj
 0001:000605b7       __ehhandler$?CloseDisc@CDiscAccess@@QAEXK@Z 100615b7 f   programcommonlibforengine:discaccess.obj
 0001:000605d2       __unwindfunclet$?OpenFile@CDiscAccess@@QAEPAXKPBDKKW4ENUM_OPEN_DISPOSITION@@@Z$0 100615d2 f   programcommonlibforengine:discaccess.obj
 0001:000605da       __ehhandler$?OpenFile@CDiscAccess@@QAEPAXKPBDKKW4ENUM_OPEN_DISPOSITION@@@Z 100615da f   programcommonlibforengine:discaccess.obj
 0001:00060602       __unwindfunclet$?CloseFile@CDiscAccess@@QAEHPAX@Z$0 10061602 f   programcommonlibforengine:discaccess.obj
 0001:0006060a       __ehhandler$?CloseFile@CDiscAccess@@QAEHPAX@Z 1006160a f   programcommonlibforengine:discaccess.obj
 0001:00060625       __unwindfunclet$?SeekFile@CDiscAccess@@QAEKPAXJW4ENUM_SEEK_ORIGIN@@@Z$0 10061625 f   programcommonlibforengine:discaccess.obj
 0001:0006062d       __ehhandler$?SeekFile@CDiscAccess@@QAEKPAXJW4ENUM_SEEK_ORIGIN@@@Z 1006162d f   programcommonlibforengine:discaccess.obj
 0001:00060648       __unwindfunclet$?ReadFile@CDiscAccess@@QAEKPAX0K@Z$0 10061648 f   programcommonlibforengine:discaccess.obj
 0001:00060650       __ehhandler$?ReadFile@CDiscAccess@@QAEKPAX0K@Z 10061650 f   programcommonlibforengine:discaccess.obj
 0001:0006066b       __unwindfunclet$?WriteFile@CDiscAccess@@QAEKPAXPBXK@Z$0 1006166b f   programcommonlibforengine:discaccess.obj
 0001:00060673       __ehhandler$?WriteFile@CDiscAccess@@QAEKPAXPBXK@Z 10061673 f   programcommonlibforengine:discaccess.obj
 0001:0006068e       __unwindfunclet$?FileExists@CDiscAccess@@QAEHKPBD@Z$0 1006168e f   programcommonlibforengine:discaccess.obj
 0001:00060696       __ehhandler$?FileExists@CDiscAccess@@QAEHKPBD@Z 10061696 f   programcommonlibforengine:discaccess.obj
 0001:000606be       __unwindfunclet$?GetFileSize@CDiscAccess@@QAEKPAX@Z$0 100616be f   programcommonlibforengine:discaccess.obj
 0001:000606c6       __ehhandler$?GetFileSize@CDiscAccess@@QAEKPAX@Z 100616c6 f   programcommonlibforengine:discaccess.obj
 0001:000606e1       __unwindfunclet$?GetFileInformationByHandle@CDiscAccess@@QAEHPAXPAUSt_FileInformation@@@Z$0 100616e1 f   programcommonlibforengine:discaccess.obj
 0001:000606e9       __ehhandler$?GetFileInformationByHandle@CDiscAccess@@QAEHPAXPAUSt_FileInformation@@@Z 100616e9 f   programcommonlibforengine:discaccess.obj
 0001:00060711       __unwindfunclet$?CopyFileA@CDiscAccess@@QAEHKPBD0@Z$0 10061711 f   programcommonlibforengine:discaccess.obj
 0001:00060719       __ehhandler$?CopyFileA@CDiscAccess@@QAEHKPBD0@Z 10061719 f   programcommonlibforengine:discaccess.obj
 0001:00060741       __unwindfunclet$?DeleteFileA@CDiscAccess@@QAEHKPBD@Z$0 10061741 f   programcommonlibforengine:discaccess.obj
 0001:00060749       __ehhandler$?DeleteFileA@CDiscAccess@@QAEHKPBD@Z 10061749 f   programcommonlibforengine:discaccess.obj
 0001:00060771       __unwindfunclet$?CreateDirectoryA@CDiscAccess@@QAEHKPBD@Z$0 10061771 f   programcommonlibforengine:discaccess.obj
 0001:00060779       __ehhandler$?CreateDirectoryA@CDiscAccess@@QAEHKPBD@Z 10061779 f   programcommonlibforengine:discaccess.obj
 0001:000607a1       __unwindfunclet$?RemoveDirectoryA@CDiscAccess@@QAEHKPBD@Z$0 100617a1 f   programcommonlibforengine:discaccess.obj
 0001:000607a9       __ehhandler$?RemoveDirectoryA@CDiscAccess@@QAEHKPBD@Z 100617a9 f   programcommonlibforengine:discaccess.obj
 0001:000607d1       __unwindfunclet$??0?$CWzHandleManager@USt_DAFileInfo@@@@QAE@XZ$0 100617d1 f   programcommonlibforengine:discaccess.obj
 0001:000607dc       __unwindfunclet$??0?$CWzHandleManager@USt_DAFileInfo@@@@QAE@XZ$1 100617dc f   programcommonlibforengine:discaccess.obj
 0001:000607e7       __unwindfunclet$??0?$CWzHandleManager@USt_DAFileInfo@@@@QAE@XZ$2 100617e7 f   programcommonlibforengine:discaccess.obj
 0001:000607f2       __ehhandler$??0?$CWzHandleManager@USt_DAFileInfo@@@@QAE@XZ 100617f2 f   programcommonlibforengine:discaccess.obj
 0001:0006080d       __unwindfunclet$??1?$CWzHandleManager@USt_DAFileInfo@@@@UAE@XZ$0 1006180d f   programcommonlibforengine:discaccess.obj
 0001:00060818       __unwindfunclet$??1?$CWzHandleManager@USt_DAFileInfo@@@@UAE@XZ$1 10061818 f   programcommonlibforengine:discaccess.obj
 0001:00060823       __ehhandler$??1?$CWzHandleManager@USt_DAFileInfo@@@@UAE@XZ 10061823 f   programcommonlibforengine:discaccess.obj
 0001:0006083e       __unwindfunclet$?_Xlen@_String_base@std@@SAXXZ$0 1006183e f   libcpmt:string.obj
 0001:0006083e       __unwindfunclet$?_Xran@_String_base@std@@SAXXZ$0 1006183e f   libcpmt:string.obj
 0001:00060846       __ehhandler$?_Xlen@_String_base@std@@SAXXZ 10061846 f   libcpmt:string.obj
 0001:00060846       __ehhandler$?_Xran@_String_base@std@@SAXXZ 10061846 f   libcpmt:string.obj
 0001:00060861       __ehhandler$?CallUnexpected@@YAXPBU_s_ESTypeList@@@Z 10061861 f   LIBCMT:frame.obj
 0001:00060880       ??__EEXTERNAL_API_INITIALIZER@@YAXXZ 10061880 f   CtrlDxEdit.obj
 0001:0006089a       ??__E?s_CandList@CCtrlDxIMEEditBox@@1UCCandList@1@A@@YAXXZ 1006189a f   CtrlDxEdit.obj
 0001:000608b6       ??__E?s_Locale@CCtrlDxIMEEditBox@@1V?$CGrowableArray@UCInputLocale@CCtrlDxIMEEditBox@@@@A@@YAXXZ 100618b6 f   CtrlDxEdit.obj
 0001:000608db       ??__E?static_stdListEditPtr@CDialogWZ@@2V?$list@PAVCControlWZ@@V?$allocator@PAVCControlWZ@@@std@@@std@@A@@YAXXZ 100618db f   DialogWZ.obj
 0001:00060900       ??__Eautofree@@YAXXZ       10061900 f   wzFilePacker_static:wzFilePacker.obj
 0001:00060910       ??__Fs_invalid_string_value@?4??FindString@CStringManager@@QAEABV?$basic_string@DU?$char_traits@D@std@@V?$allocator@D@2@@std@@K@Z@YAXXZ 10061910 f   StringManager.obj
 0001:00060926       ??__FEXTERNAL_API_INITIALIZER@@YAXXZ 10061926 f   CtrlDxEdit.obj
 0001:00060935       ??__F?s_CandList@CCtrlDxIMEEditBox@@1UCCandList@1@A@@YAXXZ 10061935 f   CtrlDxEdit.obj
 0001:00060944       ??__F?s_Locale@CCtrlDxIMEEditBox@@1V?$CGrowableArray@UCInputLocale@CCtrlDxIMEEditBox@@@@A@@YAXXZ 10061944 f   CtrlDxEdit.obj
 0001:00060955       ??__F?static_stdListEditPtr@CDialogWZ@@2V?$list@PAVCControlWZ@@V?$allocator@PAVCControlWZ@@@std@@@std@@A@@YAXXZ 10061955 f   DialogWZ.obj
 0001:000609aa       ??__Fnomem@?5???2@YAPAXI@Z@YAXXZ 100619aa f   LIBCMT:new.obj
 0001:000609c0       ??__Fautofree@@YAXXZ       100619c0 f   wzFilePacker_static:wzFilePacker.obj

 Exports

  ordinal    name

        1    _GFXDll_DialogManagerWZ
               exported name: GFXDll_DialogManagerWZ
